 dna_graphpack

 Timestamp is 5dee3708 (Mon Dec 09 18:59:04 2019)

 Preferred load address is 10000000

 Start         Length     Name                   Class
 0001:00000000 00004db4H .text$di                CODE
 0001:00004dc0 000089deH .text$mn                CODE
 0001:0000d7a0 000022c4H .text$x                 CODE
 0001:0000fa70 000015faH .text$yd                CODE
 0002:00000000 000002b8H .idata$5                DATA
 0002:000002b8 00000004H .CRT$XCA                DATA
 0002:000002bc 00000500H .CRT$XCU                DATA
 0002:000007bc 00000004H .CRT$XCZ                DATA
 0002:000007c0 00000004H .CRT$XIA                DATA
 0002:000007c4 00000004H .CRT$XIAA               DATA
 0002:000007c8 00000004H .CRT$XIC                DATA
 0002:000007cc 00000004H .CRT$XIZ                DATA
 0002:000007d0 00000f18H .rdata                  DATA
 0002:000016e8 00000074H .rdata$debug            DATA
 0002:0000175c 000008f4H .rdata$r                DATA
 0002:00002050 000002bcH .rdata$sxdata           DATA
 0002:0000230c 00000004H .rtc$IAA                DATA
 0002:00002310 00000004H .rtc$IZZ                DATA
 0002:00002314 00000004H .rtc$TAA                DATA
 0002:00002318 00000004H .rtc$TZZ                DATA
 0002:00002320 000024b4H .xdata$x                DATA
 0002:000047e0 00000056H .edata                  DATA
 0002:00004838 000000b4H .idata$2                DATA
 0002:000048ec 00000014H .idata$3                DATA
 0002:00004900 000002b8H .idata$4                DATA
 0002:00004bb8 00001b4eH .idata$6                DATA
 0003:00000000 00000694H .data                   DATA
 0003:00000694 0000049cH .data$r                 DATA
 0003:00000b30 0000077cH .bss                    DATA
 0004:00000000 00000058H .rsrc$01                DATA
 0004:00000060 00000180H .rsrc$02                DATA

  Address         Publics by Value              Rva+Base       Lib:Object

 0000:00000000       ___guard_flags             00000000     <absolute>
 0000:00000000       ___guard_fids_count        00000000     <absolute>
 0000:00000000       __except_list              00000000     <absolute>
 0000:00000000       ___guard_fids_table        00000000     <absolute>
 0000:000000af       ___safe_se_handler_count   000000af     <absolute>
 0000:00009876       __fltused                  00009876     <absolute>
 0000:00009876       __ldused                   00009876     <absolute>
 0000:00000000       ___ImageBase               10000000     <linker-defined>
 0001:00004dc0       ??$_Allocate@D@std@@YAPADIPAD@Z 10005dc0 f i BaseContentGraph.obj
 0001:00004df0       ??$addressof@D@std@@YAPADAAD@Z 10005df0 f i BaseContentGraph.obj
 0001:00004e00       ??$atomic@H@?$QAtomicOpsBySize@$03@@CAPAJPAH@Z 10005e00 f i BaseContentGraph.obj
 0001:00004e10       ??$construct@PADAAPAD@?$_Wrap_alloc@V?$allocator@D@std@@@std@@QAEXPAPADAAPAD@Z 10005e10 f i BaseContentGraph.obj
 0001:00004e30       ??$construct@PADAAPAD@?$allocator@D@std@@QAEXPAPADAAPAD@Z 10005e30 f i BaseContentGraph.obj
 0001:00004e50       ??$construct@PADAAPAD@?$allocator_traits@V?$allocator@D@std@@@std@@SAXAAV?$allocator@D@1@PAPADAAPAD@Z 10005e50 f i BaseContentGraph.obj
 0001:00004e70       ??$deref@H@?$QAtomicOpsBySize@$03@@SA_NAAH@Z 10005e70 f i BaseContentGraph.obj
 0001:00004e90       ??$destroy@PAD@?$_Wrap_alloc@V?$allocator@D@std@@@std@@QAEXPAPAD@Z 10005e90 f i BaseContentGraph.obj
 0001:00004ea0       ??$destroy@PAD@?$allocator@D@std@@QAEXPAPAD@Z 10005ea0 f i BaseContentGraph.obj
 0001:00004eb0       ??$destroy@PAD@?$allocator_traits@V?$allocator@D@std@@@std@@SAXAAV?$allocator@D@1@PAPAD@Z 10005eb0 f i BaseContentGraph.obj
 0001:00004ec0       ??$forward@AAPAD@std@@YAAAPADAAPAD@Z 10005ec0 f i BaseContentGraph.obj
 0001:00004ed0       ??$internalConstruct@UNormalDeleter@QtSharedPointer@@@?$QSharedPointer@VGSequenceGraphData@U2@@@@AAEXPAVGSequenceGraphData@U2@@UNormalDeleter@QtSharedPointer@@@Z 10005ed0 f i BaseContentGraph.obj
 0001:00004f30       ??$load@H@?$QGenericAtomicOps@U?$QAtomicOpsBySize@$03@@@@SAHABH@Z 10005f30 f i BaseContentGraph.obj
 0001:00004f40       ??$ref@H@?$QAtomicOpsBySize@$03@@SA_NAAH@Z 10005f40 f i BaseContentGraph.obj
 0001:00004f60       ??$store@HH@?$QGenericAtomicOps@U?$QAtomicOpsBySize@$03@@@@SAXAAHH@Z 10005f60 f i BaseContentGraph.obj
 0001:00004f70       ??0?$AbstractId@H@U2@@IAE@ABH@Z 10005f70 f i BaseContentGraph.obj
 0001:00004f90       ??0?$CustomDeleter@VGSequenceGraphData@U2@@UNormalDeleter@QtSharedPointer@@@QtSharedPointer@@QAE@PAVGSequenceGraphData@U2@@UNormalDeleter@1@@Z 10005f90 f i BaseContentGraph.obj
 0001:00004fa0       ??0?$QFlags@W4AllocationOption@QArrayData@@@@QAE@W4AllocationOption@QArrayData@@@Z 10005fa0 f i BaseContentGraph.obj
 0001:00004fb0       ??0?$QList@V?$QSharedPointer@VGSequenceGraphData@U2@@@@@@QAE@$$QAV0@@Z 10005fb0 f i BaseContentGraph.obj
 0001:00004fd0       ??0?$QList@V?$QSharedPointer@VGSequenceGraphData@U2@@@@@@QAE@XZ 10005fd0 f i BaseContentGraph.obj
 0001:00004fe0       ??0?$QSharedPointer@VGSequenceGraphData@U2@@@@QAE@ABV0@@Z 10005fe0 f i BaseContentGraph.obj
 0001:00005020       ??0?$QSharedPointer@VGSequenceGraphData@U2@@@@QAE@PAVGSequenceGraphData@U2@@@Z 10006020 f i BaseContentGraph.obj
 0001:00005090       ??0?$_String_alloc@$0A@U?$_String_base_types@DV?$allocator@D@std@@@std@@@std@@QAE@ABV?$allocator@D@1@@Z 10006090 f i BaseContentGraph.obj
 0001:000050b0       ??0?$_String_val@U?$_Simple_types@D@std@@@std@@QAE@XZ 100060b0 f i BaseContentGraph.obj
 0001:000050d0       ??0?$_Wrap_alloc@V?$allocator@D@std@@@std@@QAE@XZ 100060d0 f i BaseContentGraph.obj
 0001:000050e0       ??0?$allocator@D@std@@QAE@XZ 100060e0 f i BaseContentGraph.obj
 0001:000050f0       ??0?$basic_string@DU?$char_traits@D@std@@V?$allocator@D@2@@std@@QAE@PBD@Z 100060f0 f i BaseContentGraph.obj
 0001:00005150       ??0AbstractInt32Id@U2@@IAE@H@Z 10006150 f i BaseContentGraph.obj
 0001:00005170       ??0BaseContentGraphAlgorithm@U2@@QAE@ABVQBitArray@@@Z 10006170 f   BaseContentGraph.obj
 0001:000051d0       ??0BaseContentGraphFactory@U2@@QAE@W4GType@01@PAVQObject@@@Z 100061d0 f   BaseContentGraph.obj
 0001:000052b0       ??0ExternalRefCountData@QtSharedPointer@@QAE@P6AXPAU01@@Z@Z 100062b0 f i BaseContentGraph.obj
 0001:000052d0       ??0QLatin1Char@@QAE@D@Z    100062d0 f i BaseContentGraph.obj
 0001:000052e0       ??0ServiceType@U2@@QAE@H@Z 100062e0 f i BaseContentGraph.obj
 0001:00005300       ??0_Generic_error_category@std@@QAE@XZ 10006300 f i BaseContentGraph.obj
 0001:00005310       ??0_Ignore@std@@QAE@XZ     10006310 f i BaseContentGraph.obj
 0001:00005320       ??0_Iostream_error_category@std@@QAE@XZ 10006320 f i BaseContentGraph.obj
 0001:00005330       ??0_System_error_category@std@@QAE@XZ 10006330 f i BaseContentGraph.obj
 0001:00005340       ??0error_category@std@@QAE@XZ 10006340 f i BaseContentGraph.obj
 0001:00005350       ??0error_condition@std@@QAE@HABVerror_category@1@@Z 10006350 f i BaseContentGraph.obj
 0001:00005370       ??1?$AbstractId@H@U2@@MAE@XZ 10006370 f i BaseContentGraph.obj
 0001:00005380       ??1?$QList@V?$QSharedPointer@VGSequenceGraphData@U2@@@@@@QAE@XZ 10006380 f i BaseContentGraph.obj
 0001:000053d0       ??1?$QSharedPointer@VGSequenceGraphData@U2@@@@QAE@XZ 100063d0 f i BaseContentGraph.obj
 0001:00005410       ??1?$basic_string@DU?$char_traits@D@std@@V?$allocator@D@2@@std@@QAE@XZ 10006410 f i BaseContentGraph.obj
 0001:00005440       ??1AbstractInt32Id@U2@@UAE@XZ 10006440 f i BaseContentGraph.obj
 0001:00005450       ??1BaseContentGraphAlgorithm@U2@@UAE@XZ 10006450 f i BaseContentGraph.obj
 0001:000054b0       ??1BaseContentGraphFactory@U2@@UAE@XZ 100064b0 f i BaseContentGraph.obj
 0001:00005510       ??1ExternalRefCountData@QtSharedPointer@@QAE@XZ 10006510 f i BaseContentGraph.obj
 0001:00005520       ??1ServiceType@U2@@UAE@XZ  10006520 f i BaseContentGraph.obj
 0001:00005530       ??1_Generic_error_category@std@@UAE@XZ 10006530 f i BaseContentGraph.obj
 0001:00005540       ??1_Iostream_error_category@std@@UAE@XZ 10006540 f i BaseContentGraph.obj
 0001:00005550       ??1_System_error_category@std@@UAE@XZ 10006550 f i BaseContentGraph.obj
 0001:00005560       ??1error_category@std@@UAE@XZ 10006560 f i BaseContentGraph.obj
 0001:00005570       ??2@YAPAXIPAX@Z            10006570 f i BaseContentGraph.obj
 0001:00005580       ??3@YAXPAX0@Z              10006580 f i BaseContentGraph.obj
 0001:00005590       ??3ExternalRefCountData@QtSharedPointer@@SAXPAX0@Z 10006590 f i BaseContentGraph.obj
 0001:000055a0       ??3ExternalRefCountData@QtSharedPointer@@SAXPAX@Z 100065a0 f i BaseContentGraph.obj
 0001:000055b0       ??8error_category@std@@QBE_NABV01@@Z 100065b0 f i BaseContentGraph.obj
 0001:000055c0       ??8error_condition@std@@QBE_NABV01@@Z 100065c0 f i BaseContentGraph.obj
 0001:000055e0       ??C?$QSharedPointer@VGSequenceGraphData@U2@@@@QBEPAVGSequenceGraphData@U2@@XZ 100065e0 f i BaseContentGraph.obj
 0001:000055f0       ??_G?$AbstractId@H@U2@@MAEPAXI@Z 100065f0 f i BaseContentGraph.obj
 0001:000055f0       ??_E?$AbstractId@H@U2@@MAEPAXI@Z 100065f0 f i BaseContentGraph.obj
 0001:00005620       ??_G?$QSharedPointer@VGSequenceGraphData@U2@@@@QAEPAXI@Z 10006620 f i BaseContentGraph.obj
 0001:00005670       ??_GAbstractInt32Id@U2@@UAEPAXI@Z 10006670 f i BaseContentGraph.obj
 0001:00005670       ??_EAbstractInt32Id@U2@@UAEPAXI@Z 10006670 f i BaseContentGraph.obj
 0001:000056a0       ??_GBaseContentGraphAlgorithm@U2@@UAEPAXI@Z 100066a0 f i BaseContentGraph.obj
 0001:000056a0       ??_EBaseContentGraphAlgorithm@U2@@UAEPAXI@Z 100066a0 f i BaseContentGraph.obj
 0001:00005710       ??_EBaseContentGraphFactory@U2@@UAEPAXI@Z 10006710 f i BaseContentGraph.obj
 0001:00005710       ??_GBaseContentGraphFactory@U2@@UAEPAXI@Z 10006710 f i BaseContentGraph.obj
 0001:00005780       ??_GExternalRefCountData@QtSharedPointer@@QAEPAXI@Z 10006780 f i BaseContentGraph.obj
 0001:000057a0       ??_GGSequenceGraphData@U2@@UAEPAXI@Z 100067a0 f i BaseContentGraph.obj
 0001:000057a0       ??_EGSequenceGraphData@U2@@UAEPAXI@Z 100067a0 f i BaseContentGraph.obj
 0001:000057d0       ??_EServiceType@U2@@UAEPAXI@Z 100067d0 f i BaseContentGraph.obj
 0001:000057d0       ??_GServiceType@U2@@UAEPAXI@Z 100067d0 f i BaseContentGraph.obj
 0001:00005800       ??_E_Generic_error_category@std@@UAEPAXI@Z 10006800 f i BaseContentGraph.obj
 0001:00005800       ??_G_Generic_error_category@std@@UAEPAXI@Z 10006800 f i BaseContentGraph.obj
 0001:00005830       ??_G_Iostream_error_category@std@@UAEPAXI@Z 10006830 f i BaseContentGraph.obj
 0001:00005830       ??_E_Iostream_error_category@std@@UAEPAXI@Z 10006830 f i BaseContentGraph.obj
 0001:00005860       ??_E_System_error_category@std@@UAEPAXI@Z 10006860 f i BaseContentGraph.obj
 0001:00005860       ??_G_System_error_category@std@@UAEPAXI@Z 10006860 f i BaseContentGraph.obj
 0001:00005890       ??_Gerror_category@std@@UAEPAXI@Z 10006890 f i BaseContentGraph.obj
 0001:00005890       ??_Eerror_category@std@@UAEPAXI@Z 10006890 f i BaseContentGraph.obj
 0001:000058c0       ?_Copy@?$basic_string@DU?$char_traits@D@std@@V?$allocator@D@2@@std@@QAEXII@Z 100068c0 f i BaseContentGraph.obj
 0001:00005a10       ?_Eos@?$basic_string@DU?$char_traits@D@std@@V?$allocator@D@2@@std@@QAEXI@Z 10006a10 f i BaseContentGraph.obj
 0001:00005a40       ?_Getal@?$_String_alloc@$0A@U?$_String_base_types@DV?$allocator@D@std@@@std@@@std@@QBE?AU?$_Wrap_alloc@V?$allocator@D@std@@@2@XZ 10006a40 f i BaseContentGraph.obj
 0001:00005a50       ?_Grow@?$basic_string@DU?$char_traits@D@std@@V?$allocator@D@2@@std@@QAE_NI_N@Z 10006a50 f i BaseContentGraph.obj
 0001:00005b00       ?_Inside@?$basic_string@DU?$char_traits@D@std@@V?$allocator@D@2@@std@@QAE_NPBD@Z 10006b00 f i BaseContentGraph.obj
 0001:00005b40       ?_Myptr@?$_String_val@U?$_Simple_types@D@std@@@std@@QAEPADXZ 10006b40 f i BaseContentGraph.obj
 0001:00005b50       ?_Myptr@?$_String_val@U?$_Simple_types@D@std@@@std@@QBEPBDXZ 10006b50 f i BaseContentGraph.obj
 0001:00005b60       ?_Tidy@?$basic_string@DU?$char_traits@D@std@@V?$allocator@D@2@@std@@QAEX_NI@Z 10006b60 f i BaseContentGraph.obj
 0001:00005bb0       ?_Xlen@?$basic_string@DU?$char_traits@D@std@@V?$allocator@D@2@@std@@QBEXXZ 10006bb0 f i BaseContentGraph.obj
 0001:00005bc0       ?_Xran@?$basic_string@DU?$char_traits@D@std@@V?$allocator@D@2@@std@@QBEXXZ 10006bc0 f i BaseContentGraph.obj
 0001:00005bd0       ?allocate@?$QTypedArrayData@M@@SAPAU1@IV?$QFlags@W4AllocationOption@QArrayData@@@@@Z 10006bd0 f i BaseContentGraph.obj
 0001:00005bf0       ?allocate@?$_Wrap_alloc@V?$allocator@D@std@@@std@@QAEPADI@Z 10006bf0 f i BaseContentGraph.obj
 0001:00005c20       ?allocate@?$allocator@D@std@@QAEPADI@Z 10006c20 f i BaseContentGraph.obj
 0001:00005c50       ?append@?$QList@V?$QSharedPointer@VGSequenceGraphData@U2@@@@@@QAEXABV?$QSharedPointer@VGSequenceGraphData@U2@@@@@Z 10006c50 f i BaseContentGraph.obj
 0001:00005d50       ?append@?$QVector@M@@QAEXABM@Z 10006d50 f i BaseContentGraph.obj
 0001:00005dd0       ?assign@?$basic_string@DU?$char_traits@D@std@@V?$allocator@D@2@@std@@QAEAAV12@ABV12@II@Z 10006dd0 f i BaseContentGraph.obj
 0001:00005ef0       ?assign@?$basic_string@DU?$char_traits@D@std@@V?$allocator@D@2@@std@@QAEAAV12@PBD@Z 10006ef0 f i BaseContentGraph.obj
 0001:00005f30       ?assign@?$basic_string@DU?$char_traits@D@std@@V?$allocator@D@2@@std@@QAEAAV12@PBDI@Z 10006f30 f i BaseContentGraph.obj
 0001:00006030       ?assign@?$char_traits@D@std@@SAXAADABD@Z 10007030 f i BaseContentGraph.obj
 0001:00006040       ?begin@?$QTypedArrayData@M@@QAEPAMPAM@Z 10007040 f i BaseContentGraph.obj
 0001:00006050       ?calculate@BaseContentGraphAlgorithm@U2@@UAEXAAV?$QVector@M@@PAVU2SequenceObject@2@ABVU2Region@2@PBVGSequenceGraphWindowData@2@AAVU2OpStatus@2@@Z 10007050 f   BaseContentGraph.obj
 0001:000063b0       ?category@error_code@std@@QBEABVerror_category@2@XZ 100073b0 f i BaseContentGraph.obj
 0001:000063c0       ?category@error_condition@std@@QBEABVerror_category@2@XZ 100073c0 f i BaseContentGraph.obj
 0001:000063d0       ?copy@?$char_traits@D@std@@SAPADPADPBDI@Z 100073d0 f i BaseContentGraph.obj
 0001:000063f0       ?create@?$ExternalRefCountWithCustomDeleter@VGSequenceGraphData@U2@@UNormalDeleter@QtSharedPointer@@@QtSharedPointer@@SAPAU12@PAVGSequenceGraphData@U2@@UNormalDeleter@2@P6AXPAUExternalRefCountData@2@@Z@Z 100073f0 f i BaseContentGraph.obj
 0001:00006430       ?createGraphs@BaseContentGraphFactory@U2@@UAE?AV?$QList@V?$QSharedPointer@VGSequenceGraphData@U2@@@@@@PAVGSequenceGraphView@2@@Z 10007430 f   BaseContentGraph.obj
 0001:00006560       ?data@?$QSharedPointer@VGSequenceGraphData@U2@@@@QBEPAVGSequenceGraphData@U2@@XZ 10007560 f i BaseContentGraph.obj
 0001:00006570       ?data@?$QTypedArrayData@M@@QAEPAMXZ 10007570 f i BaseContentGraph.obj
 0001:00006580       ?dealloc@?$QList@V?$QSharedPointer@VGSequenceGraphData@U2@@@@@@AAEXPAUData@QListData@@@Z 10007580 f i BaseContentGraph.obj
 0001:000065b0       ?deallocate@?$QTypedArrayData@M@@SAXPAUQArrayData@@@Z 100075b0 f i BaseContentGraph.obj
 0001:000065d0       ?deallocate@?$_Wrap_alloc@V?$allocator@D@std@@@std@@QAEXPADI@Z 100075d0 f i BaseContentGraph.obj
 0001:000065f0       ?deallocate@?$allocator@D@std@@QAEXPADI@Z 100075f0 f i BaseContentGraph.obj
 0001:00006610       ?defaultConstruct@?$QVector@M@@AAEXPAM0@Z 10007610 f i BaseContentGraph.obj
 0001:00006630       ?default_error_condition@_System_error_category@std@@UBE?AVerror_condition@2@H@Z 10007630 f i BaseContentGraph.obj
 0001:00006670       ?default_error_condition@error_category@std@@UBE?AVerror_condition@2@H@Z 10007670 f i BaseContentGraph.obj
 0001:00006690       ?deleter@?$ExternalRefCountWithCustomDeleter@VGSequenceGraphData@U2@@UNormalDeleter@QtSharedPointer@@@QtSharedPointer@@SAXPAUExternalRefCountData@2@@Z 10007690 f i BaseContentGraph.obj
 0001:000066b0       ?deref@?$QBasicAtomicInteger@H@@QAE_NXZ 100076b0 f i BaseContentGraph.obj
 0001:000066c0       ?deref@?$QSharedPointer@VGSequenceGraphData@U2@@@@AAEXXZ 100076c0 f i BaseContentGraph.obj
 0001:00006700       ?deref@?$QSharedPointer@VGSequenceGraphData@U2@@@@CAXPAUExternalRefCountData@QtSharedPointer@@@Z 10007700 f i BaseContentGraph.obj
 0001:00006740       ?deref@RefCount@QtPrivate@@QAE_NXZ 10007740 f i BaseContentGraph.obj
 0001:00006760       ?destroy@ExternalRefCountData@QtSharedPointer@@QAEXXZ 10007760 f i BaseContentGraph.obj
 0001:00006770       ?destruct@?$QVector@M@@AAEXPAM0@Z 10007770 f i BaseContentGraph.obj
 0001:00006780       ?detach_helper_grow@?$QList@V?$QSharedPointer@VGSequenceGraphData@U2@@@@@@AAEPAUNode@1@HH@Z 10007780 f i BaseContentGraph.obj
 0001:000068f0       ?enableSharedFromThis@?$QSharedPointer@VGSequenceGraphData@U2@@@@AAAXZZ 100078f0 f i BaseContentGraph.obj
 0001:00006900       ?end@?$QTypedArrayData@M@@QAEPAMPAM@Z 10007900 f i BaseContentGraph.obj
 0001:00006920       ?equivalent@error_category@std@@UBE_NABVerror_code@2@H@Z 10007920 f i BaseContentGraph.obj
 0001:00006940       ?equivalent@error_category@std@@UBE_NHABVerror_condition@2@@Z 10007940 f i BaseContentGraph.obj
 0001:00006980       ?erase@?$basic_string@DU?$char_traits@D@std@@V?$allocator@D@2@@std@@QAEAAV12@I@Z 10007980 f i BaseContentGraph.obj
 0001:000069c0       ?erase@?$basic_string@DU?$char_traits@D@std@@V?$allocator@D@2@@std@@QAEAAV12@II@Z 100079c0 f i BaseContentGraph.obj
 0001:00006a60       ?execute@?$CustomDeleter@VGSequenceGraphData@U2@@UNormalDeleter@QtSharedPointer@@@QtSharedPointer@@QAEXXZ 10007a60 f i BaseContentGraph.obj
 0001:00006a70       ?freeData@?$QVector@M@@AAEXPAU?$QTypedArrayData@M@@@Z 10007a70 f i BaseContentGraph.obj
 0001:00006aa0       ?generic_category@std@@YAABVerror_category@1@XZ 10007aa0 f i BaseContentGraph.obj
 0001:00006ab0       ?isDetached@?$QVector@M@@QBE_NXZ 10007ab0 f i BaseContentGraph.obj
 0001:00006ae0       ?isEnabled@BaseContentGraphFactory@U2@@UBE_NPBVU2SequenceObject@2@@Z 10007ae0 f   BaseContentGraph.obj
 0001:00006b00       ?isShared@RefCount@QtPrivate@@QBE_NXZ 10007b00 f i BaseContentGraph.obj
 0001:00006b20       ?isValid@AbstractInt32Id@U2@@UBE_NXZ 10007b20 f i BaseContentGraph.obj
 0001:00006b30       ?length@?$char_traits@D@std@@SAIPBD@Z 10007b30 f i BaseContentGraph.obj
 0001:00006b50       ?load@?$QBasicAtomicInteger@H@@QBEHXZ 10007b50 f i BaseContentGraph.obj
 0001:00006b60       ?max_size@?$_Wrap_alloc@V?$allocator@D@std@@@std@@QBEIXZ 10007b60 f i BaseContentGraph.obj
 0001:00006b70       ?max_size@?$allocator@D@std@@QBEIXZ 10007b70 f i BaseContentGraph.obj
 0001:00006b80       ?max_size@?$allocator_traits@V?$allocator@D@std@@@std@@SAIABV?$allocator@D@2@@Z 10007b80 f i BaseContentGraph.obj
 0001:00006b90       ?max_size@?$basic_string@DU?$char_traits@D@std@@V?$allocator@D@2@@std@@QBEIXZ 10007b90 f i BaseContentGraph.obj
 0001:00006ba0       ?message@_Generic_error_category@std@@UBE?AV?$basic_string@DU?$char_traits@D@std@@V?$allocator@D@2@@2@H@Z 10007ba0 f i BaseContentGraph.obj
 0001:00006c20       ?message@_Iostream_error_category@std@@UBE?AV?$basic_string@DU?$char_traits@D@std@@V?$allocator@D@2@@2@H@Z 10007c20 f i BaseContentGraph.obj
 0001:00006c70       ?message@_System_error_category@std@@UBE?AV?$basic_string@DU?$char_traits@D@std@@V?$allocator@D@2@@2@H@Z 10007c70 f i BaseContentGraph.obj
 0001:00006cf0       ?move@?$char_traits@D@std@@SAPADPADPBDI@Z 10007cf0 f i BaseContentGraph.obj
 0001:00006d10       ?name@_Generic_error_category@std@@UBEPBDXZ 10007d10 f i BaseContentGraph.obj
 0001:00006d20       ?name@_Iostream_error_category@std@@UBEPBDXZ 10007d20 f i BaseContentGraph.obj
 0001:00006d30       ?name@_System_error_category@std@@UBEPBDXZ 10007d30 f i BaseContentGraph.obj
 0001:00006d90       ?node_construct@?$QList@V?$QSharedPointer@VGSequenceGraphData@U2@@@@@@AAEXPAUNode@1@ABV?$QSharedPointer@VGSequenceGraphData@U2@@@@@Z 10007d90 f i BaseContentGraph.obj
 0001:00006df0       ?node_copy@?$QList@V?$QSharedPointer@VGSequenceGraphData@U2@@@@@@AAEXPAUNode@1@00@Z 10007df0 f i BaseContentGraph.obj
 0001:00006ec0       ?node_destruct@?$QList@V?$QSharedPointer@VGSequenceGraphData@U2@@@@@@AAEXPAUNode@1@0@Z 10007ec0 f i BaseContentGraph.obj
 0001:00006f20       ?node_destruct@?$QList@V?$QSharedPointer@VGSequenceGraphData@U2@@@@@@AAEXPAUNode@1@@Z 10007f20 f i BaseContentGraph.obj
 0001:00006f70       ?qt_noop@@YAXXZ            10007f70 f i BaseContentGraph.obj
 0001:00006f80       ?reallocData@?$QVector@M@@AAEXHHV?$QFlags@W4AllocationOption@QArrayData@@@@@Z 10007f80 f i BaseContentGraph.obj
 0001:000071c0       ?ref@?$QBasicAtomicInteger@H@@QAE_NXZ 100081c0 f i BaseContentGraph.obj
 0001:000071e0       ?ref@?$QSharedPointer@VGSequenceGraphData@U2@@@@ABEXXZ 100081e0 f i BaseContentGraph.obj
 0001:00007200       ?reserve@?$QVector@M@@QAEXH@Z 10008200 f i BaseContentGraph.obj
 0001:00007250       ?setQObjectShared@ExternalRefCountData@QtSharedPointer@@QAAXZZ 10008250 f i BaseContentGraph.obj
 0001:00007260       ?sharedNull@?$QTypedArrayData@M@@SAPAU1@XZ 10008260 f i BaseContentGraph.obj
 0001:00007270       ?size@?$basic_string@DU?$char_traits@D@std@@V?$allocator@D@2@@std@@QBEIXZ 10008270 f i BaseContentGraph.obj
 0001:00007280       ?store@?$QBasicAtomicInteger@H@@QAEXH@Z 10008280 f i BaseContentGraph.obj
 0001:00007290       ?system_category@std@@YAABVerror_category@1@XZ 10008290 f i BaseContentGraph.obj
 0001:000072a0       ?tr@BaseContentGraphFactory@U2@@SA?AVQString@@PBD0H@Z 100082a0 f i BaseContentGraph.obj
 0001:000072d0       ?value@error_code@std@@QBEHXZ 100082d0 f i BaseContentGraph.obj
 0001:000072e0       ?value@error_condition@std@@QBEHXZ 100082e0 f i BaseContentGraph.obj
 0001:000072f0       ?windowStrategyWithoutMemorize@BaseContentGraphAlgorithm@U2@@AAEXAAV?$QVector@M@@ABVQByteArray@@HPBVGSequenceGraphWindowData@2@HAAVU2OpStatus@2@@Z 100082f0 f   BaseContentGraph.obj
 0001:00007410       _hypot                     10008410 f i BaseContentGraph.obj
 0001:00007440       ??0?$QPair@DD@@QAE@XZ      10008440 f i CumulativeSkew.obj
 0001:00007450       ??0CumulativeSkewGraphAlgorithm@U2@@QAE@ABU?$QPair@DD@@@Z 10008450 f   CumulativeSkew.obj
 0001:00007480       ??0CumulativeSkewGraphFactory@U2@@QAE@W4GCumulativeSkewType@01@PAVQObject@@@Z 10008480 f   CumulativeSkew.obj
 0001:00007520       ??1CumulativeSkewGraphAlgorithm@U2@@UAE@XZ 10008520 f i CumulativeSkew.obj
 0001:00007530       ??1CumulativeSkewGraphFactory@U2@@UAE@XZ 10008530 f i CumulativeSkew.obj
 0001:00007540       ??_GCumulativeSkewGraphAlgorithm@U2@@UAEPAXI@Z 10008540 f i CumulativeSkew.obj
 0001:00007540       ??_ECumulativeSkewGraphAlgorithm@U2@@UAEPAXI@Z 10008540 f i CumulativeSkew.obj
 0001:00007570       ??_GCumulativeSkewGraphFactory@U2@@UAEPAXI@Z 10008570 f i CumulativeSkew.obj
 0001:00007570       ??_ECumulativeSkewGraphFactory@U2@@UAEPAXI@Z 10008570 f i CumulativeSkew.obj
 0001:000075a0       ?calculate@CumulativeSkewGraphAlgorithm@U2@@UAEXAAV?$QVector@M@@PAVU2SequenceObject@2@ABVU2Region@2@PBVGSequenceGraphWindowData@2@AAVU2OpStatus@2@@Z 100085a0 f   CumulativeSkew.obj
 0001:000076e0       ?createGraphs@CumulativeSkewGraphFactory@U2@@UAE?AV?$QList@V?$QSharedPointer@VGSequenceGraphData@U2@@@@@@PAVGSequenceGraphView@2@@Z 100086e0 f   CumulativeSkew.obj
 0001:00007800       ?getValue@CumulativeSkewGraphAlgorithm@U2@@QAEMHHABVQByteArray@@@Z 10008800 f   CumulativeSkew.obj
 0001:000078d0       ?isEnabled@CumulativeSkewGraphFactory@U2@@UBE_NPBVU2SequenceObject@2@@Z 100088d0 f   CumulativeSkew.obj
 0001:00007940       ?tr@CumulativeSkewGraphFactory@U2@@SA?AVQString@@PBD0H@Z 10008940 f i CumulativeSkew.obj
 0001:00007970       ??$qobject_cast@PAVADVSingleSequenceWidget@U2@@@@YAPAVADVSingleSequenceWidget@U2@@PAVQObject@@@Z 10008970 f i DNAGraphPackPlugin.obj
 0001:00007990       ??$qobject_cast@PAVAnnotatedDNAView@U2@@@@YAPAVAnnotatedDNAView@U2@@PAVQObject@@@Z 10008990 f i DNAGraphPackPlugin.obj
 0001:000079b0       ??0?$QForeachContainer@$$CBV?$QList@PAVADVSequenceWidget@U2@@@@@@QAE@ABV?$QList@PAVADVSequenceWidget@U2@@@@@Z 100089b0 f i DNAGraphPackPlugin.obj
 0001:000079f0       ??0?$QForeachContainer@V?$QList@PAVGSequenceGraphFactory@U2@@@@@@QAE@ABV?$QList@PAVGSequenceGraphFactory@U2@@@@@Z 100089f0 f i DNAGraphPackPlugin.obj
 0001:00007a30       ??0?$QList@PAVADVSequenceWidget@U2@@@@QAE@ABV0@@Z 10008a30 f i DNAGraphPackPlugin.obj
 0001:00007af0       ??0?$QList@PAVGSequenceGraphFactory@U2@@@@QAE@ABV0@@Z 10008af0 f i DNAGraphPackPlugin.obj
 0001:00007bb0       ??0?$QList@PAVGSequenceGraphFactory@U2@@@@QAE@XZ 10008bb0 f i DNAGraphPackPlugin.obj
 0001:00007bc0       ??0DNAGraphPackPlugin@U2@@QAE@XZ 10008bc0 f   DNAGraphPackPlugin.obj
 0001:00007c90       ??0DNAGraphPackViewContext@U2@@QAE@PAVQObject@@@Z 10008c90 f   DNAGraphPackPlugin.obj
 0001:00007ea0       ??0GObjectViewFactoryId@U2@@QAE@PBD@Z 10008ea0 f i DNAGraphPackPlugin.obj
 0001:00007ee0       ??0const_iterator@?$QList@PAVADVSequenceWidget@U2@@@@QAE@PAUNode@1@@Z 10008ee0 f i DNAGraphPackPlugin.obj
 0001:00007ef0       ??0const_iterator@?$QList@PAVGSequenceGraphFactory@U2@@@@QAE@PAUNode@1@@Z 10008ef0 f i DNAGraphPackPlugin.obj
 0001:00007f00       ??1?$QForeachContainer@$$CBV?$QList@PAVADVSequenceWidget@U2@@@@@@QAE@XZ 10008f00 f i DNAGraphPackPlugin.obj
 0001:00007f30       ??1?$QForeachContainer@V?$QList@PAVGSequenceGraphFactory@U2@@@@@@QAE@XZ 10008f30 f i DNAGraphPackPlugin.obj
 0001:00007f60       ??1?$QList@PAVADVSequenceWidget@U2@@@@QAE@XZ 10008f60 f i DNAGraphPackPlugin.obj
 0001:00007f90       ??1?$QList@PAVGSequenceGraphFactory@U2@@@@QAE@XZ 10008f90 f i DNAGraphPackPlugin.obj
 0001:00007fc0       ??1DNAGraphPackPlugin@U2@@UAE@XZ 10008fc0 f i DNAGraphPackPlugin.obj
 0001:00007fd0       ??1DNAGraphPackViewContext@U2@@UAE@XZ 10008fd0 f i DNAGraphPackPlugin.obj
 0001:00008050       ??1GObjectViewFactoryId@U2@@QAE@XZ 10009050 f i DNAGraphPackPlugin.obj
 0001:00008060       ??9const_iterator@?$QList@PAVADVSequenceWidget@U2@@@@QBE_NABV01@@Z 10009060 f i DNAGraphPackPlugin.obj
 0001:00008080       ??9const_iterator@?$QList@PAVGSequenceGraphFactory@U2@@@@QBE_NABV01@@Z 10009080 f i DNAGraphPackPlugin.obj
 0001:000080a0       ??Dconst_iterator@?$QList@PAVADVSequenceWidget@U2@@@@QBEABQAVADVSequenceWidget@U2@@XZ 100090a0 f i DNAGraphPackPlugin.obj
 0001:000080b0       ??Dconst_iterator@?$QList@PAVGSequenceGraphFactory@U2@@@@QBEABQAVGSequenceGraphFactory@U2@@XZ 100090b0 f i DNAGraphPackPlugin.obj
 0001:000080c0       ??Econst_iterator@?$QList@PAVADVSequenceWidget@U2@@@@QAEAAV01@XZ 100090c0 f i DNAGraphPackPlugin.obj
 0001:000080d0       ??Econst_iterator@?$QList@PAVGSequenceGraphFactory@U2@@@@QAEAAV01@XZ 100090d0 f i DNAGraphPackPlugin.obj
 0001:000080d6       ??_EDNAGraphPackViewContext@U2@@W7AEPAXI@Z 100090d6 f i DNAGraphPackPlugin.obj
 0001:000080e0       ??_GDNAGraphPackPlugin@U2@@UAEPAXI@Z 100090e0 f i DNAGraphPackPlugin.obj
 0001:000080e0       ??_EDNAGraphPackPlugin@U2@@UAEPAXI@Z 100090e0 f i DNAGraphPackPlugin.obj
 0001:00008110       ??_GDNAGraphPackViewContext@U2@@UAEPAXI@Z 10009110 f i DNAGraphPackPlugin.obj
 0001:00008110       ??_EDNAGraphPackViewContext@U2@@UAEPAXI@Z 10009110 f i DNAGraphPackPlugin.obj
 0001:000081a0       ??_GGraphAction@U2@@UAEPAXI@Z 100091a0 f i DNAGraphPackPlugin.obj
 0001:000081a0       ??_EGraphAction@U2@@UAEPAXI@Z 100091a0 f i DNAGraphPackPlugin.obj
 0001:000081d0       ?append@?$QList@PAVGSequenceGraphFactory@U2@@@@QAEXABQAVGSequenceGraphFactory@U2@@@Z 100091d0 f i DNAGraphPackPlugin.obj
 0001:00008260       ?begin@?$QList@PAVADVSequenceWidget@U2@@@@QBE?AVconst_iterator@1@XZ 10009260 f i DNAGraphPackPlugin.obj
 0001:00008280       ?begin@?$QList@PAVGSequenceGraphFactory@U2@@@@QBE?AVconst_iterator@1@XZ 10009280 f i DNAGraphPackPlugin.obj
 0001:000082a0       ?dealloc@?$QList@PAVADVSequenceWidget@U2@@@@AAEXPAUData@QListData@@@Z 100092a0 f i DNAGraphPackPlugin.obj
 0001:000082c0       ?dealloc@?$QList@PAVGSequenceGraphFactory@U2@@@@AAEXPAUData@QListData@@@Z 100092c0 f i DNAGraphPackPlugin.obj
 0001:000082e0       ?detach_helper_grow@?$QList@PAVGSequenceGraphFactory@U2@@@@AAEPAUNode@1@HH@Z 100092e0 f i DNAGraphPackPlugin.obj
 0001:000083f0       ?end@?$QList@PAVADVSequenceWidget@U2@@@@QBE?AVconst_iterator@1@XZ 100093f0 f i DNAGraphPackPlugin.obj
 0001:00008410       ?end@?$QList@PAVGSequenceGraphFactory@U2@@@@QBE?AVconst_iterator@1@XZ 10009410 f i DNAGraphPackPlugin.obj
 0001:00008430       ?initViewContext@DNAGraphPackViewContext@U2@@EAEXPAVGObjectView@2@@Z 10009430 f   DNAGraphPackPlugin.obj
 0001:00008570       ?node_construct@?$QList@PAVGSequenceGraphFactory@U2@@@@AAEXPAUNode@1@ABQAVGSequenceGraphFactory@U2@@@Z 10009570 f i DNAGraphPackPlugin.obj
 0001:00008590       ?node_copy@?$QList@PAVADVSequenceWidget@U2@@@@AAEXPAUNode@1@00@Z 10009590 f i DNAGraphPackPlugin.obj
 0001:000085c0       ?node_copy@?$QList@PAVGSequenceGraphFactory@U2@@@@AAEXPAUNode@1@00@Z 100095c0 f i DNAGraphPackPlugin.obj
 0001:000085f0       ?node_destruct@?$QList@PAVADVSequenceWidget@U2@@@@AAEXPAUNode@1@0@Z 100095f0 f i DNAGraphPackPlugin.obj
 0001:00008600       ?node_destruct@?$QList@PAVGSequenceGraphFactory@U2@@@@AAEXPAUNode@1@0@Z 10009600 f i DNAGraphPackPlugin.obj
 0001:00008610       ?node_destruct@?$QList@PAVGSequenceGraphFactory@U2@@@@AAEXPAUNode@1@@Z 10009610 f i DNAGraphPackPlugin.obj
 0001:00008620       ?ref@RefCount@QtPrivate@@QAE_NXZ 10009620 f i DNAGraphPackPlugin.obj
 0001:00008640       ?sl_sequenceWidgetAdded@DNAGraphPackViewContext@U2@@AAEXPAVADVSequenceWidget@2@@Z 10009640 f   DNAGraphPackPlugin.obj
 0001:000087d0       ?t@Node@?$QList@PAVADVSequenceWidget@U2@@@@QAEAAPAVADVSequenceWidget@U2@@XZ 100097d0 f i DNAGraphPackPlugin.obj
 0001:000087e0       ?t@Node@?$QList@PAVGSequenceGraphFactory@U2@@@@QAEAAPAVGSequenceGraphFactory@U2@@XZ 100097e0 f i DNAGraphPackPlugin.obj
 0001:000087f0       ?tr@DNAGraphPackPlugin@U2@@SA?AVQString@@PBD0H@Z 100097f0 f i DNAGraphPackPlugin.obj
 0001:00008820       _ugene_plugin_init         10009820 f   DNAGraphPackPlugin.obj
 0001:00008850       ??$?0HH@?$QPair@HH@@QAE@$$QAU0@@Z 10009850 f i DeviationGraph.obj
 0001:00008870       ??$qMax@M@@YAABMABM0@Z     10009870 f i DeviationGraph.obj
 0001:00008890       ??0?$QFlags@W4AllocationOption@QArrayData@@@@QAE@PQPrivate@0@H@Z 10009890 f i DeviationGraph.obj
 0001:000088a0       ??0?$QPair@HH@@QAE@ABH0@Z  100098a0 f i DeviationGraph.obj
 0001:000088c0       ??0?$QVector@H@@QAE@XZ     100098c0 f i DeviationGraph.obj
 0001:000088d0       ??0?$RollingArray@H@U2@@QAE@H@Z 100098d0 f i DeviationGraph.obj
 0001:00008970       ??0DeviationGraphAlgorithm@U2@@QAE@ABU?$QPair@DD@@@Z 10009970 f   DeviationGraph.obj
 0001:000089a0       ??0DeviationGraphFactory@U2@@QAE@W4GDeviationType@01@PAVQObject@@@Z 100099a0 f   DeviationGraph.obj
 0001:00008a40       ??1?$QVector@H@@QAE@XZ     10009a40 f i DeviationGraph.obj
 0001:00008a80       ??1?$RollingArray@H@U2@@QAE@XZ 10009a80 f i DeviationGraph.obj
 0001:00008ac0       ??1DeviationGraphAlgorithm@U2@@UAE@XZ 10009ac0 f i DeviationGraph.obj
 0001:00008ad0       ??1DeviationGraphFactory@U2@@UAE@XZ 10009ad0 f i DeviationGraph.obj
 0001:00008ae0       ??A?$QVector@H@@QAEAAHH@Z  10009ae0 f i DeviationGraph.obj
 0001:00008b60       ??_EDeviationGraphAlgorithm@U2@@UAEPAXI@Z 10009b60 f i DeviationGraph.obj
 0001:00008b60       ??_GDeviationGraphAlgorithm@U2@@UAEPAXI@Z 10009b60 f i DeviationGraph.obj
 0001:00008b90       ??_EDeviationGraphFactory@U2@@UAEPAXI@Z 10009b90 f i DeviationGraph.obj
 0001:00008b90       ??_GDeviationGraphFactory@U2@@UAEPAXI@Z 10009b90 f i DeviationGraph.obj
 0001:00008bc0       ?allocate@?$QTypedArrayData@H@@SAPAU1@IV?$QFlags@W4AllocationOption@QArrayData@@@@@Z 10009bc0 f i DeviationGraph.obj
 0001:00008be0       ?begin@?$QTypedArrayData@H@@QAEPAHPAH@Z 10009be0 f i DeviationGraph.obj
 0001:00008bf0       ?calculate@DeviationGraphAlgorithm@U2@@UAEXAAV?$QVector@M@@PAVU2SequenceObject@2@ABVU2Region@2@PBVGSequenceGraphWindowData@2@AAVU2OpStatus@2@@Z 10009bf0 f   DeviationGraph.obj
 0001:00008cc0       ?createGraphs@DeviationGraphFactory@U2@@UAE?AV?$QList@V?$QSharedPointer@VGSequenceGraphData@U2@@@@@@PAVGSequenceGraphView@2@@Z 10009cc0 f   DeviationGraph.obj
 0001:00008de0       ?data@?$QTypedArrayData@H@@QAEPAHXZ 10009de0 f i DeviationGraph.obj
 0001:00008df0       ?data@?$QVector@H@@QAEPAHXZ 10009df0 f i DeviationGraph.obj
 0001:00008e50       ?deallocate@?$QTypedArrayData@H@@SAXPAUQArrayData@@@Z 10009e50 f i DeviationGraph.obj
 0001:00008e70       ?defaultConstruct@?$QVector@H@@AAEXPAH0@Z 10009e70 f i DeviationGraph.obj
 0001:00008e90       ?destruct@?$QVector@H@@AAEXPAH0@Z 10009e90 f i DeviationGraph.obj
 0001:00008ea0       ?detach@?$QVector@H@@QAEXXZ 10009ea0 f i DeviationGraph.obj
 0001:00008ef0       ?end@?$QTypedArrayData@H@@QAEPAHPAH@Z 10009ef0 f i DeviationGraph.obj
 0001:00008f10       ?freeData@?$QVector@H@@AAEXPAU?$QTypedArrayData@H@@@Z 10009f10 f i DeviationGraph.obj
 0001:00008f40       ?get@?$RollingArray@H@U2@@QAEAAHH@Z 10009f40 f i DeviationGraph.obj
 0001:00008f60       ?getMaxSize@?$RollingArray@H@U2@@QBEHXZ 10009f60 f i DeviationGraph.obj
 0001:00008f70       ?isDetached@?$QVector@H@@QBE_NXZ 10009f70 f i DeviationGraph.obj
 0001:00008fa0       ?isEnabled@DeviationGraphFactory@U2@@UBE_NPBVU2SequenceObject@2@@Z 10009fa0 f   DeviationGraph.obj
 0001:00008ff0       ?matchOnStep@DeviationGraphAlgorithm@U2@@AAE?AU?$QPair@HH@@ABVQByteArray@@HH@Z 10009ff0 f   DeviationGraph.obj
 0001:000090a0       ?pop_front@?$RollingArray@H@U2@@AAEHXZ 1000a0a0 f i DeviationGraph.obj
 0001:000090d0       ?push@?$RollingArray@H@U2@@AAEXH@Z 1000a0d0 f i DeviationGraph.obj
 0001:00009100       ?push_back_pop_front@?$RollingArray@H@U2@@QAEXH@Z 1000a100 f i DeviationGraph.obj
 0001:00009160       ?reallocData@?$QVector@H@@AAEXHHV?$QFlags@W4AllocationOption@QArrayData@@@@@Z 1000a160 f i DeviationGraph.obj
 0001:000093a0       ?resize@?$QVector@H@@QAEXH@Z 1000a3a0 f i DeviationGraph.obj
 0001:000093f0       ?sequenceStrategyWithMemorize@DeviationGraphAlgorithm@U2@@AAEXAAV?$QVector@M@@ABVQByteArray@@ABVU2Region@2@PBVGSequenceGraphWindowData@2@AAVU2OpStatus@2@@Z 1000a3f0 f   DeviationGraph.obj
 0001:000097b0       ?sharedNull@?$QTypedArrayData@H@@SAPAU1@XZ 1000a7b0 f i DeviationGraph.obj
 0001:000097c0       ?size@?$RollingArray@H@U2@@QBEHXZ 1000a7c0 f i DeviationGraph.obj
 0001:000097d0       ?toPos@?$RollingArray@H@U2@@ABEHH@Z 1000a7d0 f i DeviationGraph.obj
 0001:000097f0       ?toRollPos@?$RollingArray@H@U2@@ABEHH@Z 1000a7f0 f i DeviationGraph.obj
 0001:00009810       ?tr@DeviationGraphFactory@U2@@SA?AVQString@@PBD0H@Z 1000a810 f i DeviationGraph.obj
 0001:00009840       ?unsharableEmpty@?$QTypedArrayData@H@@SAPAU1@XZ 1000a840 f i DeviationGraph.obj
 0001:00009860       ?windowStrategyWithoutMemorize@DeviationGraphAlgorithm@U2@@AAEXAAV?$QVector@M@@ABVQByteArray@@HPBVGSequenceGraphWindowData@2@HAAVU2OpStatus@2@@Z 1000a860 f   DeviationGraph.obj
 0001:00009990       ??$qFill@PAHH@@YAXPAH0ABH@Z 1000a990 f i EntropyAlgorithm.obj
 0001:000099d0       ??0?$IndexedMapping3To1@H@U2@@QAE@ABVQByteArray@@ABH@Z 1000a9d0 f i EntropyAlgorithm.obj
 0001:00009a50       ??0EntropyGraphAlgorithm@U2@@QAE@XZ 1000aa50 f i EntropyAlgorithm.obj
 0001:00009a70       ??0EntropyGraphFactory@U2@@QAE@PAVQObject@@@Z 1000aa70 f   EntropyAlgorithm.obj
 0001:00009af0       ??1?$IndexedMapping3To1@H@U2@@QAE@XZ 1000aaf0 f i EntropyAlgorithm.obj
 0001:00009b00       ??1EntropyGraphAlgorithm@U2@@UAE@XZ 1000ab00 f i EntropyAlgorithm.obj
 0001:00009b10       ??1EntropyGraphFactory@U2@@UAE@XZ 1000ab10 f i EntropyAlgorithm.obj
 0001:00009b20       ??_EEntropyGraphAlgorithm@U2@@UAEPAXI@Z 1000ab20 f i EntropyAlgorithm.obj
 0001:00009b20       ??_GEntropyGraphAlgorithm@U2@@UAEPAXI@Z 1000ab20 f i EntropyAlgorithm.obj
 0001:00009b50       ??_GEntropyGraphFactory@U2@@UAEPAXI@Z 1000ab50 f i EntropyAlgorithm.obj
 0001:00009b50       ??_EEntropyGraphFactory@U2@@UAEPAXI@Z 1000ab50 f i EntropyAlgorithm.obj
 0001:00009b80       ?calculate@EntropyGraphAlgorithm@U2@@UAEXAAV?$QVector@M@@PAVU2SequenceObject@2@ABVU2Region@2@PBVGSequenceGraphWindowData@2@AAVU2OpStatus@2@@Z 1000ab80 f   EntropyAlgorithm.obj
 0001:00009ea0       ?createGraphs@EntropyGraphFactory@U2@@UAE?AV?$QList@V?$QSharedPointer@VGSequenceGraphData@U2@@@@@@PAVGSequenceGraphView@2@@Z 1000aea0 f   EntropyAlgorithm.obj
 0001:00009fc0       ?getMapSize@?$IndexedMapping3To1@H@U2@@QBEHXZ 1000afc0 f i EntropyAlgorithm.obj
 0001:00009fd0       ?isEnabled@EntropyGraphFactory@U2@@UBE_NPBVU2SequenceObject@2@@Z 1000afd0 f   EntropyAlgorithm.obj
 0001:0000a030       ?log10@@YAMM@Z             1000b030 f i EntropyAlgorithm.obj
 0001:0000a050       ?mapData@?$IndexedMapping3To1@H@U2@@QAEAAPAHXZ 1000b050 f i EntropyAlgorithm.obj
 0001:0000a060       ?mapNC@?$IndexedMapping3To1@H@U2@@QAEAAHPBD@Z 1000b060 f i EntropyAlgorithm.obj
 0001:0000a0c0       ?tr@EntropyGraphFactory@U2@@SA?AVQString@@PBD0H@Z 1000b0c0 f i EntropyAlgorithm.obj
 0001:0000a0f0       _log10f                    1000b0f0 f i EntropyAlgorithm.obj
 0001:0000a110       ??$qMapLessThanKey@VQString@@@@YA_NABVQString@@0@Z 1000b110 f i GCFramePlot.obj
 0001:0000a120       ??0?$QMap@VQString@@VQColor@@@@QAE@XZ 1000b120 f i GCFramePlot.obj
 0001:0000a130       ??0GCFramePlotAlgorithm@U2@@QAE@H@Z 1000b130 f   GCFramePlot.obj
 0001:0000a1d0       ??0GCFramePlotFactory@U2@@QAE@PAVQObject@@@Z 1000b1d0 f   GCFramePlot.obj
 0001:0000a250       ??0iterator@?$QMap@VQString@@VQColor@@@@QAE@PAU?$QMapNode@VQString@@VQColor@@@@@Z 1000b250 f i GCFramePlot.obj
 0001:0000a260       ??1?$QMap@VQString@@VQColor@@@@QAE@XZ 1000b260 f i GCFramePlot.obj
 0001:0000a2d0       ??1GCFramePlotAlgorithm@U2@@UAE@XZ 1000b2d0 f i GCFramePlot.obj
 0001:0000a330       ??1GCFramePlotFactory@U2@@UAE@XZ 1000b330 f i GCFramePlot.obj
 0001:0000a340       ??_EGCFramePlotAlgorithm@U2@@UAEPAXI@Z 1000b340 f i GCFramePlot.obj
 0001:0000a340       ??_GGCFramePlotAlgorithm@U2@@UAEPAXI@Z 1000b340 f i GCFramePlot.obj
 0001:0000a3b0       ??_GGCFramePlotFactory@U2@@UAEPAXI@Z 1000b3b0 f i GCFramePlot.obj
 0001:0000a3b0       ??_EGCFramePlotFactory@U2@@UAEPAXI@Z 1000b3b0 f i GCFramePlot.obj
 0001:0000a3e0       ??_GQString@@QAEPAXI@Z     1000b3e0 f i GCFramePlot.obj
 0001:0000a410       ?calculate@GCFramePlotAlgorithm@U2@@UAEXAAV?$QVector@M@@PAVU2SequenceObject@2@ABVU2Region@2@PBVGSequenceGraphWindowData@2@AAVU2OpStatus@2@@Z 1000b410 f   GCFramePlot.obj
 0001:0000a4b0       ?copy@?$QMapNode@VQString@@VQColor@@@@QBEPAU1@PAU?$QMapData@VQString@@VQColor@@@@@Z 1000b4b0 f i GCFramePlot.obj
 0001:0000a540       ?create@?$QMapData@VQString@@VQColor@@@@SAPAU1@XZ 1000b540 f i GCFramePlot.obj
 0001:0000a550       ?createGraphs@GCFramePlotFactory@U2@@UAE?AV?$QList@V?$QSharedPointer@VGSequenceGraphData@U2@@@@@@PAVGSequenceGraphView@2@@Z 1000b550 f   GCFramePlot.obj
 0001:0000a850       ?createNode@?$QMapData@VQString@@VQColor@@@@QAEPAU?$QMapNode@VQString@@VQColor@@@@ABVQString@@ABVQColor@@PAU2@_N@Z 1000b850 f i GCFramePlot.obj
 0001:0000a900       ?destroy@?$QMapData@VQString@@VQColor@@@@QAEXXZ 1000b900 f i GCFramePlot.obj
 0001:0000a950       ?destroySubTree@?$QMapNode@VQString@@VQColor@@@@QAEXXZ 1000b950 f i GCFramePlot.obj
 0001:0000a980       ?detach@?$QMap@VQString@@VQColor@@@@QAEXXZ 1000b980 f i GCFramePlot.obj
 0001:0000a9a0       ?detach_helper@?$QMap@VQString@@VQColor@@@@AAEXXZ 1000b9a0 f i GCFramePlot.obj
 0001:0000aa50       ?end@?$QMapData@VQString@@VQColor@@@@QAEPAU?$QMapNode@VQString@@VQColor@@@@XZ 1000ba50 f i GCFramePlot.obj
 0001:0000aa60       ?getDrawer@GCFramePlotFactory@U2@@UAEPAVGSequenceGraphDrawer@2@PAVGSequenceGraphView@2@@Z 1000ba60 f   GCFramePlot.obj
 0001:0000aba0       ?insert@?$QMap@VQString@@VQColor@@@@QAE?AViterator@1@ABVQString@@ABVQColor@@@Z 1000bba0 f i GCFramePlot.obj
 0001:0000ac60       ?isEnabled@GCFramePlotFactory@U2@@UBE_NPBVU2SequenceObject@2@@Z 1000bc60 f   GCFramePlot.obj
 0001:0000ac80       ?leftNode@?$QMapNode@VQString@@VQColor@@@@QBEPAU1@XZ 1000bc80 f i GCFramePlot.obj
 0001:0000ac90       ?rightNode@?$QMapNode@VQString@@VQColor@@@@QBEPAU1@XZ 1000bc90 f i GCFramePlot.obj
 0001:0000aca0       ?root@?$QMapData@VQString@@VQColor@@@@QBEPAU?$QMapNode@VQString@@VQColor@@@@XZ 1000bca0 f i GCFramePlot.obj
 0001:0000acb0       ?windowStrategyWithoutMemorize@GCFramePlotAlgorithm@U2@@AAEXAAV?$QVector@M@@ABVQByteArray@@HPBVGSequenceGraphWindowData@2@HAAVU2OpStatus@2@@Z 1000bcb0 f   GCFramePlot.obj
 0001:0000ae20       ??$qAbs@M@@YAMABM@Z        1000be20 f i KarlinSignatureDifferenceGraph.obj
 0001:0000ae50       ??0KarlinGraphAlgorithm@U2@@QAE@XZ 1000be50 f   KarlinSignatureDifferenceGraph.obj
 0001:0000aeb0       ??0KarlinGraphFactory@U2@@QAE@PAVQObject@@@Z 1000beb0 f   KarlinSignatureDifferenceGraph.obj
 0001:0000af30       ??1KarlinGraphAlgorithm@U2@@UAE@XZ 1000bf30 f   KarlinSignatureDifferenceGraph.obj
 0001:0000afa0       ??1KarlinGraphFactory@U2@@UAE@XZ 1000bfa0 f i KarlinSignatureDifferenceGraph.obj
 0001:0000afb0       ??_GKarlinGraphAlgorithm@U2@@UAEPAXI@Z 1000bfb0 f i KarlinSignatureDifferenceGraph.obj
 0001:0000afb0       ??_EKarlinGraphAlgorithm@U2@@UAEPAXI@Z 1000bfb0 f i KarlinSignatureDifferenceGraph.obj
 0001:0000b030       ??_EKarlinGraphFactory@U2@@UAEPAXI@Z 1000c030 f i KarlinSignatureDifferenceGraph.obj
 0001:0000b030       ??_GKarlinGraphFactory@U2@@UAEPAXI@Z 1000c030 f i KarlinSignatureDifferenceGraph.obj
 0001:0000b060       ?calculate@KarlinGraphAlgorithm@U2@@UAEXAAV?$QVector@M@@PAVU2SequenceObject@2@ABVU2Region@2@PBVGSequenceGraphWindowData@2@AAVU2OpStatus@2@@Z 1000c060 f   KarlinSignatureDifferenceGraph.obj
 0001:0000b260       ?calculateRelativeAbundance@KarlinGraphAlgorithm@U2@@AAEXPBDHPAMAAVU2OpStatus@2@@Z 1000c260 f   KarlinSignatureDifferenceGraph.obj
 0001:0000b680       ?createGraphs@KarlinGraphFactory@U2@@UAE?AV?$QList@V?$QSharedPointer@VGSequenceGraphData@U2@@@@@@PAVGSequenceGraphView@2@@Z 1000c680 f   KarlinSignatureDifferenceGraph.obj
 0001:0000b820       ?getValue@KarlinGraphAlgorithm@U2@@AAEMHHABVQByteArray@@AAVU2OpStatus@2@@Z 1000c820 f   KarlinSignatureDifferenceGraph.obj
 0001:0000b900       ?isEnabled@KarlinGraphFactory@U2@@UBE_NPBVU2SequenceObject@2@@Z 1000c900 f   KarlinSignatureDifferenceGraph.obj
 0001:0000b950       ?tr@KarlinGraphFactory@U2@@SA?AVQString@@PBD0H@Z 1000c950 f i KarlinSignatureDifferenceGraph.obj
 0001:0000b980       ??C?$QScopedPointer@VQObjectData@@U?$QScopedPointerDeleter@VQObjectData@@@@@@QBEPAVQObjectData@@XZ 1000c980 f i moc_BaseContentGraph.obj
 0001:0000b990       ?metaObject@BaseContentGraphFactory@U2@@UBEPBUQMetaObject@@XZ 1000c990 f   moc_BaseContentGraph.obj
 0001:0000b9b0       ?qt_metacall@BaseContentGraphFactory@U2@@UAEHW4Call@QMetaObject@@HPAPAX@Z 1000c9b0 f   moc_BaseContentGraph.obj
 0001:0000b9c0       ?qt_metacast@BaseContentGraphFactory@U2@@UAEPAXPBD@Z 1000c9c0 f   moc_BaseContentGraph.obj
 0001:0000ba20       ?qt_static_metacall@BaseContentGraphFactory@U2@@CAXPAVQObject@@W4Call@QMetaObject@@HPAPAX@Z 1000ca20 f   moc_BaseContentGraph.obj
 0001:0000ba30       ?metaObject@CumulativeSkewGraphFactory@U2@@UBEPBUQMetaObject@@XZ 1000ca30 f   moc_CumulativeSkew.obj
 0001:0000ba50       ?qt_metacall@CumulativeSkewGraphFactory@U2@@UAEHW4Call@QMetaObject@@HPAPAX@Z 1000ca50 f   moc_CumulativeSkew.obj
 0001:0000ba60       ?qt_metacast@CumulativeSkewGraphFactory@U2@@UAEPAXPBD@Z 1000ca60 f   moc_CumulativeSkew.obj
 0001:0000bac0       ?qt_static_metacall@CumulativeSkewGraphFactory@U2@@CAXPAVQObject@@W4Call@QMetaObject@@HPAPAX@Z 1000cac0 f   moc_CumulativeSkew.obj
 0001:0000bad0       ??$acquireMemoryFence@H@?$QGenericAtomicOps@U?$QAtomicOpsBySize@$03@@@@SAXABH@Z 1000cad0 f i moc_DNAGraphPackPlugin.obj
 0001:0000bae0       ??$loadAcquire@H@?$QGenericAtomicOps@U?$QAtomicOpsBySize@$03@@@@SAHABH@Z 1000cae0 f i moc_DNAGraphPackPlugin.obj
 0001:0000baf0       ??$orderedMemoryFence@H@?$QGenericAtomicOps@U?$QAtomicOpsBySize@$03@@@@SAXABH@Z 1000caf0 f i moc_DNAGraphPackPlugin.obj
 0001:0000bb00       ??$qMetaTypeId@PAVADVSequenceWidget@U2@@@@YAHXZ 1000cb00 f i moc_DNAGraphPackPlugin.obj
 0001:0000bb10       ??$qRegisterMetaType@PAVADVSequenceWidget@U2@@@@YAHXZ 1000cb10 f i moc_DNAGraphPackPlugin.obj
 0001:0000bb20       ??$qRegisterNormalizedMetaType@PAVADVSequenceWidget@U2@@@@YAHABVQByteArray@@PAPAVADVSequenceWidget@U2@@W4DefinedType@?$MetaTypeDefinedHelper@PAVADVSequenceWidget@U2@@$00@QtPrivate@@@Z 1000cb20 f i moc_DNAGraphPackPlugin.obj
 0001:0000bb80       ??$releaseMemoryFence@H@?$QGenericAtomicOps@U?$QAtomicOpsBySize@$03@@@@SAXABH@Z 1000cb80 f i moc_DNAGraphPackPlugin.obj
 0001:0000bb90       ??$storeRelease@HH@?$QGenericAtomicOps@U?$QAtomicOpsBySize@$03@@@@SAXAAHH@Z 1000cb90 f i moc_DNAGraphPackPlugin.obj
 0001:0000bba0       ??0?$QFlags@W4TypeFlag@QMetaType@@@@QAE@VQFlag@@@Z 1000cba0 f i moc_DNAGraphPackPlugin.obj
 0001:0000bbb0       ??0QFlag@@QAE@H@Z          1000cbb0 f i moc_DNAGraphPackPlugin.obj
 0001:0000bbc0       ??BQFlag@@QBEHXZ           1000cbc0 f i moc_DNAGraphPackPlugin.obj
 0001:0000bbd0       ??_5?$QFlags@W4TypeFlag@QMetaType@@@@QAEAAV0@W4TypeFlag@QMetaType@@@Z 1000cbd0 f i moc_DNAGraphPackPlugin.obj
 0001:0000bbe0       ?Construct@?$QMetaTypeFunctionHelper@PAVADVSequenceWidget@U2@@$00@QtMetaTypePrivate@@SAPAXPAXPBX@Z 1000cbe0 f i moc_DNAGraphPackPlugin.obj
 0001:0000bc10       ?Create@?$QMetaTypeFunctionHelper@PAVADVSequenceWidget@U2@@$00@QtMetaTypePrivate@@SAPAXPBX@Z 1000cc10 f i moc_DNAGraphPackPlugin.obj
 0001:0000bc50       ?Delete@?$QMetaTypeFunctionHelper@PAVADVSequenceWidget@U2@@$00@QtMetaTypePrivate@@SAXPAX@Z 1000cc50 f i moc_DNAGraphPackPlugin.obj
 0001:0000bc60       ?Destruct@?$QMetaTypeFunctionHelper@PAVADVSequenceWidget@U2@@$00@QtMetaTypePrivate@@SAXPAX@Z 1000cc60 f i moc_DNAGraphPackPlugin.obj
 0001:0000bc70       ?loadAcquire@?$QBasicAtomicInteger@H@@QBEHXZ 1000cc70 f i moc_DNAGraphPackPlugin.obj
 0001:0000bc80       ?metaObject@DNAGraphPackPlugin@U2@@UBEPBUQMetaObject@@XZ 1000cc80 f   moc_DNAGraphPackPlugin.obj
 0001:0000bca0       ?metaObject@DNAGraphPackViewContext@U2@@UBEPBUQMetaObject@@XZ 1000cca0 f   moc_DNAGraphPackPlugin.obj
 0001:0000bcc0       ?qt_metacall@DNAGraphPackPlugin@U2@@UAEHW4Call@QMetaObject@@HPAPAX@Z 1000ccc0 f   moc_DNAGraphPackPlugin.obj
 0001:0000bcd0       ?qt_metacall@DNAGraphPackViewContext@U2@@UAEHW4Call@QMetaObject@@HPAPAX@Z 1000ccd0 f   moc_DNAGraphPackPlugin.obj
 0001:0000bd30       ?qt_metacast@DNAGraphPackPlugin@U2@@UAEPAXPBD@Z 1000cd30 f   moc_DNAGraphPackPlugin.obj
 0001:0000bd90       ?qt_metacast@DNAGraphPackViewContext@U2@@UAEPAXPBD@Z 1000cd90 f   moc_DNAGraphPackPlugin.obj
 0001:0000bdf0       ?qt_metatype_id@?$QMetaTypeId2@PAVADVSequenceWidget@U2@@@@SAHXZ 1000cdf0 f i moc_DNAGraphPackPlugin.obj
 0001:0000be00       ?qt_metatype_id@?$QMetaTypeIdHelper@PAVADVSequenceWidget@U2@@$00@QtPrivate@@SAHXZ 1000ce00 f i moc_DNAGraphPackPlugin.obj
 0001:0000be10       ?qt_metatype_id@?$QMetaTypeIdQObject@PAVADVSequenceWidget@U2@@$00@@SAHXZ 1000ce10 f i moc_DNAGraphPackPlugin.obj
 0001:0000bef0       ?qt_static_metacall@DNAGraphPackPlugin@U2@@CAXPAVQObject@@W4Call@QMetaObject@@HPAPAX@Z 1000cef0 f   moc_DNAGraphPackPlugin.obj
 0001:0000bf00       ?qt_static_metacall@DNAGraphPackViewContext@U2@@CAXPAVQObject@@W4Call@QMetaObject@@HPAPAX@Z 1000cf00 f   moc_DNAGraphPackPlugin.obj
 0001:0000bf60       ?registerConverter@?$AssociativeContainerConverterHelper@PAVADVSequenceWidget@U2@@$0A@@QtPrivate@@SA_NH@Z 1000cf60 f i moc_DNAGraphPackPlugin.obj
 0001:0000bf70       ?registerConverter@?$IsPair@PAVADVSequenceWidget@U2@@@QtPrivate@@SA_NH@Z 1000cf70 f i moc_DNAGraphPackPlugin.obj
 0001:0000bf80       ?registerConverter@?$MetaTypeSmartPointerHelper@PAVADVSequenceWidget@U2@@X@QtPrivate@@SA_NH@Z 1000cf80 f i moc_DNAGraphPackPlugin.obj
 0001:0000bf90       ?registerConverter@?$SequentialContainerConverterHelper@PAVADVSequenceWidget@U2@@$0A@@QtPrivate@@SA_NH@Z 1000cf90 f i moc_DNAGraphPackPlugin.obj
 0001:0000bfa0       ?storeRelease@?$QBasicAtomicInteger@H@@QAEXH@Z 1000cfa0 f i moc_DNAGraphPackPlugin.obj
 0001:0000bfb0       ?value@?$MetaObjectForType@PAVADVSequenceWidget@U2@@$00@QtPrivate@@SAPBUQMetaObject@@XZ 1000cfb0 f i moc_DNAGraphPackPlugin.obj
 0001:0000bfc0       ?metaObject@DeviationGraphFactory@U2@@UBEPBUQMetaObject@@XZ 1000cfc0 f   moc_DeviationGraph.obj
 0001:0000bfe0       ?qt_metacall@DeviationGraphFactory@U2@@UAEHW4Call@QMetaObject@@HPAPAX@Z 1000cfe0 f   moc_DeviationGraph.obj
 0001:0000bff0       ?qt_metacast@DeviationGraphFactory@U2@@UAEPAXPBD@Z 1000cff0 f   moc_DeviationGraph.obj
 0001:0000c050       ?qt_static_metacall@DeviationGraphFactory@U2@@CAXPAVQObject@@W4Call@QMetaObject@@HPAPAX@Z 1000d050 f   moc_DeviationGraph.obj
 0001:0000c060       ?metaObject@EntropyGraphFactory@U2@@UBEPBUQMetaObject@@XZ 1000d060 f   moc_EntropyAlgorithm.obj
 0001:0000c080       ?qt_metacall@EntropyGraphFactory@U2@@UAEHW4Call@QMetaObject@@HPAPAX@Z 1000d080 f   moc_EntropyAlgorithm.obj
 0001:0000c090       ?qt_metacast@EntropyGraphFactory@U2@@UAEPAXPBD@Z 1000d090 f   moc_EntropyAlgorithm.obj
 0001:0000c0f0       ?qt_static_metacall@EntropyGraphFactory@U2@@CAXPAVQObject@@W4Call@QMetaObject@@HPAPAX@Z 1000d0f0 f   moc_EntropyAlgorithm.obj
 0001:0000c100       ?metaObject@GCFramePlotFactory@U2@@UBEPBUQMetaObject@@XZ 1000d100 f   moc_GCFramePlot.obj
 0001:0000c120       ?qt_metacall@GCFramePlotFactory@U2@@UAEHW4Call@QMetaObject@@HPAPAX@Z 1000d120 f   moc_GCFramePlot.obj
 0001:0000c130       ?qt_metacast@GCFramePlotFactory@U2@@UAEPAXPBD@Z 1000d130 f   moc_GCFramePlot.obj
 0001:0000c190       ?qt_static_metacall@GCFramePlotFactory@U2@@CAXPAVQObject@@W4Call@QMetaObject@@HPAPAX@Z 1000d190 f   moc_GCFramePlot.obj
 0001:0000c1a0       ?metaObject@KarlinGraphFactory@U2@@UBEPBUQMetaObject@@XZ 1000d1a0 f   moc_KarlinSignatureDifferenceGraph.obj
 0001:0000c1c0       ?qt_metacall@KarlinGraphFactory@U2@@UAEHW4Call@QMetaObject@@HPAPAX@Z 1000d1c0 f   moc_KarlinSignatureDifferenceGraph.obj
 0001:0000c1d0       ?qt_metacast@KarlinGraphFactory@U2@@UAEPAXPBD@Z 1000d1d0 f   moc_KarlinSignatureDifferenceGraph.obj
 0001:0000c230       ?qt_static_metacall@KarlinGraphFactory@U2@@CAXPAVQObject@@W4Call@QMetaObject@@HPAPAX@Z 1000d230 f   moc_KarlinSignatureDifferenceGraph.obj
 0001:0000c240       ??0initializer@?A0x701b237d@@QAE@XZ 1000d240 f i qrc_dna_graphpack.obj
 0001:0000c260       ??1initializer@?A0x701b237d@@QAE@XZ 1000d260 f i qrc_dna_graphpack.obj
 0001:0000c280       ?qCleanupResources_dna_graphpack@@YAHXZ 1000d280 f   qrc_dna_graphpack.obj
 0001:0000c2a0       ?qInitResources_dna_graphpack@@YAHXZ 1000d2a0 f   qrc_dna_graphpack.obj
 0001:0000c2c0       ?getAlphabet@U2SequenceObject@U2@@QBEPBVDNAAlphabet@2@XZ 1000d2c0 f   U2Core:U2Core.dll
 0001:0000c2c6       ?nullPointerError@L10N@U2@@SA?AVQString@@ABV3@@Z 1000d2c6 f   U2Core:U2Core.dll
 0001:0000c2cc       ??0Logger@U2@@QAE@ABVQString@@@Z 1000d2cc f   U2Core:U2Core.dll
 0001:0000c2d2       ??1Logger@U2@@UAE@XZ       1000d2d2 f   U2Core:U2Core.dll
 0001:0000c2d8       ?error@Logger@U2@@QAEXABVQString@@@Z 1000d2d8 f   U2Core:U2Core.dll
 0001:0000c2de       ??0Plugin@U2@@QAE@ABVQString@@0_NW4PluginState@1@@Z 1000d2de f   U2Core:U2Core.dll
 0001:0000c2e4       ??1Plugin@U2@@UAE@XZ       1000d2e4 f   U2Core:U2Core.dll
 0001:0000c2ea       ?getMainWindow@AppContext@U2@@SAPAVMainWindow@2@XZ 1000d2ea f   U2Core:U2Core.dll
 0001:0000c2f0       ?isRNA@DNAAlphabet@U2@@QBE_NXZ 1000d2f0 f   U2Core:U2Core.dll
 0001:0000c2f6       ?getAlphabetChars@DNAAlphabet@U2@@QBE?AVQByteArray@@_N@Z 1000d2f6 f   U2Core:U2Core.dll
 0001:0000c2fc       ??0Index3To1@U2@@QAE@XZ    1000d2fc f   U2Core:U2Core.dll
 0001:0000c302       ?init@Index3To1@U2@@QAEXABVQByteArray@@@Z 1000d302 f   U2Core:U2Core.dll
 0001:0000c308       ?indexOf@Index3To1@U2@@QBEHPBD@Z 1000d308 f   U2Core:U2Core.dll
 0001:0000c30e       ?indexOf@Index3To1@U2@@QBEHDDD@Z 1000d30e f   U2Core:U2Core.dll
 0001:0000c314       ?getDNATranslationRegistry@AppContext@U2@@SAPAVDNATranslationRegistry@2@XZ 1000d314 f   U2Core:U2Core.dll
 0001:0000c31a       ?lookupComplementTranslation@DNATranslationRegistry@U2@@QAEPAVDNATranslation@2@PBVDNAAlphabet@2@@Z 1000d31a f   U2Core:U2Core.dll
 0001:0000c320       ?qt_metacast@Plugin@U2@@UAEPAXPBD@Z 1000d320 f   U2Core:U2Core.dll
 0001:0000c326       ?qt_metacall@Plugin@U2@@UAEHW4Call@QMetaObject@@HPAPAX@Z 1000d326 f   U2Core:U2Core.dll
 0001:0000c32c       ??0GObjectViewWindowContext@U2@@QAE@PAVQObject@@ABVGObjectViewFactoryId@1@@Z 1000d32c f   U2Gui:U2Gui.dll
 0001:0000c332       ??1GObjectViewWindowContext@U2@@UAE@XZ 1000d332 f   U2Gui:U2Gui.dll
 0001:0000c338       ?buildMenu@GObjectViewWindowContext@U2@@MAEXPAVGObjectView@2@PAVQMenu@@@Z 1000d338 f   U2Gui:U2Gui.dll
 0001:0000c33e       ?canHandle@GObjectViewObjectHandler@U2@@UAE_NPAVGObjectView@2@PAVGObject@2@@Z 1000d33e f   U2Gui:U2Gui.dll
 0001:0000c344       ?disconnectView@GObjectViewWindowContext@U2@@MAEXPAVGObjectView@2@@Z 1000d344 f   U2Gui:U2Gui.dll
 0001:0000c34a       ?init@GObjectViewWindowContext@U2@@UAEXXZ 1000d34a f   U2Gui:U2Gui.dll
 0001:0000c350       ?onObjectAdded@GObjectViewObjectHandler@U2@@UAEXPAVGObjectView@2@PAVGObject@2@@Z 1000d350 f   U2Gui:U2Gui.dll
 0001:0000c356       ?onObjectRemoved@GObjectViewWindowContext@U2@@UAEXPAVGObjectView@2@PAVGObject@2@@Z 1000d356 f   U2Gui:U2Gui.dll
 0001:0000c35c       ?sl_buildContextMenu@GObjectViewWindowContext@U2@@MAEXPAVGObjectView@2@PAVQMenu@@@Z 1000d35c f   U2Gui:U2Gui.dll
 0001:0000c362       ?sl_buildStaticMenu@GObjectViewWindowContext@U2@@MAEXPAVGObjectView@2@PAVQMenu@@@Z 1000d362 f   U2Gui:U2Gui.dll
 0001:0000c368       ?sl_windowAdded@GObjectViewWindowContext@U2@@MAEXPAVMWMDIWindow@2@@Z 1000d368 f   U2Gui:U2Gui.dll
 0001:0000c36e       ?sl_windowClosing@GObjectViewWindowContext@U2@@MAEXPAVMWMDIWindow@2@@Z 1000d36e f   U2Gui:U2Gui.dll
 0001:0000c374       ?qt_metacast@GObjectViewWindowContext@U2@@UAEPAXPBD@Z 1000d374 f   U2Gui:U2Gui.dll
 0001:0000c37a       ?qt_metacall@GObjectViewWindowContext@U2@@UAEHW4Call@QMetaObject@@HPAPAX@Z 1000d37a f   U2Gui:U2Gui.dll
 0001:0000c380       ??1GSequenceGraphAlgorithm@U2@@UAE@XZ 1000d380 f   U2View:U2View.dll
 0001:0000c386       ??0GSequenceGraphAlgorithm@U2@@IAE@XZ 1000d386 f   U2View:U2View.dll
 0001:0000c38c       ?getSequenceData@GSequenceGraphAlgorithm@U2@@IAEABVQByteArray@@PAVU2SequenceObject@2@AAVU2OpStatus@2@@Z 1000d38c f   U2View:U2View.dll
 0001:0000c392       ??0GSequenceGraphData@U2@@QAE@ABVQString@@@Z 1000d392 f   U2View:U2View.dll
 0001:0000c398       ??1GSequenceGraphData@U2@@UAE@XZ 1000d398 f   U2View:U2View.dll
 0001:0000c39e       ?getNumSteps@GSequenceGraphUtils@U2@@SAHABVU2Region@2@HH@Z 1000d39e f   U2View:U2View.dll
 0001:0000c3a4       ??0GSequenceGraphFactory@U2@@QAE@ABVQString@@PAVQObject@@@Z 1000d3a4 f   U2View:U2View.dll
 0001:0000c3aa       ??1GSequenceGraphFactory@U2@@UAE@XZ 1000d3aa f   U2View:U2View.dll
 0001:0000c3b0       ?getDrawer@GSequenceGraphFactory@U2@@UAEPAVGSequenceGraphDrawer@2@PAVGSequenceGraphView@2@@Z 1000d3b0 f   U2View:U2View.dll
 0001:0000c3b6       ?getSequenceObject@ADVSingleSequenceWidget@U2@@QBEPAVU2SequenceObject@2@XZ 1000d3b6 f   U2View:U2View.dll
 0001:0000c3bc       ??0GraphAction@U2@@QAE@PAVGSequenceGraphFactory@1@@Z 1000d3bc f   U2View:U2View.dll
 0001:0000c3c2       ??1GraphAction@U2@@UAE@XZ  1000d3c2 f   U2View:U2View.dll
 0001:0000c3c8       ?addGraphAction@GraphMenuAction@U2@@SAXPAVADVSequenceObjectContext@2@PAVGraphAction@2@@Z 1000d3c8 f   U2View:U2View.dll
 0001:0000c3ce       ?getSequenceWidgets@AnnotatedDNAView@U2@@QBE?BV?$QList@PAVADVSequenceWidget@U2@@@@XZ 1000d3ce f   U2View:U2View.dll
 0001:0000c3d4       ?metaObject@GraphAction@U2@@UBEPBUQMetaObject@@XZ 1000d3d4 f   U2View:U2View.dll
 0001:0000c3da       ?qt_metacall@GraphAction@U2@@UAEHW4Call@QMetaObject@@HPAPAX@Z 1000d3da f   U2View:U2View.dll
 0001:0000c3e0       ?qt_metacast@GraphAction@U2@@UAEPAXPBD@Z 1000d3e0 f   U2View:U2View.dll
 0001:0000c3e6       ?setColors@GSequenceGraphDrawer@U2@@QAEXABV?$QMap@VQString@@VQColor@@@@@Z 1000d3e6 f   U2View:U2View.dll
 0001:0000c3ec       ?setEnabled@QAction@@QAEX_N@Z 1000d3ec f   Qt5Widgets:Qt5Widgets.dll
 0001:0000c3f2       ?event@QAction@@MAE_NPAVQEvent@@@Z 1000d3f2 f   Qt5Widgets:Qt5Widgets.dll
 0001:0000c3f8       ??0QColor@@QAE@W4GlobalColor@Qt@@@Z 1000d3f8 f   Qt5Gui:Qt5Gui.dll
 0001:0000c3fe       ??4QColor@@QAEAAV0@ABV0@@Z 1000d3fe f   Qt5Gui:Qt5Gui.dll
 0001:0000c404       ?qBadAlloc@@YAXXZ          1000d404 f   Qt5Core:Qt5Core.dll
 0001:0000c40a       ?data@QArrayData@@QAEPAXXZ 1000d40a f   Qt5Core:Qt5Core.dll
 0001:0000c410       ?allocate@QArrayData@@SAPAU1@IIIV?$QFlags@W4AllocationOption@QArrayData@@@@@Z 1000d410 f   Qt5Core:Qt5Core.dll
 0001:0000c416       ?deallocate@QArrayData@@SAXPAU1@II@Z 1000d416 f   Qt5Core:Qt5Core.dll
 0001:0000c41c       ?detach_grow@QListData@@QAEPAUData@1@PAHH@Z 1000d41c f   Qt5Core:Qt5Core.dll
 0001:0000c422       ?dispose@QListData@@SAXPAUData@1@@Z 1000d422 f   Qt5Core:Qt5Core.dll
 0001:0000c428       ?append@QListData@@QAEPAPAXXZ 1000d428 f   Qt5Core:Qt5Core.dll
 0001:0000c42e       ??AQByteArray@@QBEDH@Z     1000d42e f   Qt5Core:Qt5Core.dll
 0001:0000c434       ?tr@QMetaObject@@QBE?AVQString@@PBD0H@Z 1000d434 f   Qt5Core:Qt5Core.dll
 0001:0000c43a       ??0QChar@@QAE@UQLatin1Char@@@Z 1000d43a f   Qt5Core:Qt5Core.dll
 0001:0000c440       ??1QString@@QAE@XZ         1000d440 f   Qt5Core:Qt5Core.dll
 0001:0000c446       ?arg@QString@@QBE?AV1@HHHVQChar@@@Z 1000d446 f   Qt5Core:Qt5Core.dll
 0001:0000c44c       ?arg@QString@@QBE?AV1@ABV1@HVQChar@@@Z 1000d44c f   Qt5Core:Qt5Core.dll
 0001:0000c452       ?fromAscii_helper@QString@@CAPAU?$QTypedArrayData@G@@PBDH@Z 1000d452 f   Qt5Core:Qt5Core.dll
 0001:0000c458       ??0QBitArray@@QAE@H_N@Z    1000d458 f   Qt5Core:Qt5Core.dll
 0001:0000c45e       ??0QBitArray@@QAE@ABV0@@Z  1000d45e f   Qt5Core:Qt5Core.dll
 0001:0000c464       ??AQBitArray@@QAE?AVQBitRef@@H@Z 1000d464 f   Qt5Core:Qt5Core.dll
 0001:0000c46a       ??1QBitArray@@QAE@XZ       1000d46a f   Qt5Core:Qt5Core.dll
 0001:0000c470       ??BQBitRef@@QBE_NXZ        1000d470 f   Qt5Core:Qt5Core.dll
 0001:0000c476       ??4QBitRef@@QAEAAV0@ABV0@@Z 1000d476 f   Qt5Core:Qt5Core.dll
 0001:0000c47c       ??4QBitRef@@QAEAAV0@_N@Z   1000d47c f   Qt5Core:Qt5Core.dll
 0001:0000c482       ?childEvent@QObject@@MAEXPAVQChildEvent@@@Z 1000d482 f   Qt5Core:Qt5Core.dll
 0001:0000c488       ?connectNotify@QObject@@MAEXABVQMetaMethod@@@Z 1000d488 f   Qt5Core:Qt5Core.dll
 0001:0000c48e       ?customEvent@QObject@@MAEXPAVQEvent@@@Z 1000d48e f   Qt5Core:Qt5Core.dll
 0001:0000c494       ?disconnectNotify@QObject@@MAEXABVQMetaMethod@@@Z 1000d494 f   Qt5Core:Qt5Core.dll
 0001:0000c49a       ?event@QObject@@UAE_NPAVQEvent@@@Z 1000d49a f   Qt5Core:Qt5Core.dll
 0001:0000c4a0       ?eventFilter@QObject@@UAE_NPAV1@PAVQEvent@@@Z 1000d4a0 f   Qt5Core:Qt5Core.dll
 0001:0000c4a6       ?timerEvent@QObject@@MAEXPAVQTimerEvent@@@Z 1000d4a6 f   Qt5Core:Qt5Core.dll
 0001:0000c4ac       ?detach@QListData@@QAEPAUData@1@H@Z 1000d4ac f   Qt5Core:Qt5Core.dll
 0001:0000c4b2       ?cast@QMetaObject@@QBEPAVQObject@@PAV2@@Z 1000d4b2 f   Qt5Core:Qt5Core.dll
 0001:0000c4b8       ??1Connection@QMetaObject@@QAE@XZ 1000d4b8 f   Qt5Core:Qt5Core.dll
 0001:0000c4be       ?connect@QObject@@SA?AVConnection@QMetaObject@@PBV1@PBD01W4ConnectionType@Qt@@@Z 1000d4be f   Qt5Core:Qt5Core.dll
 0001:0000c4c4       ?connect@QObject@@QBE?AVConnection@QMetaObject@@PBV1@PBD1W4ConnectionType@Qt@@@Z 1000d4c4 f   Qt5Core:Qt5Core.dll
 0001:0000c4ca       ?constData@QByteArray@@QBEPBDXZ 1000d4ca f   Qt5Core:Qt5Core.dll
 0001:0000c4d0       ??1QByteArray@@QAE@XZ      1000d4d0 f   Qt5Core:Qt5Core.dll
 0001:0000c4d6       ??0QString@@QAE@ABV0@@Z    1000d4d6 f   Qt5Core:Qt5Core.dll
 0001:0000c4dc       ??M@YA_NABVQString@@0@Z    1000d4dc f   Qt5Core:Qt5Core.dll
 0001:0000c4e2       ?freeNodeAndRebalance@QMapDataBase@@QAEXPAUQMapNodeBase@@@Z 1000d4e2 f   Qt5Core:Qt5Core.dll
 0001:0000c4e8       ?recalcMostLeftNode@QMapDataBase@@QAEXXZ 1000d4e8 f   Qt5Core:Qt5Core.dll
 0001:0000c4ee       ?createNode@QMapDataBase@@QAEPAUQMapNodeBase@@HHPAU2@_N@Z 1000d4ee f   Qt5Core:Qt5Core.dll
 0001:0000c4f4       ?freeTree@QMapDataBase@@QAEXPAUQMapNodeBase@@H@Z 1000d4f4 f   Qt5Core:Qt5Core.dll
 0001:0000c4fa       ?createData@QMapDataBase@@SAPAU1@XZ 1000d4fa f   Qt5Core:Qt5Core.dll
 0001:0000c500       ?freeData@QMapDataBase@@SAXPAU1@@Z 1000d500 f   Qt5Core:Qt5Core.dll
 0001:0000c506       ??0QByteArray@@QAE@XZ      1000d506 f   Qt5Core:Qt5Core.dll
 0001:0000c50c       ??4QByteArray@@QAEAAV0@$$QAV0@@Z 1000d50c f   Qt5Core:Qt5Core.dll
 0001:0000c512       ?resize@QByteArray@@QAEXH@Z 1000d512 f   Qt5Core:Qt5Core.dll
 0001:0000c518       ?at@QByteArray@@QBEDH@Z    1000d518 f   Qt5Core:Qt5Core.dll
 0001:0000c51e       ?dynamicMetaObject@QObjectData@@QBEPAUQMetaObject@@XZ 1000d51e f   Qt5Core:Qt5Core.dll
 0001:0000c524       ?qt_metacast@QObject@@UAEPAXPBD@Z 1000d524 f   Qt5Core:Qt5Core.dll
 0001:0000c52a       ?qt_metacall@QObject@@UAEHW4Call@QMetaObject@@HPAPAX@Z 1000d52a f   Qt5Core:Qt5Core.dll
 0001:0000c530       ?reserve@QByteArray@@QAEXH@Z 1000d530 f   Qt5Core:Qt5Core.dll
 0001:0000c536       ?append@QByteArray@@QAEAAV1@D@Z 1000d536 f   Qt5Core:Qt5Core.dll
 0001:0000c53c       ?append@QByteArray@@QAEAAV1@PBD@Z 1000d53c f   Qt5Core:Qt5Core.dll
 0001:0000c542       ?className@QMetaObject@@QBEPBDXZ 1000d542 f   Qt5Core:Qt5Core.dll
 0001:0000c548       ?registerNormalizedType@QMetaType@@SAHABVQByteArray@@P6AXPAX@ZP6APAXPBX@Z2P6APAX13@ZHV?$QFlags@W4TypeFlag@QMetaType@@@@PBUQMetaObject@@@Z 1000d548 f   Qt5Core:Qt5Core.dll
 0001:0000c54e       ?registerNormalizedTypedef@QMetaType@@SAHABVQByteArray@@H@Z 1000d54e f   Qt5Core:Qt5Core.dll
 0001:0000c554       ?qRegisterResourceData@@YA_NHPBE00@Z 1000d554 f   Qt5Core:Qt5Core.dll
 0001:0000c55a       ?qUnregisterResourceData@@YA_NHPBE00@Z 1000d55a f   Qt5Core:Qt5Core.dll
 0001:0000c560       ?_Xbad_alloc@std@@YAXXZ    1000d560 f   msvcprt:MSVCP120.dll
 0001:0000c566       ?_Xlength_error@std@@YAXPBD@Z 1000d566 f   msvcprt:MSVCP120.dll
 0001:0000c56c       ?_Xout_of_range@std@@YAXPBD@Z 1000d56c f   msvcprt:MSVCP120.dll
 0001:0000c572       ?_Syserror_map@std@@YAPBDH@Z 1000d572 f   msvcprt:MSVCP120.dll
 0001:0000c578       ?_Winerror_map@std@@YAPBDH@Z 1000d578 f   msvcprt:MSVCP120.dll
 0001:0000c57e       ??_U@YAPAXI@Z              1000d57e f   msvcprt:newaop_s.obj
 0001:0000c588       __purecall                 1000d588 f   MSVCRT:MSVCR120.dll
 0001:0000c58e       ??2@YAPAXI@Z               1000d58e f   MSVCRT:MSVCR120.dll
 0001:0000c594       ??3@YAXPAX@Z               1000d594 f   MSVCRT:MSVCR120.dll
 0001:0000c59a       ___atonexitinit            1000d59a f   MSVCRT:atonexit.obj
 0001:0000c5d6       __onexit                   1000d5d6 f   MSVCRT:atonexit.obj
 0001:0000c67f       _atexit                    1000d67f f   MSVCRT:atonexit.obj
 0001:0000c694       _memmove                   1000d694 f   MSVCRT:MSVCR120.dll
 0001:0000c69a       __hypot                    1000d69a f   MSVCRT:MSVCR120.dll
 0001:0000c6a0       @__security_check_cookie@4 1000d6a0 f   MSVCRT:secchk.obj
 0001:0000c6b0       __CxxThrowException@8      1000d6b0 f   MSVCRT:MSVCR120.dll
 0001:0000c6b6       ___CxxFrameHandler3        1000d6b6 f   MSVCRT:MSVCR120.dll
 0001:0000c6c0       __ftoui3                   1000d6c0 f   MSVCRT:ftol3.obj
 0001:0000c6cf       __ftoul3                   1000d6cf f   MSVCRT:ftol3.obj
 0001:0000c6de       __ftol3                    1000d6de f   MSVCRT:ftol3.obj
 0001:0000c6eb       __ftol3_NaN                1000d6eb f   MSVCRT:ftol3.obj
 0001:0000c703       __ftol3_work               1000d703 f   MSVCRT:ftol3.obj
 0001:0000c789       __ftol3_common             1000d789 f   MSVCRT:ftol3.obj
 0001:0000c84b       __ftol3_arg_error          1000d84b f   MSVCRT:ftol3.obj
 0001:0000c85d       __ftol3_except             1000d85d f   MSVCRT:ftol3.obj
 0001:0000c8a1       __dtoui3                   1000d8a1 f   MSVCRT:ftol3.obj
 0001:0000c8b0       __dtoul3                   1000d8b0 f   MSVCRT:ftol3.obj
 0001:0000c8bf       __dtol3                    1000d8bf f   MSVCRT:ftol3.obj
 0001:0000c8cc       __dtol3_NaN                1000d8cc f   MSVCRT:ftol3.obj
 0001:0000c8e9       __dtol3_work               1000d8e9 f   MSVCRT:ftol3.obj
 0001:0000c9ce       __ultod3                   1000d9ce f   MSVCRT:ftol3.obj
 0001:0000ca5f       __ltod3                    1000da5f f   MSVCRT:ftol3.obj
 0001:0000ca8e       _memcpy                    1000da8e f   MSVCRT:MSVCR120.dll
 0001:0000ca94       _memset                    1000da94 f   MSVCRT:MSVCR120.dll
 0001:0000ca9a       ??0type_info@@AAE@ABV0@@Z  1000da9a f   MSVCRT:ti_inst.obj
 0001:0000caa5       ??4type_info@@AAEAAV0@ABV0@@Z 1000daa5 f   MSVCRT:ti_inst.obj
 0001:0000caaa       ??_Etype_info@@UAEPAXI@Z   1000daaa f i MSVCRT:ti_inst.obj
 0001:0000cb00       __alldiv                   1000db00 f   MSVCRT:lldiv.obj
 0001:0000cbb0       __allrem                   1000dbb0 f   MSVCRT:llrem.obj
 0001:0000cc62       ??_V@YAXPAX@Z              1000dc62 f   MSVCRT:MSVCR120.dll
 0001:0000cc68       __libm_sse2_log10_precise  1000dc68 f   MSVCRT:MSVCR120.dll
 0001:0000ccba       _NtCurrentTeb              1000dcba f i MSVCRT:crtdll.obj
 0001:0000ccc1       __CRT_INIT@12              1000dcc1 f   MSVCRT:crtdll.obj
 0001:0000ceb8       __DllMainCRTStartup@12     1000deb8 f   MSVCRT:crtdll.obj
 0001:0000d00e       __lock                     1000e00e f   MSVCRT:MSVCR120.dll
 0001:0000d014       __unlock                   1000e014 f   MSVCRT:MSVCR120.dll
 0001:0000d01a       __calloc_crt               1000e01a f   MSVCRT:MSVCR120.dll
 0001:0000d020       ___dllonexit               1000e020 f   MSVCRT:MSVCR120.dll
 0001:0000d030       __SEH_prolog4              1000e030 f   MSVCRT:sehprolg4.obj
 0001:0000d075       __SEH_epilog4              1000e075 f   MSVCRT:sehprolg4.obj
 0001:0000d089       __except_handler4          1000e089 f   MSVCRT:chandler4gs.obj
 0001:0000d0ac       ___raise_securityfailure   1000e0ac f   MSVCRT:gs_report.obj
 0001:0000d0e9       ___report_gsfailure        1000e0e9 f   MSVCRT:gs_report.obj
 0001:0000d1e4       ___report_rangecheckfailure 1000e1e4 f   MSVCRT:gs_report.obj
 0001:0000d1f0       ___report_securityfailure  1000e1f0 f   MSVCRT:gs_report.obj
 0001:0000d2c0       ___report_securityfailureEx 1000e2c0 f   MSVCRT:gs_report.obj
 0001:0000d3d6       __except1                  1000e3d6 f   MSVCRT:MSVCR120.dll
 0001:0000d3dc       ??_M@YGXPAXIHP6EX0@Z@Z     1000e3dc f   MSVCRT:ehvecdtr.obj
 0001:0000d464       ?__ArrayUnwind@@YGXPAXIHP6EX0@Z@Z 1000e464 f   MSVCRT:ehvecdtr.obj
 0001:0000d4c2       ??1type_info@@UAE@XZ       1000e4c2 f   MSVCRT:MSVCR120.dll
 0001:0000d4c8       ___CppXcptFilter           1000e4c8 f   MSVCRT:MSVCR120.dll
 0001:0000d4ce       __amsg_exit                1000e4ce f   MSVCRT:MSVCR120.dll
 0001:0000d4e0       __FindPESection            1000e4e0 f   MSVCRT:pesect.obj
 0001:0000d530       __IsNonwritableInCurrentImage 1000e530 f   MSVCRT:pesect.obj
 0001:0000d5f0       __ValidateImageBase        1000e5f0 f   MSVCRT:pesect.obj
 0001:0000d622       _free                      1000e622 f   MSVCRT:MSVCR120.dll
 0001:0000d628       ___security_init_cookie    1000e628 f   MSVCRT:gs_support.obj
 0001:0000d6c4       _DllMain@12                1000e6c4 f   MSVCRT:dllmain.obj
 0001:0000d6e6       __malloc_crt               1000e6e6 f   MSVCRT:MSVCR120.dll
 0001:0000d6ec       __RTC_Initialize           1000e6ec f   MSVCRT:initsect.obj
 0001:0000d70c       __RTC_Terminate            1000e70c f   MSVCRT:initsect.obj
 0001:0000d72c       __initterm                 1000e72c f   MSVCRT:MSVCR120.dll
 0001:0000d732       __initterm_e               1000e732 f   MSVCRT:MSVCR120.dll
 0001:0000d738       ___clean_type_info_names   1000e738 f   MSVCRT:tncleanup.obj
 0001:0000d744       __except_handler4_common   1000e744 f   MSVCRT:MSVCR120.dll
 0001:0000d74a       __crt_debugger_hook        1000e74a f   MSVCRT:MSVCR120.dll
 0001:0000d750       ___crtUnhandledException   1000e750 f   MSVCRT:MSVCR120.dll
 0001:0000d756       ___crtTerminateProcess     1000e756 f   MSVCRT:MSVCR120.dll
 0001:0000d75c       ?terminate@@YAXXZ          1000e75c f   MSVCRT:MSVCR120.dll
 0001:0000d762       ___clean_type_info_names_internal 1000e762 f   MSVCRT:MSVCR120.dll
 0001:0000d768       _EncodePointer@4           1000e768 f   kernel32:KERNEL32.dll
 0001:0000d76e       _DecodePointer@4           1000e76e f   kernel32:KERNEL32.dll
 0001:0000d774       _IsDebuggerPresent@0       1000e774 f   kernel32:KERNEL32.dll
 0001:0000d77a       _IsProcessorFeaturePresent@4 1000e77a f   kernel32:KERNEL32.dll
 0001:0000d780       _QueryPerformanceCounter@4 1000e780 f   kernel32:KERNEL32.dll
 0001:0000d786       _GetCurrentProcessId@0     1000e786 f   kernel32:KERNEL32.dll
 0001:0000d78c       _GetCurrentThreadId@0      1000e78c f   kernel32:KERNEL32.dll
 0001:0000d792       _GetSystemTimeAsFileTime@4 1000e792 f   kernel32:KERNEL32.dll
 0001:0000d798       _DisableThreadLibraryCalls@4 1000e798 f   kernel32:KERNEL32.dll
 0002:00000000       __imp__DisableThreadLibraryCalls@4 10013000     kernel32:KERNEL32.dll
 0002:00000004       __imp__GetSystemTimeAsFileTime@4 10013004     kernel32:KERNEL32.dll
 0002:00000008       __imp__GetCurrentThreadId@0 10013008     kernel32:KERNEL32.dll
 0002:0000000c       __imp__GetCurrentProcessId@0 1001300c     kernel32:KERNEL32.dll
 0002:00000010       __imp__QueryPerformanceCounter@4 10013010     kernel32:KERNEL32.dll
 0002:00000014       __imp__IsProcessorFeaturePresent@4 10013014     kernel32:KERNEL32.dll
 0002:00000018       __imp__IsDebuggerPresent@0 10013018     kernel32:KERNEL32.dll
 0002:0000001c       __imp__DecodePointer@4     1001301c     kernel32:KERNEL32.dll
 0002:00000020       __imp__EncodePointer@4     10013020     kernel32:KERNEL32.dll
 0002:00000024       \177KERNEL32_NULL_THUNK_DATA 10013024     kernel32:KERNEL32.dll
 0002:00000028       __imp_?_Xlength_error@std@@YAXPBD@Z 10013028     msvcprt:MSVCP120.dll
 0002:0000002c       __imp_?_Xout_of_range@std@@YAXPBD@Z 1001302c     msvcprt:MSVCP120.dll
 0002:00000030       __imp_?_Syserror_map@std@@YAPBDH@Z 10013030     msvcprt:MSVCP120.dll
 0002:00000034       __imp_?_Winerror_map@std@@YAPBDH@Z 10013034     msvcprt:MSVCP120.dll
 0002:00000038       __imp_?_Xbad_alloc@std@@YAXXZ 10013038     msvcprt:MSVCP120.dll
 0002:0000003c       \177MSVCP120_NULL_THUNK_DATA 1001303c     msvcprt:MSVCP120.dll
 0002:00000040       __imp___initterm_e         10013040     MSVCRT:MSVCR120.dll
 0002:00000044       __imp___initterm           10013044     MSVCRT:MSVCR120.dll
 0002:00000048       __imp___malloc_crt         10013048     MSVCRT:MSVCR120.dll
 0002:0000004c       __imp__free                1001304c     MSVCRT:MSVCR120.dll
 0002:00000050       __imp___amsg_exit          10013050     MSVCRT:MSVCR120.dll
 0002:00000054       __imp____CppXcptFilter     10013054     MSVCRT:MSVCR120.dll
 0002:00000058       __imp___except_handler4_common 10013058     MSVCRT:MSVCR120.dll
 0002:0000005c       __imp___except1            1001305c     MSVCRT:MSVCR120.dll
 0002:00000060       __imp___onexit             10013060     MSVCRT:MSVCR120.dll
 0002:00000064       __imp____dllonexit         10013064     MSVCRT:MSVCR120.dll
 0002:00000068       __imp___calloc_crt         10013068     MSVCRT:MSVCR120.dll
 0002:0000006c       __imp___unlock             1001306c     MSVCRT:MSVCR120.dll
 0002:00000070       __imp___lock               10013070     MSVCRT:MSVCR120.dll
 0002:00000074       __imp___libm_sse2_log10_precise 10013074     MSVCRT:MSVCR120.dll
 0002:00000078       __imp_??_V@YAXPAX@Z        10013078     MSVCRT:MSVCR120.dll
 0002:0000007c       __imp__memset              1001307c     MSVCRT:MSVCR120.dll
 0002:00000080       __imp__memcpy              10013080     MSVCRT:MSVCR120.dll
 0002:00000084       __imp____CxxFrameHandler3  10013084     MSVCRT:MSVCR120.dll
 0002:00000088       __imp___CxxThrowException@8 10013088     MSVCRT:MSVCR120.dll
 0002:0000008c       __imp___hypot              1001308c     MSVCRT:MSVCR120.dll
 0002:00000090       __imp__memmove             10013090     MSVCRT:MSVCR120.dll
 0002:00000094       __imp_??3@YAXPAX@Z         10013094     MSVCRT:MSVCR120.dll
 0002:00000098       __imp_??2@YAPAXI@Z         10013098     MSVCRT:MSVCR120.dll
 0002:0000009c       __imp___purecall           1001309c     MSVCRT:MSVCR120.dll
 0002:000000a0       __imp___crt_debugger_hook  100130a0     MSVCRT:MSVCR120.dll
 0002:000000a4       __imp____crtUnhandledException 100130a4     MSVCRT:MSVCR120.dll
 0002:000000a8       __imp____crtTerminateProcess 100130a8     MSVCRT:MSVCR120.dll
 0002:000000ac       __imp_?terminate@@YAXXZ    100130ac     MSVCRT:MSVCR120.dll
 0002:000000b0       __imp____clean_type_info_names_internal 100130b0     MSVCRT:MSVCR120.dll
 0002:000000b4       __imp_??1type_info@@UAE@XZ 100130b4     MSVCRT:MSVCR120.dll
 0002:000000b8       \177MSVCR120_NULL_THUNK_DATA 100130b8     MSVCRT:MSVCR120.dll
 0002:000000bc       __imp_?qUnregisterResourceData@@YA_NHPBE00@Z 100130bc     Qt5Core:Qt5Core.dll
 0002:000000c0       __imp_?qRegisterResourceData@@YA_NHPBE00@Z 100130c0     Qt5Core:Qt5Core.dll
 0002:000000c4       __imp_?registerNormalizedTypedef@QMetaType@@SAHABVQByteArray@@H@Z 100130c4     Qt5Core:Qt5Core.dll
 0002:000000c8       __imp_?registerNormalizedType@QMetaType@@SAHABVQByteArray@@P6AXPAX@ZP6APAXPBX@Z2P6APAX13@ZHV?$QFlags@W4TypeFlag@QMetaType@@@@PBUQMetaObject@@@Z 100130c8     Qt5Core:Qt5Core.dll
 0002:000000cc       __imp_?className@QMetaObject@@QBEPBDXZ 100130cc     Qt5Core:Qt5Core.dll
 0002:000000d0       __imp_?append@QByteArray@@QAEAAV1@PBD@Z 100130d0     Qt5Core:Qt5Core.dll
 0002:000000d4       __imp_?append@QByteArray@@QAEAAV1@D@Z 100130d4     Qt5Core:Qt5Core.dll
 0002:000000d8       __imp_?reserve@QByteArray@@QAEXH@Z 100130d8     Qt5Core:Qt5Core.dll
 0002:000000dc       __imp_?staticMetaObject@QObject@@2UQMetaObject@@B 100130dc     Qt5Core:Qt5Core.dll
 0002:000000e0       __imp_?qt_metacall@QObject@@UAEHW4Call@QMetaObject@@HPAPAX@Z 100130e0     Qt5Core:Qt5Core.dll
 0002:000000e4       __imp_?qt_metacast@QObject@@UAEPAXPBD@Z 100130e4     Qt5Core:Qt5Core.dll
 0002:000000e8       __imp_?dynamicMetaObject@QObjectData@@QBEPAUQMetaObject@@XZ 100130e8     Qt5Core:Qt5Core.dll
 0002:000000ec       __imp_?at@QByteArray@@QBEDH@Z 100130ec     Qt5Core:Qt5Core.dll
 0002:000000f0       __imp_?resize@QByteArray@@QAEXH@Z 100130f0     Qt5Core:Qt5Core.dll
 0002:000000f4       __imp_??4QByteArray@@QAEAAV0@$$QAV0@@Z 100130f4     Qt5Core:Qt5Core.dll
 0002:000000f8       __imp_??0QByteArray@@QAE@XZ 100130f8     Qt5Core:Qt5Core.dll
 0002:000000fc       __imp_?qBadAlloc@@YAXXZ    100130fc     Qt5Core:Qt5Core.dll
 0002:00000100       __imp_?data@QArrayData@@QAEPAXXZ 10013100     Qt5Core:Qt5Core.dll
 0002:00000104       __imp_?allocate@QArrayData@@SAPAU1@IIIV?$QFlags@W4AllocationOption@QArrayData@@@@@Z 10013104     Qt5Core:Qt5Core.dll
 0002:00000108       __imp_?deallocate@QArrayData@@SAXPAU1@II@Z 10013108     Qt5Core:Qt5Core.dll
 0002:0000010c       __imp_?detach_grow@QListData@@QAEPAUData@1@PAHH@Z 1001310c     Qt5Core:Qt5Core.dll
 0002:00000110       __imp_?dispose@QListData@@SAXPAUData@1@@Z 10013110     Qt5Core:Qt5Core.dll
 0002:00000114       __imp_?append@QListData@@QAEPAPAXXZ 10013114     Qt5Core:Qt5Core.dll
 0002:00000118       __imp_??AQByteArray@@QBEDH@Z 10013118     Qt5Core:Qt5Core.dll
 0002:0000011c       __imp_?tr@QMetaObject@@QBE?AVQString@@PBD0H@Z 1001311c     Qt5Core:Qt5Core.dll
 0002:00000120       __imp_??0QChar@@QAE@UQLatin1Char@@@Z 10013120     Qt5Core:Qt5Core.dll
 0002:00000124       __imp_??1QString@@QAE@XZ   10013124     Qt5Core:Qt5Core.dll
 0002:00000128       __imp_?arg@QString@@QBE?AV1@HHHVQChar@@@Z 10013128     Qt5Core:Qt5Core.dll
 0002:0000012c       __imp_?arg@QString@@QBE?AV1@ABV1@HVQChar@@@Z 1001312c     Qt5Core:Qt5Core.dll
 0002:00000130       __imp_?fromAscii_helper@QString@@CAPAU?$QTypedArrayData@G@@PBDH@Z 10013130     Qt5Core:Qt5Core.dll
 0002:00000134       __imp_??0QBitArray@@QAE@H_N@Z 10013134     Qt5Core:Qt5Core.dll
 0002:00000138       __imp_??0QBitArray@@QAE@ABV0@@Z 10013138     Qt5Core:Qt5Core.dll
 0002:0000013c       __imp_??AQBitArray@@QAE?AVQBitRef@@H@Z 1001313c     Qt5Core:Qt5Core.dll
 0002:00000140       __imp_??1QBitArray@@QAE@XZ 10013140     Qt5Core:Qt5Core.dll
 0002:00000144       __imp_??BQBitRef@@QBE_NXZ  10013144     Qt5Core:Qt5Core.dll
 0002:00000148       __imp_??4QBitRef@@QAEAAV0@ABV0@@Z 10013148     Qt5Core:Qt5Core.dll
 0002:0000014c       __imp_??4QBitRef@@QAEAAV0@_N@Z 1001314c     Qt5Core:Qt5Core.dll
 0002:00000150       __imp_?childEvent@QObject@@MAEXPAVQChildEvent@@@Z 10013150     Qt5Core:Qt5Core.dll
 0002:00000154       __imp_?connectNotify@QObject@@MAEXABVQMetaMethod@@@Z 10013154     Qt5Core:Qt5Core.dll
 0002:00000158       __imp_?customEvent@QObject@@MAEXPAVQEvent@@@Z 10013158     Qt5Core:Qt5Core.dll
 0002:0000015c       __imp_?disconnectNotify@QObject@@MAEXABVQMetaMethod@@@Z 1001315c     Qt5Core:Qt5Core.dll
 0002:00000160       __imp_?event@QObject@@UAE_NPAVQEvent@@@Z 10013160     Qt5Core:Qt5Core.dll
 0002:00000164       __imp_?eventFilter@QObject@@UAE_NPAV1@PAVQEvent@@@Z 10013164     Qt5Core:Qt5Core.dll
 0002:00000168       __imp_?timerEvent@QObject@@MAEXPAVQTimerEvent@@@Z 10013168     Qt5Core:Qt5Core.dll
 0002:0000016c       __imp_?shared_null@QArrayData@@2QBU1@B 1001316c     Qt5Core:Qt5Core.dll
 0002:00000170       __imp_?shared_null@QListData@@2UData@1@B 10013170     Qt5Core:Qt5Core.dll
 0002:00000174       __imp_?detach@QListData@@QAEPAUData@1@H@Z 10013174     Qt5Core:Qt5Core.dll
 0002:00000178       __imp_?cast@QMetaObject@@QBEPAVQObject@@PAV2@@Z 10013178     Qt5Core:Qt5Core.dll
 0002:0000017c       __imp_??1Connection@QMetaObject@@QAE@XZ 1001317c     Qt5Core:Qt5Core.dll
 0002:00000180       __imp_?connect@QObject@@SA?AVConnection@QMetaObject@@PBV1@PBD01W4ConnectionType@Qt@@@Z 10013180     Qt5Core:Qt5Core.dll
 0002:00000184       __imp_?connect@QObject@@QBE?AVConnection@QMetaObject@@PBV1@PBD1W4ConnectionType@Qt@@@Z 10013184     Qt5Core:Qt5Core.dll
 0002:00000188       __imp_?constData@QByteArray@@QBEPBDXZ 10013188     Qt5Core:Qt5Core.dll
 0002:0000018c       __imp_??1QByteArray@@QAE@XZ 1001318c     Qt5Core:Qt5Core.dll
 0002:00000190       __imp_??0QString@@QAE@ABV0@@Z 10013190     Qt5Core:Qt5Core.dll
 0002:00000194       __imp_??M@YA_NABVQString@@0@Z 10013194     Qt5Core:Qt5Core.dll
 0002:00000198       __imp_?freeNodeAndRebalance@QMapDataBase@@QAEXPAUQMapNodeBase@@@Z 10013198     Qt5Core:Qt5Core.dll
 0002:0000019c       __imp_?recalcMostLeftNode@QMapDataBase@@QAEXXZ 1001319c     Qt5Core:Qt5Core.dll
 0002:000001a0       __imp_?createNode@QMapDataBase@@QAEPAUQMapNodeBase@@HHPAU2@_N@Z 100131a0     Qt5Core:Qt5Core.dll
 0002:000001a4       __imp_?freeTree@QMapDataBase@@QAEXPAUQMapNodeBase@@H@Z 100131a4     Qt5Core:Qt5Core.dll
 0002:000001a8       __imp_?createData@QMapDataBase@@SAPAU1@XZ 100131a8     Qt5Core:Qt5Core.dll
 0002:000001ac       __imp_?freeData@QMapDataBase@@SAXPAU1@@Z 100131ac     Qt5Core:Qt5Core.dll
 0002:000001b0       __imp_?shared_null@QMapDataBase@@2U1@B 100131b0     Qt5Core:Qt5Core.dll
 0002:000001b4       \177Qt5Core_NULL_THUNK_DATA 100131b4     Qt5Core:Qt5Core.dll
 0002:000001b8       __imp_??4QColor@@QAEAAV0@ABV0@@Z 100131b8     Qt5Gui:Qt5Gui.dll
 0002:000001bc       __imp_??0QColor@@QAE@W4GlobalColor@Qt@@@Z 100131bc     Qt5Gui:Qt5Gui.dll
 0002:000001c0       \177Qt5Gui_NULL_THUNK_DATA 100131c0     Qt5Gui:Qt5Gui.dll
 0002:000001c4       __imp_?event@QAction@@MAE_NPAVQEvent@@@Z 100131c4     Qt5Widgets:Qt5Widgets.dll
 0002:000001c8       __imp_?setEnabled@QAction@@QAEX_N@Z 100131c8     Qt5Widgets:Qt5Widgets.dll
 0002:000001cc       \177Qt5Widgets_NULL_THUNK_DATA 100131cc     Qt5Widgets:Qt5Widgets.dll
 0002:000001d0       __imp_?nullPointerError@L10N@U2@@SA?AVQString@@ABV3@@Z 100131d0     U2Core:U2Core.dll
 0002:000001d4       __imp_??0Logger@U2@@QAE@ABVQString@@@Z 100131d4     U2Core:U2Core.dll
 0002:000001d8       __imp_??1Logger@U2@@UAE@XZ 100131d8     U2Core:U2Core.dll
 0002:000001dc       __imp_?error@Logger@U2@@QAEXABVQString@@@Z 100131dc     U2Core:U2Core.dll
 0002:000001e0       __imp_??0Plugin@U2@@QAE@ABVQString@@0_NW4PluginState@1@@Z 100131e0     U2Core:U2Core.dll
 0002:000001e4       __imp_??1Plugin@U2@@UAE@XZ 100131e4     U2Core:U2Core.dll
 0002:000001e8       __imp_?getMainWindow@AppContext@U2@@SAPAVMainWindow@2@XZ 100131e8     U2Core:U2Core.dll
 0002:000001ec       __imp_?isRNA@DNAAlphabet@U2@@QBE_NXZ 100131ec     U2Core:U2Core.dll
 0002:000001f0       __imp_?getAlphabetChars@DNAAlphabet@U2@@QBE?AVQByteArray@@_N@Z 100131f0     U2Core:U2Core.dll
 0002:000001f4       __imp_??0Index3To1@U2@@QAE@XZ 100131f4     U2Core:U2Core.dll
 0002:000001f8       __imp_?init@Index3To1@U2@@QAEXABVQByteArray@@@Z 100131f8     U2Core:U2Core.dll
 0002:000001fc       __imp_?indexOf@Index3To1@U2@@QBEHPBD@Z 100131fc     U2Core:U2Core.dll
 0002:00000200       __imp_?indexOf@Index3To1@U2@@QBEHDDD@Z 10013200     U2Core:U2Core.dll
 0002:00000204       __imp_?getDNATranslationRegistry@AppContext@U2@@SAPAVDNATranslationRegistry@2@XZ 10013204     U2Core:U2Core.dll
 0002:00000208       __imp_?lookupComplementTranslation@DNATranslationRegistry@U2@@QAEPAVDNATranslation@2@PBVDNAAlphabet@2@@Z 10013208     U2Core:U2Core.dll
 0002:0000020c       __imp_?qt_metacast@Plugin@U2@@UAEPAXPBD@Z 1001320c     U2Core:U2Core.dll
 0002:00000210       __imp_?qt_metacall@Plugin@U2@@UAEHW4Call@QMetaObject@@HPAPAX@Z 10013210     U2Core:U2Core.dll
 0002:00000214       __imp_?staticMetaObject@Plugin@U2@@2UQMetaObject@@B 10013214     U2Core:U2Core.dll
 0002:00000218       __imp_?getAlphabet@U2SequenceObject@U2@@QBEPBVDNAAlphabet@2@XZ 10013218     U2Core:U2Core.dll
 0002:0000021c       \177U2Core_NULL_THUNK_DATA 1001321c     U2Core:U2Core.dll
 0002:00000220       __imp_?sl_windowClosing@GObjectViewWindowContext@U2@@MAEXPAVMWMDIWindow@2@@Z 10013220     U2Gui:U2Gui.dll
 0002:00000224       __imp_??1GObjectViewWindowContext@U2@@UAE@XZ 10013224     U2Gui:U2Gui.dll
 0002:00000228       __imp_?staticMetaObject@GObjectViewWindowContext@U2@@2UQMetaObject@@B 10013228     U2Gui:U2Gui.dll
 0002:0000022c       __imp_?qt_metacall@GObjectViewWindowContext@U2@@UAEHW4Call@QMetaObject@@HPAPAX@Z 1001322c     U2Gui:U2Gui.dll
 0002:00000230       __imp_?qt_metacast@GObjectViewWindowContext@U2@@UAEPAXPBD@Z 10013230     U2Gui:U2Gui.dll
 0002:00000234       __imp_?buildMenu@GObjectViewWindowContext@U2@@MAEXPAVGObjectView@2@PAVQMenu@@@Z 10013234     U2Gui:U2Gui.dll
 0002:00000238       __imp_?sl_windowAdded@GObjectViewWindowContext@U2@@MAEXPAVMWMDIWindow@2@@Z 10013238     U2Gui:U2Gui.dll
 0002:0000023c       __imp_?sl_buildStaticMenu@GObjectViewWindowContext@U2@@MAEXPAVGObjectView@2@PAVQMenu@@@Z 1001323c     U2Gui:U2Gui.dll
 0002:00000240       __imp_?sl_buildContextMenu@GObjectViewWindowContext@U2@@MAEXPAVGObjectView@2@PAVQMenu@@@Z 10013240     U2Gui:U2Gui.dll
 0002:00000244       __imp_?onObjectRemoved@GObjectViewWindowContext@U2@@UAEXPAVGObjectView@2@PAVGObject@2@@Z 10013244     U2Gui:U2Gui.dll
 0002:00000248       __imp_?onObjectAdded@GObjectViewObjectHandler@U2@@UAEXPAVGObjectView@2@PAVGObject@2@@Z 10013248     U2Gui:U2Gui.dll
 0002:0000024c       __imp_?init@GObjectViewWindowContext@U2@@UAEXXZ 1001324c     U2Gui:U2Gui.dll
 0002:00000250       __imp_?disconnectView@GObjectViewWindowContext@U2@@MAEXPAVGObjectView@2@@Z 10013250     U2Gui:U2Gui.dll
 0002:00000254       __imp_?canHandle@GObjectViewObjectHandler@U2@@UAE_NPAVGObjectView@2@PAVGObject@2@@Z 10013254     U2Gui:U2Gui.dll
 0002:00000258       __imp_??0GObjectViewWindowContext@U2@@QAE@PAVQObject@@ABVGObjectViewFactoryId@1@@Z 10013258     U2Gui:U2Gui.dll
 0002:0000025c       \177U2Gui_NULL_THUNK_DATA  1001325c     U2Gui:U2Gui.dll
 0002:00000260       __imp_??1GSequenceGraphAlgorithm@U2@@UAE@XZ 10013260     U2View:U2View.dll
 0002:00000264       __imp_?getSequenceData@GSequenceGraphAlgorithm@U2@@IAEABVQByteArray@@PAVU2SequenceObject@2@AAVU2OpStatus@2@@Z 10013264     U2View:U2View.dll
 0002:00000268       __imp_??0GSequenceGraphData@U2@@QAE@ABVQString@@@Z 10013268     U2View:U2View.dll
 0002:0000026c       __imp_??1GSequenceGraphData@U2@@UAE@XZ 1001326c     U2View:U2View.dll
 0002:00000270       __imp_?getNumSteps@GSequenceGraphUtils@U2@@SAHABVU2Region@2@HH@Z 10013270     U2View:U2View.dll
 0002:00000274       __imp_??0GSequenceGraphFactory@U2@@QAE@ABVQString@@PAVQObject@@@Z 10013274     U2View:U2View.dll
 0002:00000278       __imp_??1GSequenceGraphFactory@U2@@UAE@XZ 10013278     U2View:U2View.dll
 0002:0000027c       __imp_?getDrawer@GSequenceGraphFactory@U2@@UAEPAVGSequenceGraphDrawer@2@PAVGSequenceGraphView@2@@Z 1001327c     U2View:U2View.dll
 0002:00000280       __imp_?getSequenceObject@ADVSingleSequenceWidget@U2@@QBEPAVU2SequenceObject@2@XZ 10013280     U2View:U2View.dll
 0002:00000284       __imp_??0GraphAction@U2@@QAE@PAVGSequenceGraphFactory@1@@Z 10013284     U2View:U2View.dll
 0002:00000288       __imp_??1GraphAction@U2@@UAE@XZ 10013288     U2View:U2View.dll
 0002:0000028c       __imp_?addGraphAction@GraphMenuAction@U2@@SAXPAVADVSequenceObjectContext@2@PAVGraphAction@2@@Z 1001328c     U2View:U2View.dll
 0002:00000290       __imp_?getSequenceWidgets@AnnotatedDNAView@U2@@QBE?BV?$QList@PAVADVSequenceWidget@U2@@@@XZ 10013290     U2View:U2View.dll
 0002:00000294       __imp_?metaObject@GraphAction@U2@@UBEPBUQMetaObject@@XZ 10013294     U2View:U2View.dll
 0002:00000298       __imp_?qt_metacall@GraphAction@U2@@UAEHW4Call@QMetaObject@@HPAPAX@Z 10013298     U2View:U2View.dll
 0002:0000029c       __imp_?qt_metacast@GraphAction@U2@@UAEPAXPBD@Z 1001329c     U2View:U2View.dll
 0002:000002a0       __imp_?staticMetaObject@ADVSingleSequenceWidget@U2@@2UQMetaObject@@B 100132a0     U2View:U2View.dll
 0002:000002a4       __imp_?staticMetaObject@AnnotatedDNAView@U2@@2UQMetaObject@@B 100132a4     U2View:U2View.dll
 0002:000002a8       __imp_?setColors@GSequenceGraphDrawer@U2@@QAEXABV?$QMap@VQString@@VQColor@@@@@Z 100132a8     U2View:U2View.dll
 0002:000002ac       __imp_?staticMetaObject@ADVSequenceWidget@U2@@2UQMetaObject@@B 100132ac     U2View:U2View.dll
 0002:000002b0       __imp_??0GSequenceGraphAlgorithm@U2@@IAE@XZ 100132b0     U2View:U2View.dll
 0002:000002b4       \177U2View_NULL_THUNK_DATA 100132b4     U2View:U2View.dll
 0002:000002b8       ___xc_a                    100132b8     MSVCRT:cinitexe.obj
 0002:000007bc       ___xc_z                    100137bc     MSVCRT:cinitexe.obj
 0002:000007c0       ___xi_a                    100137c0     MSVCRT:cinitexe.obj
 0002:000007cc       ___xi_z                    100137cc     MSVCRT:cinitexe.obj
 0002:0000080c       ??_7error_category@std@@6B@ 1001380c     BaseContentGraph.obj
 0002:00000828       ??_7_Generic_error_category@std@@6B@ 10013828     BaseContentGraph.obj
 0002:00000840       ??_C@_07DCLBNMLN@generic?$AA@ 10013840     BaseContentGraph.obj
 0002:00000848       ??_C@_0O@BFJCFAAK@unknown?5error?$AA@ 10013848     BaseContentGraph.obj
 0002:0000085c       ??_7_Iostream_error_category@std@@6B@ 1001385c     BaseContentGraph.obj
 0002:00000874       ??_C@_08LLGCOLLL@iostream?$AA@ 10013874     BaseContentGraph.obj
 0002:00000880       ??_C@_0BG@PADBLCHM@iostream?5stream?5error?$AA@ 10013880     BaseContentGraph.obj
 0002:0000089c       ??_7_System_error_category@std@@6B@ 1001389c     BaseContentGraph.obj
 0002:000008b4       ??_C@_06FHFOAHML@system?$AA@ 100138b4     BaseContentGraph.obj
 0002:000008c0       ??_7?$AbstractId@H@U2@@6B@ 100138c0     BaseContentGraph.obj
 0002:000008cc       ??_7AbstractInt32Id@U2@@6B@ 100138cc     BaseContentGraph.obj
 0002:000008d8       ??_7ServiceType@U2@@6B@    100138d8     BaseContentGraph.obj
 0002:000008e0       ??_C@_0L@JLHNEGIN@Algorithms?$AA@ 100138e0     BaseContentGraph.obj
 0002:000008ec       ??_C@_07PGLPGHFC@Console?$AA@ 100138ec     BaseContentGraph.obj
 0002:000008f4       ??_C@_0O@BOFHOPCF@Core?5Services?$AA@ 100138f4     BaseContentGraph.obj
 0002:00000904       ??_C@_0N@PPADAKBM@Input?1Output?$AA@ 10013904     BaseContentGraph.obj
 0002:00000914       ??_C@_0M@KPPBKPKK@Performance?$AA@ 10013914     BaseContentGraph.obj
 0002:00000920       ??_C@_07BFDHHBBI@Scripts?$AA@ 10013920     BaseContentGraph.obj
 0002:00000928       ??_C@_05EEGKELMG@Tasks?$AA@ 10013928     BaseContentGraph.obj
 0002:00000930       ??_C@_0P@NIIOBHGA@User?5Interface?$AA@ 10013930     BaseContentGraph.obj
 0002:00000940       ??_C@_0N@JINCGGMN@User?5Actions?$AA@ 10013940     BaseContentGraph.obj
 0002:00000954       ??_SGSequenceGraphData@U2@@6B@ 10013954     BaseContentGraph.obj
 0002:0000095c       ??_7BaseContentGraphFactory@U2@@6B@ 1001395c     BaseContentGraph.obj
 0002:00000998       ??_7BaseContentGraphAlgorithm@U2@@6B@ 10013998     BaseContentGraph.obj
 0002:000009a0       ??_C@_0P@CHCAIOCI@AG?5Content?5?$CI?$CF?$CJ?$AA@ 100139a0     BaseContentGraph.obj
 0002:000009b0       ??_C@_0P@BMHGNFMB@GC?5Content?5?$CI?$CF?$CJ?$AA@ 100139b0     BaseContentGraph.obj
 0002:000009c0       ??_C@_0CK@IGBIANDN@Trying?5to?5recover?5from?5error?3?5?$CF1@ 100139c0     BaseContentGraph.obj
 0002:000009ec       ??_C@_0N@FOAHPGLI@window?5graph?$AA@ 100139ec     BaseContentGraph.obj
 0002:000009fc       ??_C@_0BJ@JIEBGLML@src?2BaseContentGraph?4cpp?$AA@ 100139fc     BaseContentGraph.obj
 0002:00000a18       ??_C@_0BA@MFJDFJGO@sequence?5object?$AA@ 10013a18     BaseContentGraph.obj
 0002:00000a28       ??_C@_0BA@JFNIOLAK@string?5too?5long?$AA@ 10013a28     BaseContentGraph.obj
 0002:00000a38       ??_C@_0BI@CFPLBAOH@invalid?5string?5position?$AA@ 10013a38     BaseContentGraph.obj
 0002:00000a50       __real@42c80000            10013a50     BaseContentGraph.obj
 0002:00000a58       ??_7CumulativeSkewGraphFactory@U2@@6B@ 10013a58     CumulativeSkew.obj
 0002:00000a94       ??_7CumulativeSkewGraphAlgorithm@U2@@6B@ 10013a94     CumulativeSkew.obj
 0002:00000a9c       ??_C@_0BD@BKCCCCEC@AT?5Cumulative?5Skew?$AA@ 10013a9c     CumulativeSkew.obj
 0002:00000ab0       ??_C@_0BD@EIHDHPCN@GC?5Cumulative?5Skew?$AA@ 10013ab0     CumulativeSkew.obj
 0002:00000ac8       ??_SGraphAction@U2@@6B@    10013ac8     DNAGraphPackPlugin.obj
 0002:00000af8       ??_7DNAGraphPackPlugin@U2@@6B@ 10013af8     DNAGraphPackPlugin.obj
 0002:00000b28       ??_7DNAGraphPackViewContext@U2@@6BQObject@@@ 10013b28     DNAGraphPackPlugin.obj
 0002:00000b78       ??_7DNAGraphPackViewContext@U2@@6BGObjectViewObjectHandler@1@@ 10013b78     DNAGraphPackPlugin.obj
 0002:00000b88       ??_C@_0DA@BMBIEHOD@Contains?5a?5set?5of?5graphs?5for?5DNA@ 10013b88     DNAGraphPackPlugin.obj
 0002:00000bb8       ??_C@_0BG@GLPNDKCM@DNA?1RNA?5Graph?5Package?$AA@ 10013bb8     DNAGraphPackPlugin.obj
 0002:00000bd0       ??_C@_0BB@JDMPMKOK@AnnotatedDNAView?$AA@ 10013bd0     DNAGraphPackPlugin.obj
 0002:00000be4       ??_C@_0CM@JOICIJIL@1sl_sequenceWidgetAdded?$CIADVSeque@ 10013be4     DNAGraphPackPlugin.obj
 0002:00000c10       ??_C@_0CM@KILGFMLI@2si_sequenceWidgetAdded?$CIADVSeque@ 10013c10     DNAGraphPackPlugin.obj
 0002:00000c3c       ??_C@_0DN@LGKKGEKM@1sl_updateGraphView?$CIconst?5QStrin@ 10013c3c     DNAGraphPackPlugin.obj
 0002:00000c7c       ??_C@_0DN@CHPAKHJJ@2si_updateGraphView?$CIconst?5QStrin@ 10013c7c     DNAGraphPackPlugin.obj
 0002:00000cc0       ??_7DeviationGraphFactory@U2@@6B@ 10013cc0     DeviationGraph.obj
 0002:00000cfc       ??_7DeviationGraphAlgorithm@U2@@6B@ 10013cfc     DeviationGraph.obj
 0002:00000d04       ??_C@_0BJ@DABOHEFI@AT?5Deviation?5?$CIA?9T?$CJ?1?$CIA?$CLT?$CJ?$AA@ 10013d04     DeviationGraph.obj
 0002:00000d20       ??_C@_0BJ@KDILPFBK@GC?5Deviation?5?$CIG?9C?$CJ?1?$CIG?$CLC?$CJ?$AA@ 10013d20     DeviationGraph.obj
 0002:00000d3c       __real@3a83126f            10013d3c     DeviationGraph.obj
 0002:00000d44       ??_7EntropyGraphFactory@U2@@6B@ 10013d44     EntropyAlgorithm.obj
 0002:00000d80       ??_7EntropyGraphAlgorithm@U2@@6B@ 10013d80     EntropyAlgorithm.obj
 0002:00000d88       ??_C@_0BG@MEMICHPH@Informational?5Entropy?$AA@ 10013d88     EntropyAlgorithm.obj
 0002:00000da0       __real@4000000000000000    10013da0     EntropyAlgorithm.obj
 0002:00000dac       ??_7GCFramePlotFactory@U2@@6B@ 10013dac     GCFramePlot.obj
 0002:00000de8       ??_7GCFramePlotAlgorithm@U2@@6B@ 10013de8     GCFramePlot.obj
 0002:00000df0       ??_C@_0O@EBOIIKPL@GC?5Frame?5Plot?$AA@ 10013df0     GCFramePlot.obj
 0002:00000e00       ??_C@_07FODKADJO@Frame?51?$AA@ 10013e00     GCFramePlot.obj
 0002:00000e08       ??_C@_07HFBHFAFN@Frame?52?$AA@ 10013e08     GCFramePlot.obj
 0002:00000e10       ??_C@_07GMAMGBBM@Frame?53?$AA@ 10013e10     GCFramePlot.obj
 0002:00000e18       __real@40400000            10013e18     GCFramePlot.obj
 0002:00000e24       ??_7KarlinGraphFactory@U2@@6B@ 10013e24     KarlinSignatureDifferenceGraph.obj
 0002:00000e60       ??_7KarlinGraphAlgorithm@U2@@6B@ 10013e60     KarlinSignatureDifferenceGraph.obj
 0002:00000e68       ??_C@_0BM@JPBKGGCB@Karlin?5Signature?5Difference?$AA@ 10013e68     KarlinSignatureDifferenceGraph.obj
 0002:00000e84       __real@00000000            10013e84     KarlinSignatureDifferenceGraph.obj
 0002:00000e88       __real@3089705f            10013e88     KarlinSignatureDifferenceGraph.obj
 0002:00000e90       __real@3fb0000000000000    10013e90     KarlinSignatureDifferenceGraph.obj
 0002:00000ea0       __xmm@80000000800000008000000080000000 10013ea0     KarlinSignatureDifferenceGraph.obj
 0002:000015ec       ?value@?$integral_constant@_N$0A@@std@@2_NB 100145ec     msvcprt:newaop_s.obj
 0002:000015ed       ?value@?$integral_constant@_N$00@std@@2_NB 100145ed     msvcprt:newaop_s.obj
 0002:00001678       ??_7type_info@@6B@         10014678     MSVCRT:ti_inst.obj
 0002:0000167c       __pRawDllMain              1001467c     MSVCRT:crtdll.obj
 0002:0000167c       __pDefaultRawDllMain       1001467c     MSVCRT:crtdll.obj
 0002:00001688       ?ProcessDetach@NativeDll@<CrtImplementationDetails>@@0IB 10014688     MSVCRT:initsect.obj
 0002:0000168c       ?ProcessAttach@NativeDll@<CrtImplementationDetails>@@0IB 1001468c     MSVCRT:initsect.obj
 0002:00001690       ?ThreadAttach@NativeDll@<CrtImplementationDetails>@@0IB 10014690     MSVCRT:initsect.obj
 0002:00001694       ?ThreadDetach@NativeDll@<CrtImplementationDetails>@@0IB 10014694     MSVCRT:initsect.obj
 0002:00001698       ?ProcessVerifier@NativeDll@<CrtImplementationDetails>@@0IB 10014698     MSVCRT:initsect.obj
 0002:000016a0       __load_config_used         100146a0     MSVCRT:loadcfg.obj
 0002:0000175c       ??_R4error_category@std@@6B@ 1001475c     BaseContentGraph.obj
 0002:00001770       ??_R3error_category@std@@8 10014770     BaseContentGraph.obj
 0002:00001780       ??_R2error_category@std@@8 10014780     BaseContentGraph.obj
 0002:00001788       ??_R1A@?0A@EA@error_category@std@@8 10014788     BaseContentGraph.obj
 0002:000017a4       ??_R4_Generic_error_category@std@@6B@ 100147a4     BaseContentGraph.obj
 0002:000017b8       ??_R3_Generic_error_category@std@@8 100147b8     BaseContentGraph.obj
 0002:000017c8       ??_R2_Generic_error_category@std@@8 100147c8     BaseContentGraph.obj
 0002:000017d4       ??_R1A@?0A@EA@_Generic_error_category@std@@8 100147d4     BaseContentGraph.obj
 0002:000017f0       ??_R4_Iostream_error_category@std@@6B@ 100147f0     BaseContentGraph.obj
 0002:00001804       ??_R3_Iostream_error_category@std@@8 10014804     BaseContentGraph.obj
 0002:00001814       ??_R2_Iostream_error_category@std@@8 10014814     BaseContentGraph.obj
 0002:00001824       ??_R1A@?0A@EA@_Iostream_error_category@std@@8 10014824     BaseContentGraph.obj
 0002:00001840       ??_R4_System_error_category@std@@6B@ 10014840     BaseContentGraph.obj
 0002:00001854       ??_R3_System_error_category@std@@8 10014854     BaseContentGraph.obj
 0002:00001864       ??_R2_System_error_category@std@@8 10014864     BaseContentGraph.obj
 0002:00001874       ??_R1A@?0A@EA@_System_error_category@std@@8 10014874     BaseContentGraph.obj
 0002:00001890       ??_R4AbstractInt32Id@U2@@6B@ 10014890     BaseContentGraph.obj
 0002:000018a4       ??_R3AbstractInt32Id@U2@@8 100148a4     BaseContentGraph.obj
 0002:000018b4       ??_R2AbstractInt32Id@U2@@8 100148b4     BaseContentGraph.obj
 0002:000018c0       ??_R1A@?0A@EA@AbstractInt32Id@U2@@8 100148c0     BaseContentGraph.obj
 0002:000018dc       ??_R1A@?0A@EA@?$AbstractId@H@U2@@8 100148dc     BaseContentGraph.obj
 0002:000018f8       ??_R3?$AbstractId@H@U2@@8  100148f8     BaseContentGraph.obj
 0002:00001908       ??_R2?$AbstractId@H@U2@@8  10014908     BaseContentGraph.obj
 0002:00001910       ??_R4?$AbstractId@H@U2@@6B@ 10014910     BaseContentGraph.obj
 0002:00001924       ??_R4ServiceType@U2@@6B@   10014924     BaseContentGraph.obj
 0002:00001938       ??_R3ServiceType@U2@@8     10014938     BaseContentGraph.obj
 0002:00001948       ??_R2ServiceType@U2@@8     10014948     BaseContentGraph.obj
 0002:00001958       ??_R1A@?0A@EA@ServiceType@U2@@8 10014958     BaseContentGraph.obj
 0002:00001974       ??_R1A@?0A@EA@QObject@@8   10014974     BaseContentGraph.obj
 0002:00001990       ??_R3QObject@@8            10014990     BaseContentGraph.obj
 0002:000019a0       ??_R2QObject@@8            100149a0     BaseContentGraph.obj
 0002:000019a8       ??_R4GSequenceGraphData@U2@@6B@ 100149a8     BaseContentGraph.obj
 0002:000019bc       ??_R3GSequenceGraphData@U2@@8 100149bc     BaseContentGraph.obj
 0002:000019cc       ??_R2GSequenceGraphData@U2@@8 100149cc     BaseContentGraph.obj
 0002:000019d4       ??_R1A@?0A@EA@GSequenceGraphData@U2@@8 100149d4     BaseContentGraph.obj
 0002:000019f0       ??_R4BaseContentGraphFactory@U2@@6B@ 100149f0     BaseContentGraph.obj
 0002:00001a04       ??_R3BaseContentGraphFactory@U2@@8 10014a04     BaseContentGraph.obj
 0002:00001a14       ??_R2BaseContentGraphFactory@U2@@8 10014a14     BaseContentGraph.obj
 0002:00001a24       ??_R1A@?0A@EA@BaseContentGraphFactory@U2@@8 10014a24     BaseContentGraph.obj
 0002:00001a40       ??_R1A@?0A@EA@GSequenceGraphFactory@U2@@8 10014a40     BaseContentGraph.obj
 0002:00001a5c       ??_R3GSequenceGraphFactory@U2@@8 10014a5c     BaseContentGraph.obj
 0002:00001a6c       ??_R2GSequenceGraphFactory@U2@@8 10014a6c     BaseContentGraph.obj
 0002:00001a78       ??_R4BaseContentGraphAlgorithm@U2@@6B@ 10014a78     BaseContentGraph.obj
 0002:00001a8c       ??_R3BaseContentGraphAlgorithm@U2@@8 10014a8c     BaseContentGraph.obj
 0002:00001a9c       ??_R2BaseContentGraphAlgorithm@U2@@8 10014a9c     BaseContentGraph.obj
 0002:00001aa8       ??_R1A@?0A@EA@BaseContentGraphAlgorithm@U2@@8 10014aa8     BaseContentGraph.obj
 0002:00001ac4       ??_R1A@?0A@EA@GSequenceGraphAlgorithm@U2@@8 10014ac4     BaseContentGraph.obj
 0002:00001ae0       ??_R3GSequenceGraphAlgorithm@U2@@8 10014ae0     BaseContentGraph.obj
 0002:00001af0       ??_R2GSequenceGraphAlgorithm@U2@@8 10014af0     BaseContentGraph.obj
 0002:00001af8       ??_R4CumulativeSkewGraphFactory@U2@@6B@ 10014af8     CumulativeSkew.obj
 0002:00001b0c       ??_R3CumulativeSkewGraphFactory@U2@@8 10014b0c     CumulativeSkew.obj
 0002:00001b1c       ??_R2CumulativeSkewGraphFactory@U2@@8 10014b1c     CumulativeSkew.obj
 0002:00001b2c       ??_R1A@?0A@EA@CumulativeSkewGraphFactory@U2@@8 10014b2c     CumulativeSkew.obj
 0002:00001b48       ??_R4CumulativeSkewGraphAlgorithm@U2@@6B@ 10014b48     CumulativeSkew.obj
 0002:00001b5c       ??_R3CumulativeSkewGraphAlgorithm@U2@@8 10014b5c     CumulativeSkew.obj
 0002:00001b6c       ??_R2CumulativeSkewGraphAlgorithm@U2@@8 10014b6c     CumulativeSkew.obj
 0002:00001b78       ??_R1A@?0A@EA@CumulativeSkewGraphAlgorithm@U2@@8 10014b78     CumulativeSkew.obj
 0002:00001b94       ??_R4GraphAction@U2@@6B@   10014b94     DNAGraphPackPlugin.obj
 0002:00001ba8       ??_R3GraphAction@U2@@8     10014ba8     DNAGraphPackPlugin.obj
 0002:00001bb8       ??_R2GraphAction@U2@@8     10014bb8     DNAGraphPackPlugin.obj
 0002:00001bc8       ??_R1A@?0A@EA@GraphAction@U2@@8 10014bc8     DNAGraphPackPlugin.obj
 0002:00001be4       ??_R1A@?0A@EA@QAction@@8   10014be4     DNAGraphPackPlugin.obj
 0002:00001c00       ??_R3QAction@@8            10014c00     DNAGraphPackPlugin.obj
 0002:00001c10       ??_R2QAction@@8            10014c10     DNAGraphPackPlugin.obj
 0002:00001c1c       ??_R4DNAGraphPackViewContext@U2@@6BQObject@@@ 10014c1c     DNAGraphPackPlugin.obj
 0002:00001c30       ??_R3DNAGraphPackViewContext@U2@@8 10014c30     DNAGraphPackPlugin.obj
 0002:00001c40       ??_R2DNAGraphPackViewContext@U2@@8 10014c40     DNAGraphPackPlugin.obj
 0002:00001c54       ??_R1A@?0A@EA@DNAGraphPackViewContext@U2@@8 10014c54     DNAGraphPackPlugin.obj
 0002:00001c70       ??_R1A@?0A@EA@GObjectViewWindowContext@U2@@8 10014c70     DNAGraphPackPlugin.obj
 0002:00001c8c       ??_R3GObjectViewWindowContext@U2@@8 10014c8c     DNAGraphPackPlugin.obj
 0002:00001c9c       ??_R2GObjectViewWindowContext@U2@@8 10014c9c     DNAGraphPackPlugin.obj
 0002:00001cac       ??_R17?0A@EA@GObjectViewObjectHandler@U2@@8 10014cac     DNAGraphPackPlugin.obj
 0002:00001cc8       ??_R3GObjectViewObjectHandler@U2@@8 10014cc8     DNAGraphPackPlugin.obj
 0002:00001cd8       ??_R2GObjectViewObjectHandler@U2@@8 10014cd8     DNAGraphPackPlugin.obj
 0002:00001ce0       ??_R1A@?0A@EA@GObjectViewObjectHandler@U2@@8 10014ce0     DNAGraphPackPlugin.obj
 0002:00001cfc       ??_R4DNAGraphPackViewContext@U2@@6BGObjectViewObjectHandler@1@@ 10014cfc     DNAGraphPackPlugin.obj
 0002:00001d10       ??_R4DNAGraphPackPlugin@U2@@6B@ 10014d10     DNAGraphPackPlugin.obj
 0002:00001d24       ??_R3DNAGraphPackPlugin@U2@@8 10014d24     DNAGraphPackPlugin.obj
 0002:00001d34       ??_R2DNAGraphPackPlugin@U2@@8 10014d34     DNAGraphPackPlugin.obj
 0002:00001d44       ??_R1A@?0A@EA@DNAGraphPackPlugin@U2@@8 10014d44     DNAGraphPackPlugin.obj
 0002:00001d60       ??_R1A@?0A@EA@Plugin@U2@@8 10014d60     DNAGraphPackPlugin.obj
 0002:00001d7c       ??_R3Plugin@U2@@8          10014d7c     DNAGraphPackPlugin.obj
 0002:00001d8c       ??_R2Plugin@U2@@8          10014d8c     DNAGraphPackPlugin.obj
 0002:00001d98       ??_R4DeviationGraphFactory@U2@@6B@ 10014d98     DeviationGraph.obj
 0002:00001dac       ??_R3DeviationGraphFactory@U2@@8 10014dac     DeviationGraph.obj
 0002:00001dbc       ??_R2DeviationGraphFactory@U2@@8 10014dbc     DeviationGraph.obj
 0002:00001dcc       ??_R1A@?0A@EA@DeviationGraphFactory@U2@@8 10014dcc     DeviationGraph.obj
 0002:00001de8       ??_R4DeviationGraphAlgorithm@U2@@6B@ 10014de8     DeviationGraph.obj
 0002:00001dfc       ??_R3DeviationGraphAlgorithm@U2@@8 10014dfc     DeviationGraph.obj
 0002:00001e0c       ??_R2DeviationGraphAlgorithm@U2@@8 10014e0c     DeviationGraph.obj
 0002:00001e18       ??_R1A@?0A@EA@DeviationGraphAlgorithm@U2@@8 10014e18     DeviationGraph.obj
 0002:00001e34       ??_R4EntropyGraphFactory@U2@@6B@ 10014e34     EntropyAlgorithm.obj
 0002:00001e48       ??_R3EntropyGraphFactory@U2@@8 10014e48     EntropyAlgorithm.obj
 0002:00001e58       ??_R2EntropyGraphFactory@U2@@8 10014e58     EntropyAlgorithm.obj
 0002:00001e68       ??_R1A@?0A@EA@EntropyGraphFactory@U2@@8 10014e68     EntropyAlgorithm.obj
 0002:00001e84       ??_R4EntropyGraphAlgorithm@U2@@6B@ 10014e84     EntropyAlgorithm.obj
 0002:00001e98       ??_R3EntropyGraphAlgorithm@U2@@8 10014e98     EntropyAlgorithm.obj
 0002:00001ea8       ??_R2EntropyGraphAlgorithm@U2@@8 10014ea8     EntropyAlgorithm.obj
 0002:00001eb4       ??_R1A@?0A@EA@EntropyGraphAlgorithm@U2@@8 10014eb4     EntropyAlgorithm.obj
 0002:00001ed0       ??_R4GCFramePlotFactory@U2@@6B@ 10014ed0     GCFramePlot.obj
 0002:00001ee4       ??_R3GCFramePlotFactory@U2@@8 10014ee4     GCFramePlot.obj
 0002:00001ef4       ??_R2GCFramePlotFactory@U2@@8 10014ef4     GCFramePlot.obj
 0002:00001f04       ??_R1A@?0A@EA@GCFramePlotFactory@U2@@8 10014f04     GCFramePlot.obj
 0002:00001f20       ??_R4GCFramePlotAlgorithm@U2@@6B@ 10014f20     GCFramePlot.obj
 0002:00001f34       ??_R3GCFramePlotAlgorithm@U2@@8 10014f34     GCFramePlot.obj
 0002:00001f44       ??_R2GCFramePlotAlgorithm@U2@@8 10014f44     GCFramePlot.obj
 0002:00001f50       ??_R1A@?0A@EA@GCFramePlotAlgorithm@U2@@8 10014f50     GCFramePlot.obj
 0002:00001f6c       ??_R4KarlinGraphFactory@U2@@6B@ 10014f6c     KarlinSignatureDifferenceGraph.obj
 0002:00001f80       ??_R3KarlinGraphFactory@U2@@8 10014f80     KarlinSignatureDifferenceGraph.obj
 0002:00001f90       ??_R2KarlinGraphFactory@U2@@8 10014f90     KarlinSignatureDifferenceGraph.obj
 0002:00001fa0       ??_R1A@?0A@EA@KarlinGraphFactory@U2@@8 10014fa0     KarlinSignatureDifferenceGraph.obj
 0002:00001fbc       ??_R4KarlinGraphAlgorithm@U2@@6B@ 10014fbc     KarlinSignatureDifferenceGraph.obj
 0002:00001fd0       ??_R3KarlinGraphAlgorithm@U2@@8 10014fd0     KarlinSignatureDifferenceGraph.obj
 0002:00001fe0       ??_R2KarlinGraphAlgorithm@U2@@8 10014fe0     KarlinSignatureDifferenceGraph.obj
 0002:00001fec       ??_R1A@?0A@EA@KarlinGraphAlgorithm@U2@@8 10014fec     KarlinSignatureDifferenceGraph.obj
 0002:00002008       ??_R4type_info@@6B@        10015008     MSVCRT:ti_inst.obj
 0002:0000201c       ??_R3type_info@@8          1001501c     MSVCRT:ti_inst.obj
 0002:0000202c       ??_R2type_info@@8          1001502c     MSVCRT:ti_inst.obj
 0002:00002034       ??_R1A@?0A@EA@type_info@@8 10015034     MSVCRT:ti_inst.obj
 0002:00002050       ___safe_se_handler_table   10015050     <linker-defined>
 0002:0000230c       ___rtc_iaa                 1001530c     MSVCRT:initsect.obj
 0002:00002310       ___rtc_izz                 10015310     MSVCRT:initsect.obj
 0002:00002314       ___rtc_taa                 10015314     MSVCRT:initsect.obj
 0002:00002318       ___rtc_tzz                 10015318     MSVCRT:initsect.obj
 0002:00004838       __IMPORT_DESCRIPTOR_U2Core 10017838     U2Core:U2Core.dll
 0002:0000484c       __IMPORT_DESCRIPTOR_U2Gui  1001784c     U2Gui:U2Gui.dll
 0002:00004860       __IMPORT_DESCRIPTOR_U2View 10017860     U2View:U2View.dll
 0002:00004874       __IMPORT_DESCRIPTOR_Qt5Widgets 10017874     Qt5Widgets:Qt5Widgets.dll
 0002:00004888       __IMPORT_DESCRIPTOR_Qt5Gui 10017888     Qt5Gui:Qt5Gui.dll
 0002:0000489c       __IMPORT_DESCRIPTOR_Qt5Core 1001789c     Qt5Core:Qt5Core.dll
 0002:000048b0       __IMPORT_DESCRIPTOR_MSVCP120 100178b0     msvcprt:MSVCP120.dll
 0002:000048c4       __IMPORT_DESCRIPTOR_MSVCR120 100178c4     MSVCRT:MSVCR120.dll
 0002:000048d8       __IMPORT_DESCRIPTOR_KERNEL32 100178d8     kernel32:KERNEL32.dll
 0002:000048ec       __NULL_IMPORT_DESCRIPTOR   100178ec     U2Core:U2Core.dll
 0003:00000000       ?_Generic_object@?$_Error_objects@H@std@@2V_Generic_error_category@2@A 1001a000     BaseContentGraph.obj
 0003:00000004       ?_Iostream_object@?$_Error_objects@H@std@@2V_Iostream_error_category@2@A 1001a004     BaseContentGraph.obj
 0003:00000008       ?_System_object@?$_Error_objects@H@std@@2V_System_error_category@2@A 1001a008     BaseContentGraph.obj
 0003:0000034c       ?staticMetaObject@BaseContentGraphFactory@U2@@2UQMetaObject@@B 1001a34c     moc_BaseContentGraph.obj
 0003:000003cc       ?staticMetaObject@CumulativeSkewGraphFactory@U2@@2UQMetaObject@@B 1001a3cc     moc_CumulativeSkew.obj
 0003:0000044c       ?staticMetaObject@DNAGraphPackPlugin@U2@@2UQMetaObject@@B 1001a44c     moc_DNAGraphPackPlugin.obj
 0003:00000464       ?staticMetaObject@DNAGraphPackViewContext@U2@@2UQMetaObject@@B 1001a464     moc_DNAGraphPackPlugin.obj
 0003:000004e4       ?staticMetaObject@DeviationGraphFactory@U2@@2UQMetaObject@@B 1001a4e4     moc_DeviationGraph.obj
 0003:00000564       ?staticMetaObject@EntropyGraphFactory@U2@@2UQMetaObject@@B 1001a564     moc_EntropyAlgorithm.obj
 0003:000005e4       ?staticMetaObject@GCFramePlotFactory@U2@@2UQMetaObject@@B 1001a5e4     moc_GCFramePlot.obj
 0003:00000664       ?staticMetaObject@KarlinGraphFactory@U2@@2UQMetaObject@@B 1001a664     moc_KarlinSignatureDifferenceGraph.obj
 0003:00000680       ___security_cookie         1001a680     MSVCRT:gs_cookie.obj
 0003:00000684       ___security_cookie_complement 1001a684     MSVCRT:gs_cookie.obj
 0003:00000690       ___native_dllmain_reason   1001a690     MSVCRT:natstart.obj
 0003:00000694       ??_R0?AVQObject@@@8        1001a694     BaseContentGraph.obj
 0003:000006ac       ??_R0?AVerror_category@std@@@8 1001a6ac     BaseContentGraph.obj
 0003:000006d0       ??_R0?AV_Generic_error_category@std@@@8 1001a6d0     BaseContentGraph.obj
 0003:000006fc       ??_R0?AV_Iostream_error_category@std@@@8 1001a6fc     BaseContentGraph.obj
 0003:00000728       ??_R0?AV_System_error_category@std@@@8 1001a728     BaseContentGraph.obj
 0003:00000754       ??_R0?AVAbstractInt32Id@U2@@@8 1001a754     BaseContentGraph.obj
 0003:00000778       ??_R0?AV?$AbstractId@H@U2@@@8 1001a778     BaseContentGraph.obj
 0003:00000798       ??_R0?AVServiceType@U2@@@8 1001a798     BaseContentGraph.obj
 0003:000007b8       ??_R0?AVGSequenceGraphData@U2@@@8 1001a7b8     BaseContentGraph.obj
 0003:000007dc       ??_R0?AVBaseContentGraphFactory@U2@@@8 1001a7dc     BaseContentGraph.obj
 0003:00000808       ??_R0?AVGSequenceGraphFactory@U2@@@8 1001a808     BaseContentGraph.obj
 0003:00000830       ??_R0?AVBaseContentGraphAlgorithm@U2@@@8 1001a830     BaseContentGraph.obj
 0003:0000085c       ??_R0?AVGSequenceGraphAlgorithm@U2@@@8 1001a85c     BaseContentGraph.obj
 0003:00000888       ??_R0?AVCumulativeSkewGraphFactory@U2@@@8 1001a888     CumulativeSkew.obj
 0003:000008b4       ??_R0?AVCumulativeSkewGraphAlgorithm@U2@@@8 1001a8b4     CumulativeSkew.obj
 0003:000008e4       ??_R0?AVGraphAction@U2@@@8 1001a8e4     DNAGraphPackPlugin.obj
 0003:00000904       ??_R0?AVQAction@@@8        1001a904     DNAGraphPackPlugin.obj
 0003:0000091c       ??_R0?AVDNAGraphPackViewContext@U2@@@8 1001a91c     DNAGraphPackPlugin.obj
 0003:00000948       ??_R0?AVGObjectViewWindowContext@U2@@@8 1001a948     DNAGraphPackPlugin.obj
 0003:00000974       ??_R0?AVGObjectViewObjectHandler@U2@@@8 1001a974     DNAGraphPackPlugin.obj
 0003:000009a0       ??_R0?AVDNAGraphPackPlugin@U2@@@8 1001a9a0     DNAGraphPackPlugin.obj
 0003:000009c4       ??_R0?AVPlugin@U2@@@8      1001a9c4     DNAGraphPackPlugin.obj
 0003:000009dc       ??_R0?AVDeviationGraphFactory@U2@@@8 1001a9dc     DeviationGraph.obj
 0003:00000a04       ??_R0?AVDeviationGraphAlgorithm@U2@@@8 1001aa04     DeviationGraph.obj
 0003:00000a30       ??_R0?AVEntropyGraphFactory@U2@@@8 1001aa30     EntropyAlgorithm.obj
 0003:00000a58       ??_R0?AVEntropyGraphAlgorithm@U2@@@8 1001aa58     EntropyAlgorithm.obj
 0003:00000a80       ??_R0?AVGCFramePlotFactory@U2@@@8 1001aa80     GCFramePlot.obj
 0003:00000aa4       ??_R0?AVGCFramePlotAlgorithm@U2@@@8 1001aaa4     GCFramePlot.obj
 0003:00000acc       ??_R0?AVKarlinGraphFactory@U2@@@8 1001aacc     KarlinSignatureDifferenceGraph.obj
 0003:00000af0       ??_R0?AVKarlinGraphAlgorithm@U2@@@8 1001aaf0     KarlinSignatureDifferenceGraph.obj
 0003:00000b18       ??_R0?AVtype_info@@@8      1001ab18     MSVCRT:ti_inst.obj
 0003:00000b7c       ?id@?$num_put@DV?$back_insert_iterator@V?$basic_string@DU?$char_traits@D@std@@V?$allocator@D@2@@std@@@std@@@std@@2V0locale@2@A 1001ab7c     BaseContentGraph.obj
 0003:00000b80       ?id@?$num_put@_WV?$back_insert_iterator@V?$basic_string@_WU?$char_traits@_W@std@@V?$allocator@_W@2@@std@@@std@@@std@@2V0locale@2@A 1001ab80     BaseContentGraph.obj
 0003:00000e30       ?metatype_id@?1??qt_metatype_id@?$QMetaTypeIdQObject@PAVADVSequenceWidget@U2@@$00@@SAHXZ@4V?$QBasicAtomicInteger@H@@A 1001ae30     moc_DNAGraphPackPlugin.obj
 0003:00000f64       ?dummy@?A0x701b237d@@3Uinitializer@1@A 1001af64     qrc_dna_graphpack.obj
 0003:00001290       ?__type_info_root_node@@3U__type_info_node@@A 1001b290     MSVCRT:tncleanup.obj
 0003:00001298       ___native_startup_lock     1001b298     <common>
 0003:0000129c       ___native_startup_state    1001b29c     <common>
 0003:000012a0       ___dyn_tls_init_callback   1001b2a0     <common>
 0003:000012a4       ___onexitend               1001b2a4     <common>
 0003:000012a8       ___onexitbegin             1001b2a8     <common>

 entry point at        0001:0000ceb8

 Static symbols

 0000:fffe0000       .debug$S                   10000000     MSVCRT:MSVCR120.dll
 0000:fffe0000       .debug$S                   10000000     MSVCRT:MSVCR120.dll
 0000:fffe0000       .debug$S                   10000000     MSVCRT:MSVCR120.dll
 0000:fffe0000       .debug$S                   10000000     MSVCRT:MSVCR120.dll
 0000:fffe0000       .debug$S                   10000000     MSVCRT:MSVCR120.dll
 0000:fffe0000       .debug$S                   10000000     MSVCRT:MSVCR120.dll
 0000:fffe0000       .debug$S                   10000000     MSVCRT:MSVCR120.dll
 0000:fffe0000       .debug$S                   10000000     MSVCRT:MSVCR120.dll
 0000:fffe0000       .debug$S                   10000000     MSVCRT:MSVCR120.dll
 0000:fffe0000       .debug$S                   10000000     MSVCRT:MSVCR120.dll
 0001:fffff000       __ehhandler$?_Copy@?$basic_string@DU?$char_traits@D@std@@V?$allocator@D@2@@std@@QAEXII@Z 10000000 f   moc_DNAGraphPackPlugin.obj
 0000:fffe0000       .debug$S                   10000000     MSVCRT:MSVCR120.dll
 0000:fffe0000       .debug$S                   10000000     MSVCRT:MSVCR120.dll
 0000:fffe0000       .debug$S                   10000000     MSVCRT:MSVCR120.dll
 0000:fffe0000       .debug$S                   10000000     MSVCRT:MSVCR120.dll
 0002:fffed000       __catchsym$?reallocData@?$QVector@M@@AAEXHHV?$QFlags@W4AllocationOption@QArrayData@@@@@Z$5 10000000     DeviationGraph.obj
 0000:fffe0000       .debug$S                   10000000     MSVCRT:MSVCR120.dll
 0002:fffed000       ?_System_object$initializer$@?$_Error_objects@H@std@@2P6AXXZA 10000000     moc_DeviationGraph.obj
 0000:fffe0000       .debug$S                   10000000     MSVCRT:MSVCR120.dll
 0002:fffed000       ?_Iostream_object$initializer$@?$_Error_objects@H@std@@2P6AXXZA 10000000     moc_DeviationGraph.obj
 0000:fffe0000       .debug$S                   10000000     MSVCRT:MSVCR120.dll
 0002:fffed000       ?_Generic_object$initializer$@?$_Error_objects@H@std@@2P6AXXZA 10000000     moc_DeviationGraph.obj
 0000:fffe0000       .debug$S                   10000000     MSVCRT:MSVCR120.dll
 0002:fffed000       __catchsym$?append@?$QList@V?$QSharedPointer@VGSequenceGraphData@U2@@@@@@QAEXABV?$QSharedPointer@VGSequenceGraphData@U2@@@@@Z$9 10000000     DeviationGraph.obj
 0000:fffe0000       .debug$S                   10000000     MSVCRT:MSVCR120.dll
 0002:fffed000       __catchsym$?detach_helper_grow@?$QList@V?$QSharedPointer@VGSequenceGraphData@U2@@@@@@AAEPAUNode@1@HH@Z$5 10000000     DeviationGraph.obj
 0000:fffe0000       .debug$S                   10000000     MSVCRT:MSVCR120.dll
 0002:fffed000       __catchsym$?node_copy@?$QList@V?$QSharedPointer@VGSequenceGraphData@U2@@@@@@AAEXPAUNode@1@00@Z$6 10000000     DeviationGraph.obj
 0000:fffe0000       .debug$S                   10000000     MSVCRT:MSVCR120.dll
 0002:fffed000       ?_Generic_object$initializer$@?$_Error_objects@H@std@@2P6AXXZA 10000000     DeviationGraph.obj
 0000:fffe0000       .debug$S                   10000000     MSVCRT:MSVCR120.dll
 0002:fffed000       ?_Iostream_object$initializer$@?$_Error_objects@H@std@@2P6AXXZA 10000000     DeviationGraph.obj
 0000:fffe0000       .debug$S                   10000000     MSVCRT:MSVCR120.dll
 0002:fffed000       ?_System_object$initializer$@?$_Error_objects@H@std@@2P6AXXZA 10000000     DeviationGraph.obj
 0000:fffe0000       .debug$S                   10000000     MSVCRT:MSVCR120.dll
 0001:fffff000       __ehhandler$?_Copy@?$basic_string@DU?$char_traits@D@std@@V?$allocator@D@2@@std@@QAEXII@Z 10000000 f   DNAGraphPackPlugin.obj
 0000:fffe0000       .debug$S                   10000000     MSVCRT:MSVCR120.dll
 0001:fffff000       __ehhandler$?node_copy@?$QList@V?$QSharedPointer@VGSequenceGraphData@U2@@@@@@AAEXPAUNode@1@00@Z 10000000 f   DeviationGraph.obj
 0000:fffe0000       .debug$S                   10000000     MSVCRT:MSVCR120.dll
 0001:fffff000       __ehhandler$?detach_helper_grow@?$QList@V?$QSharedPointer@VGSequenceGraphData@U2@@@@@@AAEPAUNode@1@HH@Z 10000000 f   DeviationGraph.obj
 0000:fffe0000       .debug$S                   10000000     MSVCRT:MSVCR120.dll
 0001:fffff000       __ehhandler$?append@?$QList@V?$QSharedPointer@VGSequenceGraphData@U2@@@@@@QAEXABV?$QSharedPointer@VGSequenceGraphData@U2@@@@@Z 10000000 f   DeviationGraph.obj
 0000:fffe0000       .debug$S                   10000000     MSVCRT:MSVCR120.dll
 0001:fffff000       __ehhandler$?reallocData@?$QVector@M@@AAEXHHV?$QFlags@W4AllocationOption@QArrayData@@@@@Z 10000000 f   DeviationGraph.obj
 0000:fffe0000       .debug$S                   10000000     MSVCRT:MSVCR120.dll
 0001:fffff000       __ehhandler$?_Copy@?$basic_string@DU?$char_traits@D@std@@V?$allocator@D@2@@std@@QAEXII@Z 10000000 f   KarlinSignatureDifferenceGraph.obj
 0000:fffe0000       .debug$S                   10000000     MSVCRT:MSVCR120.dll
 0002:fffed000       ?_System_object$initializer$@?$_Error_objects@H@std@@2P6AXXZA 10000000     moc_BaseContentGraph.obj
 0002:fffed000       ?_Iostream_object$initializer$@?$_Error_objects@H@std@@2P6AXXZA 10000000     moc_BaseContentGraph.obj
 0002:fffed000       ?_Generic_object$initializer$@?$_Error_objects@H@std@@2P6AXXZA 10000000     moc_BaseContentGraph.obj
 0002:fffed000       __catchsym$?_Copy@?$basic_string@DU?$char_traits@D@std@@V?$allocator@D@2@@std@@QAEXII@Z$5 10000000     moc_DNAGraphPackPlugin.obj
 0001:fffff000       __ehhandler$?_Copy@?$basic_string@DU?$char_traits@D@std@@V?$allocator@D@2@@std@@QAEXII@Z 10000000 f   DeviationGraph.obj
 0001:fffff000       __ehhandler$?reallocData@?$QVector@M@@AAEXHHV?$QFlags@W4AllocationOption@QArrayData@@@@@Z 10000000 f   KarlinSignatureDifferenceGraph.obj
 0002:fffed000       __catchsym$?_Copy@?$basic_string@DU?$char_traits@D@std@@V?$allocator@D@2@@std@@QAEXII@Z$5 10000000     moc_DeviationGraph.obj
 0001:fffff000       __ehhandler$?_Copy@?$basic_string@DU?$char_traits@D@std@@V?$allocator@D@2@@std@@QAEXII@Z 10000000 f   moc_DeviationGraph.obj
 0001:fffff000       __ehhandler$?append@?$QList@V?$QSharedPointer@VGSequenceGraphData@U2@@@@@@QAEXABV?$QSharedPointer@VGSequenceGraphData@U2@@@@@Z 10000000 f   KarlinSignatureDifferenceGraph.obj
 0002:fffed000       ?_System_object$initializer$@?$_Error_objects@H@std@@2P6AXXZA 10000000     EntropyAlgorithm.obj
 0002:fffed000       ?_Iostream_object$initializer$@?$_Error_objects@H@std@@2P6AXXZA 10000000     EntropyAlgorithm.obj
 0001:fffff000       __ehhandler$?detach_helper_grow@?$QList@V?$QSharedPointer@VGSequenceGraphData@U2@@@@@@AAEPAUNode@1@HH@Z 10000000 f   KarlinSignatureDifferenceGraph.obj
 0002:fffed000       ?_Generic_object$initializer$@?$_Error_objects@H@std@@2P6AXXZA 10000000     EntropyAlgorithm.obj
 0002:fffed000       __catchsym$?node_copy@?$QList@V?$QSharedPointer@VGSequenceGraphData@U2@@@@@@AAEXPAUNode@1@00@Z$6 10000000     EntropyAlgorithm.obj
 0001:fffff000       __ehhandler$?node_copy@?$QList@V?$QSharedPointer@VGSequenceGraphData@U2@@@@@@AAEXPAUNode@1@00@Z 10000000 f   KarlinSignatureDifferenceGraph.obj
 0002:fffed000       __catchsym$?detach_helper_grow@?$QList@V?$QSharedPointer@VGSequenceGraphData@U2@@@@@@AAEPAUNode@1@HH@Z$5 10000000     EntropyAlgorithm.obj
 0000:fffe0000       .debug$S                   10000000     msvcprt:MSVCP120.dll
 0002:fffed000       __catchsym$?append@?$QList@V?$QSharedPointer@VGSequenceGraphData@U2@@@@@@QAEXABV?$QSharedPointer@VGSequenceGraphData@U2@@@@@Z$9 10000000     EntropyAlgorithm.obj
 0000:fffe0000       .debug$S                   10000000     msvcprt:MSVCP120.dll
 0001:fffff000       __ehhandler$?_Copy@?$basic_string@DU?$char_traits@D@std@@V?$allocator@D@2@@std@@QAEXII@Z 10000000 f   moc_KarlinSignatureDifferenceGraph.obj
 0002:fffed000       __catchsym$?reallocData@?$QVector@M@@AAEXHHV?$QFlags@W4AllocationOption@QArrayData@@@@@Z$5 10000000     EntropyAlgorithm.obj
 0002:fffed000       __catchsym$?_Copy@?$basic_string@DU?$char_traits@D@std@@V?$allocator@D@2@@std@@QAEXII@Z$5 10000000     DNAGraphPackPlugin.obj
 0000:fffe0000       .debug$S                   10000000     msvcprt:MSVCP120.dll
 0000:fffe0000       .debug$S                   10000000     msvcprt:MSVCP120.dll
 0000:fffe0000       .debug$S                   10000000     msvcprt:MSVCP120.dll
 0000:fffe0000       .debug$S                   10000000     kernel32:KERNEL32.dll
 0000:fffe0000       .debug$S                   10000000     kernel32:KERNEL32.dll
 0000:fffe0000       .debug$S                   10000000     kernel32:KERNEL32.dll
 0000:fffe0000       .debug$S                   10000000     kernel32:KERNEL32.dll
 0000:fffe0000       .debug$S                   10000000     kernel32:KERNEL32.dll
 0000:fffe0000       .debug$S                   10000000     kernel32:KERNEL32.dll
 0000:fffe0000       .debug$S                   10000000     kernel32:KERNEL32.dll
 0000:fffe0000       .debug$S                   10000000     kernel32:KERNEL32.dll
 0000:fffe0000       .debug$S                   10000000     kernel32:KERNEL32.dll
 0000:fffe0000       .debug$S                   10000000     Qt5Core:Qt5Core.dll
 0000:fffe0000       .debug$S                   10000000     Qt5Core:Qt5Core.dll
 0000:fffe0000       .debug$S                   10000000     Qt5Core:Qt5Core.dll
 0000:fffe0000       .debug$S                   10000000     Qt5Core:Qt5Core.dll
 0000:fffe0000       .debug$S                   10000000     Qt5Core:Qt5Core.dll
 0000:fffe0000       .debug$S                   10000000     Qt5Core:Qt5Core.dll
 0002:fffed000       ?_Generic_object$initializer$@?$_Error_objects@H@std@@2P6AXXZA 10000000     DNAGraphPackPlugin.obj
 0002:fffed000       __catchsym$?_Copy@?$basic_string@DU?$char_traits@D@std@@V?$allocator@D@2@@std@@QAEXII@Z$5 10000000     EntropyAlgorithm.obj
 0002:fffed000       ?_Iostream_object$initializer$@?$_Error_objects@H@std@@2P6AXXZA 10000000     DNAGraphPackPlugin.obj
 0002:fffed000       ?_System_object$initializer$@?$_Error_objects@H@std@@2P6AXXZA 10000000     DNAGraphPackPlugin.obj
 0002:fffed000       __catchsym$?_Copy@?$basic_string@DU?$char_traits@D@std@@V?$allocator@D@2@@std@@QAEXII@Z$5 10000000     moc_KarlinSignatureDifferenceGraph.obj
 0000:fffe0000       .debug$S                   10000000     Qt5Core:Qt5Core.dll
 0000:fffe0000       .debug$S                   10000000     Qt5Core:Qt5Core.dll
 0000:fffe0000       .debug$S                   10000000     Qt5Core:Qt5Core.dll
 0000:fffe0000       .debug$S                   10000000     Qt5Core:Qt5Core.dll
 0000:fffe0000       .debug$S                   10000000     Qt5Core:Qt5Core.dll
 0000:fffe0000       .debug$S                   10000000     Qt5Core:Qt5Core.dll
 0000:fffe0000       .debug$S                   10000000     Qt5Core:Qt5Core.dll
 0000:fffe0000       .debug$S                   10000000     Qt5Core:Qt5Core.dll
 0000:fffe0000       .debug$S                   10000000     Qt5Core:Qt5Core.dll
 0000:fffe0000       .debug$S                   10000000     Qt5Core:Qt5Core.dll
 0000:fffe0000       .debug$S                   10000000     Qt5Core:Qt5Core.dll
 0000:fffe0000       .debug$S                   10000000     Qt5Core:Qt5Core.dll
 0000:fffe0000       .debug$S                   10000000     Qt5Core:Qt5Core.dll
 0000:fffe0000       .debug$S                   10000000     Qt5Core:Qt5Core.dll
 0000:fffe0000       .debug$S                   10000000     Qt5Core:Qt5Core.dll
 0000:fffe0000       .debug$S                   10000000     Qt5Core:Qt5Core.dll
 0000:fffe0000       .debug$S                   10000000     Qt5Core:Qt5Core.dll
 0000:fffe0000       .debug$S                   10000000     Qt5Core:Qt5Core.dll
 0000:fffe0000       .debug$S                   10000000     Qt5Core:Qt5Core.dll
 0000:fffe0000       .debug$S                   10000000     Qt5Core:Qt5Core.dll
 0000:fffe0000       .debug$S                   10000000     Qt5Core:Qt5Core.dll
 0000:fffe0000       .debug$S                   10000000     Qt5Core:Qt5Core.dll
 0000:fffe0000       .debug$S                   10000000     Qt5Core:Qt5Core.dll
 0000:fffe0000       .debug$S                   10000000     Qt5Core:Qt5Core.dll
 0000:fffe0000       .debug$S                   10000000     Qt5Core:Qt5Core.dll
 0000:fffe0000       .debug$S                   10000000     Qt5Core:Qt5Core.dll
 0000:fffe0000       .debug$S                   10000000     Qt5Core:Qt5Core.dll
 0000:fffe0000       .debug$S                   10000000     Qt5Core:Qt5Core.dll
 0000:fffe0000       .debug$S                   10000000     Qt5Core:Qt5Core.dll
 0000:fffe0000       .debug$S                   10000000     Qt5Core:Qt5Core.dll
 0000:fffe0000       .debug$S                   10000000     Qt5Core:Qt5Core.dll
 0000:fffe0000       .debug$S                   10000000     Qt5Core:Qt5Core.dll
 0000:fffe0000       .debug$S                   10000000     Qt5Core:Qt5Core.dll
 0000:fffe0000       .debug$S                   10000000     Qt5Core:Qt5Core.dll
 0000:fffe0000       .debug$S                   10000000     Qt5Core:Qt5Core.dll
 0000:fffe0000       .debug$S                   10000000     Qt5Core:Qt5Core.dll
 0000:fffe0000       .debug$S                   10000000     Qt5Core:Qt5Core.dll
 0000:fffe0000       .debug$S                   10000000     Qt5Core:Qt5Core.dll
 0000:fffe0000       .debug$S                   10000000     Qt5Core:Qt5Core.dll
 0000:fffe0000       .debug$S                   10000000     Qt5Core:Qt5Core.dll
 0000:fffe0000       .debug$S                   10000000     Qt5Core:Qt5Core.dll
 0000:fffe0000       .debug$S                   10000000     Qt5Core:Qt5Core.dll
 0000:fffe0000       .debug$S                   10000000     Qt5Core:Qt5Core.dll
 0000:fffe0000       .debug$S                   10000000     Qt5Core:Qt5Core.dll
 0000:fffe0000       .debug$S                   10000000     Qt5Core:Qt5Core.dll
 0000:fffe0000       .debug$S                   10000000     Qt5Core:Qt5Core.dll
 0000:fffe0000       .debug$S                   10000000     Qt5Core:Qt5Core.dll
 0000:fffe0000       .debug$S                   10000000     Qt5Core:Qt5Core.dll
 0000:fffe0000       .debug$S                   10000000     Qt5Core:Qt5Core.dll
 0000:fffe0000       .debug$S                   10000000     Qt5Core:Qt5Core.dll
 0000:fffe0000       .debug$S                   10000000     Qt5Core:Qt5Core.dll
 0000:fffe0000       .debug$S                   10000000     Qt5Core:Qt5Core.dll
 0000:fffe0000       .debug$S                   10000000     Qt5Core:Qt5Core.dll
 0000:fffe0000       .debug$S                   10000000     Qt5Core:Qt5Core.dll
 0000:fffe0000       .debug$S                   10000000     Qt5Core:Qt5Core.dll
 0000:fffe0000       .debug$S                   10000000     Qt5Core:Qt5Core.dll
 0000:fffe0000       .debug$S                   10000000     Qt5Gui:Qt5Gui.dll
 0000:fffe0000       .debug$S                   10000000     Qt5Gui:Qt5Gui.dll
 0000:fffe0000       .debug$S                   10000000     Qt5Widgets:Qt5Widgets.dll
 0000:fffe0000       .debug$S                   10000000     Qt5Widgets:Qt5Widgets.dll
 0000:fffe0000       .debug$S                   10000000     U2View:U2View.dll
 0000:fffe0000       .debug$S                   10000000     U2View:U2View.dll
 0000:fffe0000       .debug$S                   10000000     U2View:U2View.dll
 0000:fffe0000       .debug$S                   10000000     U2View:U2View.dll
 0000:fffe0000       .debug$S                   10000000     U2View:U2View.dll
 0000:fffe0000       .debug$S                   10000000     U2View:U2View.dll
 0000:fffe0000       .debug$S                   10000000     U2View:U2View.dll
 0002:fffed000       ?_Generic_object$initializer$@?$_Error_objects@H@std@@2P6AXXZA 10000000     moc_KarlinSignatureDifferenceGraph.obj
 0002:fffed000       ?_Iostream_object$initializer$@?$_Error_objects@H@std@@2P6AXXZA 10000000     moc_KarlinSignatureDifferenceGraph.obj
 0002:fffed000       ?_System_object$initializer$@?$_Error_objects@H@std@@2P6AXXZA 10000000     moc_KarlinSignatureDifferenceGraph.obj
 0000:fffe0000       .debug$S                   10000000     U2View:U2View.dll
 0000:fffe0000       .debug$S                   10000000     U2View:U2View.dll
 0002:fffed000       ?_Generic_object$initializer$@?$_Error_objects@H@std@@2P6AXXZA 10000000     moc_DNAGraphPackPlugin.obj
 0000:fffe0000       .debug$S                   10000000     U2View:U2View.dll
 0002:fffed000       ?_Iostream_object$initializer$@?$_Error_objects@H@std@@2P6AXXZA 10000000     moc_DNAGraphPackPlugin.obj
 0000:fffe0000       .debug$S                   10000000     U2View:U2View.dll
 0002:fffed000       ?_System_object$initializer$@?$_Error_objects@H@std@@2P6AXXZA 10000000     moc_DNAGraphPackPlugin.obj
 0000:fffe0000       .debug$S                   10000000     U2View:U2View.dll
 0002:fffed000       __catchsym$?_Copy@?$basic_string@DU?$char_traits@D@std@@V?$allocator@D@2@@std@@QAEXII@Z$5 10000000     KarlinSignatureDifferenceGraph.obj
 0000:fffe0000       .debug$S                   10000000     U2View:U2View.dll
 0001:fffff000       __ehhandler$?node_copy@?$QList@V?$QSharedPointer@VGSequenceGraphData@U2@@@@@@AAEXPAUNode@1@00@Z 10000000 f   EntropyAlgorithm.obj
 0000:fffe0000       .debug$S                   10000000     U2View:U2View.dll
 0002:fffed000       ?_System_object$initializer$@?$_Error_objects@H@std@@2P6AXXZA 10000000     moc_EntropyAlgorithm.obj
 0000:fffe0000       .debug$S                   10000000     U2View:U2View.dll
 0002:fffed000       ?_Iostream_object$initializer$@?$_Error_objects@H@std@@2P6AXXZA 10000000     moc_EntropyAlgorithm.obj
 0000:fffe0000       .debug$S                   10000000     U2View:U2View.dll
 0002:fffed000       ?_Generic_object$initializer$@?$_Error_objects@H@std@@2P6AXXZA 10000000     moc_EntropyAlgorithm.obj
 0000:fffe0000       .debug$S                   10000000     U2View:U2View.dll
 0002:fffed000       __catchsym$?reallocData@?$QVector@M@@AAEXHHV?$QFlags@W4AllocationOption@QArrayData@@@@@Z$5 10000000     KarlinSignatureDifferenceGraph.obj
 0000:fffe0000       .debug$S                   10000000     U2View:U2View.dll
 0001:fffff000       __ehhandler$?_Copy@?$basic_string@DU?$char_traits@D@std@@V?$allocator@D@2@@std@@QAEXII@Z 10000000 f   CumulativeSkew.obj
 0000:fffe0000       .debug$S                   10000000     U2View:U2View.dll
 0001:fffff000       __ehhandler$?detach_helper_grow@?$QList@V?$QSharedPointer@VGSequenceGraphData@U2@@@@@@AAEPAUNode@1@HH@Z 10000000 f   EntropyAlgorithm.obj
 0000:fffe0000       .debug$S                   10000000     U2View:U2View.dll
 0001:fffff000       __ehhandler$?append@?$QList@V?$QSharedPointer@VGSequenceGraphData@U2@@@@@@QAEXABV?$QSharedPointer@VGSequenceGraphData@U2@@@@@Z 10000000 f   EntropyAlgorithm.obj
 0000:fffe0000       .debug$S                   10000000     U2View:U2View.dll
 0001:fffff000       __ehhandler$?reallocData@?$QVector@M@@AAEXHHV?$QFlags@W4AllocationOption@QArrayData@@@@@Z 10000000 f   EntropyAlgorithm.obj
 0000:fffe0000       .debug$S                   10000000     U2Gui:U2Gui.dll
 0002:fffed000       __catchsym$?append@?$QList@V?$QSharedPointer@VGSequenceGraphData@U2@@@@@@QAEXABV?$QSharedPointer@VGSequenceGraphData@U2@@@@@Z$9 10000000     KarlinSignatureDifferenceGraph.obj
 0000:fffe0000       .debug$S                   10000000     U2Gui:U2Gui.dll
 0001:fffff000       __ehhandler$?_Copy@?$basic_string@DU?$char_traits@D@std@@V?$allocator@D@2@@std@@QAEXII@Z 10000000 f   moc_CumulativeSkew.obj
 0000:fffe0000       .debug$S                   10000000     U2Gui:U2Gui.dll
 0001:fffff000       __ehhandler$?_Copy@?$basic_string@DU?$char_traits@D@std@@V?$allocator@D@2@@std@@QAEXII@Z 10000000 f   EntropyAlgorithm.obj
 0000:fffe0000       .debug$S                   10000000     U2Gui:U2Gui.dll
 0001:fffff000       __ehhandler$?reallocData@?$QVector@M@@AAEXHHV?$QFlags@W4AllocationOption@QArrayData@@@@@Z 10000000 f   CumulativeSkew.obj
 0000:fffe0000       .debug$S                   10000000     U2Gui:U2Gui.dll
 0001:fffff000       __ehhandler$?append@?$QList@V?$QSharedPointer@VGSequenceGraphData@U2@@@@@@QAEXABV?$QSharedPointer@VGSequenceGraphData@U2@@@@@Z 10000000 f   CumulativeSkew.obj
 0000:fffe0000       .debug$S                   10000000     U2Gui:U2Gui.dll
 0002:fffed000       __catchsym$?detach_helper_grow@?$QList@V?$QSharedPointer@VGSequenceGraphData@U2@@@@@@AAEPAUNode@1@HH@Z$5 10000000     KarlinSignatureDifferenceGraph.obj
 0000:fffe0000       .debug$S                   10000000     U2Gui:U2Gui.dll
 0001:fffff000       __ehhandler$?detach_helper_grow@?$QList@V?$QSharedPointer@VGSequenceGraphData@U2@@@@@@AAEPAUNode@1@HH@Z 10000000 f   CumulativeSkew.obj
 0000:fffe0000       .debug$S                   10000000     U2Gui:U2Gui.dll
 0001:fffff000       __ehhandler$?node_copy@?$QList@V?$QSharedPointer@VGSequenceGraphData@U2@@@@@@AAEXPAUNode@1@00@Z 10000000 f   CumulativeSkew.obj
 0000:fffe0000       .debug$S                   10000000     U2Gui:U2Gui.dll
 0002:fffed000       __catchsym$?_Copy@?$basic_string@DU?$char_traits@D@std@@V?$allocator@D@2@@std@@QAEXII@Z$5 10000000     moc_CumulativeSkew.obj
 0000:fffe0000       .debug$S                   10000000     U2Gui:U2Gui.dll
 0002:fffed000       __catchsym$?node_copy@?$QList@V?$QSharedPointer@VGSequenceGraphData@U2@@@@@@AAEXPAUNode@1@00@Z$6 10000000     KarlinSignatureDifferenceGraph.obj
 0002:fffed000       ?_Generic_object$initializer$@?$_Error_objects@H@std@@2P6AXXZA 10000000     KarlinSignatureDifferenceGraph.obj
 0000:fffe0000       .debug$S                   10000000     U2Gui:U2Gui.dll
 0002:fffed000       ?_Iostream_object$initializer$@?$_Error_objects@H@std@@2P6AXXZA 10000000     KarlinSignatureDifferenceGraph.obj
 0000:fffe0000       .debug$S                   10000000     U2Gui:U2Gui.dll
 0002:fffed000       ?_System_object$initializer$@?$_Error_objects@H@std@@2P6AXXZA 10000000     KarlinSignatureDifferenceGraph.obj
 0000:fffe0000       .debug$S                   10000000     U2Gui:U2Gui.dll
 0001:fffff000       __ehhandler$?_Copy@?$basic_string@DU?$char_traits@D@std@@V?$allocator@D@2@@std@@QAEXII@Z 10000000 f   moc_GCFramePlot.obj
 0002:fffed000       __catchsym$?_Copy@?$basic_string@DU?$char_traits@D@std@@V?$allocator@D@2@@std@@QAEXII@Z$5 10000000     CumulativeSkew.obj
 0002:fffed000       __catchsym$?reallocData@?$QVector@M@@AAEXHHV?$QFlags@W4AllocationOption@QArrayData@@@@@Z$5 10000000     CumulativeSkew.obj
 0000:fffe0000       .debug$S                   10000000     U2Gui:U2Gui.dll
 0000:fffe0000       .debug$S                   10000000     U2Gui:U2Gui.dll
 0000:fffe0000       .debug$S                   10000000     U2Core:U2Core.dll
 0000:fffe0000       .debug$S                   10000000     U2Core:U2Core.dll
 0000:fffe0000       .debug$S                   10000000     U2Core:U2Core.dll
 0000:fffe0000       .debug$S                   10000000     U2Core:U2Core.dll
 0000:fffe0000       .debug$S                   10000000     U2Core:U2Core.dll
 0000:fffe0000       .debug$S                   10000000     U2Core:U2Core.dll
 0000:fffe0000       .debug$S                   10000000     U2Core:U2Core.dll
 0000:fffe0000       .debug$S                   10000000     U2Core:U2Core.dll
 0000:fffe0000       .debug$S                   10000000     U2Core:U2Core.dll
 0000:fffe0000       .debug$S                   10000000     U2Core:U2Core.dll
 0000:fffe0000       .debug$S                   10000000     U2Core:U2Core.dll
 0000:fffe0000       .debug$S                   10000000     U2Core:U2Core.dll
 0000:fffe0000       .debug$S                   10000000     U2Core:U2Core.dll
 0000:fffe0000       .debug$S                   10000000     U2Core:U2Core.dll
 0000:fffe0000       .debug$S                   10000000     U2Core:U2Core.dll
 0000:fffe0000       .debug$S                   10000000     U2Core:U2Core.dll
 0002:fffed000       __catchsym$?_Copy@?$basic_string@DU?$char_traits@D@std@@V?$allocator@D@2@@std@@QAEXII@Z$5 10000000     moc_EntropyAlgorithm.obj
 0002:fffed000       __catchsym$?append@?$QList@V?$QSharedPointer@VGSequenceGraphData@U2@@@@@@QAEXABV?$QSharedPointer@VGSequenceGraphData@U2@@@@@Z$9 10000000     CumulativeSkew.obj
 0002:fffed000       __catchsym$?detach_helper_grow@?$QList@V?$QSharedPointer@VGSequenceGraphData@U2@@@@@@AAEPAUNode@1@HH@Z$5 10000000     CumulativeSkew.obj
 0002:fffed000       __catchsym$?node_copy@?$QList@V?$QSharedPointer@VGSequenceGraphData@U2@@@@@@AAEXPAUNode@1@00@Z$6 10000000     CumulativeSkew.obj
 0002:fffed000       __catchsym$?_Copy@?$basic_string@DU?$char_traits@D@std@@V?$allocator@D@2@@std@@QAEXII@Z$5 10000000     moc_GCFramePlot.obj
 0000:fffe0000       .debug$S                   10000000     U2Core:U2Core.dll
 0000:fffe0000       .debug$S                   10000000     U2Core:U2Core.dll
 0000:fffe0000       .debug$S                   10000000     U2Core:U2Core.dll
 0002:fffed000       ?_Generic_object$initializer$@?$_Error_objects@H@std@@2P6AXXZA 10000000     CumulativeSkew.obj
 0002:fffed000       ?_Iostream_object$initializer$@?$_Error_objects@H@std@@2P6AXXZA 10000000     CumulativeSkew.obj
 0002:fffed000       ?_System_object$initializer$@?$_Error_objects@H@std@@2P6AXXZA 10000000     CumulativeSkew.obj
 0001:fffff000       __ehhandler$?_Copy@?$basic_string@DU?$char_traits@D@std@@V?$allocator@D@2@@std@@QAEXII@Z 10000000 f   moc_EntropyAlgorithm.obj
 0002:fffed000       ?_System_object$initializer$@?$_Error_objects@H@std@@2P6AXXZA 10000000     GCFramePlot.obj
 0002:fffed000       ?_Iostream_object$initializer$@?$_Error_objects@H@std@@2P6AXXZA 10000000     GCFramePlot.obj
 0002:fffed000       ?_Generic_object$initializer$@?$_Error_objects@H@std@@2P6AXXZA 10000000     GCFramePlot.obj
 0002:fffed000       __catchsym$?node_copy@?$QList@V?$QSharedPointer@VGSequenceGraphData@U2@@@@@@AAEXPAUNode@1@00@Z$6 10000000     GCFramePlot.obj
 0002:fffed000       __catchsym$?detach_helper_grow@?$QList@V?$QSharedPointer@VGSequenceGraphData@U2@@@@@@AAEPAUNode@1@HH@Z$5 10000000     GCFramePlot.obj
 0002:fffed000       __catchsym$?_Copy@?$basic_string@DU?$char_traits@D@std@@V?$allocator@D@2@@std@@QAEXII@Z$5 10000000     DeviationGraph.obj
 0002:fffed000       __catchsym$?append@?$QList@V?$QSharedPointer@VGSequenceGraphData@U2@@@@@@QAEXABV?$QSharedPointer@VGSequenceGraphData@U2@@@@@Z$9 10000000     GCFramePlot.obj
 0002:fffed000       ?_System_object$initializer$@?$_Error_objects@H@std@@2P6AXXZA 10000000     moc_GCFramePlot.obj
 0002:fffed000       ?_Iostream_object$initializer$@?$_Error_objects@H@std@@2P6AXXZA 10000000     moc_GCFramePlot.obj
 0002:fffed000       ?_Generic_object$initializer$@?$_Error_objects@H@std@@2P6AXXZA 10000000     moc_GCFramePlot.obj
 0002:fffed000       __catchsym$?reallocData@?$QVector@M@@AAEXHHV?$QFlags@W4AllocationOption@QArrayData@@@@@Z$5 10000000     GCFramePlot.obj
 0002:fffed000       __catchsym$?_Copy@?$basic_string@DU?$char_traits@D@std@@V?$allocator@D@2@@std@@QAEXII@Z$5 10000000     GCFramePlot.obj
 0002:fffed000       ?_Generic_object$initializer$@?$_Error_objects@H@std@@2P6AXXZA 10000000     moc_CumulativeSkew.obj
 0002:fffed000       __catchsym$?_Copy@?$basic_string@DU?$char_traits@D@std@@V?$allocator@D@2@@std@@QAEXII@Z$5 10000000     moc_BaseContentGraph.obj
 0002:fffed000       ?_Iostream_object$initializer$@?$_Error_objects@H@std@@2P6AXXZA 10000000     moc_CumulativeSkew.obj
 0002:fffed000       ?_System_object$initializer$@?$_Error_objects@H@std@@2P6AXXZA 10000000     moc_CumulativeSkew.obj
 0001:fffff000       __ehhandler$?node_copy@?$QList@V?$QSharedPointer@VGSequenceGraphData@U2@@@@@@AAEXPAUNode@1@00@Z 10000000 f   GCFramePlot.obj
 0001:fffff000       __ehhandler$?detach_helper_grow@?$QList@V?$QSharedPointer@VGSequenceGraphData@U2@@@@@@AAEPAUNode@1@HH@Z 10000000 f   GCFramePlot.obj
 0001:fffff000       __ehhandler$?append@?$QList@V?$QSharedPointer@VGSequenceGraphData@U2@@@@@@QAEXABV?$QSharedPointer@VGSequenceGraphData@U2@@@@@Z 10000000 f   GCFramePlot.obj
 0001:fffff000       __ehhandler$?reallocData@?$QVector@M@@AAEXHHV?$QFlags@W4AllocationOption@QArrayData@@@@@Z 10000000 f   GCFramePlot.obj
 0001:fffff000       __ehhandler$?_Copy@?$basic_string@DU?$char_traits@D@std@@V?$allocator@D@2@@std@@QAEXII@Z 10000000 f   moc_BaseContentGraph.obj
 0001:fffff000       __ehhandler$?_Copy@?$basic_string@DU?$char_traits@D@std@@V?$allocator@D@2@@std@@QAEXII@Z 10000000 f   GCFramePlot.obj
 0002:fffed010       __catchsym$?_Copy@?$basic_string@DU?$char_traits@D@std@@V?$allocator@D@2@@std@@QAEXII@Z$4 10000010     moc_EntropyAlgorithm.obj
 0002:fffed010       __catchsym$?_Copy@?$basic_string@DU?$char_traits@D@std@@V?$allocator@D@2@@std@@QAEXII@Z$4 10000010     DeviationGraph.obj
 0002:fffed010       __catchsym$?detach_helper_grow@?$QList@V?$QSharedPointer@VGSequenceGraphData@U2@@@@@@AAEPAUNode@1@HH@Z$4 10000010     EntropyAlgorithm.obj
 0002:fffed010       __catchsym$?detach_helper_grow@?$QList@V?$QSharedPointer@VGSequenceGraphData@U2@@@@@@AAEPAUNode@1@HH@Z$4 10000010     CumulativeSkew.obj
 0002:fffed010       __tryblocktable$?node_copy@?$QList@V?$QSharedPointer@VGSequenceGraphData@U2@@@@@@AAEXPAUNode@1@00@Z 10000010     CumulativeSkew.obj
 0002:fffed010       __catchsym$?append@?$QList@V?$QSharedPointer@VGSequenceGraphData@U2@@@@@@QAEXABV?$QSharedPointer@VGSequenceGraphData@U2@@@@@Z$8 10000010     EntropyAlgorithm.obj
 0002:fffed010       __catchsym$?append@?$QList@V?$QSharedPointer@VGSequenceGraphData@U2@@@@@@QAEXABV?$QSharedPointer@VGSequenceGraphData@U2@@@@@Z$8 10000010     CumulativeSkew.obj
 0002:fffed010       __catchsym$?detach_helper_grow@?$QList@V?$QSharedPointer@VGSequenceGraphData@U2@@@@@@AAEPAUNode@1@HH@Z$4 10000010     DeviationGraph.obj
 0002:fffed010       __catchsym$?reallocData@?$QVector@M@@AAEXHHV?$QFlags@W4AllocationOption@QArrayData@@@@@Z$4 10000010     EntropyAlgorithm.obj
 0002:fffed010       __tryblocktable$?node_copy@?$QList@V?$QSharedPointer@VGSequenceGraphData@U2@@@@@@AAEXPAUNode@1@00@Z 10000010     GCFramePlot.obj
 0002:fffed010       __catchsym$?_Copy@?$basic_string@DU?$char_traits@D@std@@V?$allocator@D@2@@std@@QAEXII@Z$4 10000010     DNAGraphPackPlugin.obj
 0002:fffed010       __catchsym$?_Copy@?$basic_string@DU?$char_traits@D@std@@V?$allocator@D@2@@std@@QAEXII@Z$4 10000010     moc_GCFramePlot.obj
 0002:fffed010       __catchsym$?_Copy@?$basic_string@DU?$char_traits@D@std@@V?$allocator@D@2@@std@@QAEXII@Z$4 10000010     moc_DeviationGraph.obj
 0002:fffed010       __catchsym$?_Copy@?$basic_string@DU?$char_traits@D@std@@V?$allocator@D@2@@std@@QAEXII@Z$4 10000010     EntropyAlgorithm.obj
 0002:fffed010       __catchsym$?_Copy@?$basic_string@DU?$char_traits@D@std@@V?$allocator@D@2@@std@@QAEXII@Z$4 10000010     moc_KarlinSignatureDifferenceGraph.obj
 0002:fffed010       __catchsym$?reallocData@?$QVector@M@@AAEXHHV?$QFlags@W4AllocationOption@QArrayData@@@@@Z$4 10000010     CumulativeSkew.obj
 0002:fffed010       __catchsym$?detach_helper_grow@?$QList@V?$QSharedPointer@VGSequenceGraphData@U2@@@@@@AAEPAUNode@1@HH@Z$4 10000010     GCFramePlot.obj
 0002:fffed010       __catchsym$?_Copy@?$basic_string@DU?$char_traits@D@std@@V?$allocator@D@2@@std@@QAEXII@Z$4 10000010     KarlinSignatureDifferenceGraph.obj
 0002:fffed010       __catchsym$?_Copy@?$basic_string@DU?$char_traits@D@std@@V?$allocator@D@2@@std@@QAEXII@Z$4 10000010     CumulativeSkew.obj
 0002:fffed010       __catchsym$?append@?$QList@V?$QSharedPointer@VGSequenceGraphData@U2@@@@@@QAEXABV?$QSharedPointer@VGSequenceGraphData@U2@@@@@Z$8 10000010     DeviationGraph.obj
 0002:fffed010       __catchsym$?reallocData@?$QVector@M@@AAEXHHV?$QFlags@W4AllocationOption@QArrayData@@@@@Z$4 10000010     KarlinSignatureDifferenceGraph.obj
 0002:fffed010       __tryblocktable$?node_copy@?$QList@V?$QSharedPointer@VGSequenceGraphData@U2@@@@@@AAEXPAUNode@1@00@Z 10000010     EntropyAlgorithm.obj
 0002:fffed010       __catchsym$?_Copy@?$basic_string@DU?$char_traits@D@std@@V?$allocator@D@2@@std@@QAEXII@Z$4 10000010     moc_BaseContentGraph.obj
 0002:fffed010       __catchsym$?reallocData@?$QVector@M@@AAEXHHV?$QFlags@W4AllocationOption@QArrayData@@@@@Z$4 10000010     DeviationGraph.obj
 0002:fffed010       __tryblocktable$?node_copy@?$QList@V?$QSharedPointer@VGSequenceGraphData@U2@@@@@@AAEXPAUNode@1@00@Z 10000010     KarlinSignatureDifferenceGraph.obj
 0002:fffed010       __catchsym$?append@?$QList@V?$QSharedPointer@VGSequenceGraphData@U2@@@@@@QAEXABV?$QSharedPointer@VGSequenceGraphData@U2@@@@@Z$8 10000010     GCFramePlot.obj
 0002:fffed010       __catchsym$?append@?$QList@V?$QSharedPointer@VGSequenceGraphData@U2@@@@@@QAEXABV?$QSharedPointer@VGSequenceGraphData@U2@@@@@Z$8 10000010     KarlinSignatureDifferenceGraph.obj
 0002:fffed010       __catchsym$?_Copy@?$basic_string@DU?$char_traits@D@std@@V?$allocator@D@2@@std@@QAEXII@Z$4 10000010     GCFramePlot.obj
 0002:fffed010       __catchsym$?_Copy@?$basic_string@DU?$char_traits@D@std@@V?$allocator@D@2@@std@@QAEXII@Z$4 10000010     moc_CumulativeSkew.obj
 0002:fffed010       __catchsym$?detach_helper_grow@?$QList@V?$QSharedPointer@VGSequenceGraphData@U2@@@@@@AAEPAUNode@1@HH@Z$4 10000010     KarlinSignatureDifferenceGraph.obj
 0002:fffed010       __tryblocktable$?node_copy@?$QList@V?$QSharedPointer@VGSequenceGraphData@U2@@@@@@AAEXPAUNode@1@00@Z 10000010     DeviationGraph.obj
 0002:fffed010       __catchsym$?_Copy@?$basic_string@DU?$char_traits@D@std@@V?$allocator@D@2@@std@@QAEXII@Z$4 10000010     moc_DNAGraphPackPlugin.obj
 0002:fffed010       __catchsym$?reallocData@?$QVector@M@@AAEXHHV?$QFlags@W4AllocationOption@QArrayData@@@@@Z$4 10000010     GCFramePlot.obj
 0002:fffed020       __ehfuncinfo$?append@?$QList@V?$QSharedPointer@VGSequenceGraphData@U2@@@@@@QAEXABV?$QSharedPointer@VGSequenceGraphData@U2@@@@@Z 10000020     DeviationGraph.obj
 0002:fffed020       __ehfuncinfo$?append@?$QList@V?$QSharedPointer@VGSequenceGraphData@U2@@@@@@QAEXABV?$QSharedPointer@VGSequenceGraphData@U2@@@@@Z 10000020     GCFramePlot.obj
 0002:fffed020       __unwindtable$?_Copy@?$basic_string@DU?$char_traits@D@std@@V?$allocator@D@2@@std@@QAEXII@Z 10000020     moc_CumulativeSkew.obj
 0002:fffed020       __unwindtable$?detach_helper_grow@?$QList@V?$QSharedPointer@VGSequenceGraphData@U2@@@@@@AAEPAUNode@1@HH@Z 10000020     KarlinSignatureDifferenceGraph.obj
 0002:fffed020       __unwindtable$?_Copy@?$basic_string@DU?$char_traits@D@std@@V?$allocator@D@2@@std@@QAEXII@Z 10000020     GCFramePlot.obj
 0002:fffed020       __ehfuncinfo$?append@?$QList@V?$QSharedPointer@VGSequenceGraphData@U2@@@@@@QAEXABV?$QSharedPointer@VGSequenceGraphData@U2@@@@@Z 10000020     KarlinSignatureDifferenceGraph.obj
 0002:fffed020       __unwindtable$?_Copy@?$basic_string@DU?$char_traits@D@std@@V?$allocator@D@2@@std@@QAEXII@Z 10000020     moc_DeviationGraph.obj
 0002:fffed020       __unwindtable$?_Copy@?$basic_string@DU?$char_traits@D@std@@V?$allocator@D@2@@std@@QAEXII@Z 10000020     moc_BaseContentGraph.obj
 0002:fffed020       __unwindtable$?_Copy@?$basic_string@DU?$char_traits@D@std@@V?$allocator@D@2@@std@@QAEXII@Z 10000020     CumulativeSkew.obj
 0002:fffed020       __unwindtable$?detach_helper_grow@?$QList@V?$QSharedPointer@VGSequenceGraphData@U2@@@@@@AAEPAUNode@1@HH@Z 10000020     DeviationGraph.obj
 0002:fffed020       __unwindtable$?detach_helper_grow@?$QList@V?$QSharedPointer@VGSequenceGraphData@U2@@@@@@AAEPAUNode@1@HH@Z 10000020     GCFramePlot.obj
 0002:fffed020       __unwindtable$?reallocData@?$QVector@M@@AAEXHHV?$QFlags@W4AllocationOption@QArrayData@@@@@Z 10000020     KarlinSignatureDifferenceGraph.obj
 0002:fffed020       __unwindtable$?_Copy@?$basic_string@DU?$char_traits@D@std@@V?$allocator@D@2@@std@@QAEXII@Z 10000020     KarlinSignatureDifferenceGraph.obj
 0002:fffed020       __unwindtable$?reallocData@?$QVector@M@@AAEXHHV?$QFlags@W4AllocationOption@QArrayData@@@@@Z 10000020     CumulativeSkew.obj
 0002:fffed020       __unwindtable$?_Copy@?$basic_string@DU?$char_traits@D@std@@V?$allocator@D@2@@std@@QAEXII@Z 10000020     EntropyAlgorithm.obj
 0002:fffed020       __ehfuncinfo$?append@?$QList@V?$QSharedPointer@VGSequenceGraphData@U2@@@@@@QAEXABV?$QSharedPointer@VGSequenceGraphData@U2@@@@@Z 10000020     CumulativeSkew.obj
 0002:fffed020       __unwindtable$?_Copy@?$basic_string@DU?$char_traits@D@std@@V?$allocator@D@2@@std@@QAEXII@Z 10000020     moc_KarlinSignatureDifferenceGraph.obj
 0002:fffed020       __unwindtable$?_Copy@?$basic_string@DU?$char_traits@D@std@@V?$allocator@D@2@@std@@QAEXII@Z 10000020     moc_EntropyAlgorithm.obj
 0002:fffed020       __unwindtable$?reallocData@?$QVector@M@@AAEXHHV?$QFlags@W4AllocationOption@QArrayData@@@@@Z 10000020     EntropyAlgorithm.obj
 0002:fffed020       __unwindtable$?_Copy@?$basic_string@DU?$char_traits@D@std@@V?$allocator@D@2@@std@@QAEXII@Z 10000020     DeviationGraph.obj
 0002:fffed020       __unwindtable$?_Copy@?$basic_string@DU?$char_traits@D@std@@V?$allocator@D@2@@std@@QAEXII@Z 10000020     DNAGraphPackPlugin.obj
 0002:fffed020       __ehfuncinfo$?append@?$QList@V?$QSharedPointer@VGSequenceGraphData@U2@@@@@@QAEXABV?$QSharedPointer@VGSequenceGraphData@U2@@@@@Z 10000020     EntropyAlgorithm.obj
 0002:fffed020       __unwindtable$?_Copy@?$basic_string@DU?$char_traits@D@std@@V?$allocator@D@2@@std@@QAEXII@Z 10000020     moc_GCFramePlot.obj
 0002:fffed020       __unwindtable$?detach_helper_grow@?$QList@V?$QSharedPointer@VGSequenceGraphData@U2@@@@@@AAEPAUNode@1@HH@Z 10000020     CumulativeSkew.obj
 0002:fffed020       __unwindtable$?reallocData@?$QVector@M@@AAEXHHV?$QFlags@W4AllocationOption@QArrayData@@@@@Z 10000020     DeviationGraph.obj
 0002:fffed020       __unwindtable$?detach_helper_grow@?$QList@V?$QSharedPointer@VGSequenceGraphData@U2@@@@@@AAEPAUNode@1@HH@Z 10000020     EntropyAlgorithm.obj
 0002:fffed020       __unwindtable$?reallocData@?$QVector@M@@AAEXHHV?$QFlags@W4AllocationOption@QArrayData@@@@@Z 10000020     GCFramePlot.obj
 0002:fffed020       __unwindtable$?_Copy@?$basic_string@DU?$char_traits@D@std@@V?$allocator@D@2@@std@@QAEXII@Z 10000020     moc_DNAGraphPackPlugin.obj
 0002:fffed024       __unwindtable$?node_copy@?$QList@V?$QSharedPointer@VGSequenceGraphData@U2@@@@@@AAEXPAUNode@1@00@Z 10000024     GCFramePlot.obj
 0002:fffed024       __unwindtable$?node_copy@?$QList@V?$QSharedPointer@VGSequenceGraphData@U2@@@@@@AAEXPAUNode@1@00@Z 10000024     EntropyAlgorithm.obj
 0002:fffed024       __unwindtable$?node_copy@?$QList@V?$QSharedPointer@VGSequenceGraphData@U2@@@@@@AAEXPAUNode@1@00@Z 10000024     KarlinSignatureDifferenceGraph.obj
 0002:fffed024       __unwindtable$?node_copy@?$QList@V?$QSharedPointer@VGSequenceGraphData@U2@@@@@@AAEXPAUNode@1@00@Z 10000024     DeviationGraph.obj
 0002:fffed024       __unwindtable$?node_copy@?$QList@V?$QSharedPointer@VGSequenceGraphData@U2@@@@@@AAEXPAUNode@1@00@Z 10000024     CumulativeSkew.obj
 0002:fffed040       __ehfuncinfo$?detach_helper_grow@?$QList@V?$QSharedPointer@VGSequenceGraphData@U2@@@@@@AAEPAUNode@1@HH@Z 10000040     GCFramePlot.obj
 0002:fffed040       __ehfuncinfo$?_Copy@?$basic_string@DU?$char_traits@D@std@@V?$allocator@D@2@@std@@QAEXII@Z 10000040     moc_KarlinSignatureDifferenceGraph.obj
 0002:fffed040       __ehfuncinfo$?_Copy@?$basic_string@DU?$char_traits@D@std@@V?$allocator@D@2@@std@@QAEXII@Z 10000040     moc_EntropyAlgorithm.obj
 0002:fffed040       __ehfuncinfo$?reallocData@?$QVector@M@@AAEXHHV?$QFlags@W4AllocationOption@QArrayData@@@@@Z 10000040     KarlinSignatureDifferenceGraph.obj
 0002:fffed040       __ehfuncinfo$?reallocData@?$QVector@M@@AAEXHHV?$QFlags@W4AllocationOption@QArrayData@@@@@Z 10000040     EntropyAlgorithm.obj
 0002:fffed040       __ehfuncinfo$?_Copy@?$basic_string@DU?$char_traits@D@std@@V?$allocator@D@2@@std@@QAEXII@Z 10000040     moc_BaseContentGraph.obj
 0002:fffed040       __ehfuncinfo$?reallocData@?$QVector@M@@AAEXHHV?$QFlags@W4AllocationOption@QArrayData@@@@@Z 10000040     DeviationGraph.obj
 0002:fffed040       __ehfuncinfo$?_Copy@?$basic_string@DU?$char_traits@D@std@@V?$allocator@D@2@@std@@QAEXII@Z 10000040     EntropyAlgorithm.obj
 0002:fffed040       __ehfuncinfo$?detach_helper_grow@?$QList@V?$QSharedPointer@VGSequenceGraphData@U2@@@@@@AAEPAUNode@1@HH@Z 10000040     CumulativeSkew.obj
 0002:fffed040       __ehfuncinfo$?reallocData@?$QVector@M@@AAEXHHV?$QFlags@W4AllocationOption@QArrayData@@@@@Z 10000040     CumulativeSkew.obj
 0002:fffed040       __ehfuncinfo$?detach_helper_grow@?$QList@V?$QSharedPointer@VGSequenceGraphData@U2@@@@@@AAEPAUNode@1@HH@Z 10000040     DeviationGraph.obj
 0002:fffed040       __ehfuncinfo$?_Copy@?$basic_string@DU?$char_traits@D@std@@V?$allocator@D@2@@std@@QAEXII@Z 10000040     CumulativeSkew.obj
 0002:fffed040       __ehfuncinfo$?detach_helper_grow@?$QList@V?$QSharedPointer@VGSequenceGraphData@U2@@@@@@AAEPAUNode@1@HH@Z 10000040     EntropyAlgorithm.obj
 0002:fffed040       __ehfuncinfo$?_Copy@?$basic_string@DU?$char_traits@D@std@@V?$allocator@D@2@@std@@QAEXII@Z 10000040     DeviationGraph.obj
 0002:fffed040       __ehfuncinfo$?_Copy@?$basic_string@DU?$char_traits@D@std@@V?$allocator@D@2@@std@@QAEXII@Z 10000040     KarlinSignatureDifferenceGraph.obj
 0002:fffed040       __ehfuncinfo$?_Copy@?$basic_string@DU?$char_traits@D@std@@V?$allocator@D@2@@std@@QAEXII@Z 10000040     moc_DNAGraphPackPlugin.obj
 0002:fffed040       __ehfuncinfo$?_Copy@?$basic_string@DU?$char_traits@D@std@@V?$allocator@D@2@@std@@QAEXII@Z 10000040     GCFramePlot.obj
 0002:fffed040       __ehfuncinfo$?_Copy@?$basic_string@DU?$char_traits@D@std@@V?$allocator@D@2@@std@@QAEXII@Z 10000040     moc_DeviationGraph.obj
 0002:fffed040       __ehfuncinfo$?_Copy@?$basic_string@DU?$char_traits@D@std@@V?$allocator@D@2@@std@@QAEXII@Z 10000040     moc_CumulativeSkew.obj
 0002:fffed040       __ehfuncinfo$?reallocData@?$QVector@M@@AAEXHHV?$QFlags@W4AllocationOption@QArrayData@@@@@Z 10000040     GCFramePlot.obj
 0002:fffed040       __ehfuncinfo$?_Copy@?$basic_string@DU?$char_traits@D@std@@V?$allocator@D@2@@std@@QAEXII@Z 10000040     DNAGraphPackPlugin.obj
 0002:fffed040       __ehfuncinfo$?detach_helper_grow@?$QList@V?$QSharedPointer@VGSequenceGraphData@U2@@@@@@AAEPAUNode@1@HH@Z 10000040     KarlinSignatureDifferenceGraph.obj
 0002:fffed040       __ehfuncinfo$?_Copy@?$basic_string@DU?$char_traits@D@std@@V?$allocator@D@2@@std@@QAEXII@Z 10000040     moc_GCFramePlot.obj
 0002:fffed044       __ehfuncinfo$?node_copy@?$QList@V?$QSharedPointer@VGSequenceGraphData@U2@@@@@@AAEXPAUNode@1@00@Z 10000044     EntropyAlgorithm.obj
 0002:fffed044       __tryblocktable$?append@?$QList@V?$QSharedPointer@VGSequenceGraphData@U2@@@@@@QAEXABV?$QSharedPointer@VGSequenceGraphData@U2@@@@@Z 10000044     CumulativeSkew.obj
 0002:fffed044       __ehfuncinfo$?node_copy@?$QList@V?$QSharedPointer@VGSequenceGraphData@U2@@@@@@AAEXPAUNode@1@00@Z 10000044     KarlinSignatureDifferenceGraph.obj
 0002:fffed044       __ehfuncinfo$?node_copy@?$QList@V?$QSharedPointer@VGSequenceGraphData@U2@@@@@@AAEXPAUNode@1@00@Z 10000044     DeviationGraph.obj
 0002:fffed044       __tryblocktable$?append@?$QList@V?$QSharedPointer@VGSequenceGraphData@U2@@@@@@QAEXABV?$QSharedPointer@VGSequenceGraphData@U2@@@@@Z 10000044     EntropyAlgorithm.obj
 0002:fffed044       __ehfuncinfo$?node_copy@?$QList@V?$QSharedPointer@VGSequenceGraphData@U2@@@@@@AAEXPAUNode@1@00@Z 10000044     CumulativeSkew.obj
 0002:fffed044       __tryblocktable$?append@?$QList@V?$QSharedPointer@VGSequenceGraphData@U2@@@@@@QAEXABV?$QSharedPointer@VGSequenceGraphData@U2@@@@@Z 10000044     GCFramePlot.obj
 0002:fffed044       __tryblocktable$?append@?$QList@V?$QSharedPointer@VGSequenceGraphData@U2@@@@@@QAEXABV?$QSharedPointer@VGSequenceGraphData@U2@@@@@Z 10000044     KarlinSignatureDifferenceGraph.obj
 0002:fffed044       __tryblocktable$?append@?$QList@V?$QSharedPointer@VGSequenceGraphData@U2@@@@@@QAEXABV?$QSharedPointer@VGSequenceGraphData@U2@@@@@Z 10000044     DeviationGraph.obj
 0002:fffed044       __ehfuncinfo$?node_copy@?$QList@V?$QSharedPointer@VGSequenceGraphData@U2@@@@@@AAEXPAUNode@1@00@Z 10000044     GCFramePlot.obj
 0002:fffed064       __tryblocktable$?_Copy@?$basic_string@DU?$char_traits@D@std@@V?$allocator@D@2@@std@@QAEXII@Z 10000064     EntropyAlgorithm.obj
 0002:fffed064       __tryblocktable$?_Copy@?$basic_string@DU?$char_traits@D@std@@V?$allocator@D@2@@std@@QAEXII@Z 10000064     DeviationGraph.obj
 0002:fffed064       __tryblocktable$?_Copy@?$basic_string@DU?$char_traits@D@std@@V?$allocator@D@2@@std@@QAEXII@Z 10000064     moc_DeviationGraph.obj
 0002:fffed064       __tryblocktable$?reallocData@?$QVector@M@@AAEXHHV?$QFlags@W4AllocationOption@QArrayData@@@@@Z 10000064     EntropyAlgorithm.obj
 0002:fffed064       __tryblocktable$?_Copy@?$basic_string@DU?$char_traits@D@std@@V?$allocator@D@2@@std@@QAEXII@Z 10000064     DNAGraphPackPlugin.obj
 0002:fffed064       __tryblocktable$?reallocData@?$QVector@M@@AAEXHHV?$QFlags@W4AllocationOption@QArrayData@@@@@Z 10000064     DeviationGraph.obj
 0002:fffed064       __tryblocktable$?_Copy@?$basic_string@DU?$char_traits@D@std@@V?$allocator@D@2@@std@@QAEXII@Z 10000064     moc_CumulativeSkew.obj
 0002:fffed064       __tryblocktable$?_Copy@?$basic_string@DU?$char_traits@D@std@@V?$allocator@D@2@@std@@QAEXII@Z 10000064     moc_GCFramePlot.obj
 0002:fffed064       __tryblocktable$?detach_helper_grow@?$QList@V?$QSharedPointer@VGSequenceGraphData@U2@@@@@@AAEPAUNode@1@HH@Z 10000064     GCFramePlot.obj
 0002:fffed064       __tryblocktable$?detach_helper_grow@?$QList@V?$QSharedPointer@VGSequenceGraphData@U2@@@@@@AAEPAUNode@1@HH@Z 10000064     CumulativeSkew.obj
 0002:fffed064       __tryblocktable$?_Copy@?$basic_string@DU?$char_traits@D@std@@V?$allocator@D@2@@std@@QAEXII@Z 10000064     moc_BaseContentGraph.obj
 0002:fffed064       __tryblocktable$?detach_helper_grow@?$QList@V?$QSharedPointer@VGSequenceGraphData@U2@@@@@@AAEPAUNode@1@HH@Z 10000064     EntropyAlgorithm.obj
 0002:fffed064       __tryblocktable$?reallocData@?$QVector@M@@AAEXHHV?$QFlags@W4AllocationOption@QArrayData@@@@@Z 10000064     GCFramePlot.obj
 0002:fffed064       __tryblocktable$?_Copy@?$basic_string@DU?$char_traits@D@std@@V?$allocator@D@2@@std@@QAEXII@Z 10000064     KarlinSignatureDifferenceGraph.obj
 0002:fffed064       __tryblocktable$?_Copy@?$basic_string@DU?$char_traits@D@std@@V?$allocator@D@2@@std@@QAEXII@Z 10000064     moc_DNAGraphPackPlugin.obj
 0002:fffed064       __tryblocktable$?_Copy@?$basic_string@DU?$char_traits@D@std@@V?$allocator@D@2@@std@@QAEXII@Z 10000064     moc_KarlinSignatureDifferenceGraph.obj
 0002:fffed064       __tryblocktable$?_Copy@?$basic_string@DU?$char_traits@D@std@@V?$allocator@D@2@@std@@QAEXII@Z 10000064     GCFramePlot.obj
 0002:fffed064       __tryblocktable$?reallocData@?$QVector@M@@AAEXHHV?$QFlags@W4AllocationOption@QArrayData@@@@@Z 10000064     KarlinSignatureDifferenceGraph.obj
 0002:fffed064       __tryblocktable$?_Copy@?$basic_string@DU?$char_traits@D@std@@V?$allocator@D@2@@std@@QAEXII@Z 10000064     moc_EntropyAlgorithm.obj
 0002:fffed064       __tryblocktable$?_Copy@?$basic_string@DU?$char_traits@D@std@@V?$allocator@D@2@@std@@QAEXII@Z 10000064     CumulativeSkew.obj
 0002:fffed064       __tryblocktable$?detach_helper_grow@?$QList@V?$QSharedPointer@VGSequenceGraphData@U2@@@@@@AAEPAUNode@1@HH@Z 10000064     KarlinSignatureDifferenceGraph.obj
 0002:fffed064       __tryblocktable$?reallocData@?$QVector@M@@AAEXHHV?$QFlags@W4AllocationOption@QArrayData@@@@@Z 10000064     CumulativeSkew.obj
 0002:fffed064       __tryblocktable$?detach_helper_grow@?$QList@V?$QSharedPointer@VGSequenceGraphData@U2@@@@@@AAEPAUNode@1@HH@Z 10000064     DeviationGraph.obj
 0002:fffed06c       __unwindtable$?append@?$QList@V?$QSharedPointer@VGSequenceGraphData@U2@@@@@@QAEXABV?$QSharedPointer@VGSequenceGraphData@U2@@@@@Z 1000006c     GCFramePlot.obj
 0002:fffed06c       __unwindtable$?append@?$QList@V?$QSharedPointer@VGSequenceGraphData@U2@@@@@@QAEXABV?$QSharedPointer@VGSequenceGraphData@U2@@@@@Z 1000006c     EntropyAlgorithm.obj
 0002:fffed06c       __unwindtable$?append@?$QList@V?$QSharedPointer@VGSequenceGraphData@U2@@@@@@QAEXABV?$QSharedPointer@VGSequenceGraphData@U2@@@@@Z 1000006c     CumulativeSkew.obj
 0002:fffed06c       __unwindtable$?append@?$QList@V?$QSharedPointer@VGSequenceGraphData@U2@@@@@@QAEXABV?$QSharedPointer@VGSequenceGraphData@U2@@@@@Z 1000006c     DeviationGraph.obj
 0002:fffed06c       __unwindtable$?append@?$QList@V?$QSharedPointer@VGSequenceGraphData@U2@@@@@@QAEXABV?$QSharedPointer@VGSequenceGraphData@U2@@@@@Z 1000006c     KarlinSignatureDifferenceGraph.obj
 0001:fffff08e       __catch$?node_copy@?$QList@V?$QSharedPointer@VGSequenceGraphData@U2@@@@@@AAEXPAUNode@1@00@Z$0 1000008e f   EntropyAlgorithm.obj
 0001:fffff08e       __catch$?node_copy@?$QList@V?$QSharedPointer@VGSequenceGraphData@U2@@@@@@AAEXPAUNode@1@00@Z$0 1000008e f   DeviationGraph.obj
 0001:fffff08e       __catch$?node_copy@?$QList@V?$QSharedPointer@VGSequenceGraphData@U2@@@@@@AAEXPAUNode@1@00@Z$0 1000008e f   GCFramePlot.obj
 0001:fffff08e       __catch$?node_copy@?$QList@V?$QSharedPointer@VGSequenceGraphData@U2@@@@@@AAEXPAUNode@1@00@Z$0 1000008e f   KarlinSignatureDifferenceGraph.obj
 0001:fffff08e       __catch$?node_copy@?$QList@V?$QSharedPointer@VGSequenceGraphData@U2@@@@@@AAEXPAUNode@1@00@Z$0 1000008e f   CumulativeSkew.obj
 0001:fffff096       __catch$?_Copy@?$basic_string@DU?$char_traits@D@std@@V?$allocator@D@2@@std@@QAEXII@Z$0 10000096 f   GCFramePlot.obj
 0001:fffff096       __catch$?_Copy@?$basic_string@DU?$char_traits@D@std@@V?$allocator@D@2@@std@@QAEXII@Z$0 10000096 f   DNAGraphPackPlugin.obj
 0001:fffff096       __catch$?_Copy@?$basic_string@DU?$char_traits@D@std@@V?$allocator@D@2@@std@@QAEXII@Z$0 10000096 f   moc_EntropyAlgorithm.obj
 0001:fffff096       __catch$?_Copy@?$basic_string@DU?$char_traits@D@std@@V?$allocator@D@2@@std@@QAEXII@Z$0 10000096 f   moc_CumulativeSkew.obj
 0001:fffff096       __catch$?_Copy@?$basic_string@DU?$char_traits@D@std@@V?$allocator@D@2@@std@@QAEXII@Z$0 10000096 f   moc_GCFramePlot.obj
 0001:fffff096       __catch$?_Copy@?$basic_string@DU?$char_traits@D@std@@V?$allocator@D@2@@std@@QAEXII@Z$0 10000096 f   EntropyAlgorithm.obj
 0001:fffff096       __catch$?_Copy@?$basic_string@DU?$char_traits@D@std@@V?$allocator@D@2@@std@@QAEXII@Z$0 10000096 f   moc_BaseContentGraph.obj
 0001:fffff096       __catch$?_Copy@?$basic_string@DU?$char_traits@D@std@@V?$allocator@D@2@@std@@QAEXII@Z$0 10000096 f   CumulativeSkew.obj
 0001:fffff096       __catch$?_Copy@?$basic_string@DU?$char_traits@D@std@@V?$allocator@D@2@@std@@QAEXII@Z$0 10000096 f   DeviationGraph.obj
 0001:fffff096       __catch$?_Copy@?$basic_string@DU?$char_traits@D@std@@V?$allocator@D@2@@std@@QAEXII@Z$0 10000096 f   moc_DNAGraphPackPlugin.obj
 0001:fffff096       __catch$?_Copy@?$basic_string@DU?$char_traits@D@std@@V?$allocator@D@2@@std@@QAEXII@Z$0 10000096 f   moc_DeviationGraph.obj
 0001:fffff096       __catch$?_Copy@?$basic_string@DU?$char_traits@D@std@@V?$allocator@D@2@@std@@QAEXII@Z$0 10000096 f   moc_KarlinSignatureDifferenceGraph.obj
 0001:fffff096       __catch$?_Copy@?$basic_string@DU?$char_traits@D@std@@V?$allocator@D@2@@std@@QAEXII@Z$0 10000096 f   KarlinSignatureDifferenceGraph.obj
 0001:fffff0bf       __catch$?append@?$QList@V?$QSharedPointer@VGSequenceGraphData@U2@@@@@@QAEXABV?$QSharedPointer@VGSequenceGraphData@U2@@@@@Z$2 100000bf f   CumulativeSkew.obj
 0001:fffff0bf       __catch$?append@?$QList@V?$QSharedPointer@VGSequenceGraphData@U2@@@@@@QAEXABV?$QSharedPointer@VGSequenceGraphData@U2@@@@@Z$0 100000bf f   DeviationGraph.obj
 0001:fffff0bf       __catch$?append@?$QList@V?$QSharedPointer@VGSequenceGraphData@U2@@@@@@QAEXABV?$QSharedPointer@VGSequenceGraphData@U2@@@@@Z$0 100000bf f   GCFramePlot.obj
 0001:fffff0bf       __catch$?append@?$QList@V?$QSharedPointer@VGSequenceGraphData@U2@@@@@@QAEXABV?$QSharedPointer@VGSequenceGraphData@U2@@@@@Z$2 100000bf f   DeviationGraph.obj
 0001:fffff0bf       __catch$?append@?$QList@V?$QSharedPointer@VGSequenceGraphData@U2@@@@@@QAEXABV?$QSharedPointer@VGSequenceGraphData@U2@@@@@Z$0 100000bf f   CumulativeSkew.obj
 0001:fffff0bf       __catch$?append@?$QList@V?$QSharedPointer@VGSequenceGraphData@U2@@@@@@QAEXABV?$QSharedPointer@VGSequenceGraphData@U2@@@@@Z$2 100000bf f   GCFramePlot.obj
 0001:fffff0bf       __catch$?append@?$QList@V?$QSharedPointer@VGSequenceGraphData@U2@@@@@@QAEXABV?$QSharedPointer@VGSequenceGraphData@U2@@@@@Z$0 100000bf f   EntropyAlgorithm.obj
 0001:fffff0bf       __catch$?append@?$QList@V?$QSharedPointer@VGSequenceGraphData@U2@@@@@@QAEXABV?$QSharedPointer@VGSequenceGraphData@U2@@@@@Z$2 100000bf f   KarlinSignatureDifferenceGraph.obj
 0001:fffff0bf       __catch$?append@?$QList@V?$QSharedPointer@VGSequenceGraphData@U2@@@@@@QAEXABV?$QSharedPointer@VGSequenceGraphData@U2@@@@@Z$0 100000bf f   KarlinSignatureDifferenceGraph.obj
 0001:fffff0bf       __catch$?append@?$QList@V?$QSharedPointer@VGSequenceGraphData@U2@@@@@@QAEXABV?$QSharedPointer@VGSequenceGraphData@U2@@@@@Z$2 100000bf f   EntropyAlgorithm.obj
 0001:fffff0d3       __catch$?_Copy@?$basic_string@DU?$char_traits@D@std@@V?$allocator@D@2@@std@@QAEXII@Z$1 100000d3 f   moc_GCFramePlot.obj
 0001:fffff0d3       __catch$?_Copy@?$basic_string@DU?$char_traits@D@std@@V?$allocator@D@2@@std@@QAEXII@Z$1 100000d3 f   moc_BaseContentGraph.obj
 0001:fffff0d3       __catch$?_Copy@?$basic_string@DU?$char_traits@D@std@@V?$allocator@D@2@@std@@QAEXII@Z$1 100000d3 f   EntropyAlgorithm.obj
 0001:fffff0d3       __catch$?_Copy@?$basic_string@DU?$char_traits@D@std@@V?$allocator@D@2@@std@@QAEXII@Z$1 100000d3 f   moc_CumulativeSkew.obj
 0001:fffff0d3       __catch$?_Copy@?$basic_string@DU?$char_traits@D@std@@V?$allocator@D@2@@std@@QAEXII@Z$1 100000d3 f   KarlinSignatureDifferenceGraph.obj
 0001:fffff0d3       __catch$?_Copy@?$basic_string@DU?$char_traits@D@std@@V?$allocator@D@2@@std@@QAEXII@Z$1 100000d3 f   GCFramePlot.obj
 0001:fffff0d3       __catch$?_Copy@?$basic_string@DU?$char_traits@D@std@@V?$allocator@D@2@@std@@QAEXII@Z$1 100000d3 f   moc_DeviationGraph.obj
 0001:fffff0d3       __catch$?_Copy@?$basic_string@DU?$char_traits@D@std@@V?$allocator@D@2@@std@@QAEXII@Z$1 100000d3 f   DNAGraphPackPlugin.obj
 0001:fffff0d3       __catch$?_Copy@?$basic_string@DU?$char_traits@D@std@@V?$allocator@D@2@@std@@QAEXII@Z$1 100000d3 f   moc_KarlinSignatureDifferenceGraph.obj
 0001:fffff0d3       __catch$?_Copy@?$basic_string@DU?$char_traits@D@std@@V?$allocator@D@2@@std@@QAEXII@Z$1 100000d3 f   moc_DNAGraphPackPlugin.obj
 0001:fffff0d3       __catch$?_Copy@?$basic_string@DU?$char_traits@D@std@@V?$allocator@D@2@@std@@QAEXII@Z$1 100000d3 f   CumulativeSkew.obj
 0001:fffff0d3       __catch$?_Copy@?$basic_string@DU?$char_traits@D@std@@V?$allocator@D@2@@std@@QAEXII@Z$1 100000d3 f   DeviationGraph.obj
 0001:fffff0d3       __catch$?_Copy@?$basic_string@DU?$char_traits@D@std@@V?$allocator@D@2@@std@@QAEXII@Z$1 100000d3 f   moc_EntropyAlgorithm.obj
 0001:fffff10c       __catch$?detach_helper_grow@?$QList@V?$QSharedPointer@VGSequenceGraphData@U2@@@@@@AAEPAUNode@1@HH@Z$2 1000010c f   KarlinSignatureDifferenceGraph.obj
 0001:fffff10c       __catch$?detach_helper_grow@?$QList@V?$QSharedPointer@VGSequenceGraphData@U2@@@@@@AAEPAUNode@1@HH@Z$2 1000010c f   DeviationGraph.obj
 0001:fffff10c       __catch$?detach_helper_grow@?$QList@V?$QSharedPointer@VGSequenceGraphData@U2@@@@@@AAEPAUNode@1@HH@Z$2 1000010c f   EntropyAlgorithm.obj
 0001:fffff10c       __catch$?detach_helper_grow@?$QList@V?$QSharedPointer@VGSequenceGraphData@U2@@@@@@AAEPAUNode@1@HH@Z$2 1000010c f   GCFramePlot.obj
 0001:fffff10c       __catch$?detach_helper_grow@?$QList@V?$QSharedPointer@VGSequenceGraphData@U2@@@@@@AAEPAUNode@1@HH@Z$2 1000010c f   CumulativeSkew.obj
 0001:fffff147       __catch$?detach_helper_grow@?$QList@V?$QSharedPointer@VGSequenceGraphData@U2@@@@@@AAEPAUNode@1@HH@Z$0 10000147 f   GCFramePlot.obj
 0001:fffff147       __catch$?detach_helper_grow@?$QList@V?$QSharedPointer@VGSequenceGraphData@U2@@@@@@AAEPAUNode@1@HH@Z$0 10000147 f   KarlinSignatureDifferenceGraph.obj
 0001:fffff147       __catch$?detach_helper_grow@?$QList@V?$QSharedPointer@VGSequenceGraphData@U2@@@@@@AAEPAUNode@1@HH@Z$0 10000147 f   EntropyAlgorithm.obj
 0001:fffff147       __catch$?detach_helper_grow@?$QList@V?$QSharedPointer@VGSequenceGraphData@U2@@@@@@AAEPAUNode@1@HH@Z$0 10000147 f   DeviationGraph.obj
 0001:fffff147       __catch$?detach_helper_grow@?$QList@V?$QSharedPointer@VGSequenceGraphData@U2@@@@@@AAEPAUNode@1@HH@Z$0 10000147 f   CumulativeSkew.obj
 0001:fffff1a4       __catch$?reallocData@?$QVector@M@@AAEXHHV?$QFlags@W4AllocationOption@QArrayData@@@@@Z$0 100001a4 f   CumulativeSkew.obj
 0001:fffff1a4       __catch$?reallocData@?$QVector@M@@AAEXHHV?$QFlags@W4AllocationOption@QArrayData@@@@@Z$0 100001a4 f   GCFramePlot.obj
 0001:fffff1a4       __catch$?reallocData@?$QVector@M@@AAEXHHV?$QFlags@W4AllocationOption@QArrayData@@@@@Z$0 100001a4 f   EntropyAlgorithm.obj
 0001:fffff1a4       __catch$?reallocData@?$QVector@M@@AAEXHHV?$QFlags@W4AllocationOption@QArrayData@@@@@Z$0 100001a4 f   KarlinSignatureDifferenceGraph.obj
 0001:fffff1a4       __catch$?reallocData@?$QVector@M@@AAEXHHV?$QFlags@W4AllocationOption@QArrayData@@@@@Z$0 100001a4 f   DeviationGraph.obj
 0001:fffff1b6       __catch$?reallocData@?$QVector@M@@AAEXHHV?$QFlags@W4AllocationOption@QArrayData@@@@@Z$2 100001b6 f   EntropyAlgorithm.obj
 0001:fffff1b6       __catch$?reallocData@?$QVector@M@@AAEXHHV?$QFlags@W4AllocationOption@QArrayData@@@@@Z$2 100001b6 f   KarlinSignatureDifferenceGraph.obj
 0001:fffff1b6       __catch$?reallocData@?$QVector@M@@AAEXHHV?$QFlags@W4AllocationOption@QArrayData@@@@@Z$2 100001b6 f   DeviationGraph.obj
 0001:fffff1b6       __catch$?reallocData@?$QVector@M@@AAEXHHV?$QFlags@W4AllocationOption@QArrayData@@@@@Z$2 100001b6 f   GCFramePlot.obj
 0001:fffff1b6       __catch$?reallocData@?$QVector@M@@AAEXHHV?$QFlags@W4AllocationOption@QArrayData@@@@@Z$2 100001b6 f   CumulativeSkew.obj
 0001:00000000       ??__E?_Generic_object@?$_Error_objects@H@std@@2V_Generic_error_category@2@A@@YAXXZ 10001000 f   BaseContentGraph.obj
 0001:00000010       ??__E?_Iostream_object@?$_Error_objects@H@std@@2V_Iostream_error_category@2@A@@YAXXZ 10001010 f   BaseContentGraph.obj
 0001:00000020       ??__E?_System_object@?$_Error_objects@H@std@@2V_System_error_category@2@A@@YAXXZ 10001020 f   BaseContentGraph.obj
 0001:00000030       ??__EService_DNAExport@U2@@YAXXZ 10001030 f   BaseContentGraph.obj
 0001:00000040       ??__EService_DNAGraphPack@U2@@YAXXZ 10001040 f   BaseContentGraph.obj
 0001:00000050       ??__EService_ExternalToolSupport@U2@@YAXXZ 10001050 f   BaseContentGraph.obj
 0001:00000060       ??__EService_GUITesting@U2@@YAXXZ 10001060 f   BaseContentGraph.obj
 0001:00000070       ??__EService_MaxCoreServiceId@U2@@YAXXZ 10001070 f   BaseContentGraph.obj
 0001:00000080       ??__EService_MinCoreServiceId@U2@@YAXXZ 10001080 f   BaseContentGraph.obj
 0001:00000090       ??__EService_PluginViewer@U2@@YAXXZ 10001090 f   BaseContentGraph.obj
 0001:000000a0       ??__EService_Project@U2@@YAXXZ 100010a0 f   BaseContentGraph.obj
 0001:000000b0       ??__EService_ProjectView@U2@@YAXXZ 100010b0 f   BaseContentGraph.obj
 0001:000000c0       ??__EService_QueryDesigner@U2@@YAXXZ 100010c0 f   BaseContentGraph.obj
 0001:000000d0       ??__EService_ScriptRegistry@U2@@YAXXZ 100010d0 f   BaseContentGraph.obj
 0001:000000e0       ??__EService_TestRunner@U2@@YAXXZ 100010e0 f   BaseContentGraph.obj
 0001:000000f0       ??__EService_WorkflowDesigner@U2@@YAXXZ 100010f0 f   BaseContentGraph.obj
 0001:00000100       ??__EalgoLog@U2@@YAXXZ     10001100 f   BaseContentGraph.obj
 0001:00000180       ??__EcmdLog@U2@@YAXXZ      10001180 f   BaseContentGraph.obj
 0001:00000200       ??__EcoreLog@U2@@YAXXZ     10001200 f   BaseContentGraph.obj
 0001:00000280       ??__EioLog@U2@@YAXXZ       10001280 f   BaseContentGraph.obj
 0001:00000300       ??__EperfLog@U2@@YAXXZ     10001300 f   BaseContentGraph.obj
 0001:00000380       ??__EscriptLog@U2@@YAXXZ   10001380 f   BaseContentGraph.obj
 0001:00000400       ??__EtaskLog@U2@@YAXXZ     10001400 f   BaseContentGraph.obj
 0001:00000480       ??__EuiLog@U2@@YAXXZ       10001480 f   BaseContentGraph.obj
 0001:00000500       ??__EuserActLog@U2@@YAXXZ  10001500 f   BaseContentGraph.obj
 0001:00000580       ??__E?_Generic_object@?$_Error_objects@H@std@@2V_Generic_error_category@2@A@@YAXXZ 10001580 f   CumulativeSkew.obj
 0001:00000590       ??__E?_Iostream_object@?$_Error_objects@H@std@@2V_Iostream_error_category@2@A@@YAXXZ 10001590 f   CumulativeSkew.obj
 0001:000005a0       ??__E?_System_object@?$_Error_objects@H@std@@2V_System_error_category@2@A@@YAXXZ 100015a0 f   CumulativeSkew.obj
 0001:000005b0       ??__EService_DNAExport@U2@@YAXXZ 100015b0 f   CumulativeSkew.obj
 0001:000005c0       ??__EService_DNAGraphPack@U2@@YAXXZ 100015c0 f   CumulativeSkew.obj
 0001:000005d0       ??__EService_ExternalToolSupport@U2@@YAXXZ 100015d0 f   CumulativeSkew.obj
 0001:000005e0       ??__EService_GUITesting@U2@@YAXXZ 100015e0 f   CumulativeSkew.obj
 0001:000005f0       ??__EService_MaxCoreServiceId@U2@@YAXXZ 100015f0 f   CumulativeSkew.obj
 0001:00000600       ??__EService_MinCoreServiceId@U2@@YAXXZ 10001600 f   CumulativeSkew.obj
 0001:00000610       ??__EService_PluginViewer@U2@@YAXXZ 10001610 f   CumulativeSkew.obj
 0001:00000620       ??__EService_Project@U2@@YAXXZ 10001620 f   CumulativeSkew.obj
 0001:00000630       ??__EService_ProjectView@U2@@YAXXZ 10001630 f   CumulativeSkew.obj
 0001:00000640       ??__EService_QueryDesigner@U2@@YAXXZ 10001640 f   CumulativeSkew.obj
 0001:00000650       ??__EService_ScriptRegistry@U2@@YAXXZ 10001650 f   CumulativeSkew.obj
 0001:00000660       ??__EService_TestRunner@U2@@YAXXZ 10001660 f   CumulativeSkew.obj
 0001:00000670       ??__EService_WorkflowDesigner@U2@@YAXXZ 10001670 f   CumulativeSkew.obj
 0001:00000680       ??__EalgoLog@U2@@YAXXZ     10001680 f   CumulativeSkew.obj
 0001:00000700       ??__EcmdLog@U2@@YAXXZ      10001700 f   CumulativeSkew.obj
 0001:00000780       ??__EcoreLog@U2@@YAXXZ     10001780 f   CumulativeSkew.obj
 0001:00000800       ??__EioLog@U2@@YAXXZ       10001800 f   CumulativeSkew.obj
 0001:00000880       ??__EperfLog@U2@@YAXXZ     10001880 f   CumulativeSkew.obj
 0001:00000900       ??__EscriptLog@U2@@YAXXZ   10001900 f   CumulativeSkew.obj
 0001:00000980       ??__EtaskLog@U2@@YAXXZ     10001980 f   CumulativeSkew.obj
 0001:00000a00       ??__EuiLog@U2@@YAXXZ       10001a00 f   CumulativeSkew.obj
 0001:00000a80       ??__EuserActLog@U2@@YAXXZ  10001a80 f   CumulativeSkew.obj
 0001:00000b00       ??__E?_Generic_object@?$_Error_objects@H@std@@2V_Generic_error_category@2@A@@YAXXZ 10001b00 f   DNAGraphPackPlugin.obj
 0001:00000b10       ??__E?_Iostream_object@?$_Error_objects@H@std@@2V_Iostream_error_category@2@A@@YAXXZ 10001b10 f   DNAGraphPackPlugin.obj
 0001:00000b20       ??__E?_System_object@?$_Error_objects@H@std@@2V_System_error_category@2@A@@YAXXZ 10001b20 f   DNAGraphPackPlugin.obj
 0001:00000b30       ??__EService_DNAExport@U2@@YAXXZ 10001b30 f   DNAGraphPackPlugin.obj
 0001:00000b40       ??__EService_DNAGraphPack@U2@@YAXXZ 10001b40 f   DNAGraphPackPlugin.obj
 0001:00000b50       ??__EService_ExternalToolSupport@U2@@YAXXZ 10001b50 f   DNAGraphPackPlugin.obj
 0001:00000b60       ??__EService_GUITesting@U2@@YAXXZ 10001b60 f   DNAGraphPackPlugin.obj
 0001:00000b70       ??__EService_MaxCoreServiceId@U2@@YAXXZ 10001b70 f   DNAGraphPackPlugin.obj
 0001:00000b80       ??__EService_MinCoreServiceId@U2@@YAXXZ 10001b80 f   DNAGraphPackPlugin.obj
 0001:00000b90       ??__EService_PluginViewer@U2@@YAXXZ 10001b90 f   DNAGraphPackPlugin.obj
 0001:00000ba0       ??__EService_Project@U2@@YAXXZ 10001ba0 f   DNAGraphPackPlugin.obj
 0001:00000bb0       ??__EService_ProjectView@U2@@YAXXZ 10001bb0 f   DNAGraphPackPlugin.obj
 0001:00000bc0       ??__EService_QueryDesigner@U2@@YAXXZ 10001bc0 f   DNAGraphPackPlugin.obj
 0001:00000bd0       ??__EService_ScriptRegistry@U2@@YAXXZ 10001bd0 f   DNAGraphPackPlugin.obj
 0001:00000be0       ??__EService_TestRunner@U2@@YAXXZ 10001be0 f   DNAGraphPackPlugin.obj
 0001:00000bf0       ??__EService_WorkflowDesigner@U2@@YAXXZ 10001bf0 f   DNAGraphPackPlugin.obj
 0001:00000c00       ??__EalgoLog@U2@@YAXXZ     10001c00 f   DNAGraphPackPlugin.obj
 0001:00000c80       ??__EcmdLog@U2@@YAXXZ      10001c80 f   DNAGraphPackPlugin.obj
 0001:00000d00       ??__EcoreLog@U2@@YAXXZ     10001d00 f   DNAGraphPackPlugin.obj
 0001:00000d80       ??__EioLog@U2@@YAXXZ       10001d80 f   DNAGraphPackPlugin.obj
 0001:00000e00       ??__EperfLog@U2@@YAXXZ     10001e00 f   DNAGraphPackPlugin.obj
 0001:00000e80       ??__EscriptLog@U2@@YAXXZ   10001e80 f   DNAGraphPackPlugin.obj
 0001:00000f00       ??__EtaskLog@U2@@YAXXZ     10001f00 f   DNAGraphPackPlugin.obj
 0001:00000f80       ??__EuiLog@U2@@YAXXZ       10001f80 f   DNAGraphPackPlugin.obj
 0001:00001000       ??__EuserActLog@U2@@YAXXZ  10002000 f   DNAGraphPackPlugin.obj
 0001:00001080       ??__E?_Generic_object@?$_Error_objects@H@std@@2V_Generic_error_category@2@A@@YAXXZ 10002080 f   DeviationGraph.obj
 0001:00001090       ??__E?_Iostream_object@?$_Error_objects@H@std@@2V_Iostream_error_category@2@A@@YAXXZ 10002090 f   DeviationGraph.obj
 0001:000010a0       ??__E?_System_object@?$_Error_objects@H@std@@2V_System_error_category@2@A@@YAXXZ 100020a0 f   DeviationGraph.obj
 0001:000010b0       ??__EService_DNAExport@U2@@YAXXZ 100020b0 f   DeviationGraph.obj
 0001:000010c0       ??__EService_DNAGraphPack@U2@@YAXXZ 100020c0 f   DeviationGraph.obj
 0001:000010d0       ??__EService_ExternalToolSupport@U2@@YAXXZ 100020d0 f   DeviationGraph.obj
 0001:000010e0       ??__EService_GUITesting@U2@@YAXXZ 100020e0 f   DeviationGraph.obj
 0001:000010f0       ??__EService_MaxCoreServiceId@U2@@YAXXZ 100020f0 f   DeviationGraph.obj
 0001:00001100       ??__EService_MinCoreServiceId@U2@@YAXXZ 10002100 f   DeviationGraph.obj
 0001:00001110       ??__EService_PluginViewer@U2@@YAXXZ 10002110 f   DeviationGraph.obj
 0001:00001120       ??__EService_Project@U2@@YAXXZ 10002120 f   DeviationGraph.obj
 0001:00001130       ??__EService_ProjectView@U2@@YAXXZ 10002130 f   DeviationGraph.obj
 0001:00001140       ??__EService_QueryDesigner@U2@@YAXXZ 10002140 f   DeviationGraph.obj
 0001:00001150       ??__EService_ScriptRegistry@U2@@YAXXZ 10002150 f   DeviationGraph.obj
 0001:00001160       ??__EService_TestRunner@U2@@YAXXZ 10002160 f   DeviationGraph.obj
 0001:00001170       ??__EService_WorkflowDesigner@U2@@YAXXZ 10002170 f   DeviationGraph.obj
 0001:00001180       ??__EalgoLog@U2@@YAXXZ     10002180 f   DeviationGraph.obj
 0001:00001200       ??__EcmdLog@U2@@YAXXZ      10002200 f   DeviationGraph.obj
 0001:00001280       ??__EcoreLog@U2@@YAXXZ     10002280 f   DeviationGraph.obj
 0001:00001300       ??__EioLog@U2@@YAXXZ       10002300 f   DeviationGraph.obj
 0001:00001380       ??__EperfLog@U2@@YAXXZ     10002380 f   DeviationGraph.obj
 0001:00001400       ??__EscriptLog@U2@@YAXXZ   10002400 f   DeviationGraph.obj
 0001:00001480       ??__EtaskLog@U2@@YAXXZ     10002480 f   DeviationGraph.obj
 0001:00001500       ??__EuiLog@U2@@YAXXZ       10002500 f   DeviationGraph.obj
 0001:00001580       ??__EuserActLog@U2@@YAXXZ  10002580 f   DeviationGraph.obj
 0001:00001600       ??__E?_Generic_object@?$_Error_objects@H@std@@2V_Generic_error_category@2@A@@YAXXZ 10002600 f   EntropyAlgorithm.obj
 0001:00001610       ??__E?_Iostream_object@?$_Error_objects@H@std@@2V_Iostream_error_category@2@A@@YAXXZ 10002610 f   EntropyAlgorithm.obj
 0001:00001620       ??__E?_System_object@?$_Error_objects@H@std@@2V_System_error_category@2@A@@YAXXZ 10002620 f   EntropyAlgorithm.obj
 0001:00001630       ??__EService_DNAExport@U2@@YAXXZ 10002630 f   EntropyAlgorithm.obj
 0001:00001640       ??__EService_DNAGraphPack@U2@@YAXXZ 10002640 f   EntropyAlgorithm.obj
 0001:00001650       ??__EService_ExternalToolSupport@U2@@YAXXZ 10002650 f   EntropyAlgorithm.obj
 0001:00001660       ??__EService_GUITesting@U2@@YAXXZ 10002660 f   EntropyAlgorithm.obj
 0001:00001670       ??__EService_MaxCoreServiceId@U2@@YAXXZ 10002670 f   EntropyAlgorithm.obj
 0001:00001680       ??__EService_MinCoreServiceId@U2@@YAXXZ 10002680 f   EntropyAlgorithm.obj
 0001:00001690       ??__EService_PluginViewer@U2@@YAXXZ 10002690 f   EntropyAlgorithm.obj
 0001:000016a0       ??__EService_Project@U2@@YAXXZ 100026a0 f   EntropyAlgorithm.obj
 0001:000016b0       ??__EService_ProjectView@U2@@YAXXZ 100026b0 f   EntropyAlgorithm.obj
 0001:000016c0       ??__EService_QueryDesigner@U2@@YAXXZ 100026c0 f   EntropyAlgorithm.obj
 0001:000016d0       ??__EService_ScriptRegistry@U2@@YAXXZ 100026d0 f   EntropyAlgorithm.obj
 0001:000016e0       ??__EService_TestRunner@U2@@YAXXZ 100026e0 f   EntropyAlgorithm.obj
 0001:000016f0       ??__EService_WorkflowDesigner@U2@@YAXXZ 100026f0 f   EntropyAlgorithm.obj
 0001:00001700       ??__EalgoLog@U2@@YAXXZ     10002700 f   EntropyAlgorithm.obj
 0001:00001780       ??__EcmdLog@U2@@YAXXZ      10002780 f   EntropyAlgorithm.obj
 0001:00001800       ??__EcoreLog@U2@@YAXXZ     10002800 f   EntropyAlgorithm.obj
 0001:00001880       ??__EioLog@U2@@YAXXZ       10002880 f   EntropyAlgorithm.obj
 0001:00001900       ??__EperfLog@U2@@YAXXZ     10002900 f   EntropyAlgorithm.obj
 0001:00001980       ??__EscriptLog@U2@@YAXXZ   10002980 f   EntropyAlgorithm.obj
 0001:00001a00       ??__EtaskLog@U2@@YAXXZ     10002a00 f   EntropyAlgorithm.obj
 0001:00001a80       ??__EuiLog@U2@@YAXXZ       10002a80 f   EntropyAlgorithm.obj
 0001:00001b00       ??__EuserActLog@U2@@YAXXZ  10002b00 f   EntropyAlgorithm.obj
 0001:00001b80       ??__E?_Generic_object@?$_Error_objects@H@std@@2V_Generic_error_category@2@A@@YAXXZ 10002b80 f   GCFramePlot.obj
 0001:00001b90       ??__E?_Iostream_object@?$_Error_objects@H@std@@2V_Iostream_error_category@2@A@@YAXXZ 10002b90 f   GCFramePlot.obj
 0001:00001ba0       ??__E?_System_object@?$_Error_objects@H@std@@2V_System_error_category@2@A@@YAXXZ 10002ba0 f   GCFramePlot.obj
 0001:00001bb0       ??__EService_DNAExport@U2@@YAXXZ 10002bb0 f   GCFramePlot.obj
 0001:00001bc0       ??__EService_DNAGraphPack@U2@@YAXXZ 10002bc0 f   GCFramePlot.obj
 0001:00001bd0       ??__EService_ExternalToolSupport@U2@@YAXXZ 10002bd0 f   GCFramePlot.obj
 0001:00001be0       ??__EService_GUITesting@U2@@YAXXZ 10002be0 f   GCFramePlot.obj
 0001:00001bf0       ??__EService_MaxCoreServiceId@U2@@YAXXZ 10002bf0 f   GCFramePlot.obj
 0001:00001c00       ??__EService_MinCoreServiceId@U2@@YAXXZ 10002c00 f   GCFramePlot.obj
 0001:00001c10       ??__EService_PluginViewer@U2@@YAXXZ 10002c10 f   GCFramePlot.obj
 0001:00001c20       ??__EService_Project@U2@@YAXXZ 10002c20 f   GCFramePlot.obj
 0001:00001c30       ??__EService_ProjectView@U2@@YAXXZ 10002c30 f   GCFramePlot.obj
 0001:00001c40       ??__EService_QueryDesigner@U2@@YAXXZ 10002c40 f   GCFramePlot.obj
 0001:00001c50       ??__EService_ScriptRegistry@U2@@YAXXZ 10002c50 f   GCFramePlot.obj
 0001:00001c60       ??__EService_TestRunner@U2@@YAXXZ 10002c60 f   GCFramePlot.obj
 0001:00001c70       ??__EService_WorkflowDesigner@U2@@YAXXZ 10002c70 f   GCFramePlot.obj
 0001:00001c80       ??__EalgoLog@U2@@YAXXZ     10002c80 f   GCFramePlot.obj
 0001:00001d00       ??__EcmdLog@U2@@YAXXZ      10002d00 f   GCFramePlot.obj
 0001:00001d80       ??__EcoreLog@U2@@YAXXZ     10002d80 f   GCFramePlot.obj
 0001:00001e00       ??__EioLog@U2@@YAXXZ       10002e00 f   GCFramePlot.obj
 0001:00001e80       ??__EperfLog@U2@@YAXXZ     10002e80 f   GCFramePlot.obj
 0001:00001f00       ??__EscriptLog@U2@@YAXXZ   10002f00 f   GCFramePlot.obj
 0001:00001f80       ??__EtaskLog@U2@@YAXXZ     10002f80 f   GCFramePlot.obj
 0001:00002000       ??__EuiLog@U2@@YAXXZ       10003000 f   GCFramePlot.obj
 0001:00002080       ??__EuserActLog@U2@@YAXXZ  10003080 f   GCFramePlot.obj
 0001:00002100       ??__E?_Generic_object@?$_Error_objects@H@std@@2V_Generic_error_category@2@A@@YAXXZ 10003100 f   KarlinSignatureDifferenceGraph.obj
 0001:00002110       ??__E?_Iostream_object@?$_Error_objects@H@std@@2V_Iostream_error_category@2@A@@YAXXZ 10003110 f   KarlinSignatureDifferenceGraph.obj
 0001:00002120       ??__E?_System_object@?$_Error_objects@H@std@@2V_System_error_category@2@A@@YAXXZ 10003120 f   KarlinSignatureDifferenceGraph.obj
 0001:00002130       ??__EService_DNAExport@U2@@YAXXZ 10003130 f   KarlinSignatureDifferenceGraph.obj
 0001:00002140       ??__EService_DNAGraphPack@U2@@YAXXZ 10003140 f   KarlinSignatureDifferenceGraph.obj
 0001:00002150       ??__EService_ExternalToolSupport@U2@@YAXXZ 10003150 f   KarlinSignatureDifferenceGraph.obj
 0001:00002160       ??__EService_GUITesting@U2@@YAXXZ 10003160 f   KarlinSignatureDifferenceGraph.obj
 0001:00002170       ??__EService_MaxCoreServiceId@U2@@YAXXZ 10003170 f   KarlinSignatureDifferenceGraph.obj
 0001:00002180       ??__EService_MinCoreServiceId@U2@@YAXXZ 10003180 f   KarlinSignatureDifferenceGraph.obj
 0001:00002190       ??__EService_PluginViewer@U2@@YAXXZ 10003190 f   KarlinSignatureDifferenceGraph.obj
 0001:000021a0       ??__EService_Project@U2@@YAXXZ 100031a0 f   KarlinSignatureDifferenceGraph.obj
 0001:000021b0       ??__EService_ProjectView@U2@@YAXXZ 100031b0 f   KarlinSignatureDifferenceGraph.obj
 0001:000021c0       ??__EService_QueryDesigner@U2@@YAXXZ 100031c0 f   KarlinSignatureDifferenceGraph.obj
 0001:000021d0       ??__EService_ScriptRegistry@U2@@YAXXZ 100031d0 f   KarlinSignatureDifferenceGraph.obj
 0001:000021e0       ??__EService_TestRunner@U2@@YAXXZ 100031e0 f   KarlinSignatureDifferenceGraph.obj
 0001:000021f0       ??__EService_WorkflowDesigner@U2@@YAXXZ 100031f0 f   KarlinSignatureDifferenceGraph.obj
 0001:00002200       ??__EalgoLog@U2@@YAXXZ     10003200 f   KarlinSignatureDifferenceGraph.obj
 0001:00002280       ??__EcmdLog@U2@@YAXXZ      10003280 f   KarlinSignatureDifferenceGraph.obj
 0001:00002300       ??__EcoreLog@U2@@YAXXZ     10003300 f   KarlinSignatureDifferenceGraph.obj
 0001:00002380       ??__EioLog@U2@@YAXXZ       10003380 f   KarlinSignatureDifferenceGraph.obj
 0001:00002400       ??__EperfLog@U2@@YAXXZ     10003400 f   KarlinSignatureDifferenceGraph.obj
 0001:00002480       ??__EscriptLog@U2@@YAXXZ   10003480 f   KarlinSignatureDifferenceGraph.obj
 0001:00002500       ??__EtaskLog@U2@@YAXXZ     10003500 f   KarlinSignatureDifferenceGraph.obj
 0001:00002580       ??__EuiLog@U2@@YAXXZ       10003580 f   KarlinSignatureDifferenceGraph.obj
 0001:00002600       ??__EuserActLog@U2@@YAXXZ  10003600 f   KarlinSignatureDifferenceGraph.obj
 0001:00002680       ??__E?_Generic_object@?$_Error_objects@H@std@@2V_Generic_error_category@2@A@@YAXXZ 10003680 f   moc_BaseContentGraph.obj
 0001:00002690       ??__E?_Iostream_object@?$_Error_objects@H@std@@2V_Iostream_error_category@2@A@@YAXXZ 10003690 f   moc_BaseContentGraph.obj
 0001:000026a0       ??__E?_System_object@?$_Error_objects@H@std@@2V_System_error_category@2@A@@YAXXZ 100036a0 f   moc_BaseContentGraph.obj
 0001:000026b0       ??__E?staticMetaObject@BaseContentGraphFactory@U2@@2UQMetaObject@@B@@YAXXZ 100036b0 f   moc_BaseContentGraph.obj
 0001:000026c0       ??__EService_DNAExport@U2@@YAXXZ 100036c0 f   moc_BaseContentGraph.obj
 0001:000026d0       ??__EService_DNAGraphPack@U2@@YAXXZ 100036d0 f   moc_BaseContentGraph.obj
 0001:000026e0       ??__EService_ExternalToolSupport@U2@@YAXXZ 100036e0 f   moc_BaseContentGraph.obj
 0001:000026f0       ??__EService_GUITesting@U2@@YAXXZ 100036f0 f   moc_BaseContentGraph.obj
 0001:00002700       ??__EService_MaxCoreServiceId@U2@@YAXXZ 10003700 f   moc_BaseContentGraph.obj
 0001:00002710       ??__EService_MinCoreServiceId@U2@@YAXXZ 10003710 f   moc_BaseContentGraph.obj
 0001:00002720       ??__EService_PluginViewer@U2@@YAXXZ 10003720 f   moc_BaseContentGraph.obj
 0001:00002730       ??__EService_Project@U2@@YAXXZ 10003730 f   moc_BaseContentGraph.obj
 0001:00002740       ??__EService_ProjectView@U2@@YAXXZ 10003740 f   moc_BaseContentGraph.obj
 0001:00002750       ??__EService_QueryDesigner@U2@@YAXXZ 10003750 f   moc_BaseContentGraph.obj
 0001:00002760       ??__EService_ScriptRegistry@U2@@YAXXZ 10003760 f   moc_BaseContentGraph.obj
 0001:00002770       ??__EService_TestRunner@U2@@YAXXZ 10003770 f   moc_BaseContentGraph.obj
 0001:00002780       ??__EService_WorkflowDesigner@U2@@YAXXZ 10003780 f   moc_BaseContentGraph.obj
 0001:00002790       ??__EalgoLog@U2@@YAXXZ     10003790 f   moc_BaseContentGraph.obj
 0001:00002810       ??__EcmdLog@U2@@YAXXZ      10003810 f   moc_BaseContentGraph.obj
 0001:00002890       ??__EcoreLog@U2@@YAXXZ     10003890 f   moc_BaseContentGraph.obj
 0001:00002910       ??__EioLog@U2@@YAXXZ       10003910 f   moc_BaseContentGraph.obj
 0001:00002990       ??__EperfLog@U2@@YAXXZ     10003990 f   moc_BaseContentGraph.obj
 0001:00002a10       ??__EscriptLog@U2@@YAXXZ   10003a10 f   moc_BaseContentGraph.obj
 0001:00002a90       ??__EtaskLog@U2@@YAXXZ     10003a90 f   moc_BaseContentGraph.obj
 0001:00002b10       ??__EuiLog@U2@@YAXXZ       10003b10 f   moc_BaseContentGraph.obj
 0001:00002b90       ??__EuserActLog@U2@@YAXXZ  10003b90 f   moc_BaseContentGraph.obj
 0001:00002c10       ??__E?_Generic_object@?$_Error_objects@H@std@@2V_Generic_error_category@2@A@@YAXXZ 10003c10 f   moc_CumulativeSkew.obj
 0001:00002c20       ??__E?_Iostream_object@?$_Error_objects@H@std@@2V_Iostream_error_category@2@A@@YAXXZ 10003c20 f   moc_CumulativeSkew.obj
 0001:00002c30       ??__E?_System_object@?$_Error_objects@H@std@@2V_System_error_category@2@A@@YAXXZ 10003c30 f   moc_CumulativeSkew.obj
 0001:00002c40       ??__E?staticMetaObject@CumulativeSkewGraphFactory@U2@@2UQMetaObject@@B@@YAXXZ 10003c40 f   moc_CumulativeSkew.obj
 0001:00002c50       ??__EService_DNAExport@U2@@YAXXZ 10003c50 f   moc_CumulativeSkew.obj
 0001:00002c60       ??__EService_DNAGraphPack@U2@@YAXXZ 10003c60 f   moc_CumulativeSkew.obj
 0001:00002c70       ??__EService_ExternalToolSupport@U2@@YAXXZ 10003c70 f   moc_CumulativeSkew.obj
 0001:00002c80       ??__EService_GUITesting@U2@@YAXXZ 10003c80 f   moc_CumulativeSkew.obj
 0001:00002c90       ??__EService_MaxCoreServiceId@U2@@YAXXZ 10003c90 f   moc_CumulativeSkew.obj
 0001:00002ca0       ??__EService_MinCoreServiceId@U2@@YAXXZ 10003ca0 f   moc_CumulativeSkew.obj
 0001:00002cb0       ??__EService_PluginViewer@U2@@YAXXZ 10003cb0 f   moc_CumulativeSkew.obj
 0001:00002cc0       ??__EService_Project@U2@@YAXXZ 10003cc0 f   moc_CumulativeSkew.obj
 0001:00002cd0       ??__EService_ProjectView@U2@@YAXXZ 10003cd0 f   moc_CumulativeSkew.obj
 0001:00002ce0       ??__EService_QueryDesigner@U2@@YAXXZ 10003ce0 f   moc_CumulativeSkew.obj
 0001:00002cf0       ??__EService_ScriptRegistry@U2@@YAXXZ 10003cf0 f   moc_CumulativeSkew.obj
 0001:00002d00       ??__EService_TestRunner@U2@@YAXXZ 10003d00 f   moc_CumulativeSkew.obj
 0001:00002d10       ??__EService_WorkflowDesigner@U2@@YAXXZ 10003d10 f   moc_CumulativeSkew.obj
 0001:00002d20       ??__EalgoLog@U2@@YAXXZ     10003d20 f   moc_CumulativeSkew.obj
 0001:00002da0       ??__EcmdLog@U2@@YAXXZ      10003da0 f   moc_CumulativeSkew.obj
 0001:00002e20       ??__EcoreLog@U2@@YAXXZ     10003e20 f   moc_CumulativeSkew.obj
 0001:00002ea0       ??__EioLog@U2@@YAXXZ       10003ea0 f   moc_CumulativeSkew.obj
 0001:00002f20       ??__EperfLog@U2@@YAXXZ     10003f20 f   moc_CumulativeSkew.obj
 0001:00002fb0       ??__EscriptLog@U2@@YAXXZ   10003fb0 f   moc_CumulativeSkew.obj
 0001:00003030       ??__EtaskLog@U2@@YAXXZ     10004030 f   moc_CumulativeSkew.obj
 0001:000030b0       ??__EuiLog@U2@@YAXXZ       100040b0 f   moc_CumulativeSkew.obj
 0001:00003130       ??__EuserActLog@U2@@YAXXZ  10004130 f   moc_CumulativeSkew.obj
 0001:000031b0       ??__E?_Generic_object@?$_Error_objects@H@std@@2V_Generic_error_category@2@A@@YAXXZ 100041b0 f   moc_DNAGraphPackPlugin.obj
 0001:000031c0       ??__E?_Iostream_object@?$_Error_objects@H@std@@2V_Iostream_error_category@2@A@@YAXXZ 100041c0 f   moc_DNAGraphPackPlugin.obj
 0001:000031d0       ??__E?_System_object@?$_Error_objects@H@std@@2V_System_error_category@2@A@@YAXXZ 100041d0 f   moc_DNAGraphPackPlugin.obj
 0001:000031e0       ??__E?staticMetaObject@DNAGraphPackPlugin@U2@@2UQMetaObject@@B@@YAXXZ 100041e0 f   moc_DNAGraphPackPlugin.obj
 0001:000031f0       ??__E?staticMetaObject@DNAGraphPackViewContext@U2@@2UQMetaObject@@B@@YAXXZ 100041f0 f   moc_DNAGraphPackPlugin.obj
 0001:00003200       ??__EService_DNAExport@U2@@YAXXZ 10004200 f   moc_DNAGraphPackPlugin.obj
 0001:00003210       ??__EService_DNAGraphPack@U2@@YAXXZ 10004210 f   moc_DNAGraphPackPlugin.obj
 0001:00003220       ??__EService_ExternalToolSupport@U2@@YAXXZ 10004220 f   moc_DNAGraphPackPlugin.obj
 0001:00003230       ??__EService_GUITesting@U2@@YAXXZ 10004230 f   moc_DNAGraphPackPlugin.obj
 0001:00003240       ??__EService_MaxCoreServiceId@U2@@YAXXZ 10004240 f   moc_DNAGraphPackPlugin.obj
 0001:00003250       ??__EService_MinCoreServiceId@U2@@YAXXZ 10004250 f   moc_DNAGraphPackPlugin.obj
 0001:00003260       ??__EService_PluginViewer@U2@@YAXXZ 10004260 f   moc_DNAGraphPackPlugin.obj
 0001:00003270       ??__EService_Project@U2@@YAXXZ 10004270 f   moc_DNAGraphPackPlugin.obj
 0001:00003280       ??__EService_ProjectView@U2@@YAXXZ 10004280 f   moc_DNAGraphPackPlugin.obj
 0001:00003290       ??__EService_QueryDesigner@U2@@YAXXZ 10004290 f   moc_DNAGraphPackPlugin.obj
 0001:000032a0       ??__EService_ScriptRegistry@U2@@YAXXZ 100042a0 f   moc_DNAGraphPackPlugin.obj
 0001:000032b0       ??__EService_TestRunner@U2@@YAXXZ 100042b0 f   moc_DNAGraphPackPlugin.obj
 0001:000032c0       ??__EService_WorkflowDesigner@U2@@YAXXZ 100042c0 f   moc_DNAGraphPackPlugin.obj
 0001:000032d0       ??__EalgoLog@U2@@YAXXZ     100042d0 f   moc_DNAGraphPackPlugin.obj
 0001:00003350       ??__EcmdLog@U2@@YAXXZ      10004350 f   moc_DNAGraphPackPlugin.obj
 0001:000033d0       ??__EcoreLog@U2@@YAXXZ     100043d0 f   moc_DNAGraphPackPlugin.obj
 0001:00003450       ??__EioLog@U2@@YAXXZ       10004450 f   moc_DNAGraphPackPlugin.obj
 0001:000034d0       ??__EperfLog@U2@@YAXXZ     100044d0 f   moc_DNAGraphPackPlugin.obj
 0001:00003550       ??__EscriptLog@U2@@YAXXZ   10004550 f   moc_DNAGraphPackPlugin.obj
 0001:000035d0       ??__EtaskLog@U2@@YAXXZ     100045d0 f   moc_DNAGraphPackPlugin.obj
 0001:00003650       ??__EuiLog@U2@@YAXXZ       10004650 f   moc_DNAGraphPackPlugin.obj
 0001:000036d0       ??__EuserActLog@U2@@YAXXZ  100046d0 f   moc_DNAGraphPackPlugin.obj
 0001:00003750       ??__E?_Generic_object@?$_Error_objects@H@std@@2V_Generic_error_category@2@A@@YAXXZ 10004750 f   moc_DeviationGraph.obj
 0001:00003760       ??__E?_Iostream_object@?$_Error_objects@H@std@@2V_Iostream_error_category@2@A@@YAXXZ 10004760 f   moc_DeviationGraph.obj
 0001:00003770       ??__E?_System_object@?$_Error_objects@H@std@@2V_System_error_category@2@A@@YAXXZ 10004770 f   moc_DeviationGraph.obj
 0001:00003780       ??__E?staticMetaObject@DeviationGraphFactory@U2@@2UQMetaObject@@B@@YAXXZ 10004780 f   moc_DeviationGraph.obj
 0001:00003790       ??__EService_DNAExport@U2@@YAXXZ 10004790 f   moc_DeviationGraph.obj
 0001:000037a0       ??__EService_DNAGraphPack@U2@@YAXXZ 100047a0 f   moc_DeviationGraph.obj
 0001:000037b0       ??__EService_ExternalToolSupport@U2@@YAXXZ 100047b0 f   moc_DeviationGraph.obj
 0001:000037c0       ??__EService_GUITesting@U2@@YAXXZ 100047c0 f   moc_DeviationGraph.obj
 0001:000037d0       ??__EService_MaxCoreServiceId@U2@@YAXXZ 100047d0 f   moc_DeviationGraph.obj
 0001:000037e0       ??__EService_MinCoreServiceId@U2@@YAXXZ 100047e0 f   moc_DeviationGraph.obj
 0001:000037f0       ??__EService_PluginViewer@U2@@YAXXZ 100047f0 f   moc_DeviationGraph.obj
 0001:00003800       ??__EService_Project@U2@@YAXXZ 10004800 f   moc_DeviationGraph.obj
 0001:00003810       ??__EService_ProjectView@U2@@YAXXZ 10004810 f   moc_DeviationGraph.obj
 0001:00003820       ??__EService_QueryDesigner@U2@@YAXXZ 10004820 f   moc_DeviationGraph.obj
 0001:00003830       ??__EService_ScriptRegistry@U2@@YAXXZ 10004830 f   moc_DeviationGraph.obj
 0001:00003840       ??__EService_TestRunner@U2@@YAXXZ 10004840 f   moc_DeviationGraph.obj
 0001:00003850       ??__EService_WorkflowDesigner@U2@@YAXXZ 10004850 f   moc_DeviationGraph.obj
 0001:00003860       ??__EalgoLog@U2@@YAXXZ     10004860 f   moc_DeviationGraph.obj
 0001:000038e0       ??__EcmdLog@U2@@YAXXZ      100048e0 f   moc_DeviationGraph.obj
 0001:00003960       ??__EcoreLog@U2@@YAXXZ     10004960 f   moc_DeviationGraph.obj
 0001:000039e0       ??__EioLog@U2@@YAXXZ       100049e0 f   moc_DeviationGraph.obj
 0001:00003a60       ??__EperfLog@U2@@YAXXZ     10004a60 f   moc_DeviationGraph.obj
 0001:00003ae0       ??__EscriptLog@U2@@YAXXZ   10004ae0 f   moc_DeviationGraph.obj
 0001:00003b60       ??__EtaskLog@U2@@YAXXZ     10004b60 f   moc_DeviationGraph.obj
 0001:00003be0       ??__EuiLog@U2@@YAXXZ       10004be0 f   moc_DeviationGraph.obj
 0001:00003c60       ??__EuserActLog@U2@@YAXXZ  10004c60 f   moc_DeviationGraph.obj
 0001:00003ce0       ??__E?_Generic_object@?$_Error_objects@H@std@@2V_Generic_error_category@2@A@@YAXXZ 10004ce0 f   moc_EntropyAlgorithm.obj
 0001:00003cf0       ??__E?_Iostream_object@?$_Error_objects@H@std@@2V_Iostream_error_category@2@A@@YAXXZ 10004cf0 f   moc_EntropyAlgorithm.obj
 0001:00003d00       ??__E?_System_object@?$_Error_objects@H@std@@2V_System_error_category@2@A@@YAXXZ 10004d00 f   moc_EntropyAlgorithm.obj
 0001:00003d10       ??__E?staticMetaObject@EntropyGraphFactory@U2@@2UQMetaObject@@B@@YAXXZ 10004d10 f   moc_EntropyAlgorithm.obj
 0001:00003d20       ??__EService_DNAExport@U2@@YAXXZ 10004d20 f   moc_EntropyAlgorithm.obj
 0001:00003d30       ??__EService_DNAGraphPack@U2@@YAXXZ 10004d30 f   moc_EntropyAlgorithm.obj
 0001:00003d40       ??__EService_ExternalToolSupport@U2@@YAXXZ 10004d40 f   moc_EntropyAlgorithm.obj
 0001:00003d50       ??__EService_GUITesting@U2@@YAXXZ 10004d50 f   moc_EntropyAlgorithm.obj
 0001:00003d60       ??__EService_MaxCoreServiceId@U2@@YAXXZ 10004d60 f   moc_EntropyAlgorithm.obj
 0001:00003d70       ??__EService_MinCoreServiceId@U2@@YAXXZ 10004d70 f   moc_EntropyAlgorithm.obj
 0001:00003d80       ??__EService_PluginViewer@U2@@YAXXZ 10004d80 f   moc_EntropyAlgorithm.obj
 0001:00003d90       ??__EService_Project@U2@@YAXXZ 10004d90 f   moc_EntropyAlgorithm.obj
 0001:00003da0       ??__EService_ProjectView@U2@@YAXXZ 10004da0 f   moc_EntropyAlgorithm.obj
 0001:00003db0       ??__EService_QueryDesigner@U2@@YAXXZ 10004db0 f   moc_EntropyAlgorithm.obj
 0001:00003dc0       ??__EService_ScriptRegistry@U2@@YAXXZ 10004dc0 f   moc_EntropyAlgorithm.obj
 0001:00003dd0       ??__EService_TestRunner@U2@@YAXXZ 10004dd0 f   moc_EntropyAlgorithm.obj
 0001:00003de0       ??__EService_WorkflowDesigner@U2@@YAXXZ 10004de0 f   moc_EntropyAlgorithm.obj
 0001:00003df0       ??__EalgoLog@U2@@YAXXZ     10004df0 f   moc_EntropyAlgorithm.obj
 0001:00003e70       ??__EcmdLog@U2@@YAXXZ      10004e70 f   moc_EntropyAlgorithm.obj
 0001:00003ef0       ??__EcoreLog@U2@@YAXXZ     10004ef0 f   moc_EntropyAlgorithm.obj
 0001:00003f70       ??__EioLog@U2@@YAXXZ       10004f70 f   moc_EntropyAlgorithm.obj
 0001:00003ff0       ??__EperfLog@U2@@YAXXZ     10004ff0 f   moc_EntropyAlgorithm.obj
 0001:00004070       ??__EscriptLog@U2@@YAXXZ   10005070 f   moc_EntropyAlgorithm.obj
 0001:000040f0       ??__EtaskLog@U2@@YAXXZ     100050f0 f   moc_EntropyAlgorithm.obj
 0001:00004170       ??__EuiLog@U2@@YAXXZ       10005170 f   moc_EntropyAlgorithm.obj
 0001:000041f0       ??__EuserActLog@U2@@YAXXZ  100051f0 f   moc_EntropyAlgorithm.obj
 0001:00004270       ??__E?_Generic_object@?$_Error_objects@H@std@@2V_Generic_error_category@2@A@@YAXXZ 10005270 f   moc_GCFramePlot.obj
 0001:00004280       ??__E?_Iostream_object@?$_Error_objects@H@std@@2V_Iostream_error_category@2@A@@YAXXZ 10005280 f   moc_GCFramePlot.obj
 0001:00004290       ??__E?_System_object@?$_Error_objects@H@std@@2V_System_error_category@2@A@@YAXXZ 10005290 f   moc_GCFramePlot.obj
 0001:000042a0       ??__E?staticMetaObject@GCFramePlotFactory@U2@@2UQMetaObject@@B@@YAXXZ 100052a0 f   moc_GCFramePlot.obj
 0001:000042b0       ??__EService_DNAExport@U2@@YAXXZ 100052b0 f   moc_GCFramePlot.obj
 0001:000042c0       ??__EService_DNAGraphPack@U2@@YAXXZ 100052c0 f   moc_GCFramePlot.obj
 0001:000042d0       ??__EService_ExternalToolSupport@U2@@YAXXZ 100052d0 f   moc_GCFramePlot.obj
 0001:000042e0       ??__EService_GUITesting@U2@@YAXXZ 100052e0 f   moc_GCFramePlot.obj
 0001:000042f0       ??__EService_MaxCoreServiceId@U2@@YAXXZ 100052f0 f   moc_GCFramePlot.obj
 0001:00004300       ??__EService_MinCoreServiceId@U2@@YAXXZ 10005300 f   moc_GCFramePlot.obj
 0001:00004310       ??__EService_PluginViewer@U2@@YAXXZ 10005310 f   moc_GCFramePlot.obj
 0001:00004320       ??__EService_Project@U2@@YAXXZ 10005320 f   moc_GCFramePlot.obj
 0001:00004330       ??__EService_ProjectView@U2@@YAXXZ 10005330 f   moc_GCFramePlot.obj
 0001:00004340       ??__EService_QueryDesigner@U2@@YAXXZ 10005340 f   moc_GCFramePlot.obj
 0001:00004350       ??__EService_ScriptRegistry@U2@@YAXXZ 10005350 f   moc_GCFramePlot.obj
 0001:00004360       ??__EService_TestRunner@U2@@YAXXZ 10005360 f   moc_GCFramePlot.obj
 0001:00004370       ??__EService_WorkflowDesigner@U2@@YAXXZ 10005370 f   moc_GCFramePlot.obj
 0001:00004380       ??__EalgoLog@U2@@YAXXZ     10005380 f   moc_GCFramePlot.obj
 0001:00004400       ??__EcmdLog@U2@@YAXXZ      10005400 f   moc_GCFramePlot.obj
 0001:00004480       ??__EcoreLog@U2@@YAXXZ     10005480 f   moc_GCFramePlot.obj
 0001:00004500       ??__EioLog@U2@@YAXXZ       10005500 f   moc_GCFramePlot.obj
 0001:00004580       ??__EperfLog@U2@@YAXXZ     10005580 f   moc_GCFramePlot.obj
 0001:00004600       ??__EscriptLog@U2@@YAXXZ   10005600 f   moc_GCFramePlot.obj
 0001:00004680       ??__EtaskLog@U2@@YAXXZ     10005680 f   moc_GCFramePlot.obj
 0001:00004700       ??__EuiLog@U2@@YAXXZ       10005700 f   moc_GCFramePlot.obj
 0001:00004780       ??__EuserActLog@U2@@YAXXZ  10005780 f   moc_GCFramePlot.obj
 0001:00004800       ??__E?_Generic_object@?$_Error_objects@H@std@@2V_Generic_error_category@2@A@@YAXXZ 10005800 f   moc_KarlinSignatureDifferenceGraph.obj
 0001:00004810       ??__E?_Iostream_object@?$_Error_objects@H@std@@2V_Iostream_error_category@2@A@@YAXXZ 10005810 f   moc_KarlinSignatureDifferenceGraph.obj
 0001:00004820       ??__E?_System_object@?$_Error_objects@H@std@@2V_System_error_category@2@A@@YAXXZ 10005820 f   moc_KarlinSignatureDifferenceGraph.obj
 0001:00004830       ??__E?staticMetaObject@KarlinGraphFactory@U2@@2UQMetaObject@@B@@YAXXZ 10005830 f   moc_KarlinSignatureDifferenceGraph.obj
 0001:00004840       ??__EService_DNAExport@U2@@YAXXZ 10005840 f   moc_KarlinSignatureDifferenceGraph.obj
 0001:00004850       ??__EService_DNAGraphPack@U2@@YAXXZ 10005850 f   moc_KarlinSignatureDifferenceGraph.obj
 0001:00004860       ??__EService_ExternalToolSupport@U2@@YAXXZ 10005860 f   moc_KarlinSignatureDifferenceGraph.obj
 0001:00004870       ??__EService_GUITesting@U2@@YAXXZ 10005870 f   moc_KarlinSignatureDifferenceGraph.obj
 0001:00004880       ??__EService_MaxCoreServiceId@U2@@YAXXZ 10005880 f   moc_KarlinSignatureDifferenceGraph.obj
 0001:00004890       ??__EService_MinCoreServiceId@U2@@YAXXZ 10005890 f   moc_KarlinSignatureDifferenceGraph.obj
 0001:000048a0       ??__EService_PluginViewer@U2@@YAXXZ 100058a0 f   moc_KarlinSignatureDifferenceGraph.obj
 0001:000048b0       ??__EService_Project@U2@@YAXXZ 100058b0 f   moc_KarlinSignatureDifferenceGraph.obj
 0001:000048c0       ??__EService_ProjectView@U2@@YAXXZ 100058c0 f   moc_KarlinSignatureDifferenceGraph.obj
 0001:000048d0       ??__EService_QueryDesigner@U2@@YAXXZ 100058d0 f   moc_KarlinSignatureDifferenceGraph.obj
 0001:000048e0       ??__EService_ScriptRegistry@U2@@YAXXZ 100058e0 f   moc_KarlinSignatureDifferenceGraph.obj
 0001:000048f0       ??__EService_TestRunner@U2@@YAXXZ 100058f0 f   moc_KarlinSignatureDifferenceGraph.obj
 0001:00004900       ??__EService_WorkflowDesigner@U2@@YAXXZ 10005900 f   moc_KarlinSignatureDifferenceGraph.obj
 0001:00004910       ??__EalgoLog@U2@@YAXXZ     10005910 f   moc_KarlinSignatureDifferenceGraph.obj
 0001:00004990       ??__EcmdLog@U2@@YAXXZ      10005990 f   moc_KarlinSignatureDifferenceGraph.obj
 0001:00004a10       ??__EcoreLog@U2@@YAXXZ     10005a10 f   moc_KarlinSignatureDifferenceGraph.obj
 0001:00004a90       ??__EioLog@U2@@YAXXZ       10005a90 f   moc_KarlinSignatureDifferenceGraph.obj
 0001:00004b10       ??__EperfLog@U2@@YAXXZ     10005b10 f   moc_KarlinSignatureDifferenceGraph.obj
 0001:00004b90       ??__EscriptLog@U2@@YAXXZ   10005b90 f   moc_KarlinSignatureDifferenceGraph.obj
 0001:00004c10       ??__EtaskLog@U2@@YAXXZ     10005c10 f   moc_KarlinSignatureDifferenceGraph.obj
 0001:00004c90       ??__EuiLog@U2@@YAXXZ       10005c90 f   moc_KarlinSignatureDifferenceGraph.obj
 0001:00004d10       ??__EuserActLog@U2@@YAXXZ  10005d10 f   moc_KarlinSignatureDifferenceGraph.obj
 0001:00004d90       ??__Edummy@?A0x701b237d@@YAXXZ 10005d90 f   qrc_dna_graphpack.obj
 0001:00005956       __catch$?_Copy@?$basic_string@DU?$char_traits@D@std@@V?$allocator@D@2@@std@@QAEXII@Z$0 10006956 f i BaseContentGraph.obj
 0001:00005993       __catch$?_Copy@?$basic_string@DU?$char_traits@D@std@@V?$allocator@D@2@@std@@QAEXII@Z$1 10006993 f i BaseContentGraph.obj
 0001:00005d0f       __catch$?append@?$QList@V?$QSharedPointer@VGSequenceGraphData@U2@@@@@@QAEXABV?$QSharedPointer@VGSequenceGraphData@U2@@@@@Z$0 10006d0f f i BaseContentGraph.obj
 0001:00005d0f       __catch$?append@?$QList@V?$QSharedPointer@VGSequenceGraphData@U2@@@@@@QAEXABV?$QSharedPointer@VGSequenceGraphData@U2@@@@@Z$2 10006d0f f i BaseContentGraph.obj
 0001:0000688c       __catch$?detach_helper_grow@?$QList@V?$QSharedPointer@VGSequenceGraphData@U2@@@@@@AAEPAUNode@1@HH@Z$2 1000788c f i BaseContentGraph.obj
 0001:000068c7       __catch$?detach_helper_grow@?$QList@V?$QSharedPointer@VGSequenceGraphData@U2@@@@@@AAEPAUNode@1@HH@Z$0 100078c7 f i BaseContentGraph.obj
 0001:00006d40       ?nameByType@U2@@YA?AVQString@@W4GType@BaseContentGraphFactory@1@@Z 10007d40 f   BaseContentGraph.obj
 0001:00006e7e       __catch$?node_copy@?$QList@V?$QSharedPointer@VGSequenceGraphData@U2@@@@@@AAEXPAUNode@1@00@Z$0 10007e7e f i BaseContentGraph.obj
 0001:00007124       __catch$?reallocData@?$QVector@M@@AAEXHHV?$QFlags@W4AllocationOption@QArrayData@@@@@Z$0 10008124 f i BaseContentGraph.obj
 0001:00007136       __catch$?reallocData@?$QVector@M@@AAEXHHV?$QFlags@W4AllocationOption@QArrayData@@@@@Z$2 10008136 f i BaseContentGraph.obj
 0001:000078f0       ?nameByType@U2@@YA?AVQString@@W4GCumulativeSkewType@CumulativeSkewGraphFactory@1@@Z 100088f0 f   CumulativeSkew.obj
 0001:00007ace       __catch$??0?$QList@PAVADVSequenceWidget@U2@@@@QAE@ABV0@@Z$0 10008ace f i DNAGraphPackPlugin.obj
 0001:00007b8e       __catch$??0?$QList@PAVGSequenceGraphFactory@U2@@@@QAE@ABV0@@Z$0 10008b8e f i DNAGraphPackPlugin.obj
 0001:00008255       __catch$?append@?$QList@PAVGSequenceGraphFactory@U2@@@@QAEXABQAVGSequenceGraphFactory@U2@@@Z$4 10009255 f i DNAGraphPackPlugin.obj
 0001:000083d1       __catch$?detach_helper_grow@?$QList@PAVGSequenceGraphFactory@U2@@@@AAEPAUNode@1@HH@Z$0 100093d1 f i DNAGraphPackPlugin.obj
 0001:000083d1       __catch$?detach_helper_grow@?$QList@PAVGSequenceGraphFactory@U2@@@@AAEPAUNode@1@HH@Z$2 100093d1 f i DNAGraphPackPlugin.obj
 0001:00009050       ?nameByType@U2@@YA?AVQString@@W4GDeviationType@DeviationGraphFactory@1@@Z 1000a050 f   DeviationGraph.obj
 0001:00009304       __catch$?reallocData@?$QVector@H@@AAEXHHV?$QFlags@W4AllocationOption@QArrayData@@@@@Z$0 1000a304 f i DeviationGraph.obj
 0001:00009316       __catch$?reallocData@?$QVector@H@@AAEXHHV?$QFlags@W4AllocationOption@QArrayData@@@@@Z$2 1000a316 f i DeviationGraph.obj
 0001:0000a090       ?nameByType@U2@@YA?AVQString@@XZ 1000b090 f   EntropyAlgorithm.obj
 0001:0000a8e7       __catch$?createNode@?$QMapData@VQString@@VQColor@@@@QAEPAU?$QMapNode@VQString@@VQColor@@@@ABVQString@@ABVQColor@@PAU2@_N@Z$2 1000b8e7 f i GCFramePlot.obj
 0001:0000b5d4       $LN99                      1000c5d4     KarlinSignatureDifferenceGraph.obj
 0001:0000b5e8       $LN92                      1000c5e8     KarlinSignatureDifferenceGraph.obj
 0001:0000b5fc       $LN100                     1000c5fc     KarlinSignatureDifferenceGraph.obj
 0001:0000b610       $LN93                      1000c610     KarlinSignatureDifferenceGraph.obj
 0001:0000b624       $LN101                     1000c624     KarlinSignatureDifferenceGraph.obj
 0001:0000b638       $LN94                      1000c638     KarlinSignatureDifferenceGraph.obj
 0001:0000b64c       $LN102                     1000c64c     KarlinSignatureDifferenceGraph.obj
 0001:0000b660       $LN95                      1000c660     KarlinSignatureDifferenceGraph.obj
 0001:0000b7b0       ?getIndex@U2@@YAHD@Z       1000c7b0 f   KarlinSignatureDifferenceGraph.obj
 0001:0000b7f0       $LN11                      1000c7f0     KarlinSignatureDifferenceGraph.obj
 0001:0000b804       $LN9                       1000c804     KarlinSignatureDifferenceGraph.obj
 0001:0000b920       ?nameByType@U2@@YA?AVQString@@XZ 1000c920 f   KarlinSignatureDifferenceGraph.obj
 0001:0000c6c0       $$000000                   1000d6c0     MSVCRT:ftol3.obj
 0001:0000cb00       $$000000                   1000db00     MSVCRT:lldiv.obj
 0001:0000cbb0       $$000000                   1000dbb0     MSVCRT:llrem.obj
 0001:0000cc6e       _pre_c_init                1000dc6e f   MSVCRT:crtdll.obj
 0001:0000cedb       ___DllMainCRTStartup       1000dedb f   MSVCRT:crtdll.obj
 0001:0000d030       $$000000                   1000e030     MSVCRT:sehprolg4.obj
 0001:0000d44b       ?ArrayUnwindFilter@@YAHPAU_EXCEPTION_POINTERS@@@Z 1000e44b f   MSVCRT:ehvecdtr.obj
 0001:0000d7a0       __unwindfunclet$??0BaseContentGraphAlgorithm@U2@@QAE@ABVQBitArray@@@Z$0 1000e7a0 f   BaseContentGraph.obj
 0001:0000d7a9       __ehhandler$??0BaseContentGraphAlgorithm@U2@@QAE@ABVQBitArray@@@Z 1000e7a9 f   BaseContentGraph.obj
 0001:0000d7d0       __unwindfunclet$??0BaseContentGraphFactory@U2@@QAE@W4GType@01@PAVQObject@@@Z$0 1000e7d0 f   BaseContentGraph.obj
 0001:0000d7d9       __unwindfunclet$??0BaseContentGraphFactory@U2@@QAE@W4GType@01@PAVQObject@@@Z$1 1000e7d9 f   BaseContentGraph.obj
 0001:0000d7e2       __unwindfunclet$??0BaseContentGraphFactory@U2@@QAE@W4GType@01@PAVQObject@@@Z$2 1000e7e2 f   BaseContentGraph.obj
 0001:0000d7ee       __ehhandler$??0BaseContentGraphFactory@U2@@QAE@W4GType@01@PAVQObject@@@Z 1000e7ee f   BaseContentGraph.obj
 0001:0000d810       __unwindfunclet$??1BaseContentGraphAlgorithm@U2@@UAE@XZ$0 1000e810 f   BaseContentGraph.obj
 0001:0000d819       __ehhandler$??1BaseContentGraphAlgorithm@U2@@UAE@XZ 1000e819 f   BaseContentGraph.obj
 0001:0000d840       __unwindfunclet$??1BaseContentGraphFactory@U2@@UAE@XZ$0 1000e840 f   BaseContentGraph.obj
 0001:0000d849       __ehhandler$??1BaseContentGraphFactory@U2@@UAE@XZ 1000e849 f   BaseContentGraph.obj
 0001:0000d870       __unwindfunclet$??_GBaseContentGraphAlgorithm@U2@@UAEPAXI@Z$0 1000e870 f   BaseContentGraph.obj
 0001:0000d879       __ehhandler$??_GBaseContentGraphAlgorithm@U2@@UAEPAXI@Z 1000e879 f   BaseContentGraph.obj
 0001:0000d8a0       __unwindfunclet$??_GBaseContentGraphFactory@U2@@UAEPAXI@Z$0 1000e8a0 f   BaseContentGraph.obj
 0001:0000d8a9       __ehhandler$??_GBaseContentGraphFactory@U2@@UAEPAXI@Z 1000e8a9 f   BaseContentGraph.obj
 0001:0000d8d0       __unwindfunclet$??__EalgoLog@U2@@YAXXZ$0 1000e8d0 f   BaseContentGraph.obj
 0001:0000d8d9       __ehhandler$??__EalgoLog@U2@@YAXXZ 1000e8d9 f   BaseContentGraph.obj
 0001:0000d900       __unwindfunclet$??__EcmdLog@U2@@YAXXZ$0 1000e900 f   BaseContentGraph.obj
 0001:0000d909       __ehhandler$??__EcmdLog@U2@@YAXXZ 1000e909 f   BaseContentGraph.obj
 0001:0000d930       __unwindfunclet$??__EcoreLog@U2@@YAXXZ$0 1000e930 f   BaseContentGraph.obj
 0001:0000d939       __ehhandler$??__EcoreLog@U2@@YAXXZ 1000e939 f   BaseContentGraph.obj
 0001:0000d960       __unwindfunclet$??__EioLog@U2@@YAXXZ$0 1000e960 f   BaseContentGraph.obj
 0001:0000d969       __ehhandler$??__EioLog@U2@@YAXXZ 1000e969 f   BaseContentGraph.obj
 0001:0000d990       __unwindfunclet$??__EperfLog@U2@@YAXXZ$0 1000e990 f   BaseContentGraph.obj
 0001:0000d999       __ehhandler$??__EperfLog@U2@@YAXXZ 1000e999 f   BaseContentGraph.obj
 0001:0000d9c0       __unwindfunclet$??__EscriptLog@U2@@YAXXZ$0 1000e9c0 f   BaseContentGraph.obj
 0001:0000d9c9       __ehhandler$??__EscriptLog@U2@@YAXXZ 1000e9c9 f   BaseContentGraph.obj
 0001:0000d9f0       __unwindfunclet$??__EtaskLog@U2@@YAXXZ$0 1000e9f0 f   BaseContentGraph.obj
 0001:0000d9f9       __ehhandler$??__EtaskLog@U2@@YAXXZ 1000e9f9 f   BaseContentGraph.obj
 0001:0000da20       __unwindfunclet$??__EuiLog@U2@@YAXXZ$0 1000ea20 f   BaseContentGraph.obj
 0001:0000da29       __ehhandler$??__EuiLog@U2@@YAXXZ 1000ea29 f   BaseContentGraph.obj
 0001:0000da50       __unwindfunclet$??__EuserActLog@U2@@YAXXZ$0 1000ea50 f   BaseContentGraph.obj
 0001:0000da59       __ehhandler$??__EuserActLog@U2@@YAXXZ 1000ea59 f   BaseContentGraph.obj
 0001:0000da80       __ehhandler$?_Copy@?$basic_string@DU?$char_traits@D@std@@V?$allocator@D@2@@std@@QAEXII@Z 1000ea80 f   BaseContentGraph.obj
 0001:0000daa0       __ehhandler$?append@?$QList@V?$QSharedPointer@VGSequenceGraphData@U2@@@@@@QAEXABV?$QSharedPointer@VGSequenceGraphData@U2@@@@@Z 1000eaa0 f   BaseContentGraph.obj
 0001:0000dac0       __unwindfunclet$?calculate@BaseContentGraphAlgorithm@U2@@UAEXAAV?$QVector@M@@PAVU2SequenceObject@2@ABVU2Region@2@PBVGSequenceGraphWindowData@2@AAVU2OpStatus@2@@Z$0 1000eac0 f   BaseContentGraph.obj
 0001:0000dac9       __unwindfunclet$?calculate@BaseContentGraphAlgorithm@U2@@UAEXAAV?$QVector@M@@PAVU2SequenceObject@2@ABVU2Region@2@PBVGSequenceGraphWindowData@2@AAVU2OpStatus@2@@Z$1 1000eac9 f   BaseContentGraph.obj
 0001:0000dad2       __unwindfunclet$?calculate@BaseContentGraphAlgorithm@U2@@UAEXAAV?$QVector@M@@PAVU2SequenceObject@2@ABVU2Region@2@PBVGSequenceGraphWindowData@2@AAVU2OpStatus@2@@Z$2 1000ead2 f   BaseContentGraph.obj
 0001:0000dadb       __unwindfunclet$?calculate@BaseContentGraphAlgorithm@U2@@UAEXAAV?$QVector@M@@PAVU2SequenceObject@2@ABVU2Region@2@PBVGSequenceGraphWindowData@2@AAVU2OpStatus@2@@Z$3 1000eadb f   BaseContentGraph.obj
 0001:0000dae4       __unwindfunclet$?calculate@BaseContentGraphAlgorithm@U2@@UAEXAAV?$QVector@M@@PAVU2SequenceObject@2@ABVU2Region@2@PBVGSequenceGraphWindowData@2@AAVU2OpStatus@2@@Z$4 1000eae4 f   BaseContentGraph.obj
 0001:0000daed       __unwindfunclet$?calculate@BaseContentGraphAlgorithm@U2@@UAEXAAV?$QVector@M@@PAVU2SequenceObject@2@ABVU2Region@2@PBVGSequenceGraphWindowData@2@AAVU2OpStatus@2@@Z$5 1000eaed f   BaseContentGraph.obj
 0001:0000daf6       __unwindfunclet$?calculate@BaseContentGraphAlgorithm@U2@@UAEXAAV?$QVector@M@@PAVU2SequenceObject@2@ABVU2Region@2@PBVGSequenceGraphWindowData@2@AAVU2OpStatus@2@@Z$6 1000eaf6 f   BaseContentGraph.obj
 0001:0000daff       __unwindfunclet$?calculate@BaseContentGraphAlgorithm@U2@@UAEXAAV?$QVector@M@@PAVU2SequenceObject@2@ABVU2Region@2@PBVGSequenceGraphWindowData@2@AAVU2OpStatus@2@@Z$7 1000eaff f   BaseContentGraph.obj
 0001:0000db08       __unwindfunclet$?calculate@BaseContentGraphAlgorithm@U2@@UAEXAAV?$QVector@M@@PAVU2SequenceObject@2@ABVU2Region@2@PBVGSequenceGraphWindowData@2@AAVU2OpStatus@2@@Z$8 1000eb08 f   BaseContentGraph.obj
 0001:0000db11       __unwindfunclet$?calculate@BaseContentGraphAlgorithm@U2@@UAEXAAV?$QVector@M@@PAVU2SequenceObject@2@ABVU2Region@2@PBVGSequenceGraphWindowData@2@AAVU2OpStatus@2@@Z$9 1000eb11 f   BaseContentGraph.obj
 0001:0000db1a       __unwindfunclet$?calculate@BaseContentGraphAlgorithm@U2@@UAEXAAV?$QVector@M@@PAVU2SequenceObject@2@ABVU2Region@2@PBVGSequenceGraphWindowData@2@AAVU2OpStatus@2@@Z$10 1000eb1a f   BaseContentGraph.obj
 0001:0000db23       __unwindfunclet$?calculate@BaseContentGraphAlgorithm@U2@@UAEXAAV?$QVector@M@@PAVU2SequenceObject@2@ABVU2Region@2@PBVGSequenceGraphWindowData@2@AAVU2OpStatus@2@@Z$11 1000eb23 f   BaseContentGraph.obj
 0001:0000db2c       __unwindfunclet$?calculate@BaseContentGraphAlgorithm@U2@@UAEXAAV?$QVector@M@@PAVU2SequenceObject@2@ABVU2Region@2@PBVGSequenceGraphWindowData@2@AAVU2OpStatus@2@@Z$12 1000eb2c f   BaseContentGraph.obj
 0001:0000db35       __unwindfunclet$?calculate@BaseContentGraphAlgorithm@U2@@UAEXAAV?$QVector@M@@PAVU2SequenceObject@2@ABVU2Region@2@PBVGSequenceGraphWindowData@2@AAVU2OpStatus@2@@Z$13 1000eb35 f   BaseContentGraph.obj
 0001:0000db3e       __ehhandler$?calculate@BaseContentGraphAlgorithm@U2@@UAEXAAV?$QVector@M@@PAVU2SequenceObject@2@ABVU2Region@2@PBVGSequenceGraphWindowData@2@AAVU2OpStatus@2@@Z 1000eb3e f   BaseContentGraph.obj
 0001:0000db60       __unwindfunclet$?createGraphs@BaseContentGraphFactory@U2@@UAE?AV?$QList@V?$QSharedPointer@VGSequenceGraphData@U2@@@@@@PAVGSequenceGraphView@2@@Z$0 1000eb60 f   BaseContentGraph.obj
 0001:0000db79       __unwindfunclet$?createGraphs@BaseContentGraphFactory@U2@@UAE?AV?$QList@V?$QSharedPointer@VGSequenceGraphData@U2@@@@@@PAVGSequenceGraphView@2@@Z$1 1000eb79 f   BaseContentGraph.obj
 0001:0000db84       __unwindfunclet$?createGraphs@BaseContentGraphFactory@U2@@UAE?AV?$QList@V?$QSharedPointer@VGSequenceGraphData@U2@@@@@@PAVGSequenceGraphView@2@@Z$2 1000eb84 f   BaseContentGraph.obj
 0001:0000db8c       __unwindfunclet$?createGraphs@BaseContentGraphFactory@U2@@UAE?AV?$QList@V?$QSharedPointer@VGSequenceGraphData@U2@@@@@@PAVGSequenceGraphView@2@@Z$3 1000eb8c f   BaseContentGraph.obj
 0001:0000db97       __unwindfunclet$?createGraphs@BaseContentGraphFactory@U2@@UAE?AV?$QList@V?$QSharedPointer@VGSequenceGraphData@U2@@@@@@PAVGSequenceGraphView@2@@Z$4 1000eb97 f   BaseContentGraph.obj
 0001:0000dba0       __ehhandler$?createGraphs@BaseContentGraphFactory@U2@@UAE?AV?$QList@V?$QSharedPointer@VGSequenceGraphData@U2@@@@@@PAVGSequenceGraphView@2@@Z 1000eba0 f   BaseContentGraph.obj
 0001:0000dbc0       __ehhandler$?detach_helper_grow@?$QList@V?$QSharedPointer@VGSequenceGraphData@U2@@@@@@AAEPAUNode@1@HH@Z 1000ebc0 f   BaseContentGraph.obj
 0001:0000dbe0       __ehhandler$?node_copy@?$QList@V?$QSharedPointer@VGSequenceGraphData@U2@@@@@@AAEXPAUNode@1@00@Z 1000ebe0 f   BaseContentGraph.obj
 0001:0000dc00       __ehhandler$?reallocData@?$QVector@M@@AAEXHHV?$QFlags@W4AllocationOption@QArrayData@@@@@Z 1000ec00 f   BaseContentGraph.obj
 0001:0000dc20       __unwindfunclet$??0CumulativeSkewGraphFactory@U2@@QAE@W4GCumulativeSkewType@01@PAVQObject@@@Z$0 1000ec20 f   CumulativeSkew.obj
 0001:0000dc29       __unwindfunclet$??0CumulativeSkewGraphFactory@U2@@QAE@W4GCumulativeSkewType@01@PAVQObject@@@Z$1 1000ec29 f   CumulativeSkew.obj
 0001:0000dc32       __ehhandler$??0CumulativeSkewGraphFactory@U2@@QAE@W4GCumulativeSkewType@01@PAVQObject@@@Z 1000ec32 f   CumulativeSkew.obj
 0001:0000dc50       __unwindfunclet$??__EalgoLog@U2@@YAXXZ$0 1000ec50 f   CumulativeSkew.obj
 0001:0000dc59       __ehhandler$??__EalgoLog@U2@@YAXXZ 1000ec59 f   CumulativeSkew.obj
 0001:0000dc80       __unwindfunclet$??__EcmdLog@U2@@YAXXZ$0 1000ec80 f   CumulativeSkew.obj
 0001:0000dc89       __ehhandler$??__EcmdLog@U2@@YAXXZ 1000ec89 f   CumulativeSkew.obj
 0001:0000dcb0       __unwindfunclet$??__EcoreLog@U2@@YAXXZ$0 1000ecb0 f   CumulativeSkew.obj
 0001:0000dcb9       __ehhandler$??__EcoreLog@U2@@YAXXZ 1000ecb9 f   CumulativeSkew.obj
 0001:0000dce0       __unwindfunclet$??__EioLog@U2@@YAXXZ$0 1000ece0 f   CumulativeSkew.obj
 0001:0000dce9       __ehhandler$??__EioLog@U2@@YAXXZ 1000ece9 f   CumulativeSkew.obj
 0001:0000dd10       __unwindfunclet$??__EperfLog@U2@@YAXXZ$0 1000ed10 f   CumulativeSkew.obj
 0001:0000dd19       __ehhandler$??__EperfLog@U2@@YAXXZ 1000ed19 f   CumulativeSkew.obj
 0001:0000dd40       __unwindfunclet$??__EscriptLog@U2@@YAXXZ$0 1000ed40 f   CumulativeSkew.obj
 0001:0000dd49       __ehhandler$??__EscriptLog@U2@@YAXXZ 1000ed49 f   CumulativeSkew.obj
 0001:0000dd70       __unwindfunclet$??__EtaskLog@U2@@YAXXZ$0 1000ed70 f   CumulativeSkew.obj
 0001:0000dd79       __ehhandler$??__EtaskLog@U2@@YAXXZ 1000ed79 f   CumulativeSkew.obj
 0001:0000dda0       __unwindfunclet$??__EuiLog@U2@@YAXXZ$0 1000eda0 f   CumulativeSkew.obj
 0001:0000dda9       __ehhandler$??__EuiLog@U2@@YAXXZ 1000eda9 f   CumulativeSkew.obj
 0001:0000ddd0       __unwindfunclet$??__EuserActLog@U2@@YAXXZ$0 1000edd0 f   CumulativeSkew.obj
 0001:0000ddd9       __ehhandler$??__EuserActLog@U2@@YAXXZ 1000edd9 f   CumulativeSkew.obj
 0001:0000de00       __unwindfunclet$?createGraphs@CumulativeSkewGraphFactory@U2@@UAE?AV?$QList@V?$QSharedPointer@VGSequenceGraphData@U2@@@@@@PAVGSequenceGraphView@2@@Z$0 1000ee00 f   CumulativeSkew.obj
 0001:0000de19       __unwindfunclet$?createGraphs@CumulativeSkewGraphFactory@U2@@UAE?AV?$QList@V?$QSharedPointer@VGSequenceGraphData@U2@@@@@@PAVGSequenceGraphView@2@@Z$1 1000ee19 f   CumulativeSkew.obj
 0001:0000de24       __unwindfunclet$?createGraphs@CumulativeSkewGraphFactory@U2@@UAE?AV?$QList@V?$QSharedPointer@VGSequenceGraphData@U2@@@@@@PAVGSequenceGraphView@2@@Z$2 1000ee24 f   CumulativeSkew.obj
 0001:0000de2c       __unwindfunclet$?createGraphs@CumulativeSkewGraphFactory@U2@@UAE?AV?$QList@V?$QSharedPointer@VGSequenceGraphData@U2@@@@@@PAVGSequenceGraphView@2@@Z$3 1000ee2c f   CumulativeSkew.obj
 0001:0000de37       __ehhandler$?createGraphs@CumulativeSkewGraphFactory@U2@@UAE?AV?$QList@V?$QSharedPointer@VGSequenceGraphData@U2@@@@@@PAVGSequenceGraphView@2@@Z 1000ee37 f   CumulativeSkew.obj
 0001:0000de60       __ehhandler$??0?$QList@PAVADVSequenceWidget@U2@@@@QAE@ABV0@@Z 1000ee60 f   DNAGraphPackPlugin.obj
 0001:0000de80       __ehhandler$??0?$QList@PAVGSequenceGraphFactory@U2@@@@QAE@ABV0@@Z 1000ee80 f   DNAGraphPackPlugin.obj
 0001:0000dea0       __unwindfunclet$??0DNAGraphPackPlugin@U2@@QAE@XZ$0 1000eea0 f   DNAGraphPackPlugin.obj
 0001:0000dea9       __unwindfunclet$??0DNAGraphPackPlugin@U2@@QAE@XZ$1 1000eea9 f   DNAGraphPackPlugin.obj
 0001:0000deb2       __unwindfunclet$??0DNAGraphPackPlugin@U2@@QAE@XZ$2 1000eeb2 f   DNAGraphPackPlugin.obj
 0001:0000debb       __unwindfunclet$??0DNAGraphPackPlugin@U2@@QAE@XZ$3 1000eebb f   DNAGraphPackPlugin.obj
 0001:0000dec6       __ehhandler$??0DNAGraphPackPlugin@U2@@QAE@XZ 1000eec6 f   DNAGraphPackPlugin.obj
 0001:0000def0       __unwindfunclet$??0DNAGraphPackViewContext@U2@@QAE@PAVQObject@@@Z$0 1000eef0 f   DNAGraphPackPlugin.obj
 0001:0000def8       __unwindfunclet$??0DNAGraphPackViewContext@U2@@QAE@PAVQObject@@@Z$1 1000eef8 f   DNAGraphPackPlugin.obj
 0001:0000df01       __unwindfunclet$??0DNAGraphPackViewContext@U2@@QAE@PAVQObject@@@Z$2 1000ef01 f   DNAGraphPackPlugin.obj
 0001:0000df0c       __unwindfunclet$??0DNAGraphPackViewContext@U2@@QAE@PAVQObject@@@Z$3 1000ef0c f   DNAGraphPackPlugin.obj
 0001:0000df17       __unwindfunclet$??0DNAGraphPackViewContext@U2@@QAE@PAVQObject@@@Z$4 1000ef17 f   DNAGraphPackPlugin.obj
 0001:0000df22       __unwindfunclet$??0DNAGraphPackViewContext@U2@@QAE@PAVQObject@@@Z$5 1000ef22 f   DNAGraphPackPlugin.obj
 0001:0000df2d       __unwindfunclet$??0DNAGraphPackViewContext@U2@@QAE@PAVQObject@@@Z$6 1000ef2d f   DNAGraphPackPlugin.obj
 0001:0000df38       __unwindfunclet$??0DNAGraphPackViewContext@U2@@QAE@PAVQObject@@@Z$7 1000ef38 f   DNAGraphPackPlugin.obj
 0001:0000df43       __unwindfunclet$??0DNAGraphPackViewContext@U2@@QAE@PAVQObject@@@Z$8 1000ef43 f   DNAGraphPackPlugin.obj
 0001:0000df4e       __unwindfunclet$??0DNAGraphPackViewContext@U2@@QAE@PAVQObject@@@Z$9 1000ef4e f   DNAGraphPackPlugin.obj
 0001:0000df59       __ehhandler$??0DNAGraphPackViewContext@U2@@QAE@PAVQObject@@@Z 1000ef59 f   DNAGraphPackPlugin.obj
 0001:0000df80       __unwindfunclet$??1DNAGraphPackViewContext@U2@@UAE@XZ$0 1000ef80 f   DNAGraphPackPlugin.obj
 0001:0000df89       __ehhandler$??1DNAGraphPackViewContext@U2@@UAE@XZ 1000ef89 f   DNAGraphPackPlugin.obj
 0001:0000dfb0       __unwindfunclet$??_GDNAGraphPackViewContext@U2@@UAEPAXI@Z$0 1000efb0 f   DNAGraphPackPlugin.obj
 0001:0000dfb9       __ehhandler$??_GDNAGraphPackViewContext@U2@@UAEPAXI@Z 1000efb9 f   DNAGraphPackPlugin.obj
 0001:0000dfe0       __unwindfunclet$??__EalgoLog@U2@@YAXXZ$0 1000efe0 f   DNAGraphPackPlugin.obj
 0001:0000dfe9       __ehhandler$??__EalgoLog@U2@@YAXXZ 1000efe9 f   DNAGraphPackPlugin.obj
 0001:0000e010       __unwindfunclet$??__EcmdLog@U2@@YAXXZ$0 1000f010 f   DNAGraphPackPlugin.obj
 0001:0000e019       __ehhandler$??__EcmdLog@U2@@YAXXZ 1000f019 f   DNAGraphPackPlugin.obj
 0001:0000e040       __unwindfunclet$??__EcoreLog@U2@@YAXXZ$0 1000f040 f   DNAGraphPackPlugin.obj
 0001:0000e049       __ehhandler$??__EcoreLog@U2@@YAXXZ 1000f049 f   DNAGraphPackPlugin.obj
 0001:0000e070       __unwindfunclet$??__EioLog@U2@@YAXXZ$0 1000f070 f   DNAGraphPackPlugin.obj
 0001:0000e079       __ehhandler$??__EioLog@U2@@YAXXZ 1000f079 f   DNAGraphPackPlugin.obj
 0001:0000e0a0       __unwindfunclet$??__EperfLog@U2@@YAXXZ$0 1000f0a0 f   DNAGraphPackPlugin.obj
 0001:0000e0a9       __ehhandler$??__EperfLog@U2@@YAXXZ 1000f0a9 f   DNAGraphPackPlugin.obj
 0001:0000e0d0       __unwindfunclet$??__EscriptLog@U2@@YAXXZ$0 1000f0d0 f   DNAGraphPackPlugin.obj
 0001:0000e0d9       __ehhandler$??__EscriptLog@U2@@YAXXZ 1000f0d9 f   DNAGraphPackPlugin.obj
 0001:0000e100       __unwindfunclet$??__EtaskLog@U2@@YAXXZ$0 1000f100 f   DNAGraphPackPlugin.obj
 0001:0000e109       __ehhandler$??__EtaskLog@U2@@YAXXZ 1000f109 f   DNAGraphPackPlugin.obj
 0001:0000e130       __unwindfunclet$??__EuiLog@U2@@YAXXZ$0 1000f130 f   DNAGraphPackPlugin.obj
 0001:0000e139       __ehhandler$??__EuiLog@U2@@YAXXZ 1000f139 f   DNAGraphPackPlugin.obj
 0001:0000e160       __unwindfunclet$??__EuserActLog@U2@@YAXXZ$0 1000f160 f   DNAGraphPackPlugin.obj
 0001:0000e169       __ehhandler$??__EuserActLog@U2@@YAXXZ 1000f169 f   DNAGraphPackPlugin.obj
 0001:0000e190       __ehhandler$?append@?$QList@PAVGSequenceGraphFactory@U2@@@@QAEXABQAVGSequenceGraphFactory@U2@@@Z 1000f190 f   DNAGraphPackPlugin.obj
 0001:0000e1b0       __ehhandler$?detach_helper_grow@?$QList@PAVGSequenceGraphFactory@U2@@@@AAEPAUNode@1@HH@Z 1000f1b0 f   DNAGraphPackPlugin.obj
 0001:0000e1d0       __unwindfunclet$?initViewContext@DNAGraphPackViewContext@U2@@EAEXPAVGObjectView@2@@Z$1 1000f1d0 f   DNAGraphPackPlugin.obj
 0001:0000e1d8       __unwindfunclet$?initViewContext@DNAGraphPackViewContext@U2@@EAEXPAVGObjectView@2@@Z$2 1000f1d8 f   DNAGraphPackPlugin.obj
 0001:0000e1e0       __ehhandler$?initViewContext@DNAGraphPackViewContext@U2@@EAEXPAVGObjectView@2@@Z 1000f1e0 f   DNAGraphPackPlugin.obj
 0001:0000e200       __unwindfunclet$?sl_sequenceWidgetAdded@DNAGraphPackViewContext@U2@@AAEXPAVADVSequenceWidget@2@@Z$0 1000f200 f   DNAGraphPackPlugin.obj
 0001:0000e208       __unwindfunclet$?sl_sequenceWidgetAdded@DNAGraphPackViewContext@U2@@AAEXPAVADVSequenceWidget@2@@Z$1 1000f208 f   DNAGraphPackPlugin.obj
 0001:0000e213       __ehhandler$?sl_sequenceWidgetAdded@DNAGraphPackViewContext@U2@@AAEXPAVADVSequenceWidget@2@@Z 1000f213 f   DNAGraphPackPlugin.obj
 0001:0000e230       __unwindfunclet$??0?$RollingArray@H@U2@@QAE@H@Z$0 1000f230 f   DeviationGraph.obj
 0001:0000e238       __ehhandler$??0?$RollingArray@H@U2@@QAE@H@Z 1000f238 f   DeviationGraph.obj
 0001:0000e260       __unwindfunclet$??0DeviationGraphFactory@U2@@QAE@W4GDeviationType@01@PAVQObject@@@Z$0 1000f260 f   DeviationGraph.obj
 0001:0000e269       __unwindfunclet$??0DeviationGraphFactory@U2@@QAE@W4GDeviationType@01@PAVQObject@@@Z$1 1000f269 f   DeviationGraph.obj
 0001:0000e272       __ehhandler$??0DeviationGraphFactory@U2@@QAE@W4GDeviationType@01@PAVQObject@@@Z 1000f272 f   DeviationGraph.obj
 0001:0000e290       __unwindfunclet$??__EalgoLog@U2@@YAXXZ$0 1000f290 f   DeviationGraph.obj
 0001:0000e299       __ehhandler$??__EalgoLog@U2@@YAXXZ 1000f299 f   DeviationGraph.obj
 0001:0000e2c0       __unwindfunclet$??__EcmdLog@U2@@YAXXZ$0 1000f2c0 f   DeviationGraph.obj
 0001:0000e2c9       __ehhandler$??__EcmdLog@U2@@YAXXZ 1000f2c9 f   DeviationGraph.obj
 0001:0000e2f0       __unwindfunclet$??__EcoreLog@U2@@YAXXZ$0 1000f2f0 f   DeviationGraph.obj
 0001:0000e2f9       __ehhandler$??__EcoreLog@U2@@YAXXZ 1000f2f9 f   DeviationGraph.obj
 0001:0000e320       __unwindfunclet$??__EioLog@U2@@YAXXZ$0 1000f320 f   DeviationGraph.obj
 0001:0000e329       __ehhandler$??__EioLog@U2@@YAXXZ 1000f329 f   DeviationGraph.obj
 0001:0000e350       __unwindfunclet$??__EperfLog@U2@@YAXXZ$0 1000f350 f   DeviationGraph.obj
 0001:0000e359       __ehhandler$??__EperfLog@U2@@YAXXZ 1000f359 f   DeviationGraph.obj
 0001:0000e380       __unwindfunclet$??__EscriptLog@U2@@YAXXZ$0 1000f380 f   DeviationGraph.obj
 0001:0000e389       __ehhandler$??__EscriptLog@U2@@YAXXZ 1000f389 f   DeviationGraph.obj
 0001:0000e3b0       __unwindfunclet$??__EtaskLog@U2@@YAXXZ$0 1000f3b0 f   DeviationGraph.obj
 0001:0000e3b9       __ehhandler$??__EtaskLog@U2@@YAXXZ 1000f3b9 f   DeviationGraph.obj
 0001:0000e3e0       __unwindfunclet$??__EuiLog@U2@@YAXXZ$0 1000f3e0 f   DeviationGraph.obj
 0001:0000e3e9       __ehhandler$??__EuiLog@U2@@YAXXZ 1000f3e9 f   DeviationGraph.obj
 0001:0000e410       __unwindfunclet$??__EuserActLog@U2@@YAXXZ$0 1000f410 f   DeviationGraph.obj
 0001:0000e419       __ehhandler$??__EuserActLog@U2@@YAXXZ 1000f419 f   DeviationGraph.obj
 0001:0000e440       __unwindfunclet$?createGraphs@DeviationGraphFactory@U2@@UAE?AV?$QList@V?$QSharedPointer@VGSequenceGraphData@U2@@@@@@PAVGSequenceGraphView@2@@Z$0 1000f440 f   DeviationGraph.obj
 0001:0000e459       __unwindfunclet$?createGraphs@DeviationGraphFactory@U2@@UAE?AV?$QList@V?$QSharedPointer@VGSequenceGraphData@U2@@@@@@PAVGSequenceGraphView@2@@Z$1 1000f459 f   DeviationGraph.obj
 0001:0000e464       __unwindfunclet$?createGraphs@DeviationGraphFactory@U2@@UAE?AV?$QList@V?$QSharedPointer@VGSequenceGraphData@U2@@@@@@PAVGSequenceGraphView@2@@Z$2 1000f464 f   DeviationGraph.obj
 0001:0000e46c       __unwindfunclet$?createGraphs@DeviationGraphFactory@U2@@UAE?AV?$QList@V?$QSharedPointer@VGSequenceGraphData@U2@@@@@@PAVGSequenceGraphView@2@@Z$3 1000f46c f   DeviationGraph.obj
 0001:0000e477       __ehhandler$?createGraphs@DeviationGraphFactory@U2@@UAE?AV?$QList@V?$QSharedPointer@VGSequenceGraphData@U2@@@@@@PAVGSequenceGraphView@2@@Z 1000f477 f   DeviationGraph.obj
 0001:0000e4a0       __ehhandler$?reallocData@?$QVector@H@@AAEXHHV?$QFlags@W4AllocationOption@QArrayData@@@@@Z 1000f4a0 f   DeviationGraph.obj
 0001:0000e4c0       __unwindfunclet$?sequenceStrategyWithMemorize@DeviationGraphAlgorithm@U2@@AAEXAAV?$QVector@M@@ABVQByteArray@@ABVU2Region@2@PBVGSequenceGraphWindowData@2@AAVU2OpStatus@2@@Z$0 1000f4c0 f   DeviationGraph.obj
 0001:0000e4c8       __unwindfunclet$?sequenceStrategyWithMemorize@DeviationGraphAlgorithm@U2@@AAEXAAV?$QVector@M@@ABVQByteArray@@ABVU2Region@2@PBVGSequenceGraphWindowData@2@AAVU2OpStatus@2@@Z$1 1000f4c8 f   DeviationGraph.obj
 0001:0000e4d0       __ehhandler$?sequenceStrategyWithMemorize@DeviationGraphAlgorithm@U2@@AAEXAAV?$QVector@M@@ABVQByteArray@@ABVU2Region@2@PBVGSequenceGraphWindowData@2@AAVU2OpStatus@2@@Z 1000f4d0 f   DeviationGraph.obj
 0001:0000e4f0       __unwindfunclet$??0EntropyGraphFactory@U2@@QAE@PAVQObject@@@Z$0 1000f4f0 f   EntropyAlgorithm.obj
 0001:0000e4f9       __unwindfunclet$??0EntropyGraphFactory@U2@@QAE@PAVQObject@@@Z$1 1000f4f9 f   EntropyAlgorithm.obj
 0001:0000e502       __ehhandler$??0EntropyGraphFactory@U2@@QAE@PAVQObject@@@Z 1000f502 f   EntropyAlgorithm.obj
 0001:0000e520       __unwindfunclet$??__EalgoLog@U2@@YAXXZ$0 1000f520 f   EntropyAlgorithm.obj
 0001:0000e529       __ehhandler$??__EalgoLog@U2@@YAXXZ 1000f529 f   EntropyAlgorithm.obj
 0001:0000e550       __unwindfunclet$??__EcmdLog@U2@@YAXXZ$0 1000f550 f   EntropyAlgorithm.obj
 0001:0000e559       __ehhandler$??__EcmdLog@U2@@YAXXZ 1000f559 f   EntropyAlgorithm.obj
 0001:0000e580       __unwindfunclet$??__EcoreLog@U2@@YAXXZ$0 1000f580 f   EntropyAlgorithm.obj
 0001:0000e589       __ehhandler$??__EcoreLog@U2@@YAXXZ 1000f589 f   EntropyAlgorithm.obj
 0001:0000e5b0       __unwindfunclet$??__EioLog@U2@@YAXXZ$0 1000f5b0 f   EntropyAlgorithm.obj
 0001:0000e5b9       __ehhandler$??__EioLog@U2@@YAXXZ 1000f5b9 f   EntropyAlgorithm.obj
 0001:0000e5e0       __unwindfunclet$??__EperfLog@U2@@YAXXZ$0 1000f5e0 f   EntropyAlgorithm.obj
 0001:0000e5e9       __ehhandler$??__EperfLog@U2@@YAXXZ 1000f5e9 f   EntropyAlgorithm.obj
 0001:0000e610       __unwindfunclet$??__EscriptLog@U2@@YAXXZ$0 1000f610 f   EntropyAlgorithm.obj
 0001:0000e619       __ehhandler$??__EscriptLog@U2@@YAXXZ 1000f619 f   EntropyAlgorithm.obj
 0001:0000e640       __unwindfunclet$??__EtaskLog@U2@@YAXXZ$0 1000f640 f   EntropyAlgorithm.obj
 0001:0000e649       __ehhandler$??__EtaskLog@U2@@YAXXZ 1000f649 f   EntropyAlgorithm.obj
 0001:0000e670       __unwindfunclet$??__EuiLog@U2@@YAXXZ$0 1000f670 f   EntropyAlgorithm.obj
 0001:0000e679       __ehhandler$??__EuiLog@U2@@YAXXZ 1000f679 f   EntropyAlgorithm.obj
 0001:0000e6a0       __unwindfunclet$??__EuserActLog@U2@@YAXXZ$0 1000f6a0 f   EntropyAlgorithm.obj
 0001:0000e6a9       __ehhandler$??__EuserActLog@U2@@YAXXZ 1000f6a9 f   EntropyAlgorithm.obj
 0001:0000e6d0       __unwindfunclet$?calculate@EntropyGraphAlgorithm@U2@@UAEXAAV?$QVector@M@@PAVU2SequenceObject@2@ABVU2Region@2@PBVGSequenceGraphWindowData@2@AAVU2OpStatus@2@@Z$0 1000f6d0 f   EntropyAlgorithm.obj
 0001:0000e6dc       __unwindfunclet$?calculate@EntropyGraphAlgorithm@U2@@UAEXAAV?$QVector@M@@PAVU2SequenceObject@2@ABVU2Region@2@PBVGSequenceGraphWindowData@2@AAVU2OpStatus@2@@Z$1 1000f6dc f   EntropyAlgorithm.obj
 0001:0000e6e7       __ehhandler$?calculate@EntropyGraphAlgorithm@U2@@UAEXAAV?$QVector@M@@PAVU2SequenceObject@2@ABVU2Region@2@PBVGSequenceGraphWindowData@2@AAVU2OpStatus@2@@Z 1000f6e7 f   EntropyAlgorithm.obj
 0001:0000e710       __unwindfunclet$?createGraphs@EntropyGraphFactory@U2@@UAE?AV?$QList@V?$QSharedPointer@VGSequenceGraphData@U2@@@@@@PAVGSequenceGraphView@2@@Z$0 1000f710 f   EntropyAlgorithm.obj
 0001:0000e729       __unwindfunclet$?createGraphs@EntropyGraphFactory@U2@@UAE?AV?$QList@V?$QSharedPointer@VGSequenceGraphData@U2@@@@@@PAVGSequenceGraphView@2@@Z$1 1000f729 f   EntropyAlgorithm.obj
 0001:0000e734       __unwindfunclet$?createGraphs@EntropyGraphFactory@U2@@UAE?AV?$QList@V?$QSharedPointer@VGSequenceGraphData@U2@@@@@@PAVGSequenceGraphView@2@@Z$2 1000f734 f   EntropyAlgorithm.obj
 0001:0000e73c       __unwindfunclet$?createGraphs@EntropyGraphFactory@U2@@UAE?AV?$QList@V?$QSharedPointer@VGSequenceGraphData@U2@@@@@@PAVGSequenceGraphView@2@@Z$3 1000f73c f   EntropyAlgorithm.obj
 0001:0000e747       __ehhandler$?createGraphs@EntropyGraphFactory@U2@@UAE?AV?$QList@V?$QSharedPointer@VGSequenceGraphData@U2@@@@@@PAVGSequenceGraphView@2@@Z 1000f747 f   EntropyAlgorithm.obj
 0001:0000e770       __unwindfunclet$??0GCFramePlotAlgorithm@U2@@QAE@H@Z$0 1000f770 f   GCFramePlot.obj
 0001:0000e779       __unwindfunclet$??0GCFramePlotAlgorithm@U2@@QAE@H@Z$1 1000f779 f   GCFramePlot.obj
 0001:0000e785       __ehhandler$??0GCFramePlotAlgorithm@U2@@QAE@H@Z 1000f785 f   GCFramePlot.obj
 0001:0000e7a0       __unwindfunclet$??0GCFramePlotFactory@U2@@QAE@PAVQObject@@@Z$0 1000f7a0 f   GCFramePlot.obj
 0001:0000e7a9       __unwindfunclet$??0GCFramePlotFactory@U2@@QAE@PAVQObject@@@Z$1 1000f7a9 f   GCFramePlot.obj
 0001:0000e7b2       __ehhandler$??0GCFramePlotFactory@U2@@QAE@PAVQObject@@@Z 1000f7b2 f   GCFramePlot.obj
 0001:0000e7d0       __unwindfunclet$??1GCFramePlotAlgorithm@U2@@UAE@XZ$0 1000f7d0 f   GCFramePlot.obj
 0001:0000e7d9       __ehhandler$??1GCFramePlotAlgorithm@U2@@UAE@XZ 1000f7d9 f   GCFramePlot.obj
 0001:0000e800       __unwindfunclet$??_GGCFramePlotAlgorithm@U2@@UAEPAXI@Z$0 1000f800 f   GCFramePlot.obj
 0001:0000e809       __ehhandler$??_GGCFramePlotAlgorithm@U2@@UAEPAXI@Z 1000f809 f   GCFramePlot.obj
 0001:0000e830       __unwindfunclet$??__EalgoLog@U2@@YAXXZ$0 1000f830 f   GCFramePlot.obj
 0001:0000e839       __ehhandler$??__EalgoLog@U2@@YAXXZ 1000f839 f   GCFramePlot.obj
 0001:0000e860       __unwindfunclet$??__EcmdLog@U2@@YAXXZ$0 1000f860 f   GCFramePlot.obj
 0001:0000e869       __ehhandler$??__EcmdLog@U2@@YAXXZ 1000f869 f   GCFramePlot.obj
 0001:0000e890       __unwindfunclet$??__EcoreLog@U2@@YAXXZ$0 1000f890 f   GCFramePlot.obj
 0001:0000e899       __ehhandler$??__EcoreLog@U2@@YAXXZ 1000f899 f   GCFramePlot.obj
 0001:0000e8c0       __unwindfunclet$??__EioLog@U2@@YAXXZ$0 1000f8c0 f   GCFramePlot.obj
 0001:0000e8c9       __ehhandler$??__EioLog@U2@@YAXXZ 1000f8c9 f   GCFramePlot.obj
 0001:0000e8f0       __unwindfunclet$??__EperfLog@U2@@YAXXZ$0 1000f8f0 f   GCFramePlot.obj
 0001:0000e8f9       __ehhandler$??__EperfLog@U2@@YAXXZ 1000f8f9 f   GCFramePlot.obj
 0001:0000e920       __unwindfunclet$??__EscriptLog@U2@@YAXXZ$0 1000f920 f   GCFramePlot.obj
 0001:0000e929       __ehhandler$??__EscriptLog@U2@@YAXXZ 1000f929 f   GCFramePlot.obj
 0001:0000e950       __unwindfunclet$??__EtaskLog@U2@@YAXXZ$0 1000f950 f   GCFramePlot.obj
 0001:0000e959       __ehhandler$??__EtaskLog@U2@@YAXXZ 1000f959 f   GCFramePlot.obj
 0001:0000e980       __unwindfunclet$??__EuiLog@U2@@YAXXZ$0 1000f980 f   GCFramePlot.obj
 0001:0000e989       __ehhandler$??__EuiLog@U2@@YAXXZ 1000f989 f   GCFramePlot.obj
 0001:0000e9b0       __unwindfunclet$??__EuserActLog@U2@@YAXXZ$0 1000f9b0 f   GCFramePlot.obj
 0001:0000e9b9       __ehhandler$??__EuserActLog@U2@@YAXXZ 1000f9b9 f   GCFramePlot.obj
 0001:0000e9e0       __unwindfunclet$?createGraphs@GCFramePlotFactory@U2@@UAE?AV?$QList@V?$QSharedPointer@VGSequenceGraphData@U2@@@@@@PAVGSequenceGraphView@2@@Z$0 1000f9e0 f   GCFramePlot.obj
 0001:0000e9f9       __unwindfunclet$?createGraphs@GCFramePlotFactory@U2@@UAE?AV?$QList@V?$QSharedPointer@VGSequenceGraphData@U2@@@@@@PAVGSequenceGraphView@2@@Z$1 1000f9f9 f   GCFramePlot.obj
 0001:0000ea04       __unwindfunclet$?createGraphs@GCFramePlotFactory@U2@@UAE?AV?$QList@V?$QSharedPointer@VGSequenceGraphData@U2@@@@@@PAVGSequenceGraphView@2@@Z$2 1000fa04 f   GCFramePlot.obj
 0001:0000ea1e       __unwindfunclet$?createGraphs@GCFramePlotFactory@U2@@UAE?AV?$QList@V?$QSharedPointer@VGSequenceGraphData@U2@@@@@@PAVGSequenceGraphView@2@@Z$3 1000fa1e f   GCFramePlot.obj
 0001:0000ea26       __unwindfunclet$?createGraphs@GCFramePlotFactory@U2@@UAE?AV?$QList@V?$QSharedPointer@VGSequenceGraphData@U2@@@@@@PAVGSequenceGraphView@2@@Z$4 1000fa26 f   GCFramePlot.obj
 0001:0000ea31       __unwindfunclet$?createGraphs@GCFramePlotFactory@U2@@UAE?AV?$QList@V?$QSharedPointer@VGSequenceGraphData@U2@@@@@@PAVGSequenceGraphView@2@@Z$5 1000fa31 f   GCFramePlot.obj
 0001:0000ea3c       __unwindfunclet$?createGraphs@GCFramePlotFactory@U2@@UAE?AV?$QList@V?$QSharedPointer@VGSequenceGraphData@U2@@@@@@PAVGSequenceGraphView@2@@Z$6 1000fa3c f   GCFramePlot.obj
 0001:0000ea56       __unwindfunclet$?createGraphs@GCFramePlotFactory@U2@@UAE?AV?$QList@V?$QSharedPointer@VGSequenceGraphData@U2@@@@@@PAVGSequenceGraphView@2@@Z$7 1000fa56 f   GCFramePlot.obj
 0001:0000ea5e       __unwindfunclet$?createGraphs@GCFramePlotFactory@U2@@UAE?AV?$QList@V?$QSharedPointer@VGSequenceGraphData@U2@@@@@@PAVGSequenceGraphView@2@@Z$8 1000fa5e f   GCFramePlot.obj
 0001:0000ea69       __unwindfunclet$?createGraphs@GCFramePlotFactory@U2@@UAE?AV?$QList@V?$QSharedPointer@VGSequenceGraphData@U2@@@@@@PAVGSequenceGraphView@2@@Z$9 1000fa69 f   GCFramePlot.obj
 0001:0000ea74       __unwindfunclet$?createGraphs@GCFramePlotFactory@U2@@UAE?AV?$QList@V?$QSharedPointer@VGSequenceGraphData@U2@@@@@@PAVGSequenceGraphView@2@@Z$10 1000fa74 f   GCFramePlot.obj
 0001:0000ea8e       __unwindfunclet$?createGraphs@GCFramePlotFactory@U2@@UAE?AV?$QList@V?$QSharedPointer@VGSequenceGraphData@U2@@@@@@PAVGSequenceGraphView@2@@Z$11 1000fa8e f   GCFramePlot.obj
 0001:0000ea96       __unwindfunclet$?createGraphs@GCFramePlotFactory@U2@@UAE?AV?$QList@V?$QSharedPointer@VGSequenceGraphData@U2@@@@@@PAVGSequenceGraphView@2@@Z$12 1000fa96 f   GCFramePlot.obj
 0001:0000eaa1       __ehhandler$?createGraphs@GCFramePlotFactory@U2@@UAE?AV?$QList@V?$QSharedPointer@VGSequenceGraphData@U2@@@@@@PAVGSequenceGraphView@2@@Z 1000faa1 f   GCFramePlot.obj
 0001:0000eac0       __unwindfunclet$?createNode@?$QMapData@VQString@@VQColor@@@@QAEPAU?$QMapNode@VQString@@VQColor@@@@ABVQString@@ABVQColor@@PAU2@_N@Z$4 1000fac0 f   GCFramePlot.obj
 0001:0000ead4       __ehhandler$?createNode@?$QMapData@VQString@@VQColor@@@@QAEPAU?$QMapNode@VQString@@VQColor@@@@ABVQString@@ABVQColor@@PAU2@_N@Z 1000fad4 f   GCFramePlot.obj
 0001:0000eaf0       __unwindfunclet$?getDrawer@GCFramePlotFactory@U2@@UAEPAVGSequenceGraphDrawer@2@PAVGSequenceGraphView@2@@Z$0 1000faf0 f   GCFramePlot.obj
 0001:0000eaf8       __unwindfunclet$?getDrawer@GCFramePlotFactory@U2@@UAEPAVGSequenceGraphDrawer@2@PAVGSequenceGraphView@2@@Z$1 1000faf8 f   GCFramePlot.obj
 0001:0000eb01       __unwindfunclet$?getDrawer@GCFramePlotFactory@U2@@UAEPAVGSequenceGraphDrawer@2@PAVGSequenceGraphView@2@@Z$2 1000fb01 f   GCFramePlot.obj
 0001:0000eb0a       __unwindfunclet$?getDrawer@GCFramePlotFactory@U2@@UAEPAVGSequenceGraphDrawer@2@PAVGSequenceGraphView@2@@Z$3 1000fb0a f   GCFramePlot.obj
 0001:0000eb13       __ehhandler$?getDrawer@GCFramePlotFactory@U2@@UAEPAVGSequenceGraphDrawer@2@PAVGSequenceGraphView@2@@Z 1000fb13 f   GCFramePlot.obj
 0001:0000eb40       __unwindfunclet$??0KarlinGraphAlgorithm@U2@@QAE@XZ$0 1000fb40 f   KarlinSignatureDifferenceGraph.obj
 0001:0000eb49       __ehhandler$??0KarlinGraphAlgorithm@U2@@QAE@XZ 1000fb49 f   KarlinSignatureDifferenceGraph.obj
 0001:0000eb70       __unwindfunclet$??0KarlinGraphFactory@U2@@QAE@PAVQObject@@@Z$0 1000fb70 f   KarlinSignatureDifferenceGraph.obj
 0001:0000eb79       __unwindfunclet$??0KarlinGraphFactory@U2@@QAE@PAVQObject@@@Z$1 1000fb79 f   KarlinSignatureDifferenceGraph.obj
 0001:0000eb82       __ehhandler$??0KarlinGraphFactory@U2@@QAE@PAVQObject@@@Z 1000fb82 f   KarlinSignatureDifferenceGraph.obj
 0001:0000eba0       __unwindfunclet$??1KarlinGraphAlgorithm@U2@@UAE@XZ$0 1000fba0 f   KarlinSignatureDifferenceGraph.obj
 0001:0000eba9       __ehhandler$??1KarlinGraphAlgorithm@U2@@UAE@XZ 1000fba9 f   KarlinSignatureDifferenceGraph.obj
 0001:0000ebd0       __unwindfunclet$??_GKarlinGraphAlgorithm@U2@@UAEPAXI@Z$0 1000fbd0 f   KarlinSignatureDifferenceGraph.obj
 0001:0000ebd9       __ehhandler$??_GKarlinGraphAlgorithm@U2@@UAEPAXI@Z 1000fbd9 f   KarlinSignatureDifferenceGraph.obj
 0001:0000ec00       __unwindfunclet$??__EalgoLog@U2@@YAXXZ$0 1000fc00 f   KarlinSignatureDifferenceGraph.obj
 0001:0000ec09       __ehhandler$??__EalgoLog@U2@@YAXXZ 1000fc09 f   KarlinSignatureDifferenceGraph.obj
 0001:0000ec30       __unwindfunclet$??__EcmdLog@U2@@YAXXZ$0 1000fc30 f   KarlinSignatureDifferenceGraph.obj
 0001:0000ec39       __ehhandler$??__EcmdLog@U2@@YAXXZ 1000fc39 f   KarlinSignatureDifferenceGraph.obj
 0001:0000ec60       __unwindfunclet$??__EcoreLog@U2@@YAXXZ$0 1000fc60 f   KarlinSignatureDifferenceGraph.obj
 0001:0000ec69       __ehhandler$??__EcoreLog@U2@@YAXXZ 1000fc69 f   KarlinSignatureDifferenceGraph.obj
 0001:0000ec90       __unwindfunclet$??__EioLog@U2@@YAXXZ$0 1000fc90 f   KarlinSignatureDifferenceGraph.obj
 0001:0000ec99       __ehhandler$??__EioLog@U2@@YAXXZ 1000fc99 f   KarlinSignatureDifferenceGraph.obj
 0001:0000ecc0       __unwindfunclet$??__EperfLog@U2@@YAXXZ$0 1000fcc0 f   KarlinSignatureDifferenceGraph.obj
 0001:0000ecc9       __ehhandler$??__EperfLog@U2@@YAXXZ 1000fcc9 f   KarlinSignatureDifferenceGraph.obj
 0001:0000ecf0       __unwindfunclet$??__EscriptLog@U2@@YAXXZ$0 1000fcf0 f   KarlinSignatureDifferenceGraph.obj
 0001:0000ecf9       __ehhandler$??__EscriptLog@U2@@YAXXZ 1000fcf9 f   KarlinSignatureDifferenceGraph.obj
 0001:0000ed20       __unwindfunclet$??__EtaskLog@U2@@YAXXZ$0 1000fd20 f   KarlinSignatureDifferenceGraph.obj
 0001:0000ed29       __ehhandler$??__EtaskLog@U2@@YAXXZ 1000fd29 f   KarlinSignatureDifferenceGraph.obj
 0001:0000ed50       __unwindfunclet$??__EuiLog@U2@@YAXXZ$0 1000fd50 f   KarlinSignatureDifferenceGraph.obj
 0001:0000ed59       __ehhandler$??__EuiLog@U2@@YAXXZ 1000fd59 f   KarlinSignatureDifferenceGraph.obj
 0001:0000ed80       __unwindfunclet$??__EuserActLog@U2@@YAXXZ$0 1000fd80 f   KarlinSignatureDifferenceGraph.obj
 0001:0000ed89       __ehhandler$??__EuserActLog@U2@@YAXXZ 1000fd89 f   KarlinSignatureDifferenceGraph.obj
 0001:0000edb0       __unwindfunclet$?calculate@KarlinGraphAlgorithm@U2@@UAEXAAV?$QVector@M@@PAVU2SequenceObject@2@ABVU2Region@2@PBVGSequenceGraphWindowData@2@AAVU2OpStatus@2@@Z$0 1000fdb0 f   KarlinSignatureDifferenceGraph.obj
 0001:0000edb9       __ehhandler$?calculate@KarlinGraphAlgorithm@U2@@UAEXAAV?$QVector@M@@PAVU2SequenceObject@2@ABVU2Region@2@PBVGSequenceGraphWindowData@2@AAVU2OpStatus@2@@Z 1000fdb9 f   KarlinSignatureDifferenceGraph.obj
 0001:0000ede0       __unwindfunclet$?calculateRelativeAbundance@KarlinGraphAlgorithm@U2@@AAEXPBDHPAMAAVU2OpStatus@2@@Z$0 1000fde0 f   KarlinSignatureDifferenceGraph.obj
 0001:0000ede9       __ehhandler$?calculateRelativeAbundance@KarlinGraphAlgorithm@U2@@AAEXPBDHPAMAAVU2OpStatus@2@@Z 1000fde9 f   KarlinSignatureDifferenceGraph.obj
 0001:0000ee10       __unwindfunclet$?createGraphs@KarlinGraphFactory@U2@@UAE?AV?$QList@V?$QSharedPointer@VGSequenceGraphData@U2@@@@@@PAVGSequenceGraphView@2@@Z$0 1000fe10 f   KarlinSignatureDifferenceGraph.obj
 0001:0000ee29       __unwindfunclet$?createGraphs@KarlinGraphFactory@U2@@UAE?AV?$QList@V?$QSharedPointer@VGSequenceGraphData@U2@@@@@@PAVGSequenceGraphView@2@@Z$1 1000fe29 f   KarlinSignatureDifferenceGraph.obj
 0001:0000ee34       __unwindfunclet$?createGraphs@KarlinGraphFactory@U2@@UAE?AV?$QList@V?$QSharedPointer@VGSequenceGraphData@U2@@@@@@PAVGSequenceGraphView@2@@Z$2 1000fe34 f   KarlinSignatureDifferenceGraph.obj
 0001:0000ee3c       __unwindfunclet$?createGraphs@KarlinGraphFactory@U2@@UAE?AV?$QList@V?$QSharedPointer@VGSequenceGraphData@U2@@@@@@PAVGSequenceGraphView@2@@Z$3 1000fe3c f   KarlinSignatureDifferenceGraph.obj
 0001:0000ee47       __unwindfunclet$?createGraphs@KarlinGraphFactory@U2@@UAE?AV?$QList@V?$QSharedPointer@VGSequenceGraphData@U2@@@@@@PAVGSequenceGraphView@2@@Z$4 1000fe47 f   KarlinSignatureDifferenceGraph.obj
 0001:0000ee50       __ehhandler$?createGraphs@KarlinGraphFactory@U2@@UAE?AV?$QList@V?$QSharedPointer@VGSequenceGraphData@U2@@@@@@PAVGSequenceGraphView@2@@Z 1000fe50 f   KarlinSignatureDifferenceGraph.obj
 0001:0000ee70       __unwindfunclet$??__EalgoLog@U2@@YAXXZ$0 1000fe70 f   moc_BaseContentGraph.obj
 0001:0000ee79       __ehhandler$??__EalgoLog@U2@@YAXXZ 1000fe79 f   moc_BaseContentGraph.obj
 0001:0000eea0       __unwindfunclet$??__EcmdLog@U2@@YAXXZ$0 1000fea0 f   moc_BaseContentGraph.obj
 0001:0000eea9       __ehhandler$??__EcmdLog@U2@@YAXXZ 1000fea9 f   moc_BaseContentGraph.obj
 0001:0000eed0       __unwindfunclet$??__EcoreLog@U2@@YAXXZ$0 1000fed0 f   moc_BaseContentGraph.obj
 0001:0000eed9       __ehhandler$??__EcoreLog@U2@@YAXXZ 1000fed9 f   moc_BaseContentGraph.obj
 0001:0000ef00       __unwindfunclet$??__EioLog@U2@@YAXXZ$0 1000ff00 f   moc_BaseContentGraph.obj
 0001:0000ef09       __ehhandler$??__EioLog@U2@@YAXXZ 1000ff09 f   moc_BaseContentGraph.obj
 0001:0000ef30       __unwindfunclet$??__EperfLog@U2@@YAXXZ$0 1000ff30 f   moc_BaseContentGraph.obj
 0001:0000ef39       __ehhandler$??__EperfLog@U2@@YAXXZ 1000ff39 f   moc_BaseContentGraph.obj
 0001:0000ef60       __unwindfunclet$??__EscriptLog@U2@@YAXXZ$0 1000ff60 f   moc_BaseContentGraph.obj
 0001:0000ef69       __ehhandler$??__EscriptLog@U2@@YAXXZ 1000ff69 f   moc_BaseContentGraph.obj
 0001:0000ef90       __unwindfunclet$??__EtaskLog@U2@@YAXXZ$0 1000ff90 f   moc_BaseContentGraph.obj
 0001:0000ef99       __ehhandler$??__EtaskLog@U2@@YAXXZ 1000ff99 f   moc_BaseContentGraph.obj
 0001:0000efc0       __unwindfunclet$??__EuiLog@U2@@YAXXZ$0 1000ffc0 f   moc_BaseContentGraph.obj
 0001:0000efc9       __ehhandler$??__EuiLog@U2@@YAXXZ 1000ffc9 f   moc_BaseContentGraph.obj
 0001:0000eff0       __unwindfunclet$??__EuserActLog@U2@@YAXXZ$0 1000fff0 f   moc_BaseContentGraph.obj
 0001:0000eff9       __ehhandler$??__EuserActLog@U2@@YAXXZ 1000fff9 f   moc_BaseContentGraph.obj
 0001:0000f020       __unwindfunclet$??__EalgoLog@U2@@YAXXZ$0 10010020 f   moc_CumulativeSkew.obj
 0001:0000f029       __ehhandler$??__EalgoLog@U2@@YAXXZ 10010029 f   moc_CumulativeSkew.obj
 0001:0000f050       __unwindfunclet$??__EcmdLog@U2@@YAXXZ$0 10010050 f   moc_CumulativeSkew.obj
 0001:0000f059       __ehhandler$??__EcmdLog@U2@@YAXXZ 10010059 f   moc_CumulativeSkew.obj
 0001:0000f080       __unwindfunclet$??__EcoreLog@U2@@YAXXZ$0 10010080 f   moc_CumulativeSkew.obj
 0001:0000f089       __ehhandler$??__EcoreLog@U2@@YAXXZ 10010089 f   moc_CumulativeSkew.obj
 0001:0000f0b0       __unwindfunclet$??__EioLog@U2@@YAXXZ$0 100100b0 f   moc_CumulativeSkew.obj
 0001:0000f0b9       __ehhandler$??__EioLog@U2@@YAXXZ 100100b9 f   moc_CumulativeSkew.obj
 0001:0000f0e0       __unwindfunclet$??__EperfLog@U2@@YAXXZ$0 100100e0 f   moc_CumulativeSkew.obj
 0001:0000f0e9       __ehhandler$??__EperfLog@U2@@YAXXZ 100100e9 f   moc_CumulativeSkew.obj
 0001:0000f110       __unwindfunclet$??__EscriptLog@U2@@YAXXZ$0 10010110 f   moc_CumulativeSkew.obj
 0001:0000f119       __ehhandler$??__EscriptLog@U2@@YAXXZ 10010119 f   moc_CumulativeSkew.obj
 0001:0000f140       __unwindfunclet$??__EtaskLog@U2@@YAXXZ$0 10010140 f   moc_CumulativeSkew.obj
 0001:0000f149       __ehhandler$??__EtaskLog@U2@@YAXXZ 10010149 f   moc_CumulativeSkew.obj
 0001:0000f170       __unwindfunclet$??__EuiLog@U2@@YAXXZ$0 10010170 f   moc_CumulativeSkew.obj
 0001:0000f179       __ehhandler$??__EuiLog@U2@@YAXXZ 10010179 f   moc_CumulativeSkew.obj
 0001:0000f1a0       __unwindfunclet$??__EuserActLog@U2@@YAXXZ$0 100101a0 f   moc_CumulativeSkew.obj
 0001:0000f1a9       __ehhandler$??__EuserActLog@U2@@YAXXZ 100101a9 f   moc_CumulativeSkew.obj
 0001:0000f1d0       __unwindfunclet$??__EalgoLog@U2@@YAXXZ$0 100101d0 f   moc_DNAGraphPackPlugin.obj
 0001:0000f1d9       __ehhandler$??__EalgoLog@U2@@YAXXZ 100101d9 f   moc_DNAGraphPackPlugin.obj
 0001:0000f200       __unwindfunclet$??__EcmdLog@U2@@YAXXZ$0 10010200 f   moc_DNAGraphPackPlugin.obj
 0001:0000f209       __ehhandler$??__EcmdLog@U2@@YAXXZ 10010209 f   moc_DNAGraphPackPlugin.obj
 0001:0000f230       __unwindfunclet$??__EcoreLog@U2@@YAXXZ$0 10010230 f   moc_DNAGraphPackPlugin.obj
 0001:0000f239       __ehhandler$??__EcoreLog@U2@@YAXXZ 10010239 f   moc_DNAGraphPackPlugin.obj
 0001:0000f260       __unwindfunclet$??__EioLog@U2@@YAXXZ$0 10010260 f   moc_DNAGraphPackPlugin.obj
 0001:0000f269       __ehhandler$??__EioLog@U2@@YAXXZ 10010269 f   moc_DNAGraphPackPlugin.obj
 0001:0000f290       __unwindfunclet$??__EperfLog@U2@@YAXXZ$0 10010290 f   moc_DNAGraphPackPlugin.obj
 0001:0000f299       __ehhandler$??__EperfLog@U2@@YAXXZ 10010299 f   moc_DNAGraphPackPlugin.obj
 0001:0000f2c0       __unwindfunclet$??__EscriptLog@U2@@YAXXZ$0 100102c0 f   moc_DNAGraphPackPlugin.obj
 0001:0000f2c9       __ehhandler$??__EscriptLog@U2@@YAXXZ 100102c9 f   moc_DNAGraphPackPlugin.obj
 0001:0000f2f0       __unwindfunclet$??__EtaskLog@U2@@YAXXZ$0 100102f0 f   moc_DNAGraphPackPlugin.obj
 0001:0000f2f9       __ehhandler$??__EtaskLog@U2@@YAXXZ 100102f9 f   moc_DNAGraphPackPlugin.obj
 0001:0000f320       __unwindfunclet$??__EuiLog@U2@@YAXXZ$0 10010320 f   moc_DNAGraphPackPlugin.obj
 0001:0000f329       __ehhandler$??__EuiLog@U2@@YAXXZ 10010329 f   moc_DNAGraphPackPlugin.obj
 0001:0000f350       __unwindfunclet$??__EuserActLog@U2@@YAXXZ$0 10010350 f   moc_DNAGraphPackPlugin.obj
 0001:0000f359       __ehhandler$??__EuserActLog@U2@@YAXXZ 10010359 f   moc_DNAGraphPackPlugin.obj
 0001:0000f380       __unwindfunclet$?qt_metatype_id@?$QMetaTypeIdQObject@PAVADVSequenceWidget@U2@@$00@@SAHXZ$0 10010380 f   moc_DNAGraphPackPlugin.obj
 0001:0000f389       __ehhandler$?qt_metatype_id@?$QMetaTypeIdQObject@PAVADVSequenceWidget@U2@@$00@@SAHXZ 10010389 f   moc_DNAGraphPackPlugin.obj
 0001:0000f3b0       __unwindfunclet$??__EalgoLog@U2@@YAXXZ$0 100103b0 f   moc_DeviationGraph.obj
 0001:0000f3b9       __ehhandler$??__EalgoLog@U2@@YAXXZ 100103b9 f   moc_DeviationGraph.obj
 0001:0000f3e0       __unwindfunclet$??__EcmdLog@U2@@YAXXZ$0 100103e0 f   moc_DeviationGraph.obj
 0001:0000f3e9       __ehhandler$??__EcmdLog@U2@@YAXXZ 100103e9 f   moc_DeviationGraph.obj
 0001:0000f410       __unwindfunclet$??__EcoreLog@U2@@YAXXZ$0 10010410 f   moc_DeviationGraph.obj
 0001:0000f419       __ehhandler$??__EcoreLog@U2@@YAXXZ 10010419 f   moc_DeviationGraph.obj
 0001:0000f440       __unwindfunclet$??__EioLog@U2@@YAXXZ$0 10010440 f   moc_DeviationGraph.obj
 0001:0000f449       __ehhandler$??__EioLog@U2@@YAXXZ 10010449 f   moc_DeviationGraph.obj
 0001:0000f470       __unwindfunclet$??__EperfLog@U2@@YAXXZ$0 10010470 f   moc_DeviationGraph.obj
 0001:0000f479       __ehhandler$??__EperfLog@U2@@YAXXZ 10010479 f   moc_DeviationGraph.obj
 0001:0000f4a0       __unwindfunclet$??__EscriptLog@U2@@YAXXZ$0 100104a0 f   moc_DeviationGraph.obj
 0001:0000f4a9       __ehhandler$??__EscriptLog@U2@@YAXXZ 100104a9 f   moc_DeviationGraph.obj
 0001:0000f4d0       __unwindfunclet$??__EtaskLog@U2@@YAXXZ$0 100104d0 f   moc_DeviationGraph.obj
 0001:0000f4d9       __ehhandler$??__EtaskLog@U2@@YAXXZ 100104d9 f   moc_DeviationGraph.obj
 0001:0000f500       __unwindfunclet$??__EuiLog@U2@@YAXXZ$0 10010500 f   moc_DeviationGraph.obj
 0001:0000f509       __ehhandler$??__EuiLog@U2@@YAXXZ 10010509 f   moc_DeviationGraph.obj
 0001:0000f530       __unwindfunclet$??__EuserActLog@U2@@YAXXZ$0 10010530 f   moc_DeviationGraph.obj
 0001:0000f539       __ehhandler$??__EuserActLog@U2@@YAXXZ 10010539 f   moc_DeviationGraph.obj
 0001:0000f560       __unwindfunclet$??__EalgoLog@U2@@YAXXZ$0 10010560 f   moc_EntropyAlgorithm.obj
 0001:0000f569       __ehhandler$??__EalgoLog@U2@@YAXXZ 10010569 f   moc_EntropyAlgorithm.obj
 0001:0000f590       __unwindfunclet$??__EcmdLog@U2@@YAXXZ$0 10010590 f   moc_EntropyAlgorithm.obj
 0001:0000f599       __ehhandler$??__EcmdLog@U2@@YAXXZ 10010599 f   moc_EntropyAlgorithm.obj
 0001:0000f5c0       __unwindfunclet$??__EcoreLog@U2@@YAXXZ$0 100105c0 f   moc_EntropyAlgorithm.obj
 0001:0000f5c9       __ehhandler$??__EcoreLog@U2@@YAXXZ 100105c9 f   moc_EntropyAlgorithm.obj
 0001:0000f5f0       __unwindfunclet$??__EioLog@U2@@YAXXZ$0 100105f0 f   moc_EntropyAlgorithm.obj
 0001:0000f5f9       __ehhandler$??__EioLog@U2@@YAXXZ 100105f9 f   moc_EntropyAlgorithm.obj
 0001:0000f620       __unwindfunclet$??__EperfLog@U2@@YAXXZ$0 10010620 f   moc_EntropyAlgorithm.obj
 0001:0000f629       __ehhandler$??__EperfLog@U2@@YAXXZ 10010629 f   moc_EntropyAlgorithm.obj
 0001:0000f650       __unwindfunclet$??__EscriptLog@U2@@YAXXZ$0 10010650 f   moc_EntropyAlgorithm.obj
 0001:0000f659       __ehhandler$??__EscriptLog@U2@@YAXXZ 10010659 f   moc_EntropyAlgorithm.obj
 0001:0000f680       __unwindfunclet$??__EtaskLog@U2@@YAXXZ$0 10010680 f   moc_EntropyAlgorithm.obj
 0001:0000f689       __ehhandler$??__EtaskLog@U2@@YAXXZ 10010689 f   moc_EntropyAlgorithm.obj
 0001:0000f6b0       __unwindfunclet$??__EuiLog@U2@@YAXXZ$0 100106b0 f   moc_EntropyAlgorithm.obj
 0001:0000f6b9       __ehhandler$??__EuiLog@U2@@YAXXZ 100106b9 f   moc_EntropyAlgorithm.obj
 0001:0000f6e0       __unwindfunclet$??__EuserActLog@U2@@YAXXZ$0 100106e0 f   moc_EntropyAlgorithm.obj
 0001:0000f6e9       __ehhandler$??__EuserActLog@U2@@YAXXZ 100106e9 f   moc_EntropyAlgorithm.obj
 0001:0000f710       __unwindfunclet$??__EalgoLog@U2@@YAXXZ$0 10010710 f   moc_GCFramePlot.obj
 0001:0000f719       __ehhandler$??__EalgoLog@U2@@YAXXZ 10010719 f   moc_GCFramePlot.obj
 0001:0000f740       __unwindfunclet$??__EcmdLog@U2@@YAXXZ$0 10010740 f   moc_GCFramePlot.obj
 0001:0000f749       __ehhandler$??__EcmdLog@U2@@YAXXZ 10010749 f   moc_GCFramePlot.obj
 0001:0000f770       __unwindfunclet$??__EcoreLog@U2@@YAXXZ$0 10010770 f   moc_GCFramePlot.obj
 0001:0000f779       __ehhandler$??__EcoreLog@U2@@YAXXZ 10010779 f   moc_GCFramePlot.obj
 0001:0000f7a0       __unwindfunclet$??__EioLog@U2@@YAXXZ$0 100107a0 f   moc_GCFramePlot.obj
 0001:0000f7a9       __ehhandler$??__EioLog@U2@@YAXXZ 100107a9 f   moc_GCFramePlot.obj
 0001:0000f7d0       __unwindfunclet$??__EperfLog@U2@@YAXXZ$0 100107d0 f   moc_GCFramePlot.obj
 0001:0000f7d9       __ehhandler$??__EperfLog@U2@@YAXXZ 100107d9 f   moc_GCFramePlot.obj
 0001:0000f800       __unwindfunclet$??__EscriptLog@U2@@YAXXZ$0 10010800 f   moc_GCFramePlot.obj
 0001:0000f809       __ehhandler$??__EscriptLog@U2@@YAXXZ 10010809 f   moc_GCFramePlot.obj
 0001:0000f830       __unwindfunclet$??__EtaskLog@U2@@YAXXZ$0 10010830 f   moc_GCFramePlot.obj
 0001:0000f839       __ehhandler$??__EtaskLog@U2@@YAXXZ 10010839 f   moc_GCFramePlot.obj
 0001:0000f860       __unwindfunclet$??__EuiLog@U2@@YAXXZ$0 10010860 f   moc_GCFramePlot.obj
 0001:0000f869       __ehhandler$??__EuiLog@U2@@YAXXZ 10010869 f   moc_GCFramePlot.obj
 0001:0000f890       __unwindfunclet$??__EuserActLog@U2@@YAXXZ$0 10010890 f   moc_GCFramePlot.obj
 0001:0000f899       __ehhandler$??__EuserActLog@U2@@YAXXZ 10010899 f   moc_GCFramePlot.obj
 0001:0000f8c0       __unwindfunclet$??__EalgoLog@U2@@YAXXZ$0 100108c0 f   moc_KarlinSignatureDifferenceGraph.obj
 0001:0000f8c9       __ehhandler$??__EalgoLog@U2@@YAXXZ 100108c9 f   moc_KarlinSignatureDifferenceGraph.obj
 0001:0000f8f0       __unwindfunclet$??__EcmdLog@U2@@YAXXZ$0 100108f0 f   moc_KarlinSignatureDifferenceGraph.obj
 0001:0000f8f9       __ehhandler$??__EcmdLog@U2@@YAXXZ 100108f9 f   moc_KarlinSignatureDifferenceGraph.obj
 0001:0000f920       __unwindfunclet$??__EcoreLog@U2@@YAXXZ$0 10010920 f   moc_KarlinSignatureDifferenceGraph.obj
 0001:0000f929       __ehhandler$??__EcoreLog@U2@@YAXXZ 10010929 f   moc_KarlinSignatureDifferenceGraph.obj
 0001:0000f950       __unwindfunclet$??__EioLog@U2@@YAXXZ$0 10010950 f   moc_KarlinSignatureDifferenceGraph.obj
 0001:0000f959       __ehhandler$??__EioLog@U2@@YAXXZ 10010959 f   moc_KarlinSignatureDifferenceGraph.obj
 0001:0000f980       __unwindfunclet$??__EperfLog@U2@@YAXXZ$0 10010980 f   moc_KarlinSignatureDifferenceGraph.obj
 0001:0000f989       __ehhandler$??__EperfLog@U2@@YAXXZ 10010989 f   moc_KarlinSignatureDifferenceGraph.obj
 0001:0000f9b0       __unwindfunclet$??__EscriptLog@U2@@YAXXZ$0 100109b0 f   moc_KarlinSignatureDifferenceGraph.obj
 0001:0000f9b9       __ehhandler$??__EscriptLog@U2@@YAXXZ 100109b9 f   moc_KarlinSignatureDifferenceGraph.obj
 0001:0000f9e0       __unwindfunclet$??__EtaskLog@U2@@YAXXZ$0 100109e0 f   moc_KarlinSignatureDifferenceGraph.obj
 0001:0000f9e9       __ehhandler$??__EtaskLog@U2@@YAXXZ 100109e9 f   moc_KarlinSignatureDifferenceGraph.obj
 0001:0000fa10       __unwindfunclet$??__EuiLog@U2@@YAXXZ$0 10010a10 f   moc_KarlinSignatureDifferenceGraph.obj
 0001:0000fa19       __ehhandler$??__EuiLog@U2@@YAXXZ 10010a19 f   moc_KarlinSignatureDifferenceGraph.obj
 0001:0000fa40       __unwindfunclet$??__EuserActLog@U2@@YAXXZ$0 10010a40 f   moc_KarlinSignatureDifferenceGraph.obj
 0001:0000fa49       __ehhandler$??__EuserActLog@U2@@YAXXZ 10010a49 f   moc_KarlinSignatureDifferenceGraph.obj
 0001:0000fa70       ??__F?_Generic_object@?$_Error_objects@H@std@@2V_Generic_error_category@2@A@@YAXXZ 10010a70 f   BaseContentGraph.obj
 0001:0000fa80       ??__F?_Iostream_object@?$_Error_objects@H@std@@2V_Iostream_error_category@2@A@@YAXXZ 10010a80 f   BaseContentGraph.obj
 0001:0000fa90       ??__F?_System_object@?$_Error_objects@H@std@@2V_System_error_category@2@A@@YAXXZ 10010a90 f   BaseContentGraph.obj
 0001:0000faa0       ??__FService_DNAExport@U2@@YAXXZ 10010aa0 f   BaseContentGraph.obj
 0001:0000fab0       ??__FService_DNAGraphPack@U2@@YAXXZ 10010ab0 f   BaseContentGraph.obj
 0001:0000fac0       ??__FService_ExternalToolSupport@U2@@YAXXZ 10010ac0 f   BaseContentGraph.obj
 0001:0000fad0       ??__FService_GUITesting@U2@@YAXXZ 10010ad0 f   BaseContentGraph.obj
 0001:0000fae0       ??__FService_MaxCoreServiceId@U2@@YAXXZ 10010ae0 f   BaseContentGraph.obj
 0001:0000faf0       ??__FService_MinCoreServiceId@U2@@YAXXZ 10010af0 f   BaseContentGraph.obj
 0001:0000fb00       ??__FService_PluginViewer@U2@@YAXXZ 10010b00 f   BaseContentGraph.obj
 0001:0000fb10       ??__FService_Project@U2@@YAXXZ 10010b10 f   BaseContentGraph.obj
 0001:0000fb20       ??__FService_ProjectView@U2@@YAXXZ 10010b20 f   BaseContentGraph.obj
 0001:0000fb30       ??__FService_QueryDesigner@U2@@YAXXZ 10010b30 f   BaseContentGraph.obj
 0001:0000fb40       ??__FService_ScriptRegistry@U2@@YAXXZ 10010b40 f   BaseContentGraph.obj
 0001:0000fb50       ??__FService_TestRunner@U2@@YAXXZ 10010b50 f   BaseContentGraph.obj
 0001:0000fb60       ??__FService_WorkflowDesigner@U2@@YAXXZ 10010b60 f   BaseContentGraph.obj
 0001:0000fb70       ??__FalgoLog@U2@@YAXXZ     10010b70 f   BaseContentGraph.obj
 0001:0000fb80       ??__FcmdLog@U2@@YAXXZ      10010b80 f   BaseContentGraph.obj
 0001:0000fb90       ??__FcoreLog@U2@@YAXXZ     10010b90 f   BaseContentGraph.obj
 0001:0000fba0       ??__FioLog@U2@@YAXXZ       10010ba0 f   BaseContentGraph.obj
 0001:0000fbb0       ??__FperfLog@U2@@YAXXZ     10010bb0 f   BaseContentGraph.obj
 0001:0000fbc0       ??__FscriptLog@U2@@YAXXZ   10010bc0 f   BaseContentGraph.obj
 0001:0000fbd0       ??__FtaskLog@U2@@YAXXZ     10010bd0 f   BaseContentGraph.obj
 0001:0000fbe0       ??__FuiLog@U2@@YAXXZ       10010be0 f   BaseContentGraph.obj
 0001:0000fbf0       ??__FuserActLog@U2@@YAXXZ  10010bf0 f   BaseContentGraph.obj
 0001:0000fc00       ??__F?_Generic_object@?$_Error_objects@H@std@@2V_Generic_error_category@2@A@@YAXXZ 10010c00 f   CumulativeSkew.obj
 0001:0000fc10       ??__F?_Iostream_object@?$_Error_objects@H@std@@2V_Iostream_error_category@2@A@@YAXXZ 10010c10 f   CumulativeSkew.obj
 0001:0000fc20       ??__F?_System_object@?$_Error_objects@H@std@@2V_System_error_category@2@A@@YAXXZ 10010c20 f   CumulativeSkew.obj
 0001:0000fc30       ??__FService_DNAExport@U2@@YAXXZ 10010c30 f   CumulativeSkew.obj
 0001:0000fc40       ??__FService_DNAGraphPack@U2@@YAXXZ 10010c40 f   CumulativeSkew.obj
 0001:0000fc50       ??__FService_ExternalToolSupport@U2@@YAXXZ 10010c50 f   CumulativeSkew.obj
 0001:0000fc60       ??__FService_GUITesting@U2@@YAXXZ 10010c60 f   CumulativeSkew.obj
 0001:0000fc70       ??__FService_MaxCoreServiceId@U2@@YAXXZ 10010c70 f   CumulativeSkew.obj
 0001:0000fc80       ??__FService_MinCoreServiceId@U2@@YAXXZ 10010c80 f   CumulativeSkew.obj
 0001:0000fc90       ??__FService_PluginViewer@U2@@YAXXZ 10010c90 f   CumulativeSkew.obj
 0001:0000fca0       ??__FService_Project@U2@@YAXXZ 10010ca0 f   CumulativeSkew.obj
 0001:0000fcb0       ??__FService_ProjectView@U2@@YAXXZ 10010cb0 f   CumulativeSkew.obj
 0001:0000fcc0       ??__FService_QueryDesigner@U2@@YAXXZ 10010cc0 f   CumulativeSkew.obj
 0001:0000fcd0       ??__FService_ScriptRegistry@U2@@YAXXZ 10010cd0 f   CumulativeSkew.obj
 0001:0000fce0       ??__FService_TestRunner@U2@@YAXXZ 10010ce0 f   CumulativeSkew.obj
 0001:0000fcf0       ??__FService_WorkflowDesigner@U2@@YAXXZ 10010cf0 f   CumulativeSkew.obj
 0001:0000fd00       ??__FalgoLog@U2@@YAXXZ     10010d00 f   CumulativeSkew.obj
 0001:0000fd10       ??__FcmdLog@U2@@YAXXZ      10010d10 f   CumulativeSkew.obj
 0001:0000fd20       ??__FcoreLog@U2@@YAXXZ     10010d20 f   CumulativeSkew.obj
 0001:0000fd30       ??__FioLog@U2@@YAXXZ       10010d30 f   CumulativeSkew.obj
 0001:0000fd40       ??__FperfLog@U2@@YAXXZ     10010d40 f   CumulativeSkew.obj
 0001:0000fd50       ??__FscriptLog@U2@@YAXXZ   10010d50 f   CumulativeSkew.obj
 0001:0000fd60       ??__FtaskLog@U2@@YAXXZ     10010d60 f   CumulativeSkew.obj
 0001:0000fd70       ??__FuiLog@U2@@YAXXZ       10010d70 f   CumulativeSkew.obj
 0001:0000fd80       ??__FuserActLog@U2@@YAXXZ  10010d80 f   CumulativeSkew.obj
 0001:0000fd90       ??__F?_Generic_object@?$_Error_objects@H@std@@2V_Generic_error_category@2@A@@YAXXZ 10010d90 f   DNAGraphPackPlugin.obj
 0001:0000fda0       ??__F?_Iostream_object@?$_Error_objects@H@std@@2V_Iostream_error_category@2@A@@YAXXZ 10010da0 f   DNAGraphPackPlugin.obj
 0001:0000fdb0       ??__F?_System_object@?$_Error_objects@H@std@@2V_System_error_category@2@A@@YAXXZ 10010db0 f   DNAGraphPackPlugin.obj
 0001:0000fdc0       ??__FService_DNAExport@U2@@YAXXZ 10010dc0 f   DNAGraphPackPlugin.obj
 0001:0000fdd0       ??__FService_DNAGraphPack@U2@@YAXXZ 10010dd0 f   DNAGraphPackPlugin.obj
 0001:0000fde0       ??__FService_ExternalToolSupport@U2@@YAXXZ 10010de0 f   DNAGraphPackPlugin.obj
 0001:0000fdf0       ??__FService_GUITesting@U2@@YAXXZ 10010df0 f   DNAGraphPackPlugin.obj
 0001:0000fe00       ??__FService_MaxCoreServiceId@U2@@YAXXZ 10010e00 f   DNAGraphPackPlugin.obj
 0001:0000fe10       ??__FService_MinCoreServiceId@U2@@YAXXZ 10010e10 f   DNAGraphPackPlugin.obj
 0001:0000fe20       ??__FService_PluginViewer@U2@@YAXXZ 10010e20 f   DNAGraphPackPlugin.obj
 0001:0000fe30       ??__FService_Project@U2@@YAXXZ 10010e30 f   DNAGraphPackPlugin.obj
 0001:0000fe40       ??__FService_ProjectView@U2@@YAXXZ 10010e40 f   DNAGraphPackPlugin.obj
 0001:0000fe50       ??__FService_QueryDesigner@U2@@YAXXZ 10010e50 f   DNAGraphPackPlugin.obj
 0001:0000fe60       ??__FService_ScriptRegistry@U2@@YAXXZ 10010e60 f   DNAGraphPackPlugin.obj
 0001:0000fe70       ??__FService_TestRunner@U2@@YAXXZ 10010e70 f   DNAGraphPackPlugin.obj
 0001:0000fe80       ??__FService_WorkflowDesigner@U2@@YAXXZ 10010e80 f   DNAGraphPackPlugin.obj
 0001:0000fe90       ??__FalgoLog@U2@@YAXXZ     10010e90 f   DNAGraphPackPlugin.obj
 0001:0000fea0       ??__FcmdLog@U2@@YAXXZ      10010ea0 f   DNAGraphPackPlugin.obj
 0001:0000feb0       ??__FcoreLog@U2@@YAXXZ     10010eb0 f   DNAGraphPackPlugin.obj
 0001:0000fec0       ??__FioLog@U2@@YAXXZ       10010ec0 f   DNAGraphPackPlugin.obj
 0001:0000fed0       ??__FperfLog@U2@@YAXXZ     10010ed0 f   DNAGraphPackPlugin.obj
 0001:0000fee0       ??__FscriptLog@U2@@YAXXZ   10010ee0 f   DNAGraphPackPlugin.obj
 0001:0000fef0       ??__FtaskLog@U2@@YAXXZ     10010ef0 f   DNAGraphPackPlugin.obj
 0001:0000ff00       ??__FuiLog@U2@@YAXXZ       10010f00 f   DNAGraphPackPlugin.obj
 0001:0000ff10       ??__FuserActLog@U2@@YAXXZ  10010f10 f   DNAGraphPackPlugin.obj
 0001:0000ff20       ??__F?_Generic_object@?$_Error_objects@H@std@@2V_Generic_error_category@2@A@@YAXXZ 10010f20 f   DeviationGraph.obj
 0001:0000ff30       ??__F?_Iostream_object@?$_Error_objects@H@std@@2V_Iostream_error_category@2@A@@YAXXZ 10010f30 f   DeviationGraph.obj
 0001:0000ff40       ??__F?_System_object@?$_Error_objects@H@std@@2V_System_error_category@2@A@@YAXXZ 10010f40 f   DeviationGraph.obj
 0001:0000ff50       ??__FService_DNAExport@U2@@YAXXZ 10010f50 f   DeviationGraph.obj
 0001:0000ff60       ??__FService_DNAGraphPack@U2@@YAXXZ 10010f60 f   DeviationGraph.obj
 0001:0000ff70       ??__FService_ExternalToolSupport@U2@@YAXXZ 10010f70 f   DeviationGraph.obj
 0001:0000ff80       ??__FService_GUITesting@U2@@YAXXZ 10010f80 f   DeviationGraph.obj
 0001:0000ff90       ??__FService_MaxCoreServiceId@U2@@YAXXZ 10010f90 f   DeviationGraph.obj
 0001:0000ffa0       ??__FService_MinCoreServiceId@U2@@YAXXZ 10010fa0 f   DeviationGraph.obj
 0001:0000ffb0       ??__FService_PluginViewer@U2@@YAXXZ 10010fb0 f   DeviationGraph.obj
 0001:0000ffc0       ??__FService_Project@U2@@YAXXZ 10010fc0 f   DeviationGraph.obj
 0001:0000ffd0       ??__FService_ProjectView@U2@@YAXXZ 10010fd0 f   DeviationGraph.obj
 0001:0000ffe0       ??__FService_QueryDesigner@U2@@YAXXZ 10010fe0 f   DeviationGraph.obj
 0001:0000fff0       ??__FService_ScriptRegistry@U2@@YAXXZ 10010ff0 f   DeviationGraph.obj
 0001:00010000       ??__FService_TestRunner@U2@@YAXXZ 10011000 f   DeviationGraph.obj
 0001:00010010       ??__FService_WorkflowDesigner@U2@@YAXXZ 10011010 f   DeviationGraph.obj
 0001:00010020       ??__FalgoLog@U2@@YAXXZ     10011020 f   DeviationGraph.obj
 0001:00010030       ??__FcmdLog@U2@@YAXXZ      10011030 f   DeviationGraph.obj
 0001:00010040       ??__FcoreLog@U2@@YAXXZ     10011040 f   DeviationGraph.obj
 0001:00010050       ??__FioLog@U2@@YAXXZ       10011050 f   DeviationGraph.obj
 0001:00010060       ??__FperfLog@U2@@YAXXZ     10011060 f   DeviationGraph.obj
 0001:00010070       ??__FscriptLog@U2@@YAXXZ   10011070 f   DeviationGraph.obj
 0001:00010080       ??__FtaskLog@U2@@YAXXZ     10011080 f   DeviationGraph.obj
 0001:00010090       ??__FuiLog@U2@@YAXXZ       10011090 f   DeviationGraph.obj
 0001:000100a0       ??__FuserActLog@U2@@YAXXZ  100110a0 f   DeviationGraph.obj
 0001:000100b0       ??__F?_Generic_object@?$_Error_objects@H@std@@2V_Generic_error_category@2@A@@YAXXZ 100110b0 f   EntropyAlgorithm.obj
 0001:000100c0       ??__F?_Iostream_object@?$_Error_objects@H@std@@2V_Iostream_error_category@2@A@@YAXXZ 100110c0 f   EntropyAlgorithm.obj
 0001:000100d0       ??__F?_System_object@?$_Error_objects@H@std@@2V_System_error_category@2@A@@YAXXZ 100110d0 f   EntropyAlgorithm.obj
 0001:000100e0       ??__FService_DNAExport@U2@@YAXXZ 100110e0 f   EntropyAlgorithm.obj
 0001:000100f0       ??__FService_DNAGraphPack@U2@@YAXXZ 100110f0 f   EntropyAlgorithm.obj
 0001:00010100       ??__FService_ExternalToolSupport@U2@@YAXXZ 10011100 f   EntropyAlgorithm.obj
 0001:00010110       ??__FService_GUITesting@U2@@YAXXZ 10011110 f   EntropyAlgorithm.obj
 0001:00010120       ??__FService_MaxCoreServiceId@U2@@YAXXZ 10011120 f   EntropyAlgorithm.obj
 0001:00010130       ??__FService_MinCoreServiceId@U2@@YAXXZ 10011130 f   EntropyAlgorithm.obj
 0001:00010140       ??__FService_PluginViewer@U2@@YAXXZ 10011140 f   EntropyAlgorithm.obj
 0001:00010150       ??__FService_Project@U2@@YAXXZ 10011150 f   EntropyAlgorithm.obj
 0001:00010160       ??__FService_ProjectView@U2@@YAXXZ 10011160 f   EntropyAlgorithm.obj
 0001:00010170       ??__FService_QueryDesigner@U2@@YAXXZ 10011170 f   EntropyAlgorithm.obj
 0001:00010180       ??__FService_ScriptRegistry@U2@@YAXXZ 10011180 f   EntropyAlgorithm.obj
 0001:00010190       ??__FService_TestRunner@U2@@YAXXZ 10011190 f   EntropyAlgorithm.obj
 0001:000101a0       ??__FService_WorkflowDesigner@U2@@YAXXZ 100111a0 f   EntropyAlgorithm.obj
 0001:000101b0       ??__FalgoLog@U2@@YAXXZ     100111b0 f   EntropyAlgorithm.obj
 0001:000101c0       ??__FcmdLog@U2@@YAXXZ      100111c0 f   EntropyAlgorithm.obj
 0001:000101d0       ??__FcoreLog@U2@@YAXXZ     100111d0 f   EntropyAlgorithm.obj
 0001:000101e0       ??__FioLog@U2@@YAXXZ       100111e0 f   EntropyAlgorithm.obj
 0001:000101f0       ??__FperfLog@U2@@YAXXZ     100111f0 f   EntropyAlgorithm.obj
 0001:00010200       ??__FscriptLog@U2@@YAXXZ   10011200 f   EntropyAlgorithm.obj
 0001:00010210       ??__FtaskLog@U2@@YAXXZ     10011210 f   EntropyAlgorithm.obj
 0001:00010220       ??__FuiLog@U2@@YAXXZ       10011220 f   EntropyAlgorithm.obj
 0001:00010230       ??__FuserActLog@U2@@YAXXZ  10011230 f   EntropyAlgorithm.obj
 0001:00010240       ??__F?_Generic_object@?$_Error_objects@H@std@@2V_Generic_error_category@2@A@@YAXXZ 10011240 f   GCFramePlot.obj
 0001:00010250       ??__F?_Iostream_object@?$_Error_objects@H@std@@2V_Iostream_error_category@2@A@@YAXXZ 10011250 f   GCFramePlot.obj
 0001:00010260       ??__F?_System_object@?$_Error_objects@H@std@@2V_System_error_category@2@A@@YAXXZ 10011260 f   GCFramePlot.obj
 0001:00010270       ??__FService_DNAExport@U2@@YAXXZ 10011270 f   GCFramePlot.obj
 0001:00010280       ??__FService_DNAGraphPack@U2@@YAXXZ 10011280 f   GCFramePlot.obj
 0001:00010290       ??__FService_ExternalToolSupport@U2@@YAXXZ 10011290 f   GCFramePlot.obj
 0001:000102a0       ??__FService_GUITesting@U2@@YAXXZ 100112a0 f   GCFramePlot.obj
 0001:000102b0       ??__FService_MaxCoreServiceId@U2@@YAXXZ 100112b0 f   GCFramePlot.obj
 0001:000102c0       ??__FService_MinCoreServiceId@U2@@YAXXZ 100112c0 f   GCFramePlot.obj
 0001:000102d0       ??__FService_PluginViewer@U2@@YAXXZ 100112d0 f   GCFramePlot.obj
 0001:000102e0       ??__FService_Project@U2@@YAXXZ 100112e0 f   GCFramePlot.obj
 0001:000102f0       ??__FService_ProjectView@U2@@YAXXZ 100112f0 f   GCFramePlot.obj
 0001:00010300       ??__FService_QueryDesigner@U2@@YAXXZ 10011300 f   GCFramePlot.obj
 0001:00010310       ??__FService_ScriptRegistry@U2@@YAXXZ 10011310 f   GCFramePlot.obj
 0001:00010320       ??__FService_TestRunner@U2@@YAXXZ 10011320 f   GCFramePlot.obj
 0001:00010330       ??__FService_WorkflowDesigner@U2@@YAXXZ 10011330 f   GCFramePlot.obj
 0001:00010340       ??__FalgoLog@U2@@YAXXZ     10011340 f   GCFramePlot.obj
 0001:00010350       ??__FcmdLog@U2@@YAXXZ      10011350 f   GCFramePlot.obj
 0001:00010360       ??__FcoreLog@U2@@YAXXZ     10011360 f   GCFramePlot.obj
 0001:00010370       ??__FioLog@U2@@YAXXZ       10011370 f   GCFramePlot.obj
 0001:00010380       ??__FperfLog@U2@@YAXXZ     10011380 f   GCFramePlot.obj
 0001:00010390       ??__FscriptLog@U2@@YAXXZ   10011390 f   GCFramePlot.obj
 0001:000103a0       ??__FtaskLog@U2@@YAXXZ     100113a0 f   GCFramePlot.obj
 0001:000103b0       ??__FuiLog@U2@@YAXXZ       100113b0 f   GCFramePlot.obj
 0001:000103c0       ??__FuserActLog@U2@@YAXXZ  100113c0 f   GCFramePlot.obj
 0001:000103d0       ??__F?_Generic_object@?$_Error_objects@H@std@@2V_Generic_error_category@2@A@@YAXXZ 100113d0 f   KarlinSignatureDifferenceGraph.obj
 0001:000103e0       ??__F?_Iostream_object@?$_Error_objects@H@std@@2V_Iostream_error_category@2@A@@YAXXZ 100113e0 f   KarlinSignatureDifferenceGraph.obj
 0001:000103f0       ??__F?_System_object@?$_Error_objects@H@std@@2V_System_error_category@2@A@@YAXXZ 100113f0 f   KarlinSignatureDifferenceGraph.obj
 0001:00010400       ??__FService_DNAExport@U2@@YAXXZ 10011400 f   KarlinSignatureDifferenceGraph.obj
 0001:00010410       ??__FService_DNAGraphPack@U2@@YAXXZ 10011410 f   KarlinSignatureDifferenceGraph.obj
 0001:00010420       ??__FService_ExternalToolSupport@U2@@YAXXZ 10011420 f   KarlinSignatureDifferenceGraph.obj
 0001:00010430       ??__FService_GUITesting@U2@@YAXXZ 10011430 f   KarlinSignatureDifferenceGraph.obj
 0001:00010440       ??__FService_MaxCoreServiceId@U2@@YAXXZ 10011440 f   KarlinSignatureDifferenceGraph.obj
 0001:00010450       ??__FService_MinCoreServiceId@U2@@YAXXZ 10011450 f   KarlinSignatureDifferenceGraph.obj
 0001:00010460       ??__FService_PluginViewer@U2@@YAXXZ 10011460 f   KarlinSignatureDifferenceGraph.obj
 0001:00010470       ??__FService_Project@U2@@YAXXZ 10011470 f   KarlinSignatureDifferenceGraph.obj
 0001:00010480       ??__FService_ProjectView@U2@@YAXXZ 10011480 f   KarlinSignatureDifferenceGraph.obj
 0001:00010490       ??__FService_QueryDesigner@U2@@YAXXZ 10011490 f   KarlinSignatureDifferenceGraph.obj
 0001:000104a0       ??__FService_ScriptRegistry@U2@@YAXXZ 100114a0 f   KarlinSignatureDifferenceGraph.obj
 0001:000104b0       ??__FService_TestRunner@U2@@YAXXZ 100114b0 f   KarlinSignatureDifferenceGraph.obj
 0001:000104c0       ??__FService_WorkflowDesigner@U2@@YAXXZ 100114c0 f   KarlinSignatureDifferenceGraph.obj
 0001:000104d0       ??__FalgoLog@U2@@YAXXZ     100114d0 f   KarlinSignatureDifferenceGraph.obj
 0001:000104e0       ??__FcmdLog@U2@@YAXXZ      100114e0 f   KarlinSignatureDifferenceGraph.obj
 0001:000104f0       ??__FcoreLog@U2@@YAXXZ     100114f0 f   KarlinSignatureDifferenceGraph.obj
 0001:00010500       ??__FioLog@U2@@YAXXZ       10011500 f   KarlinSignatureDifferenceGraph.obj
 0001:00010510       ??__FperfLog@U2@@YAXXZ     10011510 f   KarlinSignatureDifferenceGraph.obj
 0001:00010520       ??__FscriptLog@U2@@YAXXZ   10011520 f   KarlinSignatureDifferenceGraph.obj
 0001:00010530       ??__FtaskLog@U2@@YAXXZ     10011530 f   KarlinSignatureDifferenceGraph.obj
 0001:00010540       ??__FuiLog@U2@@YAXXZ       10011540 f   KarlinSignatureDifferenceGraph.obj
 0001:00010550       ??__FuserActLog@U2@@YAXXZ  10011550 f   KarlinSignatureDifferenceGraph.obj
 0001:00010560       ??__F?_Generic_object@?$_Error_objects@H@std@@2V_Generic_error_category@2@A@@YAXXZ 10011560 f   moc_BaseContentGraph.obj
 0001:00010570       ??__F?_Iostream_object@?$_Error_objects@H@std@@2V_Iostream_error_category@2@A@@YAXXZ 10011570 f   moc_BaseContentGraph.obj
 0001:00010580       ??__F?_System_object@?$_Error_objects@H@std@@2V_System_error_category@2@A@@YAXXZ 10011580 f   moc_BaseContentGraph.obj
 0001:00010590       ??__FService_DNAExport@U2@@YAXXZ 10011590 f   moc_BaseContentGraph.obj
 0001:000105a0       ??__FService_DNAGraphPack@U2@@YAXXZ 100115a0 f   moc_BaseContentGraph.obj
 0001:000105b0       ??__FService_ExternalToolSupport@U2@@YAXXZ 100115b0 f   moc_BaseContentGraph.obj
 0001:000105c0       ??__FService_GUITesting@U2@@YAXXZ 100115c0 f   moc_BaseContentGraph.obj
 0001:000105d0       ??__FService_MaxCoreServiceId@U2@@YAXXZ 100115d0 f   moc_BaseContentGraph.obj
 0001:000105e0       ??__FService_MinCoreServiceId@U2@@YAXXZ 100115e0 f   moc_BaseContentGraph.obj
 0001:000105f0       ??__FService_PluginViewer@U2@@YAXXZ 100115f0 f   moc_BaseContentGraph.obj
 0001:00010600       ??__FService_Project@U2@@YAXXZ 10011600 f   moc_BaseContentGraph.obj
 0001:00010610       ??__FService_ProjectView@U2@@YAXXZ 10011610 f   moc_BaseContentGraph.obj
 0001:00010620       ??__FService_QueryDesigner@U2@@YAXXZ 10011620 f   moc_BaseContentGraph.obj
 0001:00010630       ??__FService_ScriptRegistry@U2@@YAXXZ 10011630 f   moc_BaseContentGraph.obj
 0001:00010640       ??__FService_TestRunner@U2@@YAXXZ 10011640 f   moc_BaseContentGraph.obj
 0001:00010650       ??__FService_WorkflowDesigner@U2@@YAXXZ 10011650 f   moc_BaseContentGraph.obj
 0001:00010660       ??__FalgoLog@U2@@YAXXZ     10011660 f   moc_BaseContentGraph.obj
 0001:00010670       ??__FcmdLog@U2@@YAXXZ      10011670 f   moc_BaseContentGraph.obj
 0001:00010680       ??__FcoreLog@U2@@YAXXZ     10011680 f   moc_BaseContentGraph.obj
 0001:00010690       ??__FioLog@U2@@YAXXZ       10011690 f   moc_BaseContentGraph.obj
 0001:000106a0       ??__FperfLog@U2@@YAXXZ     100116a0 f   moc_BaseContentGraph.obj
 0001:000106b0       ??__FscriptLog@U2@@YAXXZ   100116b0 f   moc_BaseContentGraph.obj
 0001:000106c0       ??__FtaskLog@U2@@YAXXZ     100116c0 f   moc_BaseContentGraph.obj
 0001:000106d0       ??__FuiLog@U2@@YAXXZ       100116d0 f   moc_BaseContentGraph.obj
 0001:000106e0       ??__FuserActLog@U2@@YAXXZ  100116e0 f   moc_BaseContentGraph.obj
 0001:000106f0       ??__F?_Generic_object@?$_Error_objects@H@std@@2V_Generic_error_category@2@A@@YAXXZ 100116f0 f   moc_CumulativeSkew.obj
 0001:00010700       ??__F?_Iostream_object@?$_Error_objects@H@std@@2V_Iostream_error_category@2@A@@YAXXZ 10011700 f   moc_CumulativeSkew.obj
 0001:00010710       ??__F?_System_object@?$_Error_objects@H@std@@2V_System_error_category@2@A@@YAXXZ 10011710 f   moc_CumulativeSkew.obj
 0001:00010720       ??__FService_DNAExport@U2@@YAXXZ 10011720 f   moc_CumulativeSkew.obj
 0001:00010730       ??__FService_DNAGraphPack@U2@@YAXXZ 10011730 f   moc_CumulativeSkew.obj
 0001:00010740       ??__FService_ExternalToolSupport@U2@@YAXXZ 10011740 f   moc_CumulativeSkew.obj
 0001:00010750       ??__FService_GUITesting@U2@@YAXXZ 10011750 f   moc_CumulativeSkew.obj
 0001:00010760       ??__FService_MaxCoreServiceId@U2@@YAXXZ 10011760 f   moc_CumulativeSkew.obj
 0001:00010770       ??__FService_MinCoreServiceId@U2@@YAXXZ 10011770 f   moc_CumulativeSkew.obj
 0001:00010780       ??__FService_PluginViewer@U2@@YAXXZ 10011780 f   moc_CumulativeSkew.obj
 0001:00010790       ??__FService_Project@U2@@YAXXZ 10011790 f   moc_CumulativeSkew.obj
 0001:000107a0       ??__FService_ProjectView@U2@@YAXXZ 100117a0 f   moc_CumulativeSkew.obj
 0001:000107b0       ??__FService_QueryDesigner@U2@@YAXXZ 100117b0 f   moc_CumulativeSkew.obj
 0001:000107c0       ??__FService_ScriptRegistry@U2@@YAXXZ 100117c0 f   moc_CumulativeSkew.obj
 0001:000107d0       ??__FService_TestRunner@U2@@YAXXZ 100117d0 f   moc_CumulativeSkew.obj
 0001:000107e0       ??__FService_WorkflowDesigner@U2@@YAXXZ 100117e0 f   moc_CumulativeSkew.obj
 0001:000107f0       ??__FalgoLog@U2@@YAXXZ     100117f0 f   moc_CumulativeSkew.obj
 0001:00010800       ??__FcmdLog@U2@@YAXXZ      10011800 f   moc_CumulativeSkew.obj
 0001:00010810       ??__FcoreLog@U2@@YAXXZ     10011810 f   moc_CumulativeSkew.obj
 0001:00010820       ??__FioLog@U2@@YAXXZ       10011820 f   moc_CumulativeSkew.obj
 0001:00010830       ??__FperfLog@U2@@YAXXZ     10011830 f   moc_CumulativeSkew.obj
 0001:00010840       ??__FscriptLog@U2@@YAXXZ   10011840 f   moc_CumulativeSkew.obj
 0001:00010850       ??__FtaskLog@U2@@YAXXZ     10011850 f   moc_CumulativeSkew.obj
 0001:00010860       ??__FuiLog@U2@@YAXXZ       10011860 f   moc_CumulativeSkew.obj
 0001:00010870       ??__FuserActLog@U2@@YAXXZ  10011870 f   moc_CumulativeSkew.obj
 0001:00010880       ??__F?_Generic_object@?$_Error_objects@H@std@@2V_Generic_error_category@2@A@@YAXXZ 10011880 f   moc_DNAGraphPackPlugin.obj
 0001:00010890       ??__F?_Iostream_object@?$_Error_objects@H@std@@2V_Iostream_error_category@2@A@@YAXXZ 10011890 f   moc_DNAGraphPackPlugin.obj
 0001:000108a0       ??__F?_System_object@?$_Error_objects@H@std@@2V_System_error_category@2@A@@YAXXZ 100118a0 f   moc_DNAGraphPackPlugin.obj
 0001:000108b0       ??__FService_DNAExport@U2@@YAXXZ 100118b0 f   moc_DNAGraphPackPlugin.obj
 0001:000108c0       ??__FService_DNAGraphPack@U2@@YAXXZ 100118c0 f   moc_DNAGraphPackPlugin.obj
 0001:000108d0       ??__FService_ExternalToolSupport@U2@@YAXXZ 100118d0 f   moc_DNAGraphPackPlugin.obj
 0001:000108e0       ??__FService_GUITesting@U2@@YAXXZ 100118e0 f   moc_DNAGraphPackPlugin.obj
 0001:000108f0       ??__FService_MaxCoreServiceId@U2@@YAXXZ 100118f0 f   moc_DNAGraphPackPlugin.obj
 0001:00010900       ??__FService_MinCoreServiceId@U2@@YAXXZ 10011900 f   moc_DNAGraphPackPlugin.obj
 0001:00010910       ??__FService_PluginViewer@U2@@YAXXZ 10011910 f   moc_DNAGraphPackPlugin.obj
 0001:00010920       ??__FService_Project@U2@@YAXXZ 10011920 f   moc_DNAGraphPackPlugin.obj
 0001:00010930       ??__FService_ProjectView@U2@@YAXXZ 10011930 f   moc_DNAGraphPackPlugin.obj
 0001:00010940       ??__FService_QueryDesigner@U2@@YAXXZ 10011940 f   moc_DNAGraphPackPlugin.obj
 0001:00010950       ??__FService_ScriptRegistry@U2@@YAXXZ 10011950 f   moc_DNAGraphPackPlugin.obj
 0001:00010960       ??__FService_TestRunner@U2@@YAXXZ 10011960 f   moc_DNAGraphPackPlugin.obj
 0001:00010970       ??__FService_WorkflowDesigner@U2@@YAXXZ 10011970 f   moc_DNAGraphPackPlugin.obj
 0001:00010980       ??__FalgoLog@U2@@YAXXZ     10011980 f   moc_DNAGraphPackPlugin.obj
 0001:00010990       ??__FcmdLog@U2@@YAXXZ      10011990 f   moc_DNAGraphPackPlugin.obj
 0001:000109a0       ??__FcoreLog@U2@@YAXXZ     100119a0 f   moc_DNAGraphPackPlugin.obj
 0001:000109b0       ??__FioLog@U2@@YAXXZ       100119b0 f   moc_DNAGraphPackPlugin.obj
 0001:000109c0       ??__FperfLog@U2@@YAXXZ     100119c0 f   moc_DNAGraphPackPlugin.obj
 0001:000109d0       ??__FscriptLog@U2@@YAXXZ   100119d0 f   moc_DNAGraphPackPlugin.obj
 0001:000109e0       ??__FtaskLog@U2@@YAXXZ     100119e0 f   moc_DNAGraphPackPlugin.obj
 0001:000109f0       ??__FuiLog@U2@@YAXXZ       100119f0 f   moc_DNAGraphPackPlugin.obj
 0001:00010a00       ??__FuserActLog@U2@@YAXXZ  10011a00 f   moc_DNAGraphPackPlugin.obj
 0001:00010a10       ??__F?_Generic_object@?$_Error_objects@H@std@@2V_Generic_error_category@2@A@@YAXXZ 10011a10 f   moc_DeviationGraph.obj
 0001:00010a20       ??__F?_Iostream_object@?$_Error_objects@H@std@@2V_Iostream_error_category@2@A@@YAXXZ 10011a20 f   moc_DeviationGraph.obj
 0001:00010a30       ??__F?_System_object@?$_Error_objects@H@std@@2V_System_error_category@2@A@@YAXXZ 10011a30 f   moc_DeviationGraph.obj
 0001:00010a40       ??__FService_DNAExport@U2@@YAXXZ 10011a40 f   moc_DeviationGraph.obj
 0001:00010a50       ??__FService_DNAGraphPack@U2@@YAXXZ 10011a50 f   moc_DeviationGraph.obj
 0001:00010a60       ??__FService_ExternalToolSupport@U2@@YAXXZ 10011a60 f   moc_DeviationGraph.obj
 0001:00010a70       ??__FService_GUITesting@U2@@YAXXZ 10011a70 f   moc_DeviationGraph.obj
 0001:00010a80       ??__FService_MaxCoreServiceId@U2@@YAXXZ 10011a80 f   moc_DeviationGraph.obj
 0001:00010a90       ??__FService_MinCoreServiceId@U2@@YAXXZ 10011a90 f   moc_DeviationGraph.obj
 0001:00010aa0       ??__FService_PluginViewer@U2@@YAXXZ 10011aa0 f   moc_DeviationGraph.obj
 0001:00010ab0       ??__FService_Project@U2@@YAXXZ 10011ab0 f   moc_DeviationGraph.obj
 0001:00010ac0       ??__FService_ProjectView@U2@@YAXXZ 10011ac0 f   moc_DeviationGraph.obj
 0001:00010ad0       ??__FService_QueryDesigner@U2@@YAXXZ 10011ad0 f   moc_DeviationGraph.obj
 0001:00010ae0       ??__FService_ScriptRegistry@U2@@YAXXZ 10011ae0 f   moc_DeviationGraph.obj
 0001:00010af0       ??__FService_TestRunner@U2@@YAXXZ 10011af0 f   moc_DeviationGraph.obj
 0001:00010b00       ??__FService_WorkflowDesigner@U2@@YAXXZ 10011b00 f   moc_DeviationGraph.obj
 0001:00010b10       ??__FalgoLog@U2@@YAXXZ     10011b10 f   moc_DeviationGraph.obj
 0001:00010b20       ??__FcmdLog@U2@@YAXXZ      10011b20 f   moc_DeviationGraph.obj
 0001:00010b30       ??__FcoreLog@U2@@YAXXZ     10011b30 f   moc_DeviationGraph.obj
 0001:00010b40       ??__FioLog@U2@@YAXXZ       10011b40 f   moc_DeviationGraph.obj
 0001:00010b50       ??__FperfLog@U2@@YAXXZ     10011b50 f   moc_DeviationGraph.obj
 0001:00010b60       ??__FscriptLog@U2@@YAXXZ   10011b60 f   moc_DeviationGraph.obj
 0001:00010b70       ??__FtaskLog@U2@@YAXXZ     10011b70 f   moc_DeviationGraph.obj
 0001:00010b80       ??__FuiLog@U2@@YAXXZ       10011b80 f   moc_DeviationGraph.obj
 0001:00010b90       ??__FuserActLog@U2@@YAXXZ  10011b90 f   moc_DeviationGraph.obj
 0001:00010ba0       ??__F?_Generic_object@?$_Error_objects@H@std@@2V_Generic_error_category@2@A@@YAXXZ 10011ba0 f   moc_EntropyAlgorithm.obj
 0001:00010bb0       ??__F?_Iostream_object@?$_Error_objects@H@std@@2V_Iostream_error_category@2@A@@YAXXZ 10011bb0 f   moc_EntropyAlgorithm.obj
 0001:00010bc0       ??__F?_System_object@?$_Error_objects@H@std@@2V_System_error_category@2@A@@YAXXZ 10011bc0 f   moc_EntropyAlgorithm.obj
 0001:00010bd0       ??__FService_DNAExport@U2@@YAXXZ 10011bd0 f   moc_EntropyAlgorithm.obj
 0001:00010be0       ??__FService_DNAGraphPack@U2@@YAXXZ 10011be0 f   moc_EntropyAlgorithm.obj
 0001:00010bf0       ??__FService_ExternalToolSupport@U2@@YAXXZ 10011bf0 f   moc_EntropyAlgorithm.obj
 0001:00010c00       ??__FService_GUITesting@U2@@YAXXZ 10011c00 f   moc_EntropyAlgorithm.obj
 0001:00010c10       ??__FService_MaxCoreServiceId@U2@@YAXXZ 10011c10 f   moc_EntropyAlgorithm.obj
 0001:00010c20       ??__FService_MinCoreServiceId@U2@@YAXXZ 10011c20 f   moc_EntropyAlgorithm.obj
 0001:00010c30       ??__FService_PluginViewer@U2@@YAXXZ 10011c30 f   moc_EntropyAlgorithm.obj
 0001:00010c40       ??__FService_Project@U2@@YAXXZ 10011c40 f   moc_EntropyAlgorithm.obj
 0001:00010c50       ??__FService_ProjectView@U2@@YAXXZ 10011c50 f   moc_EntropyAlgorithm.obj
 0001:00010c60       ??__FService_QueryDesigner@U2@@YAXXZ 10011c60 f   moc_EntropyAlgorithm.obj
 0001:00010c70       ??__FService_ScriptRegistry@U2@@YAXXZ 10011c70 f   moc_EntropyAlgorithm.obj
 0001:00010c80       ??__FService_TestRunner@U2@@YAXXZ 10011c80 f   moc_EntropyAlgorithm.obj
 0001:00010c90       ??__FService_WorkflowDesigner@U2@@YAXXZ 10011c90 f   moc_EntropyAlgorithm.obj
 0001:00010ca0       ??__FalgoLog@U2@@YAXXZ     10011ca0 f   moc_EntropyAlgorithm.obj
 0001:00010cb0       ??__FcmdLog@U2@@YAXXZ      10011cb0 f   moc_EntropyAlgorithm.obj
 0001:00010cc0       ??__FcoreLog@U2@@YAXXZ     10011cc0 f   moc_EntropyAlgorithm.obj
 0001:00010cd0       ??__FioLog@U2@@YAXXZ       10011cd0 f   moc_EntropyAlgorithm.obj
 0001:00010ce0       ??__FperfLog@U2@@YAXXZ     10011ce0 f   moc_EntropyAlgorithm.obj
 0001:00010cf0       ??__FscriptLog@U2@@YAXXZ   10011cf0 f   moc_EntropyAlgorithm.obj
 0001:00010d00       ??__FtaskLog@U2@@YAXXZ     10011d00 f   moc_EntropyAlgorithm.obj
 0001:00010d10       ??__FuiLog@U2@@YAXXZ       10011d10 f   moc_EntropyAlgorithm.obj
 0001:00010d20       ??__FuserActLog@U2@@YAXXZ  10011d20 f   moc_EntropyAlgorithm.obj
 0001:00010d30       ??__F?_Generic_object@?$_Error_objects@H@std@@2V_Generic_error_category@2@A@@YAXXZ 10011d30 f   moc_GCFramePlot.obj
 0001:00010d40       ??__F?_Iostream_object@?$_Error_objects@H@std@@2V_Iostream_error_category@2@A@@YAXXZ 10011d40 f   moc_GCFramePlot.obj
 0001:00010d50       ??__F?_System_object@?$_Error_objects@H@std@@2V_System_error_category@2@A@@YAXXZ 10011d50 f   moc_GCFramePlot.obj
 0001:00010d60       ??__FService_DNAExport@U2@@YAXXZ 10011d60 f   moc_GCFramePlot.obj
 0001:00010d70       ??__FService_DNAGraphPack@U2@@YAXXZ 10011d70 f   moc_GCFramePlot.obj
 0001:00010d80       ??__FService_ExternalToolSupport@U2@@YAXXZ 10011d80 f   moc_GCFramePlot.obj
 0001:00010d90       ??__FService_GUITesting@U2@@YAXXZ 10011d90 f   moc_GCFramePlot.obj
 0001:00010da0       ??__FService_MaxCoreServiceId@U2@@YAXXZ 10011da0 f   moc_GCFramePlot.obj
 0001:00010db0       ??__FService_MinCoreServiceId@U2@@YAXXZ 10011db0 f   moc_GCFramePlot.obj
 0001:00010dc0       ??__FService_PluginViewer@U2@@YAXXZ 10011dc0 f   moc_GCFramePlot.obj
 0001:00010dd0       ??__FService_Project@U2@@YAXXZ 10011dd0 f   moc_GCFramePlot.obj
 0001:00010de0       ??__FService_ProjectView@U2@@YAXXZ 10011de0 f   moc_GCFramePlot.obj
 0001:00010df0       ??__FService_QueryDesigner@U2@@YAXXZ 10011df0 f   moc_GCFramePlot.obj
 0001:00010e00       ??__FService_ScriptRegistry@U2@@YAXXZ 10011e00 f   moc_GCFramePlot.obj
 0001:00010e10       ??__FService_TestRunner@U2@@YAXXZ 10011e10 f   moc_GCFramePlot.obj
 0001:00010e20       ??__FService_WorkflowDesigner@U2@@YAXXZ 10011e20 f   moc_GCFramePlot.obj
 0001:00010e30       ??__FalgoLog@U2@@YAXXZ     10011e30 f   moc_GCFramePlot.obj
 0001:00010e40       ??__FcmdLog@U2@@YAXXZ      10011e40 f   moc_GCFramePlot.obj
 0001:00010e50       ??__FcoreLog@U2@@YAXXZ     10011e50 f   moc_GCFramePlot.obj
 0001:00010e60       ??__FioLog@U2@@YAXXZ       10011e60 f   moc_GCFramePlot.obj
 0001:00010e70       ??__FperfLog@U2@@YAXXZ     10011e70 f   moc_GCFramePlot.obj
 0001:00010e80       ??__FscriptLog@U2@@YAXXZ   10011e80 f   moc_GCFramePlot.obj
 0001:00010e90       ??__FtaskLog@U2@@YAXXZ     10011e90 f   moc_GCFramePlot.obj
 0001:00010ea0       ??__FuiLog@U2@@YAXXZ       10011ea0 f   moc_GCFramePlot.obj
 0001:00010eb0       ??__FuserActLog@U2@@YAXXZ  10011eb0 f   moc_GCFramePlot.obj
 0001:00010ec0       ??__F?_Generic_object@?$_Error_objects@H@std@@2V_Generic_error_category@2@A@@YAXXZ 10011ec0 f   moc_KarlinSignatureDifferenceGraph.obj
 0001:00010ed0       ??__F?_Iostream_object@?$_Error_objects@H@std@@2V_Iostream_error_category@2@A@@YAXXZ 10011ed0 f   moc_KarlinSignatureDifferenceGraph.obj
 0001:00010ee0       ??__F?_System_object@?$_Error_objects@H@std@@2V_System_error_category@2@A@@YAXXZ 10011ee0 f   moc_KarlinSignatureDifferenceGraph.obj
 0001:00010ef0       ??__FService_DNAExport@U2@@YAXXZ 10011ef0 f   moc_KarlinSignatureDifferenceGraph.obj
 0001:00010f00       ??__FService_DNAGraphPack@U2@@YAXXZ 10011f00 f   moc_KarlinSignatureDifferenceGraph.obj
 0001:00010f10       ??__FService_ExternalToolSupport@U2@@YAXXZ 10011f10 f   moc_KarlinSignatureDifferenceGraph.obj
 0001:00010f20       ??__FService_GUITesting@U2@@YAXXZ 10011f20 f   moc_KarlinSignatureDifferenceGraph.obj
 0001:00010f30       ??__FService_MaxCoreServiceId@U2@@YAXXZ 10011f30 f   moc_KarlinSignatureDifferenceGraph.obj
 0001:00010f40       ??__FService_MinCoreServiceId@U2@@YAXXZ 10011f40 f   moc_KarlinSignatureDifferenceGraph.obj
 0001:00010f50       ??__FService_PluginViewer@U2@@YAXXZ 10011f50 f   moc_KarlinSignatureDifferenceGraph.obj
 0001:00010f60       ??__FService_Project@U2@@YAXXZ 10011f60 f   moc_KarlinSignatureDifferenceGraph.obj
 0001:00010f70       ??__FService_ProjectView@U2@@YAXXZ 10011f70 f   moc_KarlinSignatureDifferenceGraph.obj
 0001:00010f80       ??__FService_QueryDesigner@U2@@YAXXZ 10011f80 f   moc_KarlinSignatureDifferenceGraph.obj
 0001:00010f90       ??__FService_ScriptRegistry@U2@@YAXXZ 10011f90 f   moc_KarlinSignatureDifferenceGraph.obj
 0001:00010fa0       ??__FService_TestRunner@U2@@YAXXZ 10011fa0 f   moc_KarlinSignatureDifferenceGraph.obj
 0001:00010fb0       ??__FService_WorkflowDesigner@U2@@YAXXZ 10011fb0 f   moc_KarlinSignatureDifferenceGraph.obj
 0001:00010fc0       ??__FalgoLog@U2@@YAXXZ     10011fc0 f   moc_KarlinSignatureDifferenceGraph.obj
 0001:00010fd0       ??__FcmdLog@U2@@YAXXZ      10011fd0 f   moc_KarlinSignatureDifferenceGraph.obj
 0001:00010fe0       ??__FcoreLog@U2@@YAXXZ     10011fe0 f   moc_KarlinSignatureDifferenceGraph.obj
 0001:00010ff0       ??__FioLog@U2@@YAXXZ       10011ff0 f   moc_KarlinSignatureDifferenceGraph.obj
 0001:00011000       ??__FperfLog@U2@@YAXXZ     10012000 f   moc_KarlinSignatureDifferenceGraph.obj
 0001:00011010       ??__FscriptLog@U2@@YAXXZ   10012010 f   moc_KarlinSignatureDifferenceGraph.obj
 0001:00011020       ??__FtaskLog@U2@@YAXXZ     10012020 f   moc_KarlinSignatureDifferenceGraph.obj
 0001:00011030       ??__FuiLog@U2@@YAXXZ       10012030 f   moc_KarlinSignatureDifferenceGraph.obj
 0001:00011040       ??__FuserActLog@U2@@YAXXZ  10012040 f   moc_KarlinSignatureDifferenceGraph.obj
 0001:00011050       ??__Fdummy@?A0x701b237d@@YAXXZ 10012050 f   qrc_dna_graphpack.obj
 0002:000002bc       _Service_PluginViewer$initializer$ 100132bc     BaseContentGraph.obj
 0002:000002c0       _Service_Project$initializer$ 100132c0     BaseContentGraph.obj
 0002:000002c4       _Service_ProjectView$initializer$ 100132c4     BaseContentGraph.obj
 0002:000002c8       _Service_DNAGraphPack$initializer$ 100132c8     BaseContentGraph.obj
 0002:000002cc       _Service_DNAExport$initializer$ 100132cc     BaseContentGraph.obj
 0002:000002d0       _Service_TestRunner$initializer$ 100132d0     BaseContentGraph.obj
 0002:000002d4       _Service_ScriptRegistry$initializer$ 100132d4     BaseContentGraph.obj
 0002:000002d8       _Service_ExternalToolSupport$initializer$ 100132d8     BaseContentGraph.obj
 0002:000002dc       _Service_GUITesting$initializer$ 100132dc     BaseContentGraph.obj
 0002:000002e0       _Service_WorkflowDesigner$initializer$ 100132e0     BaseContentGraph.obj
 0002:000002e4       _Service_QueryDesigner$initializer$ 100132e4     BaseContentGraph.obj
 0002:000002e8       _Service_MinCoreServiceId$initializer$ 100132e8     BaseContentGraph.obj
 0002:000002ec       _Service_MaxCoreServiceId$initializer$ 100132ec     BaseContentGraph.obj
 0002:000002f0       _algoLog$initializer$      100132f0     BaseContentGraph.obj
 0002:000002f4       _cmdLog$initializer$       100132f4     BaseContentGraph.obj
 0002:000002f8       _coreLog$initializer$      100132f8     BaseContentGraph.obj
 0002:000002fc       _ioLog$initializer$        100132fc     BaseContentGraph.obj
 0002:00000300       _perfLog$initializer$      10013300     BaseContentGraph.obj
 0002:00000304       _scriptLog$initializer$    10013304     BaseContentGraph.obj
 0002:00000308       _taskLog$initializer$      10013308     BaseContentGraph.obj
 0002:0000030c       _uiLog$initializer$        1001330c     BaseContentGraph.obj
 0002:00000310       _userActLog$initializer$   10013310     BaseContentGraph.obj
 0002:00000314       ?_Generic_object$initializer$@?$_Error_objects@H@std@@2P6AXXZA 10013314     BaseContentGraph.obj
 0002:00000318       ?_Iostream_object$initializer$@?$_Error_objects@H@std@@2P6AXXZA 10013318     BaseContentGraph.obj
 0002:0000031c       ?_System_object$initializer$@?$_Error_objects@H@std@@2P6AXXZA 1001331c     BaseContentGraph.obj
 0002:00000320       _Service_PluginViewer$initializer$ 10013320     CumulativeSkew.obj
 0002:00000324       _Service_Project$initializer$ 10013324     CumulativeSkew.obj
 0002:00000328       _Service_ProjectView$initializer$ 10013328     CumulativeSkew.obj
 0002:0000032c       _Service_DNAGraphPack$initializer$ 1001332c     CumulativeSkew.obj
 0002:00000330       _Service_DNAExport$initializer$ 10013330     CumulativeSkew.obj
 0002:00000334       _Service_TestRunner$initializer$ 10013334     CumulativeSkew.obj
 0002:00000338       _Service_ScriptRegistry$initializer$ 10013338     CumulativeSkew.obj
 0002:0000033c       _Service_ExternalToolSupport$initializer$ 1001333c     CumulativeSkew.obj
 0002:00000340       _Service_GUITesting$initializer$ 10013340     CumulativeSkew.obj
 0002:00000344       _Service_WorkflowDesigner$initializer$ 10013344     CumulativeSkew.obj
 0002:00000348       _Service_QueryDesigner$initializer$ 10013348     CumulativeSkew.obj
 0002:0000034c       _Service_MinCoreServiceId$initializer$ 1001334c     CumulativeSkew.obj
 0002:00000350       _Service_MaxCoreServiceId$initializer$ 10013350     CumulativeSkew.obj
 0002:00000354       _algoLog$initializer$      10013354     CumulativeSkew.obj
 0002:00000358       _cmdLog$initializer$       10013358     CumulativeSkew.obj
 0002:0000035c       _coreLog$initializer$      1001335c     CumulativeSkew.obj
 0002:00000360       _ioLog$initializer$        10013360     CumulativeSkew.obj
 0002:00000364       _perfLog$initializer$      10013364     CumulativeSkew.obj
 0002:00000368       _scriptLog$initializer$    10013368     CumulativeSkew.obj
 0002:0000036c       _taskLog$initializer$      1001336c     CumulativeSkew.obj
 0002:00000370       _uiLog$initializer$        10013370     CumulativeSkew.obj
 0002:00000374       _userActLog$initializer$   10013374     CumulativeSkew.obj
 0002:00000378       _Service_PluginViewer$initializer$ 10013378     DNAGraphPackPlugin.obj
 0002:0000037c       _Service_Project$initializer$ 1001337c     DNAGraphPackPlugin.obj
 0002:00000380       _Service_ProjectView$initializer$ 10013380     DNAGraphPackPlugin.obj
 0002:00000384       _Service_DNAGraphPack$initializer$ 10013384     DNAGraphPackPlugin.obj
 0002:00000388       _Service_DNAExport$initializer$ 10013388     DNAGraphPackPlugin.obj
 0002:0000038c       _Service_TestRunner$initializer$ 1001338c     DNAGraphPackPlugin.obj
 0002:00000390       _Service_ScriptRegistry$initializer$ 10013390     DNAGraphPackPlugin.obj
 0002:00000394       _Service_ExternalToolSupport$initializer$ 10013394     DNAGraphPackPlugin.obj
 0002:00000398       _Service_GUITesting$initializer$ 10013398     DNAGraphPackPlugin.obj
 0002:0000039c       _Service_WorkflowDesigner$initializer$ 1001339c     DNAGraphPackPlugin.obj
 0002:000003a0       _Service_QueryDesigner$initializer$ 100133a0     DNAGraphPackPlugin.obj
 0002:000003a4       _Service_MinCoreServiceId$initializer$ 100133a4     DNAGraphPackPlugin.obj
 0002:000003a8       _Service_MaxCoreServiceId$initializer$ 100133a8     DNAGraphPackPlugin.obj
 0002:000003ac       _algoLog$initializer$      100133ac     DNAGraphPackPlugin.obj
 0002:000003b0       _cmdLog$initializer$       100133b0     DNAGraphPackPlugin.obj
 0002:000003b4       _coreLog$initializer$      100133b4     DNAGraphPackPlugin.obj
 0002:000003b8       _ioLog$initializer$        100133b8     DNAGraphPackPlugin.obj
 0002:000003bc       _perfLog$initializer$      100133bc     DNAGraphPackPlugin.obj
 0002:000003c0       _scriptLog$initializer$    100133c0     DNAGraphPackPlugin.obj
 0002:000003c4       _taskLog$initializer$      100133c4     DNAGraphPackPlugin.obj
 0002:000003c8       _uiLog$initializer$        100133c8     DNAGraphPackPlugin.obj
 0002:000003cc       _userActLog$initializer$   100133cc     DNAGraphPackPlugin.obj
 0002:000003d0       _Service_PluginViewer$initializer$ 100133d0     DeviationGraph.obj
 0002:000003d4       _Service_Project$initializer$ 100133d4     DeviationGraph.obj
 0002:000003d8       _Service_ProjectView$initializer$ 100133d8     DeviationGraph.obj
 0002:000003dc       _Service_DNAGraphPack$initializer$ 100133dc     DeviationGraph.obj
 0002:000003e0       _Service_DNAExport$initializer$ 100133e0     DeviationGraph.obj
 0002:000003e4       _Service_TestRunner$initializer$ 100133e4     DeviationGraph.obj
 0002:000003e8       _Service_ScriptRegistry$initializer$ 100133e8     DeviationGraph.obj
 0002:000003ec       _Service_ExternalToolSupport$initializer$ 100133ec     DeviationGraph.obj
 0002:000003f0       _Service_GUITesting$initializer$ 100133f0     DeviationGraph.obj
 0002:000003f4       _Service_WorkflowDesigner$initializer$ 100133f4     DeviationGraph.obj
 0002:000003f8       _Service_QueryDesigner$initializer$ 100133f8     DeviationGraph.obj
 0002:000003fc       _Service_MinCoreServiceId$initializer$ 100133fc     DeviationGraph.obj
 0002:00000400       _Service_MaxCoreServiceId$initializer$ 10013400     DeviationGraph.obj
 0002:00000404       _algoLog$initializer$      10013404     DeviationGraph.obj
 0002:00000408       _cmdLog$initializer$       10013408     DeviationGraph.obj
 0002:0000040c       _coreLog$initializer$      1001340c     DeviationGraph.obj
 0002:00000410       _ioLog$initializer$        10013410     DeviationGraph.obj
 0002:00000414       _perfLog$initializer$      10013414     DeviationGraph.obj
 0002:00000418       _scriptLog$initializer$    10013418     DeviationGraph.obj
 0002:0000041c       _taskLog$initializer$      1001341c     DeviationGraph.obj
 0002:00000420       _uiLog$initializer$        10013420     DeviationGraph.obj
 0002:00000424       _userActLog$initializer$   10013424     DeviationGraph.obj
 0002:00000428       _Service_PluginViewer$initializer$ 10013428     EntropyAlgorithm.obj
 0002:0000042c       _Service_Project$initializer$ 1001342c     EntropyAlgorithm.obj
 0002:00000430       _Service_ProjectView$initializer$ 10013430     EntropyAlgorithm.obj
 0002:00000434       _Service_DNAGraphPack$initializer$ 10013434     EntropyAlgorithm.obj
 0002:00000438       _Service_DNAExport$initializer$ 10013438     EntropyAlgorithm.obj
 0002:0000043c       _Service_TestRunner$initializer$ 1001343c     EntropyAlgorithm.obj
 0002:00000440       _Service_ScriptRegistry$initializer$ 10013440     EntropyAlgorithm.obj
 0002:00000444       _Service_ExternalToolSupport$initializer$ 10013444     EntropyAlgorithm.obj
 0002:00000448       _Service_GUITesting$initializer$ 10013448     EntropyAlgorithm.obj
 0002:0000044c       _Service_WorkflowDesigner$initializer$ 1001344c     EntropyAlgorithm.obj
 0002:00000450       _Service_QueryDesigner$initializer$ 10013450     EntropyAlgorithm.obj
 0002:00000454       _Service_MinCoreServiceId$initializer$ 10013454     EntropyAlgorithm.obj
 0002:00000458       _Service_MaxCoreServiceId$initializer$ 10013458     EntropyAlgorithm.obj
 0002:0000045c       _algoLog$initializer$      1001345c     EntropyAlgorithm.obj
 0002:00000460       _cmdLog$initializer$       10013460     EntropyAlgorithm.obj
 0002:00000464       _coreLog$initializer$      10013464     EntropyAlgorithm.obj
 0002:00000468       _ioLog$initializer$        10013468     EntropyAlgorithm.obj
 0002:0000046c       _perfLog$initializer$      1001346c     EntropyAlgorithm.obj
 0002:00000470       _scriptLog$initializer$    10013470     EntropyAlgorithm.obj
 0002:00000474       _taskLog$initializer$      10013474     EntropyAlgorithm.obj
 0002:00000478       _uiLog$initializer$        10013478     EntropyAlgorithm.obj
 0002:0000047c       _userActLog$initializer$   1001347c     EntropyAlgorithm.obj
 0002:00000480       _Service_PluginViewer$initializer$ 10013480     GCFramePlot.obj
 0002:00000484       _Service_Project$initializer$ 10013484     GCFramePlot.obj
 0002:00000488       _Service_ProjectView$initializer$ 10013488     GCFramePlot.obj
 0002:0000048c       _Service_DNAGraphPack$initializer$ 1001348c     GCFramePlot.obj
 0002:00000490       _Service_DNAExport$initializer$ 10013490     GCFramePlot.obj
 0002:00000494       _Service_TestRunner$initializer$ 10013494     GCFramePlot.obj
 0002:00000498       _Service_ScriptRegistry$initializer$ 10013498     GCFramePlot.obj
 0002:0000049c       _Service_ExternalToolSupport$initializer$ 1001349c     GCFramePlot.obj
 0002:000004a0       _Service_GUITesting$initializer$ 100134a0     GCFramePlot.obj
 0002:000004a4       _Service_WorkflowDesigner$initializer$ 100134a4     GCFramePlot.obj
 0002:000004a8       _Service_QueryDesigner$initializer$ 100134a8     GCFramePlot.obj
 0002:000004ac       _Service_MinCoreServiceId$initializer$ 100134ac     GCFramePlot.obj
 0002:000004b0       _Service_MaxCoreServiceId$initializer$ 100134b0     GCFramePlot.obj
 0002:000004b4       _algoLog$initializer$      100134b4     GCFramePlot.obj
 0002:000004b8       _cmdLog$initializer$       100134b8     GCFramePlot.obj
 0002:000004bc       _coreLog$initializer$      100134bc     GCFramePlot.obj
 0002:000004c0       _ioLog$initializer$        100134c0     GCFramePlot.obj
 0002:000004c4       _perfLog$initializer$      100134c4     GCFramePlot.obj
 0002:000004c8       _scriptLog$initializer$    100134c8     GCFramePlot.obj
 0002:000004cc       _taskLog$initializer$      100134cc     GCFramePlot.obj
 0002:000004d0       _uiLog$initializer$        100134d0     GCFramePlot.obj
 0002:000004d4       _userActLog$initializer$   100134d4     GCFramePlot.obj
 0002:000004d8       _Service_PluginViewer$initializer$ 100134d8     KarlinSignatureDifferenceGraph.obj
 0002:000004dc       _Service_Project$initializer$ 100134dc     KarlinSignatureDifferenceGraph.obj
 0002:000004e0       _Service_ProjectView$initializer$ 100134e0     KarlinSignatureDifferenceGraph.obj
 0002:000004e4       _Service_DNAGraphPack$initializer$ 100134e4     KarlinSignatureDifferenceGraph.obj
 0002:000004e8       _Service_DNAExport$initializer$ 100134e8     KarlinSignatureDifferenceGraph.obj
 0002:000004ec       _Service_TestRunner$initializer$ 100134ec     KarlinSignatureDifferenceGraph.obj
 0002:000004f0       _Service_ScriptRegistry$initializer$ 100134f0     KarlinSignatureDifferenceGraph.obj
 0002:000004f4       _Service_ExternalToolSupport$initializer$ 100134f4     KarlinSignatureDifferenceGraph.obj
 0002:000004f8       _Service_GUITesting$initializer$ 100134f8     KarlinSignatureDifferenceGraph.obj
 0002:000004fc       _Service_WorkflowDesigner$initializer$ 100134fc     KarlinSignatureDifferenceGraph.obj
 0002:00000500       _Service_QueryDesigner$initializer$ 10013500     KarlinSignatureDifferenceGraph.obj
 0002:00000504       _Service_MinCoreServiceId$initializer$ 10013504     KarlinSignatureDifferenceGraph.obj
 0002:00000508       _Service_MaxCoreServiceId$initializer$ 10013508     KarlinSignatureDifferenceGraph.obj
 0002:0000050c       _algoLog$initializer$      1001350c     KarlinSignatureDifferenceGraph.obj
 0002:00000510       _cmdLog$initializer$       10013510     KarlinSignatureDifferenceGraph.obj
 0002:00000514       _coreLog$initializer$      10013514     KarlinSignatureDifferenceGraph.obj
 0002:00000518       _ioLog$initializer$        10013518     KarlinSignatureDifferenceGraph.obj
 0002:0000051c       _perfLog$initializer$      1001351c     KarlinSignatureDifferenceGraph.obj
 0002:00000520       _scriptLog$initializer$    10013520     KarlinSignatureDifferenceGraph.obj
 0002:00000524       _taskLog$initializer$      10013524     KarlinSignatureDifferenceGraph.obj
 0002:00000528       _uiLog$initializer$        10013528     KarlinSignatureDifferenceGraph.obj
 0002:0000052c       _userActLog$initializer$   1001352c     KarlinSignatureDifferenceGraph.obj
 0002:00000530       _Service_PluginViewer$initializer$ 10013530     moc_BaseContentGraph.obj
 0002:00000534       _Service_Project$initializer$ 10013534     moc_BaseContentGraph.obj
 0002:00000538       _Service_ProjectView$initializer$ 10013538     moc_BaseContentGraph.obj
 0002:0000053c       _Service_DNAGraphPack$initializer$ 1001353c     moc_BaseContentGraph.obj
 0002:00000540       _Service_DNAExport$initializer$ 10013540     moc_BaseContentGraph.obj
 0002:00000544       _Service_TestRunner$initializer$ 10013544     moc_BaseContentGraph.obj
 0002:00000548       _Service_ScriptRegistry$initializer$ 10013548     moc_BaseContentGraph.obj
 0002:0000054c       _Service_ExternalToolSupport$initializer$ 1001354c     moc_BaseContentGraph.obj
 0002:00000550       _Service_GUITesting$initializer$ 10013550     moc_BaseContentGraph.obj
 0002:00000554       _Service_WorkflowDesigner$initializer$ 10013554     moc_BaseContentGraph.obj
 0002:00000558       _Service_QueryDesigner$initializer$ 10013558     moc_BaseContentGraph.obj
 0002:0000055c       _Service_MinCoreServiceId$initializer$ 1001355c     moc_BaseContentGraph.obj
 0002:00000560       _Service_MaxCoreServiceId$initializer$ 10013560     moc_BaseContentGraph.obj
 0002:00000564       _algoLog$initializer$      10013564     moc_BaseContentGraph.obj
 0002:00000568       _cmdLog$initializer$       10013568     moc_BaseContentGraph.obj
 0002:0000056c       _coreLog$initializer$      1001356c     moc_BaseContentGraph.obj
 0002:00000570       _ioLog$initializer$        10013570     moc_BaseContentGraph.obj
 0002:00000574       _perfLog$initializer$      10013574     moc_BaseContentGraph.obj
 0002:00000578       _scriptLog$initializer$    10013578     moc_BaseContentGraph.obj
 0002:0000057c       _taskLog$initializer$      1001357c     moc_BaseContentGraph.obj
 0002:00000580       _uiLog$initializer$        10013580     moc_BaseContentGraph.obj
 0002:00000584       _userActLog$initializer$   10013584     moc_BaseContentGraph.obj
 0002:00000588       ?staticMetaObject$initializer$@BaseContentGraphFactory@U2@@2P6AXXZA 10013588     moc_BaseContentGraph.obj
 0002:0000058c       _Service_PluginViewer$initializer$ 1001358c     moc_CumulativeSkew.obj
 0002:00000590       _Service_Project$initializer$ 10013590     moc_CumulativeSkew.obj
 0002:00000594       _Service_ProjectView$initializer$ 10013594     moc_CumulativeSkew.obj
 0002:00000598       _Service_DNAGraphPack$initializer$ 10013598     moc_CumulativeSkew.obj
 0002:0000059c       _Service_DNAExport$initializer$ 1001359c     moc_CumulativeSkew.obj
 0002:000005a0       _Service_TestRunner$initializer$ 100135a0     moc_CumulativeSkew.obj
 0002:000005a4       _Service_ScriptRegistry$initializer$ 100135a4     moc_CumulativeSkew.obj
 0002:000005a8       _Service_ExternalToolSupport$initializer$ 100135a8     moc_CumulativeSkew.obj
 0002:000005ac       _Service_GUITesting$initializer$ 100135ac     moc_CumulativeSkew.obj
 0002:000005b0       _Service_WorkflowDesigner$initializer$ 100135b0     moc_CumulativeSkew.obj
 0002:000005b4       _Service_QueryDesigner$initializer$ 100135b4     moc_CumulativeSkew.obj
 0002:000005b8       _Service_MinCoreServiceId$initializer$ 100135b8     moc_CumulativeSkew.obj
 0002:000005bc       _Service_MaxCoreServiceId$initializer$ 100135bc     moc_CumulativeSkew.obj
 0002:000005c0       _algoLog$initializer$      100135c0     moc_CumulativeSkew.obj
 0002:000005c4       _cmdLog$initializer$       100135c4     moc_CumulativeSkew.obj
 0002:000005c8       _coreLog$initializer$      100135c8     moc_CumulativeSkew.obj
 0002:000005cc       _ioLog$initializer$        100135cc     moc_CumulativeSkew.obj
 0002:000005d0       _perfLog$initializer$      100135d0     moc_CumulativeSkew.obj
 0002:000005d4       _scriptLog$initializer$    100135d4     moc_CumulativeSkew.obj
 0002:000005d8       _taskLog$initializer$      100135d8     moc_CumulativeSkew.obj
 0002:000005dc       _uiLog$initializer$        100135dc     moc_CumulativeSkew.obj
 0002:000005e0       _userActLog$initializer$   100135e0     moc_CumulativeSkew.obj
 0002:000005e4       ?staticMetaObject$initializer$@CumulativeSkewGraphFactory@U2@@2P6AXXZA 100135e4     moc_CumulativeSkew.obj
 0002:000005e8       _Service_PluginViewer$initializer$ 100135e8     moc_DNAGraphPackPlugin.obj
 0002:000005ec       _Service_Project$initializer$ 100135ec     moc_DNAGraphPackPlugin.obj
 0002:000005f0       _Service_ProjectView$initializer$ 100135f0     moc_DNAGraphPackPlugin.obj
 0002:000005f4       _Service_DNAGraphPack$initializer$ 100135f4     moc_DNAGraphPackPlugin.obj
 0002:000005f8       _Service_DNAExport$initializer$ 100135f8     moc_DNAGraphPackPlugin.obj
 0002:000005fc       _Service_TestRunner$initializer$ 100135fc     moc_DNAGraphPackPlugin.obj
 0002:00000600       _Service_ScriptRegistry$initializer$ 10013600     moc_DNAGraphPackPlugin.obj
 0002:00000604       _Service_ExternalToolSupport$initializer$ 10013604     moc_DNAGraphPackPlugin.obj
 0002:00000608       _Service_GUITesting$initializer$ 10013608     moc_DNAGraphPackPlugin.obj
 0002:0000060c       _Service_WorkflowDesigner$initializer$ 1001360c     moc_DNAGraphPackPlugin.obj
 0002:00000610       _Service_QueryDesigner$initializer$ 10013610     moc_DNAGraphPackPlugin.obj
 0002:00000614       _Service_MinCoreServiceId$initializer$ 10013614     moc_DNAGraphPackPlugin.obj
 0002:00000618       _Service_MaxCoreServiceId$initializer$ 10013618     moc_DNAGraphPackPlugin.obj
 0002:0000061c       _algoLog$initializer$      1001361c     moc_DNAGraphPackPlugin.obj
 0002:00000620       _cmdLog$initializer$       10013620     moc_DNAGraphPackPlugin.obj
 0002:00000624       _coreLog$initializer$      10013624     moc_DNAGraphPackPlugin.obj
 0002:00000628       _ioLog$initializer$        10013628     moc_DNAGraphPackPlugin.obj
 0002:0000062c       _perfLog$initializer$      1001362c     moc_DNAGraphPackPlugin.obj
 0002:00000630       _scriptLog$initializer$    10013630     moc_DNAGraphPackPlugin.obj
 0002:00000634       _taskLog$initializer$      10013634     moc_DNAGraphPackPlugin.obj
 0002:00000638       _uiLog$initializer$        10013638     moc_DNAGraphPackPlugin.obj
 0002:0000063c       _userActLog$initializer$   1001363c     moc_DNAGraphPackPlugin.obj
 0002:00000640       ?staticMetaObject$initializer$@DNAGraphPackPlugin@U2@@2P6AXXZA 10013640     moc_DNAGraphPackPlugin.obj
 0002:00000644       ?staticMetaObject$initializer$@DNAGraphPackViewContext@U2@@2P6AXXZA 10013644     moc_DNAGraphPackPlugin.obj
 0002:00000648       _Service_PluginViewer$initializer$ 10013648     moc_DeviationGraph.obj
 0002:0000064c       _Service_Project$initializer$ 1001364c     moc_DeviationGraph.obj
 0002:00000650       _Service_ProjectView$initializer$ 10013650     moc_DeviationGraph.obj
 0002:00000654       _Service_DNAGraphPack$initializer$ 10013654     moc_DeviationGraph.obj
 0002:00000658       _Service_DNAExport$initializer$ 10013658     moc_DeviationGraph.obj
 0002:0000065c       _Service_TestRunner$initializer$ 1001365c     moc_DeviationGraph.obj
 0002:00000660       _Service_ScriptRegistry$initializer$ 10013660     moc_DeviationGraph.obj
 0002:00000664       _Service_ExternalToolSupport$initializer$ 10013664     moc_DeviationGraph.obj
 0002:00000668       _Service_GUITesting$initializer$ 10013668     moc_DeviationGraph.obj
 0002:0000066c       _Service_WorkflowDesigner$initializer$ 1001366c     moc_DeviationGraph.obj
 0002:00000670       _Service_QueryDesigner$initializer$ 10013670     moc_DeviationGraph.obj
 0002:00000674       _Service_MinCoreServiceId$initializer$ 10013674     moc_DeviationGraph.obj
 0002:00000678       _Service_MaxCoreServiceId$initializer$ 10013678     moc_DeviationGraph.obj
 0002:0000067c       _algoLog$initializer$      1001367c     moc_DeviationGraph.obj
 0002:00000680       _cmdLog$initializer$       10013680     moc_DeviationGraph.obj
 0002:00000684       _coreLog$initializer$      10013684     moc_DeviationGraph.obj
 0002:00000688       _ioLog$initializer$        10013688     moc_DeviationGraph.obj
 0002:0000068c       _perfLog$initializer$      1001368c     moc_DeviationGraph.obj
 0002:00000690       _scriptLog$initializer$    10013690     moc_DeviationGraph.obj
 0002:00000694       _taskLog$initializer$      10013694     moc_DeviationGraph.obj
 0002:00000698       _uiLog$initializer$        10013698     moc_DeviationGraph.obj
 0002:0000069c       _userActLog$initializer$   1001369c     moc_DeviationGraph.obj
 0002:000006a0       ?staticMetaObject$initializer$@DeviationGraphFactory@U2@@2P6AXXZA 100136a0     moc_DeviationGraph.obj
 0002:000006a4       _Service_PluginViewer$initializer$ 100136a4     moc_EntropyAlgorithm.obj
 0002:000006a8       _Service_Project$initializer$ 100136a8     moc_EntropyAlgorithm.obj
 0002:000006ac       _Service_ProjectView$initializer$ 100136ac     moc_EntropyAlgorithm.obj
 0002:000006b0       _Service_DNAGraphPack$initializer$ 100136b0     moc_EntropyAlgorithm.obj
 0002:000006b4       _Service_DNAExport$initializer$ 100136b4     moc_EntropyAlgorithm.obj
 0002:000006b8       _Service_TestRunner$initializer$ 100136b8     moc_EntropyAlgorithm.obj
 0002:000006bc       _Service_ScriptRegistry$initializer$ 100136bc     moc_EntropyAlgorithm.obj
 0002:000006c0       _Service_ExternalToolSupport$initializer$ 100136c0     moc_EntropyAlgorithm.obj
 0002:000006c4       _Service_GUITesting$initializer$ 100136c4     moc_EntropyAlgorithm.obj
 0002:000006c8       _Service_WorkflowDesigner$initializer$ 100136c8     moc_EntropyAlgorithm.obj
 0002:000006cc       _Service_QueryDesigner$initializer$ 100136cc     moc_EntropyAlgorithm.obj
 0002:000006d0       _Service_MinCoreServiceId$initializer$ 100136d0     moc_EntropyAlgorithm.obj
 0002:000006d4       _Service_MaxCoreServiceId$initializer$ 100136d4     moc_EntropyAlgorithm.obj
 0002:000006d8       _algoLog$initializer$      100136d8     moc_EntropyAlgorithm.obj
 0002:000006dc       _cmdLog$initializer$       100136dc     moc_EntropyAlgorithm.obj
 0002:000006e0       _coreLog$initializer$      100136e0     moc_EntropyAlgorithm.obj
 0002:000006e4       _ioLog$initializer$        100136e4     moc_EntropyAlgorithm.obj
 0002:000006e8       _perfLog$initializer$      100136e8     moc_EntropyAlgorithm.obj
 0002:000006ec       _scriptLog$initializer$    100136ec     moc_EntropyAlgorithm.obj
 0002:000006f0       _taskLog$initializer$      100136f0     moc_EntropyAlgorithm.obj
 0002:000006f4       _uiLog$initializer$        100136f4     moc_EntropyAlgorithm.obj
 0002:000006f8       _userActLog$initializer$   100136f8     moc_EntropyAlgorithm.obj
 0002:000006fc       ?staticMetaObject$initializer$@EntropyGraphFactory@U2@@2P6AXXZA 100136fc     moc_EntropyAlgorithm.obj
 0002:00000700       _Service_PluginViewer$initializer$ 10013700     moc_GCFramePlot.obj
 0002:00000704       _Service_Project$initializer$ 10013704     moc_GCFramePlot.obj
 0002:00000708       _Service_ProjectView$initializer$ 10013708     moc_GCFramePlot.obj
 0002:0000070c       _Service_DNAGraphPack$initializer$ 1001370c     moc_GCFramePlot.obj
 0002:00000710       _Service_DNAExport$initializer$ 10013710     moc_GCFramePlot.obj
 0002:00000714       _Service_TestRunner$initializer$ 10013714     moc_GCFramePlot.obj
 0002:00000718       _Service_ScriptRegistry$initializer$ 10013718     moc_GCFramePlot.obj
 0002:0000071c       _Service_ExternalToolSupport$initializer$ 1001371c     moc_GCFramePlot.obj
 0002:00000720       _Service_GUITesting$initializer$ 10013720     moc_GCFramePlot.obj
 0002:00000724       _Service_WorkflowDesigner$initializer$ 10013724     moc_GCFramePlot.obj
 0002:00000728       _Service_QueryDesigner$initializer$ 10013728     moc_GCFramePlot.obj
 0002:0000072c       _Service_MinCoreServiceId$initializer$ 1001372c     moc_GCFramePlot.obj
 0002:00000730       _Service_MaxCoreServiceId$initializer$ 10013730     moc_GCFramePlot.obj
 0002:00000734       _algoLog$initializer$      10013734     moc_GCFramePlot.obj
 0002:00000738       _cmdLog$initializer$       10013738     moc_GCFramePlot.obj
 0002:0000073c       _coreLog$initializer$      1001373c     moc_GCFramePlot.obj
 0002:00000740       _ioLog$initializer$        10013740     moc_GCFramePlot.obj
 0002:00000744       _perfLog$initializer$      10013744     moc_GCFramePlot.obj
 0002:00000748       _scriptLog$initializer$    10013748     moc_GCFramePlot.obj
 0002:0000074c       _taskLog$initializer$      1001374c     moc_GCFramePlot.obj
 0002:00000750       _uiLog$initializer$        10013750     moc_GCFramePlot.obj
 0002:00000754       _userActLog$initializer$   10013754     moc_GCFramePlot.obj
 0002:00000758       ?staticMetaObject$initializer$@GCFramePlotFactory@U2@@2P6AXXZA 10013758     moc_GCFramePlot.obj
 0002:0000075c       _Service_PluginViewer$initializer$ 1001375c     moc_KarlinSignatureDifferenceGraph.obj
 0002:00000760       _Service_Project$initializer$ 10013760     moc_KarlinSignatureDifferenceGraph.obj
 0002:00000764       _Service_ProjectView$initializer$ 10013764     moc_KarlinSignatureDifferenceGraph.obj
 0002:00000768       _Service_DNAGraphPack$initializer$ 10013768     moc_KarlinSignatureDifferenceGraph.obj
 0002:0000076c       _Service_DNAExport$initializer$ 1001376c     moc_KarlinSignatureDifferenceGraph.obj
 0002:00000770       _Service_TestRunner$initializer$ 10013770     moc_KarlinSignatureDifferenceGraph.obj
 0002:00000774       _Service_ScriptRegistry$initializer$ 10013774     moc_KarlinSignatureDifferenceGraph.obj
 0002:00000778       _Service_ExternalToolSupport$initializer$ 10013778     moc_KarlinSignatureDifferenceGraph.obj
 0002:0000077c       _Service_GUITesting$initializer$ 1001377c     moc_KarlinSignatureDifferenceGraph.obj
 0002:00000780       _Service_WorkflowDesigner$initializer$ 10013780     moc_KarlinSignatureDifferenceGraph.obj
 0002:00000784       _Service_QueryDesigner$initializer$ 10013784     moc_KarlinSignatureDifferenceGraph.obj
 0002:00000788       _Service_MinCoreServiceId$initializer$ 10013788     moc_KarlinSignatureDifferenceGraph.obj
 0002:0000078c       _Service_MaxCoreServiceId$initializer$ 1001378c     moc_KarlinSignatureDifferenceGraph.obj
 0002:00000790       _algoLog$initializer$      10013790     moc_KarlinSignatureDifferenceGraph.obj
 0002:00000794       _cmdLog$initializer$       10013794     moc_KarlinSignatureDifferenceGraph.obj
 0002:00000798       _coreLog$initializer$      10013798     moc_KarlinSignatureDifferenceGraph.obj
 0002:0000079c       _ioLog$initializer$        1001379c     moc_KarlinSignatureDifferenceGraph.obj
 0002:000007a0       _perfLog$initializer$      100137a0     moc_KarlinSignatureDifferenceGraph.obj
 0002:000007a4       _scriptLog$initializer$    100137a4     moc_KarlinSignatureDifferenceGraph.obj
 0002:000007a8       _taskLog$initializer$      100137a8     moc_KarlinSignatureDifferenceGraph.obj
 0002:000007ac       _uiLog$initializer$        100137ac     moc_KarlinSignatureDifferenceGraph.obj
 0002:000007b0       _userActLog$initializer$   100137b0     moc_KarlinSignatureDifferenceGraph.obj
 0002:000007b4       ?staticMetaObject$initializer$@KarlinGraphFactory@U2@@2P6AXXZA 100137b4     moc_KarlinSignatureDifferenceGraph.obj
 0002:000007b8       _dummy$initializer$        100137b8     qrc_dna_graphpack.obj
 0002:000007c4       _pcinit                    100137c4     MSVCRT:crtdll.obj
 0002:000007c8       _pinit                     100137c8     MSVCRT:atonexit.obj
 0002:00000e1c       _FLOAT_MIN                 10013e1c     KarlinSignatureDifferenceGraph.obj
 0002:00000eb0       _qt_meta_stringdata_U2__BaseContentGraphFactory 10013eb0     moc_BaseContentGraph.obj
 0002:00000edc       _qt_meta_data_U2__BaseContentGraphFactory 10013edc     moc_BaseContentGraph.obj
 0002:00000f18       _qt_meta_stringdata_U2__CumulativeSkewGraphFactory 10013f18     moc_CumulativeSkew.obj
 0002:00000f48       _qt_meta_data_U2__CumulativeSkewGraphFactory 10013f48     moc_CumulativeSkew.obj
 0002:00000f88       _qt_meta_stringdata_U2__DNAGraphPackPlugin 10013f88     moc_DNAGraphPackPlugin.obj
 0002:00000fb0       _qt_meta_data_U2__DNAGraphPackPlugin 10013fb0     moc_DNAGraphPackPlugin.obj
 0002:00000ff0       _qt_meta_stringdata_U2__DNAGraphPackViewContext 10013ff0     moc_DNAGraphPackPlugin.obj
 0002:00001078       _qt_meta_data_U2__DNAGraphPackViewContext 10014078     moc_DNAGraphPackPlugin.obj
 0002:000010d4       _qt_meta_stringdata_U2__DeviationGraphFactory 100140d4     moc_DeviationGraph.obj
 0002:00001100       _qt_meta_data_U2__DeviationGraphFactory 10014100     moc_DeviationGraph.obj
 0002:0000113c       _qt_meta_stringdata_U2__EntropyGraphFactory 1001413c     moc_EntropyAlgorithm.obj
 0002:00001164       _qt_meta_data_U2__EntropyGraphFactory 10014164     moc_EntropyAlgorithm.obj
 0002:000011a0       _qt_meta_stringdata_U2__GCFramePlotFactory 100141a0     moc_GCFramePlot.obj
 0002:000011c8       _qt_meta_data_U2__GCFramePlotFactory 100141c8     moc_GCFramePlot.obj
 0002:00001204       _qt_meta_stringdata_U2__KarlinGraphFactory 10014204     moc_KarlinSignatureDifferenceGraph.obj
 0002:0000122c       _qt_meta_data_U2__KarlinGraphFactory 1001422c     moc_KarlinSignatureDifferenceGraph.obj
 0002:00001268       _qt_resource_data          10014268     qrc_dna_graphpack.obj
 0002:00001568       _qt_resource_name          10014568     qrc_dna_graphpack.obj
 0002:000015b4       _qt_resource_struct        100145b4     qrc_dna_graphpack.obj
 0002:000015f0       _Int32ToUInt32             100145f0     MSVCRT:ftol3.obj
 0002:00001600       _MantissaMask              10014600     MSVCRT:ftol3.obj
 0002:00001608       _IntegerBit                10014608     MSVCRT:ftol3.obj
 0002:00001610       _SignBit64                 10014610     MSVCRT:ftol3.obj
 0002:00001618       _MinFP64                   10014618     MSVCRT:ftol3.obj
 0002:00001620       _MinInt64                  10014620     MSVCRT:ftol3.obj
 0002:00001628       _MaxInt64                  10014628     MSVCRT:ftol3.obj
 0002:00001630       _MaxUInt64                 10014630     MSVCRT:ftol3.obj
 0002:00001638       _MaxFP32                   10014638     MSVCRT:ftol3.obj
 0002:00001640       _MinFP32                   10014640     MSVCRT:ftol3.obj
 0002:00001648       _MinSubInexact             10014648     MSVCRT:ftol3.obj
 0002:00001650       _FpExcptTable              10014650     MSVCRT:ftol3.obj
 0002:00001660       _i1075                     10014660     MSVCRT:ftol3.obj
 0002:00001664       _i1087                     10014664     MSVCRT:ftol3.obj
 0002:00001668       _x0800                     10014668     MSVCRT:ftol3.obj
 0002:0000166c       _x17FF                     1001466c     MSVCRT:ftol3.obj
 0002:00001670       _CWMask                    10014670     MSVCRT:ftol3.obj
 0002:00001680       _GS_ExceptionPointers      10014680     MSVCRT:gs_report.obj
 0002:00002320       __catchsym$?_Copy@?$basic_string@DU?$char_traits@D@std@@V?$allocator@D@2@@std@@QAEXII@Z$5 10015320     BaseContentGraph.obj
 0002:00002330       __catchsym$?_Copy@?$basic_string@DU?$char_traits@D@std@@V?$allocator@D@2@@std@@QAEXII@Z$4 10015330     BaseContentGraph.obj
 0002:00002340       __unwindtable$?_Copy@?$basic_string@DU?$char_traits@D@std@@V?$allocator@D@2@@std@@QAEXII@Z 10015340     BaseContentGraph.obj
 0002:00002360       __ehfuncinfo$?_Copy@?$basic_string@DU?$char_traits@D@std@@V?$allocator@D@2@@std@@QAEXII@Z 10015360     BaseContentGraph.obj
 0002:00002384       __tryblocktable$?_Copy@?$basic_string@DU?$char_traits@D@std@@V?$allocator@D@2@@std@@QAEXII@Z 10015384     BaseContentGraph.obj
 0002:000023ac       __unwindtable$??__EalgoLog@U2@@YAXXZ 100153ac     BaseContentGraph.obj
 0002:000023b4       __ehfuncinfo$??__EalgoLog@U2@@YAXXZ 100153b4     BaseContentGraph.obj
 0002:000023d8       __unwindtable$??__EcmdLog@U2@@YAXXZ 100153d8     BaseContentGraph.obj
 0002:000023e0       __ehfuncinfo$??__EcmdLog@U2@@YAXXZ 100153e0     BaseContentGraph.obj
 0002:00002404       __unwindtable$??__EcoreLog@U2@@YAXXZ 10015404     BaseContentGraph.obj
 0002:0000240c       __ehfuncinfo$??__EcoreLog@U2@@YAXXZ 1001540c     BaseContentGraph.obj
 0002:00002430       __unwindtable$??__EioLog@U2@@YAXXZ 10015430     BaseContentGraph.obj
 0002:00002438       __ehfuncinfo$??__EioLog@U2@@YAXXZ 10015438     BaseContentGraph.obj
 0002:0000245c       __unwindtable$??__EperfLog@U2@@YAXXZ 1001545c     BaseContentGraph.obj
 0002:00002464       __ehfuncinfo$??__EperfLog@U2@@YAXXZ 10015464     BaseContentGraph.obj
 0002:00002488       __unwindtable$??__EscriptLog@U2@@YAXXZ 10015488     BaseContentGraph.obj
 0002:00002490       __ehfuncinfo$??__EscriptLog@U2@@YAXXZ 10015490     BaseContentGraph.obj
 0002:000024b4       __unwindtable$??__EtaskLog@U2@@YAXXZ 100154b4     BaseContentGraph.obj
 0002:000024bc       __ehfuncinfo$??__EtaskLog@U2@@YAXXZ 100154bc     BaseContentGraph.obj
 0002:000024e0       __unwindtable$??__EuiLog@U2@@YAXXZ 100154e0     BaseContentGraph.obj
 0002:000024e8       __ehfuncinfo$??__EuiLog@U2@@YAXXZ 100154e8     BaseContentGraph.obj
 0002:0000250c       __unwindtable$??__EuserActLog@U2@@YAXXZ 1001550c     BaseContentGraph.obj
 0002:00002514       __ehfuncinfo$??__EuserActLog@U2@@YAXXZ 10015514     BaseContentGraph.obj
 0002:00002538       __catchsym$?reallocData@?$QVector@M@@AAEXHHV?$QFlags@W4AllocationOption@QArrayData@@@@@Z$5 10015538     BaseContentGraph.obj
 0002:00002548       __catchsym$?reallocData@?$QVector@M@@AAEXHHV?$QFlags@W4AllocationOption@QArrayData@@@@@Z$4 10015548     BaseContentGraph.obj
 0002:00002558       __unwindtable$?reallocData@?$QVector@M@@AAEXHHV?$QFlags@W4AllocationOption@QArrayData@@@@@Z 10015558     BaseContentGraph.obj
 0002:00002578       __ehfuncinfo$?reallocData@?$QVector@M@@AAEXHHV?$QFlags@W4AllocationOption@QArrayData@@@@@Z 10015578     BaseContentGraph.obj
 0002:0000259c       __tryblocktable$?reallocData@?$QVector@M@@AAEXHHV?$QFlags@W4AllocationOption@QArrayData@@@@@Z 1001559c     BaseContentGraph.obj
 0002:000025c4       __catchsym$?append@?$QList@V?$QSharedPointer@VGSequenceGraphData@U2@@@@@@QAEXABV?$QSharedPointer@VGSequenceGraphData@U2@@@@@Z$9 100155c4     BaseContentGraph.obj
 0002:000025d4       __catchsym$?append@?$QList@V?$QSharedPointer@VGSequenceGraphData@U2@@@@@@QAEXABV?$QSharedPointer@VGSequenceGraphData@U2@@@@@Z$8 100155d4     BaseContentGraph.obj
 0002:000025e4       __ehfuncinfo$?append@?$QList@V?$QSharedPointer@VGSequenceGraphData@U2@@@@@@QAEXABV?$QSharedPointer@VGSequenceGraphData@U2@@@@@Z 100155e4     BaseContentGraph.obj
 0002:00002608       __tryblocktable$?append@?$QList@V?$QSharedPointer@VGSequenceGraphData@U2@@@@@@QAEXABV?$QSharedPointer@VGSequenceGraphData@U2@@@@@Z 10015608     BaseContentGraph.obj
 0002:00002630       __unwindtable$?append@?$QList@V?$QSharedPointer@VGSequenceGraphData@U2@@@@@@QAEXABV?$QSharedPointer@VGSequenceGraphData@U2@@@@@Z 10015630     BaseContentGraph.obj
 0002:00002660       __catchsym$?detach_helper_grow@?$QList@V?$QSharedPointer@VGSequenceGraphData@U2@@@@@@AAEPAUNode@1@HH@Z$5 10015660     BaseContentGraph.obj
 0002:00002670       __catchsym$?detach_helper_grow@?$QList@V?$QSharedPointer@VGSequenceGraphData@U2@@@@@@AAEPAUNode@1@HH@Z$4 10015670     BaseContentGraph.obj
 0002:00002680       __unwindtable$?detach_helper_grow@?$QList@V?$QSharedPointer@VGSequenceGraphData@U2@@@@@@AAEPAUNode@1@HH@Z 10015680     BaseContentGraph.obj
 0002:000026a0       __ehfuncinfo$?detach_helper_grow@?$QList@V?$QSharedPointer@VGSequenceGraphData@U2@@@@@@AAEPAUNode@1@HH@Z 100156a0     BaseContentGraph.obj
 0002:000026c4       __tryblocktable$?detach_helper_grow@?$QList@V?$QSharedPointer@VGSequenceGraphData@U2@@@@@@AAEPAUNode@1@HH@Z 100156c4     BaseContentGraph.obj
 0002:000026ec       __catchsym$?node_copy@?$QList@V?$QSharedPointer@VGSequenceGraphData@U2@@@@@@AAEXPAUNode@1@00@Z$6 100156ec     BaseContentGraph.obj
 0002:000026fc       __tryblocktable$?node_copy@?$QList@V?$QSharedPointer@VGSequenceGraphData@U2@@@@@@AAEXPAUNode@1@00@Z 100156fc     BaseContentGraph.obj
 0002:00002710       __unwindtable$?node_copy@?$QList@V?$QSharedPointer@VGSequenceGraphData@U2@@@@@@AAEXPAUNode@1@00@Z 10015710     BaseContentGraph.obj
 0002:00002730       __ehfuncinfo$?node_copy@?$QList@V?$QSharedPointer@VGSequenceGraphData@U2@@@@@@AAEXPAUNode@1@00@Z 10015730     BaseContentGraph.obj
 0002:00002754       __unwindtable$??0BaseContentGraphFactory@U2@@QAE@W4GType@01@PAVQObject@@@Z 10015754     BaseContentGraph.obj
 0002:00002774       __ehfuncinfo$??0BaseContentGraphFactory@U2@@QAE@W4GType@01@PAVQObject@@@Z 10015774     BaseContentGraph.obj
 0002:00002798       __ehfuncinfo$?createGraphs@BaseContentGraphFactory@U2@@UAE?AV?$QList@V?$QSharedPointer@VGSequenceGraphData@U2@@@@@@PAVGSequenceGraphView@2@@Z 10015798     BaseContentGraph.obj
 0002:000027bc       __unwindtable$?createGraphs@BaseContentGraphFactory@U2@@UAE?AV?$QList@V?$QSharedPointer@VGSequenceGraphData@U2@@@@@@PAVGSequenceGraphView@2@@Z 100157bc     BaseContentGraph.obj
 0002:000027e4       __unwindtable$??1BaseContentGraphFactory@U2@@UAE@XZ 100157e4     BaseContentGraph.obj
 0002:000027ec       __ehfuncinfo$??1BaseContentGraphFactory@U2@@UAE@XZ 100157ec     BaseContentGraph.obj
 0002:00002810       __unwindtable$??_GBaseContentGraphFactory@U2@@UAEPAXI@Z 10015810     BaseContentGraph.obj
 0002:00002818       __ehfuncinfo$??_GBaseContentGraphFactory@U2@@UAEPAXI@Z 10015818     BaseContentGraph.obj
 0002:0000283c       __unwindtable$??0BaseContentGraphAlgorithm@U2@@QAE@ABVQBitArray@@@Z 1001583c     BaseContentGraph.obj
 0002:00002844       __ehfuncinfo$??0BaseContentGraphAlgorithm@U2@@QAE@ABVQBitArray@@@Z 10015844     BaseContentGraph.obj
 0002:00002868       __ehfuncinfo$?calculate@BaseContentGraphAlgorithm@U2@@UAEXAAV?$QVector@M@@PAVU2SequenceObject@2@ABVU2Region@2@PBVGSequenceGraphWindowData@2@AAVU2OpStatus@2@@Z 10015868     BaseContentGraph.obj
 0002:0000288c       __unwindtable$?calculate@BaseContentGraphAlgorithm@U2@@UAEXAAV?$QVector@M@@PAVU2SequenceObject@2@ABVU2Region@2@PBVGSequenceGraphWindowData@2@AAVU2OpStatus@2@@Z 1001588c     BaseContentGraph.obj
 0002:000028fc       __unwindtable$??1BaseContentGraphAlgorithm@U2@@UAE@XZ 100158fc     BaseContentGraph.obj
 0002:00002904       __ehfuncinfo$??1BaseContentGraphAlgorithm@U2@@UAE@XZ 10015904     BaseContentGraph.obj
 0002:00002928       __unwindtable$??_GBaseContentGraphAlgorithm@U2@@UAEPAXI@Z 10015928     BaseContentGraph.obj
 0002:00002930       __ehfuncinfo$??_GBaseContentGraphAlgorithm@U2@@UAEPAXI@Z 10015930     BaseContentGraph.obj
 0002:00002954       __unwindtable$??__EalgoLog@U2@@YAXXZ 10015954     CumulativeSkew.obj
 0002:0000295c       __ehfuncinfo$??__EalgoLog@U2@@YAXXZ 1001595c     CumulativeSkew.obj
 0002:00002980       __unwindtable$??__EcmdLog@U2@@YAXXZ 10015980     CumulativeSkew.obj
 0002:00002988       __ehfuncinfo$??__EcmdLog@U2@@YAXXZ 10015988     CumulativeSkew.obj
 0002:000029ac       __unwindtable$??__EcoreLog@U2@@YAXXZ 100159ac     CumulativeSkew.obj
 0002:000029b4       __ehfuncinfo$??__EcoreLog@U2@@YAXXZ 100159b4     CumulativeSkew.obj
 0002:000029d8       __unwindtable$??__EioLog@U2@@YAXXZ 100159d8     CumulativeSkew.obj
 0002:000029e0       __ehfuncinfo$??__EioLog@U2@@YAXXZ 100159e0     CumulativeSkew.obj
 0002:00002a04       __unwindtable$??__EperfLog@U2@@YAXXZ 10015a04     CumulativeSkew.obj
 0002:00002a0c       __ehfuncinfo$??__EperfLog@U2@@YAXXZ 10015a0c     CumulativeSkew.obj
 0002:00002a30       __unwindtable$??__EscriptLog@U2@@YAXXZ 10015a30     CumulativeSkew.obj
 0002:00002a38       __ehfuncinfo$??__EscriptLog@U2@@YAXXZ 10015a38     CumulativeSkew.obj
 0002:00002a5c       __unwindtable$??__EtaskLog@U2@@YAXXZ 10015a5c     CumulativeSkew.obj
 0002:00002a64       __ehfuncinfo$??__EtaskLog@U2@@YAXXZ 10015a64     CumulativeSkew.obj
 0002:00002a88       __unwindtable$??__EuiLog@U2@@YAXXZ 10015a88     CumulativeSkew.obj
 0002:00002a90       __ehfuncinfo$??__EuiLog@U2@@YAXXZ 10015a90     CumulativeSkew.obj
 0002:00002ab4       __unwindtable$??__EuserActLog@U2@@YAXXZ 10015ab4     CumulativeSkew.obj
 0002:00002abc       __ehfuncinfo$??__EuserActLog@U2@@YAXXZ 10015abc     CumulativeSkew.obj
 0002:00002ae0       __unwindtable$??0CumulativeSkewGraphFactory@U2@@QAE@W4GCumulativeSkewType@01@PAVQObject@@@Z 10015ae0     CumulativeSkew.obj
 0002:00002af8       __ehfuncinfo$??0CumulativeSkewGraphFactory@U2@@QAE@W4GCumulativeSkewType@01@PAVQObject@@@Z 10015af8     CumulativeSkew.obj
 0002:00002b1c       __unwindtable$?createGraphs@CumulativeSkewGraphFactory@U2@@UAE?AV?$QList@V?$QSharedPointer@VGSequenceGraphData@U2@@@@@@PAVGSequenceGraphView@2@@Z 10015b1c     CumulativeSkew.obj
 0002:00002b3c       __ehfuncinfo$?createGraphs@CumulativeSkewGraphFactory@U2@@UAE?AV?$QList@V?$QSharedPointer@VGSequenceGraphData@U2@@@@@@PAVGSequenceGraphView@2@@Z 10015b3c     CumulativeSkew.obj
 0002:00002b60       __unwindtable$??__EalgoLog@U2@@YAXXZ 10015b60     DNAGraphPackPlugin.obj
 0002:00002b68       __ehfuncinfo$??__EalgoLog@U2@@YAXXZ 10015b68     DNAGraphPackPlugin.obj
 0002:00002b8c       __unwindtable$??__EcmdLog@U2@@YAXXZ 10015b8c     DNAGraphPackPlugin.obj
 0002:00002b94       __ehfuncinfo$??__EcmdLog@U2@@YAXXZ 10015b94     DNAGraphPackPlugin.obj
 0002:00002bb8       __unwindtable$??__EcoreLog@U2@@YAXXZ 10015bb8     DNAGraphPackPlugin.obj
 0002:00002bc0       __ehfuncinfo$??__EcoreLog@U2@@YAXXZ 10015bc0     DNAGraphPackPlugin.obj
 0002:00002be4       __unwindtable$??__EioLog@U2@@YAXXZ 10015be4     DNAGraphPackPlugin.obj
 0002:00002bec       __ehfuncinfo$??__EioLog@U2@@YAXXZ 10015bec     DNAGraphPackPlugin.obj
 0002:00002c10       __unwindtable$??__EperfLog@U2@@YAXXZ 10015c10     DNAGraphPackPlugin.obj
 0002:00002c18       __ehfuncinfo$??__EperfLog@U2@@YAXXZ 10015c18     DNAGraphPackPlugin.obj
 0002:00002c3c       __unwindtable$??__EscriptLog@U2@@YAXXZ 10015c3c     DNAGraphPackPlugin.obj
 0002:00002c44       __ehfuncinfo$??__EscriptLog@U2@@YAXXZ 10015c44     DNAGraphPackPlugin.obj
 0002:00002c68       __unwindtable$??__EtaskLog@U2@@YAXXZ 10015c68     DNAGraphPackPlugin.obj
 0002:00002c70       __ehfuncinfo$??__EtaskLog@U2@@YAXXZ 10015c70     DNAGraphPackPlugin.obj
 0002:00002c94       __unwindtable$??__EuiLog@U2@@YAXXZ 10015c94     DNAGraphPackPlugin.obj
 0002:00002c9c       __ehfuncinfo$??__EuiLog@U2@@YAXXZ 10015c9c     DNAGraphPackPlugin.obj
 0002:00002cc0       __unwindtable$??__EuserActLog@U2@@YAXXZ 10015cc0     DNAGraphPackPlugin.obj
 0002:00002cc8       __ehfuncinfo$??__EuserActLog@U2@@YAXXZ 10015cc8     DNAGraphPackPlugin.obj
 0002:00002cec       __ehfuncinfo$??0DNAGraphPackPlugin@U2@@QAE@XZ 10015cec     DNAGraphPackPlugin.obj
 0002:00002d10       __unwindtable$??0DNAGraphPackPlugin@U2@@QAE@XZ 10015d10     DNAGraphPackPlugin.obj
 0002:00002d40       __ehfuncinfo$??0DNAGraphPackViewContext@U2@@QAE@PAVQObject@@@Z 10015d40     DNAGraphPackPlugin.obj
 0002:00002d64       __unwindtable$??0DNAGraphPackViewContext@U2@@QAE@PAVQObject@@@Z 10015d64     DNAGraphPackPlugin.obj
 0002:00002dbc       __catchsym$??0?$QList@PAVGSequenceGraphFactory@U2@@@@QAE@ABV0@@Z$2 10015dbc     DNAGraphPackPlugin.obj
 0002:00002dcc       __unwindtable$??0?$QList@PAVGSequenceGraphFactory@U2@@@@QAE@ABV0@@Z 10015dcc     DNAGraphPackPlugin.obj
 0002:00002ddc       __tryblocktable$??0?$QList@PAVGSequenceGraphFactory@U2@@@@QAE@ABV0@@Z 10015ddc     DNAGraphPackPlugin.obj
 0002:00002df0       __ehfuncinfo$??0?$QList@PAVGSequenceGraphFactory@U2@@@@QAE@ABV0@@Z 10015df0     DNAGraphPackPlugin.obj
 0002:00002e14       __catchsym$?append@?$QList@PAVGSequenceGraphFactory@U2@@@@QAEXABQAVGSequenceGraphFactory@U2@@@Z$6 10015e14     DNAGraphPackPlugin.obj
 0002:00002e24       __tryblocktable$?append@?$QList@PAVGSequenceGraphFactory@U2@@@@QAEXABQAVGSequenceGraphFactory@U2@@@Z 10015e24     DNAGraphPackPlugin.obj
 0002:00002e38       __ehfuncinfo$?append@?$QList@PAVGSequenceGraphFactory@U2@@@@QAEXABQAVGSequenceGraphFactory@U2@@@Z 10015e38     DNAGraphPackPlugin.obj
 0002:00002e5c       __unwindtable$?append@?$QList@PAVGSequenceGraphFactory@U2@@@@QAEXABQAVGSequenceGraphFactory@U2@@@Z 10015e5c     DNAGraphPackPlugin.obj
 0002:00002e8c       __catchsym$?detach_helper_grow@?$QList@PAVGSequenceGraphFactory@U2@@@@AAEPAUNode@1@HH@Z$5 10015e8c     DNAGraphPackPlugin.obj
 0002:00002e9c       __catchsym$?detach_helper_grow@?$QList@PAVGSequenceGraphFactory@U2@@@@AAEPAUNode@1@HH@Z$4 10015e9c     DNAGraphPackPlugin.obj
 0002:00002eac       __unwindtable$?detach_helper_grow@?$QList@PAVGSequenceGraphFactory@U2@@@@AAEPAUNode@1@HH@Z 10015eac     DNAGraphPackPlugin.obj
 0002:00002ecc       __ehfuncinfo$?detach_helper_grow@?$QList@PAVGSequenceGraphFactory@U2@@@@AAEPAUNode@1@HH@Z 10015ecc     DNAGraphPackPlugin.obj
 0002:00002ef0       __tryblocktable$?detach_helper_grow@?$QList@PAVGSequenceGraphFactory@U2@@@@AAEPAUNode@1@HH@Z 10015ef0     DNAGraphPackPlugin.obj
 0002:00002f18       __unwindtable$?initViewContext@DNAGraphPackViewContext@U2@@EAEXPAVGObjectView@2@@Z 10015f18     DNAGraphPackPlugin.obj
 0002:00002f30       __ehfuncinfo$?initViewContext@DNAGraphPackViewContext@U2@@EAEXPAVGObjectView@2@@Z 10015f30     DNAGraphPackPlugin.obj
 0002:00002f54       __unwindtable$?sl_sequenceWidgetAdded@DNAGraphPackViewContext@U2@@AAEXPAVADVSequenceWidget@2@@Z 10015f54     DNAGraphPackPlugin.obj
 0002:00002f64       __ehfuncinfo$?sl_sequenceWidgetAdded@DNAGraphPackViewContext@U2@@AAEXPAVADVSequenceWidget@2@@Z 10015f64     DNAGraphPackPlugin.obj
 0002:00002f88       __unwindtable$??1DNAGraphPackViewContext@U2@@UAE@XZ 10015f88     DNAGraphPackPlugin.obj
 0002:00002f90       __ehfuncinfo$??1DNAGraphPackViewContext@U2@@UAE@XZ 10015f90     DNAGraphPackPlugin.obj
 0002:00002fb4       __unwindtable$??_GDNAGraphPackViewContext@U2@@UAEPAXI@Z 10015fb4     DNAGraphPackPlugin.obj
 0002:00002fbc       __ehfuncinfo$??_GDNAGraphPackViewContext@U2@@UAEPAXI@Z 10015fbc     DNAGraphPackPlugin.obj
 0002:00002fe0       __catchsym$??0?$QList@PAVADVSequenceWidget@U2@@@@QAE@ABV0@@Z$2 10015fe0     DNAGraphPackPlugin.obj
 0002:00002ff0       __unwindtable$??0?$QList@PAVADVSequenceWidget@U2@@@@QAE@ABV0@@Z 10015ff0     DNAGraphPackPlugin.obj
 0002:00003000       __tryblocktable$??0?$QList@PAVADVSequenceWidget@U2@@@@QAE@ABV0@@Z 10016000     DNAGraphPackPlugin.obj
 0002:00003014       __ehfuncinfo$??0?$QList@PAVADVSequenceWidget@U2@@@@QAE@ABV0@@Z 10016014     DNAGraphPackPlugin.obj
 0002:00003038       __unwindtable$??__EalgoLog@U2@@YAXXZ 10016038     DeviationGraph.obj
 0002:00003040       __ehfuncinfo$??__EalgoLog@U2@@YAXXZ 10016040     DeviationGraph.obj
 0002:00003064       __unwindtable$??__EcmdLog@U2@@YAXXZ 10016064     DeviationGraph.obj
 0002:0000306c       __ehfuncinfo$??__EcmdLog@U2@@YAXXZ 1001606c     DeviationGraph.obj
 0002:00003090       __unwindtable$??__EcoreLog@U2@@YAXXZ 10016090     DeviationGraph.obj
 0002:00003098       __ehfuncinfo$??__EcoreLog@U2@@YAXXZ 10016098     DeviationGraph.obj
 0002:000030bc       __unwindtable$??__EioLog@U2@@YAXXZ 100160bc     DeviationGraph.obj
 0002:000030c4       __ehfuncinfo$??__EioLog@U2@@YAXXZ 100160c4     DeviationGraph.obj
 0002:000030e8       __unwindtable$??__EperfLog@U2@@YAXXZ 100160e8     DeviationGraph.obj
 0002:000030f0       __ehfuncinfo$??__EperfLog@U2@@YAXXZ 100160f0     DeviationGraph.obj
 0002:00003114       __unwindtable$??__EscriptLog@U2@@YAXXZ 10016114     DeviationGraph.obj
 0002:0000311c       __ehfuncinfo$??__EscriptLog@U2@@YAXXZ 1001611c     DeviationGraph.obj
 0002:00003140       __unwindtable$??__EtaskLog@U2@@YAXXZ 10016140     DeviationGraph.obj
 0002:00003148       __ehfuncinfo$??__EtaskLog@U2@@YAXXZ 10016148     DeviationGraph.obj
 0002:0000316c       __unwindtable$??__EuiLog@U2@@YAXXZ 1001616c     DeviationGraph.obj
 0002:00003174       __ehfuncinfo$??__EuiLog@U2@@YAXXZ 10016174     DeviationGraph.obj
 0002:00003198       __unwindtable$??__EuserActLog@U2@@YAXXZ 10016198     DeviationGraph.obj
 0002:000031a0       __ehfuncinfo$??__EuserActLog@U2@@YAXXZ 100161a0     DeviationGraph.obj
 0002:000031c4       __unwindtable$??0DeviationGraphFactory@U2@@QAE@W4GDeviationType@01@PAVQObject@@@Z 100161c4     DeviationGraph.obj
 0002:000031dc       __ehfuncinfo$??0DeviationGraphFactory@U2@@QAE@W4GDeviationType@01@PAVQObject@@@Z 100161dc     DeviationGraph.obj
 0002:00003200       __unwindtable$?createGraphs@DeviationGraphFactory@U2@@UAE?AV?$QList@V?$QSharedPointer@VGSequenceGraphData@U2@@@@@@PAVGSequenceGraphView@2@@Z 10016200     DeviationGraph.obj
 0002:00003220       __ehfuncinfo$?createGraphs@DeviationGraphFactory@U2@@UAE?AV?$QList@V?$QSharedPointer@VGSequenceGraphData@U2@@@@@@PAVGSequenceGraphView@2@@Z 10016220     DeviationGraph.obj
 0002:00003244       __unwindtable$?sequenceStrategyWithMemorize@DeviationGraphAlgorithm@U2@@AAEXAAV?$QVector@M@@ABVQByteArray@@ABVU2Region@2@PBVGSequenceGraphWindowData@2@AAVU2OpStatus@2@@Z 10016244     DeviationGraph.obj
 0002:00003254       __ehfuncinfo$?sequenceStrategyWithMemorize@DeviationGraphAlgorithm@U2@@AAEXAAV?$QVector@M@@ABVQByteArray@@ABVU2Region@2@PBVGSequenceGraphWindowData@2@AAVU2OpStatus@2@@Z 10016254     DeviationGraph.obj
 0002:00003278       __unwindtable$??0?$RollingArray@H@U2@@QAE@H@Z 10016278     DeviationGraph.obj
 0002:00003280       __ehfuncinfo$??0?$RollingArray@H@U2@@QAE@H@Z 10016280     DeviationGraph.obj
 0002:000032a4       __catchsym$?reallocData@?$QVector@H@@AAEXHHV?$QFlags@W4AllocationOption@QArrayData@@@@@Z$5 100162a4     DeviationGraph.obj
 0002:000032b4       __catchsym$?reallocData@?$QVector@H@@AAEXHHV?$QFlags@W4AllocationOption@QArrayData@@@@@Z$4 100162b4     DeviationGraph.obj
 0002:000032c4       __unwindtable$?reallocData@?$QVector@H@@AAEXHHV?$QFlags@W4AllocationOption@QArrayData@@@@@Z 100162c4     DeviationGraph.obj
 0002:000032e4       __ehfuncinfo$?reallocData@?$QVector@H@@AAEXHHV?$QFlags@W4AllocationOption@QArrayData@@@@@Z 100162e4     DeviationGraph.obj
 0002:00003308       __tryblocktable$?reallocData@?$QVector@H@@AAEXHHV?$QFlags@W4AllocationOption@QArrayData@@@@@Z 10016308     DeviationGraph.obj
 0002:00003330       __unwindtable$??__EalgoLog@U2@@YAXXZ 10016330     EntropyAlgorithm.obj
 0002:00003338       __ehfuncinfo$??__EalgoLog@U2@@YAXXZ 10016338     EntropyAlgorithm.obj
 0002:0000335c       __unwindtable$??__EcmdLog@U2@@YAXXZ 1001635c     EntropyAlgorithm.obj
 0002:00003364       __ehfuncinfo$??__EcmdLog@U2@@YAXXZ 10016364     EntropyAlgorithm.obj
 0002:00003388       __unwindtable$??__EcoreLog@U2@@YAXXZ 10016388     EntropyAlgorithm.obj
 0002:00003390       __ehfuncinfo$??__EcoreLog@U2@@YAXXZ 10016390     EntropyAlgorithm.obj
 0002:000033b4       __unwindtable$??__EioLog@U2@@YAXXZ 100163b4     EntropyAlgorithm.obj
 0002:000033bc       __ehfuncinfo$??__EioLog@U2@@YAXXZ 100163bc     EntropyAlgorithm.obj
 0002:000033e0       __unwindtable$??__EperfLog@U2@@YAXXZ 100163e0     EntropyAlgorithm.obj
 0002:000033e8       __ehfuncinfo$??__EperfLog@U2@@YAXXZ 100163e8     EntropyAlgorithm.obj
 0002:0000340c       __unwindtable$??__EscriptLog@U2@@YAXXZ 1001640c     EntropyAlgorithm.obj
 0002:00003414       __ehfuncinfo$??__EscriptLog@U2@@YAXXZ 10016414     EntropyAlgorithm.obj
 0002:00003438       __unwindtable$??__EtaskLog@U2@@YAXXZ 10016438     EntropyAlgorithm.obj
 0002:00003440       __ehfuncinfo$??__EtaskLog@U2@@YAXXZ 10016440     EntropyAlgorithm.obj
 0002:00003464       __unwindtable$??__EuiLog@U2@@YAXXZ 10016464     EntropyAlgorithm.obj
 0002:0000346c       __ehfuncinfo$??__EuiLog@U2@@YAXXZ 1001646c     EntropyAlgorithm.obj
 0002:00003490       __unwindtable$??__EuserActLog@U2@@YAXXZ 10016490     EntropyAlgorithm.obj
 0002:00003498       __ehfuncinfo$??__EuserActLog@U2@@YAXXZ 10016498     EntropyAlgorithm.obj
 0002:000034bc       __unwindtable$??0EntropyGraphFactory@U2@@QAE@PAVQObject@@@Z 100164bc     EntropyAlgorithm.obj
 0002:000034d4       __ehfuncinfo$??0EntropyGraphFactory@U2@@QAE@PAVQObject@@@Z 100164d4     EntropyAlgorithm.obj
 0002:000034f8       __unwindtable$?createGraphs@EntropyGraphFactory@U2@@UAE?AV?$QList@V?$QSharedPointer@VGSequenceGraphData@U2@@@@@@PAVGSequenceGraphView@2@@Z 100164f8     EntropyAlgorithm.obj
 0002:00003518       __ehfuncinfo$?createGraphs@EntropyGraphFactory@U2@@UAE?AV?$QList@V?$QSharedPointer@VGSequenceGraphData@U2@@@@@@PAVGSequenceGraphView@2@@Z 10016518     EntropyAlgorithm.obj
 0002:0000353c       __unwindtable$?calculate@EntropyGraphAlgorithm@U2@@UAEXAAV?$QVector@M@@PAVU2SequenceObject@2@ABVU2Region@2@PBVGSequenceGraphWindowData@2@AAVU2OpStatus@2@@Z 1001653c     EntropyAlgorithm.obj
 0002:00003554       __ehfuncinfo$?calculate@EntropyGraphAlgorithm@U2@@UAEXAAV?$QVector@M@@PAVU2SequenceObject@2@ABVU2Region@2@PBVGSequenceGraphWindowData@2@AAVU2OpStatus@2@@Z 10016554     EntropyAlgorithm.obj
 0002:00003578       __unwindtable$??__EalgoLog@U2@@YAXXZ 10016578     GCFramePlot.obj
 0002:00003580       __ehfuncinfo$??__EalgoLog@U2@@YAXXZ 10016580     GCFramePlot.obj
 0002:000035a4       __unwindtable$??__EcmdLog@U2@@YAXXZ 100165a4     GCFramePlot.obj
 0002:000035ac       __ehfuncinfo$??__EcmdLog@U2@@YAXXZ 100165ac     GCFramePlot.obj
 0002:000035d0       __unwindtable$??__EcoreLog@U2@@YAXXZ 100165d0     GCFramePlot.obj
 0002:000035d8       __ehfuncinfo$??__EcoreLog@U2@@YAXXZ 100165d8     GCFramePlot.obj
 0002:000035fc       __unwindtable$??__EioLog@U2@@YAXXZ 100165fc     GCFramePlot.obj
 0002:00003604       __ehfuncinfo$??__EioLog@U2@@YAXXZ 10016604     GCFramePlot.obj
 0002:00003628       __unwindtable$??__EperfLog@U2@@YAXXZ 10016628     GCFramePlot.obj
 0002:00003630       __ehfuncinfo$??__EperfLog@U2@@YAXXZ 10016630     GCFramePlot.obj
 0002:00003654       __unwindtable$??__EscriptLog@U2@@YAXXZ 10016654     GCFramePlot.obj
 0002:0000365c       __ehfuncinfo$??__EscriptLog@U2@@YAXXZ 1001665c     GCFramePlot.obj
 0002:00003680       __unwindtable$??__EtaskLog@U2@@YAXXZ 10016680     GCFramePlot.obj
 0002:00003688       __ehfuncinfo$??__EtaskLog@U2@@YAXXZ 10016688     GCFramePlot.obj
 0002:000036ac       __unwindtable$??__EuiLog@U2@@YAXXZ 100166ac     GCFramePlot.obj
 0002:000036b4       __ehfuncinfo$??__EuiLog@U2@@YAXXZ 100166b4     GCFramePlot.obj
 0002:000036d8       __unwindtable$??__EuserActLog@U2@@YAXXZ 100166d8     GCFramePlot.obj
 0002:000036e0       __ehfuncinfo$??__EuserActLog@U2@@YAXXZ 100166e0     GCFramePlot.obj
 0002:00003704       __unwindtable$??0GCFramePlotFactory@U2@@QAE@PAVQObject@@@Z 10016704     GCFramePlot.obj
 0002:0000371c       __ehfuncinfo$??0GCFramePlotFactory@U2@@QAE@PAVQObject@@@Z 1001671c     GCFramePlot.obj
 0002:00003740       __ehfuncinfo$?createGraphs@GCFramePlotFactory@U2@@UAE?AV?$QList@V?$QSharedPointer@VGSequenceGraphData@U2@@@@@@PAVGSequenceGraphView@2@@Z 10016740     GCFramePlot.obj
 0002:00003764       __unwindtable$?createGraphs@GCFramePlotFactory@U2@@UAE?AV?$QList@V?$QSharedPointer@VGSequenceGraphData@U2@@@@@@PAVGSequenceGraphView@2@@Z 10016764     GCFramePlot.obj
 0002:000037fc       __unwindtable$?getDrawer@GCFramePlotFactory@U2@@UAEPAVGSequenceGraphDrawer@2@PAVGSequenceGraphView@2@@Z 100167fc     GCFramePlot.obj
 0002:0000381c       __ehfuncinfo$?getDrawer@GCFramePlotFactory@U2@@UAEPAVGSequenceGraphDrawer@2@PAVGSequenceGraphView@2@@Z 1001681c     GCFramePlot.obj
 0002:00003840       __unwindtable$??0GCFramePlotAlgorithm@U2@@QAE@H@Z 10016840     GCFramePlot.obj
 0002:00003850       __ehfuncinfo$??0GCFramePlotAlgorithm@U2@@QAE@H@Z 10016850     GCFramePlot.obj
 0002:00003874       __unwindtable$??1GCFramePlotAlgorithm@U2@@UAE@XZ 10016874     GCFramePlot.obj
 0002:0000387c       __ehfuncinfo$??1GCFramePlotAlgorithm@U2@@UAE@XZ 1001687c     GCFramePlot.obj
 0002:000038a0       __unwindtable$??_GGCFramePlotAlgorithm@U2@@UAEPAXI@Z 100168a0     GCFramePlot.obj
 0002:000038a8       __ehfuncinfo$??_GGCFramePlotAlgorithm@U2@@UAEPAXI@Z 100168a8     GCFramePlot.obj
 0002:000038cc       __catchsym$?createNode@?$QMapData@VQString@@VQColor@@@@QAEPAU?$QMapNode@VQString@@VQColor@@@@ABVQString@@ABVQColor@@PAU2@_N@Z$6 100168cc     GCFramePlot.obj
 0002:000038dc       __tryblocktable$?createNode@?$QMapData@VQString@@VQColor@@@@QAEPAU?$QMapNode@VQString@@VQColor@@@@ABVQString@@ABVQColor@@PAU2@_N@Z 100168dc     GCFramePlot.obj
 0002:000038f0       __ehfuncinfo$?createNode@?$QMapData@VQString@@VQColor@@@@QAEPAU?$QMapNode@VQString@@VQColor@@@@ABVQString@@ABVQColor@@PAU2@_N@Z 100168f0     GCFramePlot.obj
 0002:00003914       __unwindtable$?createNode@?$QMapData@VQString@@VQColor@@@@QAEPAU?$QMapNode@VQString@@VQColor@@@@ABVQString@@ABVQColor@@PAU2@_N@Z 10016914     GCFramePlot.obj
 0002:0000393c       __unwindtable$??__EalgoLog@U2@@YAXXZ 1001693c     KarlinSignatureDifferenceGraph.obj
 0002:00003944       __ehfuncinfo$??__EalgoLog@U2@@YAXXZ 10016944     KarlinSignatureDifferenceGraph.obj
 0002:00003968       __unwindtable$??__EcmdLog@U2@@YAXXZ 10016968     KarlinSignatureDifferenceGraph.obj
 0002:00003970       __ehfuncinfo$??__EcmdLog@U2@@YAXXZ 10016970     KarlinSignatureDifferenceGraph.obj
 0002:00003994       __unwindtable$??__EcoreLog@U2@@YAXXZ 10016994     KarlinSignatureDifferenceGraph.obj
 0002:0000399c       __ehfuncinfo$??__EcoreLog@U2@@YAXXZ 1001699c     KarlinSignatureDifferenceGraph.obj
 0002:000039c0       __unwindtable$??__EioLog@U2@@YAXXZ 100169c0     KarlinSignatureDifferenceGraph.obj
 0002:000039c8       __ehfuncinfo$??__EioLog@U2@@YAXXZ 100169c8     KarlinSignatureDifferenceGraph.obj
 0002:000039ec       __unwindtable$??__EperfLog@U2@@YAXXZ 100169ec     KarlinSignatureDifferenceGraph.obj
 0002:000039f4       __ehfuncinfo$??__EperfLog@U2@@YAXXZ 100169f4     KarlinSignatureDifferenceGraph.obj
 0002:00003a18       __unwindtable$??__EscriptLog@U2@@YAXXZ 10016a18     KarlinSignatureDifferenceGraph.obj
 0002:00003a20       __ehfuncinfo$??__EscriptLog@U2@@YAXXZ 10016a20     KarlinSignatureDifferenceGraph.obj
 0002:00003a44       __unwindtable$??__EtaskLog@U2@@YAXXZ 10016a44     KarlinSignatureDifferenceGraph.obj
 0002:00003a4c       __ehfuncinfo$??__EtaskLog@U2@@YAXXZ 10016a4c     KarlinSignatureDifferenceGraph.obj
 0002:00003a70       __unwindtable$??__EuiLog@U2@@YAXXZ 10016a70     KarlinSignatureDifferenceGraph.obj
 0002:00003a78       __ehfuncinfo$??__EuiLog@U2@@YAXXZ 10016a78     KarlinSignatureDifferenceGraph.obj
 0002:00003a9c       __unwindtable$??__EuserActLog@U2@@YAXXZ 10016a9c     KarlinSignatureDifferenceGraph.obj
 0002:00003aa4       __ehfuncinfo$??__EuserActLog@U2@@YAXXZ 10016aa4     KarlinSignatureDifferenceGraph.obj
 0002:00003ac8       __unwindtable$??0KarlinGraphFactory@U2@@QAE@PAVQObject@@@Z 10016ac8     KarlinSignatureDifferenceGraph.obj
 0002:00003ae0       __ehfuncinfo$??0KarlinGraphFactory@U2@@QAE@PAVQObject@@@Z 10016ae0     KarlinSignatureDifferenceGraph.obj
 0002:00003b04       __ehfuncinfo$?createGraphs@KarlinGraphFactory@U2@@UAE?AV?$QList@V?$QSharedPointer@VGSequenceGraphData@U2@@@@@@PAVGSequenceGraphView@2@@Z 10016b04     KarlinSignatureDifferenceGraph.obj
 0002:00003b28       __unwindtable$?createGraphs@KarlinGraphFactory@U2@@UAE?AV?$QList@V?$QSharedPointer@VGSequenceGraphData@U2@@@@@@PAVGSequenceGraphView@2@@Z 10016b28     KarlinSignatureDifferenceGraph.obj
 0002:00003b50       __unwindtable$??0KarlinGraphAlgorithm@U2@@QAE@XZ 10016b50     KarlinSignatureDifferenceGraph.obj
 0002:00003b58       __ehfuncinfo$??0KarlinGraphAlgorithm@U2@@QAE@XZ 10016b58     KarlinSignatureDifferenceGraph.obj
 0002:00003b7c       __unwindtable$??1KarlinGraphAlgorithm@U2@@UAE@XZ 10016b7c     KarlinSignatureDifferenceGraph.obj
 0002:00003b84       __ehfuncinfo$??1KarlinGraphAlgorithm@U2@@UAE@XZ 10016b84     KarlinSignatureDifferenceGraph.obj
 0002:00003ba8       __unwindtable$?calculate@KarlinGraphAlgorithm@U2@@UAEXAAV?$QVector@M@@PAVU2SequenceObject@2@ABVU2Region@2@PBVGSequenceGraphWindowData@2@AAVU2OpStatus@2@@Z 10016ba8     KarlinSignatureDifferenceGraph.obj
 0002:00003bb0       __ehfuncinfo$?calculate@KarlinGraphAlgorithm@U2@@UAEXAAV?$QVector@M@@PAVU2SequenceObject@2@ABVU2Region@2@PBVGSequenceGraphWindowData@2@AAVU2OpStatus@2@@Z 10016bb0     KarlinSignatureDifferenceGraph.obj
 0002:00003bd4       __unwindtable$?calculateRelativeAbundance@KarlinGraphAlgorithm@U2@@AAEXPBDHPAMAAVU2OpStatus@2@@Z 10016bd4     KarlinSignatureDifferenceGraph.obj
 0002:00003bdc       __ehfuncinfo$?calculateRelativeAbundance@KarlinGraphAlgorithm@U2@@AAEXPBDHPAMAAVU2OpStatus@2@@Z 10016bdc     KarlinSignatureDifferenceGraph.obj
 0002:00003c00       __unwindtable$??_GKarlinGraphAlgorithm@U2@@UAEPAXI@Z 10016c00     KarlinSignatureDifferenceGraph.obj
 0002:00003c08       __ehfuncinfo$??_GKarlinGraphAlgorithm@U2@@UAEPAXI@Z 10016c08     KarlinSignatureDifferenceGraph.obj
 0002:00003c2c       __unwindtable$??__EalgoLog@U2@@YAXXZ 10016c2c     moc_BaseContentGraph.obj
 0002:00003c34       __ehfuncinfo$??__EalgoLog@U2@@YAXXZ 10016c34     moc_BaseContentGraph.obj
 0002:00003c58       __unwindtable$??__EcmdLog@U2@@YAXXZ 10016c58     moc_BaseContentGraph.obj
 0002:00003c60       __ehfuncinfo$??__EcmdLog@U2@@YAXXZ 10016c60     moc_BaseContentGraph.obj
 0002:00003c84       __unwindtable$??__EcoreLog@U2@@YAXXZ 10016c84     moc_BaseContentGraph.obj
 0002:00003c8c       __ehfuncinfo$??__EcoreLog@U2@@YAXXZ 10016c8c     moc_BaseContentGraph.obj
 0002:00003cb0       __unwindtable$??__EioLog@U2@@YAXXZ 10016cb0     moc_BaseContentGraph.obj
 0002:00003cb8       __ehfuncinfo$??__EioLog@U2@@YAXXZ 10016cb8     moc_BaseContentGraph.obj
 0002:00003cdc       __unwindtable$??__EperfLog@U2@@YAXXZ 10016cdc     moc_BaseContentGraph.obj
 0002:00003ce4       __ehfuncinfo$??__EperfLog@U2@@YAXXZ 10016ce4     moc_BaseContentGraph.obj
 0002:00003d08       __unwindtable$??__EscriptLog@U2@@YAXXZ 10016d08     moc_BaseContentGraph.obj
 0002:00003d10       __ehfuncinfo$??__EscriptLog@U2@@YAXXZ 10016d10     moc_BaseContentGraph.obj
 0002:00003d34       __unwindtable$??__EtaskLog@U2@@YAXXZ 10016d34     moc_BaseContentGraph.obj
 0002:00003d3c       __ehfuncinfo$??__EtaskLog@U2@@YAXXZ 10016d3c     moc_BaseContentGraph.obj
 0002:00003d60       __unwindtable$??__EuiLog@U2@@YAXXZ 10016d60     moc_BaseContentGraph.obj
 0002:00003d68       __ehfuncinfo$??__EuiLog@U2@@YAXXZ 10016d68     moc_BaseContentGraph.obj
 0002:00003d8c       __unwindtable$??__EuserActLog@U2@@YAXXZ 10016d8c     moc_BaseContentGraph.obj
 0002:00003d94       __ehfuncinfo$??__EuserActLog@U2@@YAXXZ 10016d94     moc_BaseContentGraph.obj
 0002:00003db8       __unwindtable$??__EalgoLog@U2@@YAXXZ 10016db8     moc_CumulativeSkew.obj
 0002:00003dc0       __ehfuncinfo$??__EalgoLog@U2@@YAXXZ 10016dc0     moc_CumulativeSkew.obj
 0002:00003de4       __unwindtable$??__EcmdLog@U2@@YAXXZ 10016de4     moc_CumulativeSkew.obj
 0002:00003dec       __ehfuncinfo$??__EcmdLog@U2@@YAXXZ 10016dec     moc_CumulativeSkew.obj
 0002:00003e10       __unwindtable$??__EcoreLog@U2@@YAXXZ 10016e10     moc_CumulativeSkew.obj
 0002:00003e18       __ehfuncinfo$??__EcoreLog@U2@@YAXXZ 10016e18     moc_CumulativeSkew.obj
 0002:00003e3c       __unwindtable$??__EioLog@U2@@YAXXZ 10016e3c     moc_CumulativeSkew.obj
 0002:00003e44       __ehfuncinfo$??__EioLog@U2@@YAXXZ 10016e44     moc_CumulativeSkew.obj
 0002:00003e68       __unwindtable$??__EperfLog@U2@@YAXXZ 10016e68     moc_CumulativeSkew.obj
 0002:00003e70       __ehfuncinfo$??__EperfLog@U2@@YAXXZ 10016e70     moc_CumulativeSkew.obj
 0002:00003e94       __unwindtable$??__EscriptLog@U2@@YAXXZ 10016e94     moc_CumulativeSkew.obj
 0002:00003e9c       __ehfuncinfo$??__EscriptLog@U2@@YAXXZ 10016e9c     moc_CumulativeSkew.obj
 0002:00003ec0       __unwindtable$??__EtaskLog@U2@@YAXXZ 10016ec0     moc_CumulativeSkew.obj
 0002:00003ec8       __ehfuncinfo$??__EtaskLog@U2@@YAXXZ 10016ec8     moc_CumulativeSkew.obj
 0002:00003eec       __unwindtable$??__EuiLog@U2@@YAXXZ 10016eec     moc_CumulativeSkew.obj
 0002:00003ef4       __ehfuncinfo$??__EuiLog@U2@@YAXXZ 10016ef4     moc_CumulativeSkew.obj
 0002:00003f18       __unwindtable$??__EuserActLog@U2@@YAXXZ 10016f18     moc_CumulativeSkew.obj
 0002:00003f20       __ehfuncinfo$??__EuserActLog@U2@@YAXXZ 10016f20     moc_CumulativeSkew.obj
 0002:00003f44       __unwindtable$??__EalgoLog@U2@@YAXXZ 10016f44     moc_DNAGraphPackPlugin.obj
 0002:00003f4c       __ehfuncinfo$??__EalgoLog@U2@@YAXXZ 10016f4c     moc_DNAGraphPackPlugin.obj
 0002:00003f70       __unwindtable$??__EcmdLog@U2@@YAXXZ 10016f70     moc_DNAGraphPackPlugin.obj
 0002:00003f78       __ehfuncinfo$??__EcmdLog@U2@@YAXXZ 10016f78     moc_DNAGraphPackPlugin.obj
 0002:00003f9c       __unwindtable$??__EcoreLog@U2@@YAXXZ 10016f9c     moc_DNAGraphPackPlugin.obj
 0002:00003fa4       __ehfuncinfo$??__EcoreLog@U2@@YAXXZ 10016fa4     moc_DNAGraphPackPlugin.obj
 0002:00003fc8       __unwindtable$??__EioLog@U2@@YAXXZ 10016fc8     moc_DNAGraphPackPlugin.obj
 0002:00003fd0       __ehfuncinfo$??__EioLog@U2@@YAXXZ 10016fd0     moc_DNAGraphPackPlugin.obj
 0002:00003ff4       __unwindtable$??__EperfLog@U2@@YAXXZ 10016ff4     moc_DNAGraphPackPlugin.obj
 0002:00003ffc       __ehfuncinfo$??__EperfLog@U2@@YAXXZ 10016ffc     moc_DNAGraphPackPlugin.obj
 0002:00004020       __unwindtable$??__EscriptLog@U2@@YAXXZ 10017020     moc_DNAGraphPackPlugin.obj
 0002:00004028       __ehfuncinfo$??__EscriptLog@U2@@YAXXZ 10017028     moc_DNAGraphPackPlugin.obj
 0002:0000404c       __unwindtable$??__EtaskLog@U2@@YAXXZ 1001704c     moc_DNAGraphPackPlugin.obj
 0002:00004054       __ehfuncinfo$??__EtaskLog@U2@@YAXXZ 10017054     moc_DNAGraphPackPlugin.obj
 0002:00004078       __unwindtable$??__EuiLog@U2@@YAXXZ 10017078     moc_DNAGraphPackPlugin.obj
 0002:00004080       __ehfuncinfo$??__EuiLog@U2@@YAXXZ 10017080     moc_DNAGraphPackPlugin.obj
 0002:000040a4       __unwindtable$??__EuserActLog@U2@@YAXXZ 100170a4     moc_DNAGraphPackPlugin.obj
 0002:000040ac       __ehfuncinfo$??__EuserActLog@U2@@YAXXZ 100170ac     moc_DNAGraphPackPlugin.obj
 0002:000040d0       __unwindtable$?qt_metatype_id@?$QMetaTypeIdQObject@PAVADVSequenceWidget@U2@@$00@@SAHXZ 100170d0     moc_DNAGraphPackPlugin.obj
 0002:000040d8       __ehfuncinfo$?qt_metatype_id@?$QMetaTypeIdQObject@PAVADVSequenceWidget@U2@@$00@@SAHXZ 100170d8     moc_DNAGraphPackPlugin.obj
 0002:000040fc       __unwindtable$??__EalgoLog@U2@@YAXXZ 100170fc     moc_DeviationGraph.obj
 0002:00004104       __ehfuncinfo$??__EalgoLog@U2@@YAXXZ 10017104     moc_DeviationGraph.obj
 0002:00004128       __unwindtable$??__EcmdLog@U2@@YAXXZ 10017128     moc_DeviationGraph.obj
 0002:00004130       __ehfuncinfo$??__EcmdLog@U2@@YAXXZ 10017130     moc_DeviationGraph.obj
 0002:00004154       __unwindtable$??__EcoreLog@U2@@YAXXZ 10017154     moc_DeviationGraph.obj
 0002:0000415c       __ehfuncinfo$??__EcoreLog@U2@@YAXXZ 1001715c     moc_DeviationGraph.obj
 0002:00004180       __unwindtable$??__EioLog@U2@@YAXXZ 10017180     moc_DeviationGraph.obj
 0002:00004188       __ehfuncinfo$??__EioLog@U2@@YAXXZ 10017188     moc_DeviationGraph.obj
 0002:000041ac       __unwindtable$??__EperfLog@U2@@YAXXZ 100171ac     moc_DeviationGraph.obj
 0002:000041b4       __ehfuncinfo$??__EperfLog@U2@@YAXXZ 100171b4     moc_DeviationGraph.obj
 0002:000041d8       __unwindtable$??__EscriptLog@U2@@YAXXZ 100171d8     moc_DeviationGraph.obj
 0002:000041e0       __ehfuncinfo$??__EscriptLog@U2@@YAXXZ 100171e0     moc_DeviationGraph.obj
 0002:00004204       __unwindtable$??__EtaskLog@U2@@YAXXZ 10017204     moc_DeviationGraph.obj
 0002:0000420c       __ehfuncinfo$??__EtaskLog@U2@@YAXXZ 1001720c     moc_DeviationGraph.obj
 0002:00004230       __unwindtable$??__EuiLog@U2@@YAXXZ 10017230     moc_DeviationGraph.obj
 0002:00004238       __ehfuncinfo$??__EuiLog@U2@@YAXXZ 10017238     moc_DeviationGraph.obj
 0002:0000425c       __unwindtable$??__EuserActLog@U2@@YAXXZ 1001725c     moc_DeviationGraph.obj
 0002:00004264       __ehfuncinfo$??__EuserActLog@U2@@YAXXZ 10017264     moc_DeviationGraph.obj
 0002:00004288       __unwindtable$??__EalgoLog@U2@@YAXXZ 10017288     moc_EntropyAlgorithm.obj
 0002:00004290       __ehfuncinfo$??__EalgoLog@U2@@YAXXZ 10017290     moc_EntropyAlgorithm.obj
 0002:000042b4       __unwindtable$??__EcmdLog@U2@@YAXXZ 100172b4     moc_EntropyAlgorithm.obj
 0002:000042bc       __ehfuncinfo$??__EcmdLog@U2@@YAXXZ 100172bc     moc_EntropyAlgorithm.obj
 0002:000042e0       __unwindtable$??__EcoreLog@U2@@YAXXZ 100172e0     moc_EntropyAlgorithm.obj
 0002:000042e8       __ehfuncinfo$??__EcoreLog@U2@@YAXXZ 100172e8     moc_EntropyAlgorithm.obj
 0002:0000430c       __unwindtable$??__EioLog@U2@@YAXXZ 1001730c     moc_EntropyAlgorithm.obj
 0002:00004314       __ehfuncinfo$??__EioLog@U2@@YAXXZ 10017314     moc_EntropyAlgorithm.obj
 0002:00004338       __unwindtable$??__EperfLog@U2@@YAXXZ 10017338     moc_EntropyAlgorithm.obj
 0002:00004340       __ehfuncinfo$??__EperfLog@U2@@YAXXZ 10017340     moc_EntropyAlgorithm.obj
 0002:00004364       __unwindtable$??__EscriptLog@U2@@YAXXZ 10017364     moc_EntropyAlgorithm.obj
 0002:0000436c       __ehfuncinfo$??__EscriptLog@U2@@YAXXZ 1001736c     moc_EntropyAlgorithm.obj
 0002:00004390       __unwindtable$??__EtaskLog@U2@@YAXXZ 10017390     moc_EntropyAlgorithm.obj
 0002:00004398       __ehfuncinfo$??__EtaskLog@U2@@YAXXZ 10017398     moc_EntropyAlgorithm.obj
 0002:000043bc       __unwindtable$??__EuiLog@U2@@YAXXZ 100173bc     moc_EntropyAlgorithm.obj
 0002:000043c4       __ehfuncinfo$??__EuiLog@U2@@YAXXZ 100173c4     moc_EntropyAlgorithm.obj
 0002:000043e8       __unwindtable$??__EuserActLog@U2@@YAXXZ 100173e8     moc_EntropyAlgorithm.obj
 0002:000043f0       __ehfuncinfo$??__EuserActLog@U2@@YAXXZ 100173f0     moc_EntropyAlgorithm.obj
 0002:00004414       __unwindtable$??__EalgoLog@U2@@YAXXZ 10017414     moc_GCFramePlot.obj
 0002:0000441c       __ehfuncinfo$??__EalgoLog@U2@@YAXXZ 1001741c     moc_GCFramePlot.obj
 0002:00004440       __unwindtable$??__EcmdLog@U2@@YAXXZ 10017440     moc_GCFramePlot.obj
 0002:00004448       __ehfuncinfo$??__EcmdLog@U2@@YAXXZ 10017448     moc_GCFramePlot.obj
 0002:0000446c       __unwindtable$??__EcoreLog@U2@@YAXXZ 1001746c     moc_GCFramePlot.obj
 0002:00004474       __ehfuncinfo$??__EcoreLog@U2@@YAXXZ 10017474     moc_GCFramePlot.obj
 0002:00004498       __unwindtable$??__EioLog@U2@@YAXXZ 10017498     moc_GCFramePlot.obj
 0002:000044a0       __ehfuncinfo$??__EioLog@U2@@YAXXZ 100174a0     moc_GCFramePlot.obj
 0002:000044c4       __unwindtable$??__EperfLog@U2@@YAXXZ 100174c4     moc_GCFramePlot.obj
 0002:000044cc       __ehfuncinfo$??__EperfLog@U2@@YAXXZ 100174cc     moc_GCFramePlot.obj
 0002:000044f0       __unwindtable$??__EscriptLog@U2@@YAXXZ 100174f0     moc_GCFramePlot.obj
 0002:000044f8       __ehfuncinfo$??__EscriptLog@U2@@YAXXZ 100174f8     moc_GCFramePlot.obj
 0002:0000451c       __unwindtable$??__EtaskLog@U2@@YAXXZ 1001751c     moc_GCFramePlot.obj
 0002:00004524       __ehfuncinfo$??__EtaskLog@U2@@YAXXZ 10017524     moc_GCFramePlot.obj
 0002:00004548       __unwindtable$??__EuiLog@U2@@YAXXZ 10017548     moc_GCFramePlot.obj
 0002:00004550       __ehfuncinfo$??__EuiLog@U2@@YAXXZ 10017550     moc_GCFramePlot.obj
 0002:00004574       __unwindtable$??__EuserActLog@U2@@YAXXZ 10017574     moc_GCFramePlot.obj
 0002:0000457c       __ehfuncinfo$??__EuserActLog@U2@@YAXXZ 1001757c     moc_GCFramePlot.obj
 0002:000045a0       __unwindtable$??__EalgoLog@U2@@YAXXZ 100175a0     moc_KarlinSignatureDifferenceGraph.obj
 0002:000045a8       __ehfuncinfo$??__EalgoLog@U2@@YAXXZ 100175a8     moc_KarlinSignatureDifferenceGraph.obj
 0002:000045cc       __unwindtable$??__EcmdLog@U2@@YAXXZ 100175cc     moc_KarlinSignatureDifferenceGraph.obj
 0002:000045d4       __ehfuncinfo$??__EcmdLog@U2@@YAXXZ 100175d4     moc_KarlinSignatureDifferenceGraph.obj
 0002:000045f8       __unwindtable$??__EcoreLog@U2@@YAXXZ 100175f8     moc_KarlinSignatureDifferenceGraph.obj
 0002:00004600       __ehfuncinfo$??__EcoreLog@U2@@YAXXZ 10017600     moc_KarlinSignatureDifferenceGraph.obj
 0002:00004624       __unwindtable$??__EioLog@U2@@YAXXZ 10017624     moc_KarlinSignatureDifferenceGraph.obj
 0002:0000462c       __ehfuncinfo$??__EioLog@U2@@YAXXZ 1001762c     moc_KarlinSignatureDifferenceGraph.obj
 0002:00004650       __unwindtable$??__EperfLog@U2@@YAXXZ 10017650     moc_KarlinSignatureDifferenceGraph.obj
 0002:00004658       __ehfuncinfo$??__EperfLog@U2@@YAXXZ 10017658     moc_KarlinSignatureDifferenceGraph.obj
 0002:0000467c       __unwindtable$??__EscriptLog@U2@@YAXXZ 1001767c     moc_KarlinSignatureDifferenceGraph.obj
 0002:00004684       __ehfuncinfo$??__EscriptLog@U2@@YAXXZ 10017684     moc_KarlinSignatureDifferenceGraph.obj
 0002:000046a8       __unwindtable$??__EtaskLog@U2@@YAXXZ 100176a8     moc_KarlinSignatureDifferenceGraph.obj
 0002:000046b0       __ehfuncinfo$??__EtaskLog@U2@@YAXXZ 100176b0     moc_KarlinSignatureDifferenceGraph.obj
 0002:000046d4       __unwindtable$??__EuiLog@U2@@YAXXZ 100176d4     moc_KarlinSignatureDifferenceGraph.obj
 0002:000046dc       __ehfuncinfo$??__EuiLog@U2@@YAXXZ 100176dc     moc_KarlinSignatureDifferenceGraph.obj
 0002:00004700       __unwindtable$??__EuserActLog@U2@@YAXXZ 10017700     moc_KarlinSignatureDifferenceGraph.obj
 0002:00004708       __ehfuncinfo$??__EuserActLog@U2@@YAXXZ 10017708     moc_KarlinSignatureDifferenceGraph.obj
 0002:00004730       __sehtable$__onexit        10017730     MSVCRT:atonexit.obj
 0002:00004750       __sehtable$___DllMainCRTStartup 10017750     MSVCRT:crtdll.obj
 0002:00004778       __sehtable$??_M@YGXPAXIHP6EX0@Z@Z 10017778     MSVCRT:ehvecdtr.obj
 0002:00004798       __sehtable$?__ArrayUnwind@@YGXPAXIHP6EX0@Z@Z 10017798     MSVCRT:ehvecdtr.obj
 0002:000047b8       __sehtable$__IsNonwritableInCurrentImage 100177b8     MSVCRT:pesect.obj
 0002:000047e0       .edata                     100177e0     dna_graphpack.exp
 0002:00004808       rgpv                       10017808     dna_graphpack.exp
 0002:0000480c       rgszName                   1001780c     dna_graphpack.exp
 0002:00004810       rgwOrd                     10017810     dna_graphpack.exp
 0002:00004812       szName                     10017812     dna_graphpack.exp
 0002:00004824       $N00001                    10017824     dna_graphpack.exp
 0002:00004f42       .idata$6                   10017f42     U2Core:U2Core.dll
 0002:00005388       .idata$6                   10018388     U2Gui:U2Gui.dll
 0002:0000589c       .idata$6                   1001889c     U2View:U2View.dll
 0002:000058ee       .idata$6                   100188ee     Qt5Widgets:Qt5Widgets.dll
 0002:00005942       .idata$6                   10018942     Qt5Gui:Qt5Gui.dll
 0002:00006378       .idata$6                   10019378     Qt5Core:Qt5Core.dll
 0002:0000641e       .idata$6                   1001941e     msvcprt:MSVCP120.dll
 0002:000064d8       .idata$6                   100194d8     MSVCRT:MSVCR120.dll
 0002:000066f8       .idata$6                   100196f8     kernel32:KERNEL32.dll
 0003:0000000c       _Service_PluginViewer      1001a00c     BaseContentGraph.obj
 0003:00000014       _Service_Project           1001a014     BaseContentGraph.obj
 0003:0000001c       _Service_ProjectView       1001a01c     BaseContentGraph.obj
 0003:00000024       _Service_DNAGraphPack      1001a024     BaseContentGraph.obj
 0003:0000002c       _Service_DNAExport         1001a02c     BaseContentGraph.obj
 0003:00000034       _Service_TestRunner        1001a034     BaseContentGraph.obj
 0003:0000003c       _Service_ScriptRegistry    1001a03c     BaseContentGraph.obj
 0003:00000044       _Service_ExternalToolSupport 1001a044     BaseContentGraph.obj
 0003:0000004c       _Service_GUITesting        1001a04c     BaseContentGraph.obj
 0003:00000054       _Service_WorkflowDesigner  1001a054     BaseContentGraph.obj
 0003:0000005c       _Service_QueryDesigner     1001a05c     BaseContentGraph.obj
 0003:00000064       _Service_MinCoreServiceId  1001a064     BaseContentGraph.obj
 0003:0000006c       _Service_MaxCoreServiceId  1001a06c     BaseContentGraph.obj
 0003:00000074       _Service_PluginViewer      1001a074     CumulativeSkew.obj
 0003:0000007c       _Service_Project           1001a07c     CumulativeSkew.obj
 0003:00000084       _Service_ProjectView       1001a084     CumulativeSkew.obj
 0003:0000008c       _Service_DNAGraphPack      1001a08c     CumulativeSkew.obj
 0003:00000094       _Service_DNAExport         1001a094     CumulativeSkew.obj
 0003:0000009c       _Service_TestRunner        1001a09c     CumulativeSkew.obj
 0003:000000a4       _Service_ScriptRegistry    1001a0a4     CumulativeSkew.obj
 0003:000000ac       _Service_ExternalToolSupport 1001a0ac     CumulativeSkew.obj
 0003:000000b4       _Service_GUITesting        1001a0b4     CumulativeSkew.obj
 0003:000000bc       _Service_WorkflowDesigner  1001a0bc     CumulativeSkew.obj
 0003:000000c4       _Service_QueryDesigner     1001a0c4     CumulativeSkew.obj
 0003:000000cc       _Service_MinCoreServiceId  1001a0cc     CumulativeSkew.obj
 0003:000000d4       _Service_MaxCoreServiceId  1001a0d4     CumulativeSkew.obj
 0003:000000dc       _Service_PluginViewer      1001a0dc     DNAGraphPackPlugin.obj
 0003:000000e4       _Service_Project           1001a0e4     DNAGraphPackPlugin.obj
 0003:000000ec       _Service_ProjectView       1001a0ec     DNAGraphPackPlugin.obj
 0003:000000f4       _Service_DNAGraphPack      1001a0f4     DNAGraphPackPlugin.obj
 0003:000000fc       _Service_DNAExport         1001a0fc     DNAGraphPackPlugin.obj
 0003:00000104       _Service_TestRunner        1001a104     DNAGraphPackPlugin.obj
 0003:0000010c       _Service_ScriptRegistry    1001a10c     DNAGraphPackPlugin.obj
 0003:00000114       _Service_ExternalToolSupport 1001a114     DNAGraphPackPlugin.obj
 0003:0000011c       _Service_GUITesting        1001a11c     DNAGraphPackPlugin.obj
 0003:00000124       _Service_WorkflowDesigner  1001a124     DNAGraphPackPlugin.obj
 0003:0000012c       _Service_QueryDesigner     1001a12c     DNAGraphPackPlugin.obj
 0003:00000134       _Service_MinCoreServiceId  1001a134     DNAGraphPackPlugin.obj
 0003:0000013c       _Service_MaxCoreServiceId  1001a13c     DNAGraphPackPlugin.obj
 0003:00000144       _Service_PluginViewer      1001a144     DeviationGraph.obj
 0003:0000014c       _Service_Project           1001a14c     DeviationGraph.obj
 0003:00000154       _Service_ProjectView       1001a154     DeviationGraph.obj
 0003:0000015c       _Service_DNAGraphPack      1001a15c     DeviationGraph.obj
 0003:00000164       _Service_DNAExport         1001a164     DeviationGraph.obj
 0003:0000016c       _Service_TestRunner        1001a16c     DeviationGraph.obj
 0003:00000174       _Service_ScriptRegistry    1001a174     DeviationGraph.obj
 0003:0000017c       _Service_ExternalToolSupport 1001a17c     DeviationGraph.obj
 0003:00000184       _Service_GUITesting        1001a184     DeviationGraph.obj
 0003:0000018c       _Service_WorkflowDesigner  1001a18c     DeviationGraph.obj
 0003:00000194       _Service_QueryDesigner     1001a194     DeviationGraph.obj
 0003:0000019c       _Service_MinCoreServiceId  1001a19c     DeviationGraph.obj
 0003:000001a4       _Service_MaxCoreServiceId  1001a1a4     DeviationGraph.obj
 0003:000001ac       _Service_PluginViewer      1001a1ac     EntropyAlgorithm.obj
 0003:000001b4       _Service_Project           1001a1b4     EntropyAlgorithm.obj
 0003:000001bc       _Service_ProjectView       1001a1bc     EntropyAlgorithm.obj
 0003:000001c4       _Service_DNAGraphPack      1001a1c4     EntropyAlgorithm.obj
 0003:000001cc       _Service_DNAExport         1001a1cc     EntropyAlgorithm.obj
 0003:000001d4       _Service_TestRunner        1001a1d4     EntropyAlgorithm.obj
 0003:000001dc       _Service_ScriptRegistry    1001a1dc     EntropyAlgorithm.obj
 0003:000001e4       _Service_ExternalToolSupport 1001a1e4     EntropyAlgorithm.obj
 0003:000001ec       _Service_GUITesting        1001a1ec     EntropyAlgorithm.obj
 0003:000001f4       _Service_WorkflowDesigner  1001a1f4     EntropyAlgorithm.obj
 0003:000001fc       _Service_QueryDesigner     1001a1fc     EntropyAlgorithm.obj
 0003:00000204       _Service_MinCoreServiceId  1001a204     EntropyAlgorithm.obj
 0003:0000020c       _Service_MaxCoreServiceId  1001a20c     EntropyAlgorithm.obj
 0003:00000214       _Service_PluginViewer      1001a214     GCFramePlot.obj
 0003:0000021c       _Service_Project           1001a21c     GCFramePlot.obj
 0003:00000224       _Service_ProjectView       1001a224     GCFramePlot.obj
 0003:0000022c       _Service_DNAGraphPack      1001a22c     GCFramePlot.obj
 0003:00000234       _Service_DNAExport         1001a234     GCFramePlot.obj
 0003:0000023c       _Service_TestRunner        1001a23c     GCFramePlot.obj
 0003:00000244       _Service_ScriptRegistry    1001a244     GCFramePlot.obj
 0003:0000024c       _Service_ExternalToolSupport 1001a24c     GCFramePlot.obj
 0003:00000254       _Service_GUITesting        1001a254     GCFramePlot.obj
 0003:0000025c       _Service_WorkflowDesigner  1001a25c     GCFramePlot.obj
 0003:00000264       _Service_QueryDesigner     1001a264     GCFramePlot.obj
 0003:0000026c       _Service_MinCoreServiceId  1001a26c     GCFramePlot.obj
 0003:00000274       _Service_MaxCoreServiceId  1001a274     GCFramePlot.obj
 0003:0000027c       _Service_PluginViewer      1001a27c     KarlinSignatureDifferenceGraph.obj
 0003:00000284       _Service_Project           1001a284     KarlinSignatureDifferenceGraph.obj
 0003:0000028c       _Service_ProjectView       1001a28c     KarlinSignatureDifferenceGraph.obj
 0003:00000294       _Service_DNAGraphPack      1001a294     KarlinSignatureDifferenceGraph.obj
 0003:0000029c       _Service_DNAExport         1001a29c     KarlinSignatureDifferenceGraph.obj
 0003:000002a4       _Service_TestRunner        1001a2a4     KarlinSignatureDifferenceGraph.obj
 0003:000002ac       _Service_ScriptRegistry    1001a2ac     KarlinSignatureDifferenceGraph.obj
 0003:000002b4       _Service_ExternalToolSupport 1001a2b4     KarlinSignatureDifferenceGraph.obj
 0003:000002bc       _Service_GUITesting        1001a2bc     KarlinSignatureDifferenceGraph.obj
 0003:000002c4       _Service_WorkflowDesigner  1001a2c4     KarlinSignatureDifferenceGraph.obj
 0003:000002cc       _Service_QueryDesigner     1001a2cc     KarlinSignatureDifferenceGraph.obj
 0003:000002d4       _Service_MinCoreServiceId  1001a2d4     KarlinSignatureDifferenceGraph.obj
 0003:000002dc       _Service_MaxCoreServiceId  1001a2dc     KarlinSignatureDifferenceGraph.obj
 0003:000002e4       _Service_PluginViewer      1001a2e4     moc_BaseContentGraph.obj
 0003:000002ec       _Service_Project           1001a2ec     moc_BaseContentGraph.obj
 0003:000002f4       _Service_ProjectView       1001a2f4     moc_BaseContentGraph.obj
 0003:000002fc       _Service_DNAGraphPack      1001a2fc     moc_BaseContentGraph.obj
 0003:00000304       _Service_DNAExport         1001a304     moc_BaseContentGraph.obj
 0003:0000030c       _Service_TestRunner        1001a30c     moc_BaseContentGraph.obj
 0003:00000314       _Service_ScriptRegistry    1001a314     moc_BaseContentGraph.obj
 0003:0000031c       _Service_ExternalToolSupport 1001a31c     moc_BaseContentGraph.obj
 0003:00000324       _Service_GUITesting        1001a324     moc_BaseContentGraph.obj
 0003:0000032c       _Service_WorkflowDesigner  1001a32c     moc_BaseContentGraph.obj
 0003:00000334       _Service_QueryDesigner     1001a334     moc_BaseContentGraph.obj
 0003:0000033c       _Service_MinCoreServiceId  1001a33c     moc_BaseContentGraph.obj
 0003:00000344       _Service_MaxCoreServiceId  1001a344     moc_BaseContentGraph.obj
 0003:00000364       _Service_PluginViewer      1001a364     moc_CumulativeSkew.obj
 0003:0000036c       _Service_Project           1001a36c     moc_CumulativeSkew.obj
 0003:00000374       _Service_ProjectView       1001a374     moc_CumulativeSkew.obj
 0003:0000037c       _Service_DNAGraphPack      1001a37c     moc_CumulativeSkew.obj
 0003:00000384       _Service_DNAExport         1001a384     moc_CumulativeSkew.obj
 0003:0000038c       _Service_TestRunner        1001a38c     moc_CumulativeSkew.obj
 0003:00000394       _Service_ScriptRegistry    1001a394     moc_CumulativeSkew.obj
 0003:0000039c       _Service_ExternalToolSupport 1001a39c     moc_CumulativeSkew.obj
 0003:000003a4       _Service_GUITesting        1001a3a4     moc_CumulativeSkew.obj
 0003:000003ac       _Service_WorkflowDesigner  1001a3ac     moc_CumulativeSkew.obj
 0003:000003b4       _Service_QueryDesigner     1001a3b4     moc_CumulativeSkew.obj
 0003:000003bc       _Service_MinCoreServiceId  1001a3bc     moc_CumulativeSkew.obj
 0003:000003c4       _Service_MaxCoreServiceId  1001a3c4     moc_CumulativeSkew.obj
 0003:000003e4       _Service_PluginViewer      1001a3e4     moc_DNAGraphPackPlugin.obj
 0003:000003ec       _Service_Project           1001a3ec     moc_DNAGraphPackPlugin.obj
 0003:000003f4       _Service_ProjectView       1001a3f4     moc_DNAGraphPackPlugin.obj
 0003:000003fc       _Service_DNAGraphPack      1001a3fc     moc_DNAGraphPackPlugin.obj
 0003:00000404       _Service_DNAExport         1001a404     moc_DNAGraphPackPlugin.obj
 0003:0000040c       _Service_TestRunner        1001a40c     moc_DNAGraphPackPlugin.obj
 0003:00000414       _Service_ScriptRegistry    1001a414     moc_DNAGraphPackPlugin.obj
 0003:0000041c       _Service_ExternalToolSupport 1001a41c     moc_DNAGraphPackPlugin.obj
 0003:00000424       _Service_GUITesting        1001a424     moc_DNAGraphPackPlugin.obj
 0003:0000042c       _Service_WorkflowDesigner  1001a42c     moc_DNAGraphPackPlugin.obj
 0003:00000434       _Service_QueryDesigner     1001a434     moc_DNAGraphPackPlugin.obj
 0003:0000043c       _Service_MinCoreServiceId  1001a43c     moc_DNAGraphPackPlugin.obj
 0003:00000444       _Service_MaxCoreServiceId  1001a444     moc_DNAGraphPackPlugin.obj
 0003:0000047c       _Service_PluginViewer      1001a47c     moc_DeviationGraph.obj
 0003:00000484       _Service_Project           1001a484     moc_DeviationGraph.obj
 0003:0000048c       _Service_ProjectView       1001a48c     moc_DeviationGraph.obj
 0003:00000494       _Service_DNAGraphPack      1001a494     moc_DeviationGraph.obj
 0003:0000049c       _Service_DNAExport         1001a49c     moc_DeviationGraph.obj
 0003:000004a4       _Service_TestRunner        1001a4a4     moc_DeviationGraph.obj
 0003:000004ac       _Service_ScriptRegistry    1001a4ac     moc_DeviationGraph.obj
 0003:000004b4       _Service_ExternalToolSupport 1001a4b4     moc_DeviationGraph.obj
 0003:000004bc       _Service_GUITesting        1001a4bc     moc_DeviationGraph.obj
 0003:000004c4       _Service_WorkflowDesigner  1001a4c4     moc_DeviationGraph.obj
 0003:000004cc       _Service_QueryDesigner     1001a4cc     moc_DeviationGraph.obj
 0003:000004d4       _Service_MinCoreServiceId  1001a4d4     moc_DeviationGraph.obj
 0003:000004dc       _Service_MaxCoreServiceId  1001a4dc     moc_DeviationGraph.obj
 0003:000004fc       _Service_PluginViewer      1001a4fc     moc_EntropyAlgorithm.obj
 0003:00000504       _Service_Project           1001a504     moc_EntropyAlgorithm.obj
 0003:0000050c       _Service_ProjectView       1001a50c     moc_EntropyAlgorithm.obj
 0003:00000514       _Service_DNAGraphPack      1001a514     moc_EntropyAlgorithm.obj
 0003:0000051c       _Service_DNAExport         1001a51c     moc_EntropyAlgorithm.obj
 0003:00000524       _Service_TestRunner        1001a524     moc_EntropyAlgorithm.obj
 0003:0000052c       _Service_ScriptRegistry    1001a52c     moc_EntropyAlgorithm.obj
 0003:00000534       _Service_ExternalToolSupport 1001a534     moc_EntropyAlgorithm.obj
 0003:0000053c       _Service_GUITesting        1001a53c     moc_EntropyAlgorithm.obj
 0003:00000544       _Service_WorkflowDesigner  1001a544     moc_EntropyAlgorithm.obj
 0003:0000054c       _Service_QueryDesigner     1001a54c     moc_EntropyAlgorithm.obj
 0003:00000554       _Service_MinCoreServiceId  1001a554     moc_EntropyAlgorithm.obj
 0003:0000055c       _Service_MaxCoreServiceId  1001a55c     moc_EntropyAlgorithm.obj
 0003:0000057c       _Service_PluginViewer      1001a57c     moc_GCFramePlot.obj
 0003:00000584       _Service_Project           1001a584     moc_GCFramePlot.obj
 0003:0000058c       _Service_ProjectView       1001a58c     moc_GCFramePlot.obj
 0003:00000594       _Service_DNAGraphPack      1001a594     moc_GCFramePlot.obj
 0003:0000059c       _Service_DNAExport         1001a59c     moc_GCFramePlot.obj
 0003:000005a4       _Service_TestRunner        1001a5a4     moc_GCFramePlot.obj
 0003:000005ac       _Service_ScriptRegistry    1001a5ac     moc_GCFramePlot.obj
 0003:000005b4       _Service_ExternalToolSupport 1001a5b4     moc_GCFramePlot.obj
 0003:000005bc       _Service_GUITesting        1001a5bc     moc_GCFramePlot.obj
 0003:000005c4       _Service_WorkflowDesigner  1001a5c4     moc_GCFramePlot.obj
 0003:000005cc       _Service_QueryDesigner     1001a5cc     moc_GCFramePlot.obj
 0003:000005d4       _Service_MinCoreServiceId  1001a5d4     moc_GCFramePlot.obj
 0003:000005dc       _Service_MaxCoreServiceId  1001a5dc     moc_GCFramePlot.obj
 0003:000005fc       _Service_PluginViewer      1001a5fc     moc_KarlinSignatureDifferenceGraph.obj
 0003:00000604       _Service_Project           1001a604     moc_KarlinSignatureDifferenceGraph.obj
 0003:0000060c       _Service_ProjectView       1001a60c     moc_KarlinSignatureDifferenceGraph.obj
 0003:00000614       _Service_DNAGraphPack      1001a614     moc_KarlinSignatureDifferenceGraph.obj
 0003:0000061c       _Service_DNAExport         1001a61c     moc_KarlinSignatureDifferenceGraph.obj
 0003:00000624       _Service_TestRunner        1001a624     moc_KarlinSignatureDifferenceGraph.obj
 0003:0000062c       _Service_ScriptRegistry    1001a62c     moc_KarlinSignatureDifferenceGraph.obj
 0003:00000634       _Service_ExternalToolSupport 1001a634     moc_KarlinSignatureDifferenceGraph.obj
 0003:0000063c       _Service_GUITesting        1001a63c     moc_KarlinSignatureDifferenceGraph.obj
 0003:00000644       _Service_WorkflowDesigner  1001a644     moc_KarlinSignatureDifferenceGraph.obj
 0003:0000064c       _Service_QueryDesigner     1001a64c     moc_KarlinSignatureDifferenceGraph.obj
 0003:00000654       _Service_MinCoreServiceId  1001a654     moc_KarlinSignatureDifferenceGraph.obj
 0003:0000065c       _Service_MaxCoreServiceId  1001a65c     moc_KarlinSignatureDifferenceGraph.obj
 0003:00000b30       __Tuple_alloc              1001ab30     BaseContentGraph.obj
 0003:00000b31       _ignore                    1001ab31     BaseContentGraph.obj
 0003:00000b32       _allocator_arg             1001ab32     BaseContentGraph.obj
 0003:00000b33       _piecewise_construct       1001ab33     BaseContentGraph.obj
 0003:00000b34       _taskLog                   1001ab34     BaseContentGraph.obj
 0003:00000b3c       _algoLog                   1001ab3c     BaseContentGraph.obj
 0003:00000b44       _userActLog                1001ab44     BaseContentGraph.obj
 0003:00000b4c       _ioLog                     1001ab4c     BaseContentGraph.obj
 0003:00000b54       _coreLog                   1001ab54     BaseContentGraph.obj
 0003:00000b5c       _uiLog                     1001ab5c     BaseContentGraph.obj
 0003:00000b64       _scriptLog                 1001ab64     BaseContentGraph.obj
 0003:00000b6c       _perfLog                   1001ab6c     BaseContentGraph.obj
 0003:00000b74       _cmdLog                    1001ab74     BaseContentGraph.obj
 0003:00000b84       __Tuple_alloc              1001ab84     CumulativeSkew.obj
 0003:00000b85       _ignore                    1001ab85     CumulativeSkew.obj
 0003:00000b86       _allocator_arg             1001ab86     CumulativeSkew.obj
 0003:00000b87       _piecewise_construct       1001ab87     CumulativeSkew.obj
 0003:00000b88       _taskLog                   1001ab88     CumulativeSkew.obj
 0003:00000b90       _algoLog                   1001ab90     CumulativeSkew.obj
 0003:00000b98       _userActLog                1001ab98     CumulativeSkew.obj
 0003:00000ba0       _ioLog                     1001aba0     CumulativeSkew.obj
 0003:00000ba8       _coreLog                   1001aba8     CumulativeSkew.obj
 0003:00000bb0       _uiLog                     1001abb0     CumulativeSkew.obj
 0003:00000bb8       _scriptLog                 1001abb8     CumulativeSkew.obj
 0003:00000bc0       _perfLog                   1001abc0     CumulativeSkew.obj
 0003:00000bc8       _cmdLog                    1001abc8     CumulativeSkew.obj
 0003:00000bd0       __Tuple_alloc              1001abd0     DNAGraphPackPlugin.obj
 0003:00000bd1       _ignore                    1001abd1     DNAGraphPackPlugin.obj
 0003:00000bd2       _allocator_arg             1001abd2     DNAGraphPackPlugin.obj
 0003:00000bd3       _piecewise_construct       1001abd3     DNAGraphPackPlugin.obj
 0003:00000bd4       _taskLog                   1001abd4     DNAGraphPackPlugin.obj
 0003:00000bdc       _algoLog                   1001abdc     DNAGraphPackPlugin.obj
 0003:00000be4       _userActLog                1001abe4     DNAGraphPackPlugin.obj
 0003:00000bec       _ioLog                     1001abec     DNAGraphPackPlugin.obj
 0003:00000bf4       _coreLog                   1001abf4     DNAGraphPackPlugin.obj
 0003:00000bfc       _uiLog                     1001abfc     DNAGraphPackPlugin.obj
 0003:00000c04       _scriptLog                 1001ac04     DNAGraphPackPlugin.obj
 0003:00000c0c       _perfLog                   1001ac0c     DNAGraphPackPlugin.obj
 0003:00000c14       _cmdLog                    1001ac14     DNAGraphPackPlugin.obj
 0003:00000c1c       __Tuple_alloc              1001ac1c     DeviationGraph.obj
 0003:00000c1d       _ignore                    1001ac1d     DeviationGraph.obj
 0003:00000c1e       _allocator_arg             1001ac1e     DeviationGraph.obj
 0003:00000c1f       _piecewise_construct       1001ac1f     DeviationGraph.obj
 0003:00000c20       _taskLog                   1001ac20     DeviationGraph.obj
 0003:00000c28       _algoLog                   1001ac28     DeviationGraph.obj
 0003:00000c30       _userActLog                1001ac30     DeviationGraph.obj
 0003:00000c38       _ioLog                     1001ac38     DeviationGraph.obj
 0003:00000c40       _coreLog                   1001ac40     DeviationGraph.obj
 0003:00000c48       _uiLog                     1001ac48     DeviationGraph.obj
 0003:00000c50       _scriptLog                 1001ac50     DeviationGraph.obj
 0003:00000c58       _perfLog                   1001ac58     DeviationGraph.obj
 0003:00000c60       _cmdLog                    1001ac60     DeviationGraph.obj
 0003:00000c68       __Tuple_alloc              1001ac68     EntropyAlgorithm.obj
 0003:00000c69       _ignore                    1001ac69     EntropyAlgorithm.obj
 0003:00000c6a       _allocator_arg             1001ac6a     EntropyAlgorithm.obj
 0003:00000c6b       _piecewise_construct       1001ac6b     EntropyAlgorithm.obj
 0003:00000c6c       _taskLog                   1001ac6c     EntropyAlgorithm.obj
 0003:00000c74       _algoLog                   1001ac74     EntropyAlgorithm.obj
 0003:00000c7c       _userActLog                1001ac7c     EntropyAlgorithm.obj
 0003:00000c84       _ioLog                     1001ac84     EntropyAlgorithm.obj
 0003:00000c8c       _coreLog                   1001ac8c     EntropyAlgorithm.obj
 0003:00000c94       _uiLog                     1001ac94     EntropyAlgorithm.obj
 0003:00000c9c       _scriptLog                 1001ac9c     EntropyAlgorithm.obj
 0003:00000ca4       _perfLog                   1001aca4     EntropyAlgorithm.obj
 0003:00000cac       _cmdLog                    1001acac     EntropyAlgorithm.obj
 0003:00000cb4       __Tuple_alloc              1001acb4     GCFramePlot.obj
 0003:00000cb5       _ignore                    1001acb5     GCFramePlot.obj
 0003:00000cb6       _allocator_arg             1001acb6     GCFramePlot.obj
 0003:00000cb7       _piecewise_construct       1001acb7     GCFramePlot.obj
 0003:00000cb8       _taskLog                   1001acb8     GCFramePlot.obj
 0003:00000cc0       _algoLog                   1001acc0     GCFramePlot.obj
 0003:00000cc8       _userActLog                1001acc8     GCFramePlot.obj
 0003:00000cd0       _ioLog                     1001acd0     GCFramePlot.obj
 0003:00000cd8       _coreLog                   1001acd8     GCFramePlot.obj
 0003:00000ce0       _uiLog                     1001ace0     GCFramePlot.obj
 0003:00000ce8       _scriptLog                 1001ace8     GCFramePlot.obj
 0003:00000cf0       _perfLog                   1001acf0     GCFramePlot.obj
 0003:00000cf8       _cmdLog                    1001acf8     GCFramePlot.obj
 0003:00000d00       __Tuple_alloc              1001ad00     KarlinSignatureDifferenceGraph.obj
 0003:00000d01       _ignore                    1001ad01     KarlinSignatureDifferenceGraph.obj
 0003:00000d02       _allocator_arg             1001ad02     KarlinSignatureDifferenceGraph.obj
 0003:00000d03       _piecewise_construct       1001ad03     KarlinSignatureDifferenceGraph.obj
 0003:00000d04       _taskLog                   1001ad04     KarlinSignatureDifferenceGraph.obj
 0003:00000d0c       _algoLog                   1001ad0c     KarlinSignatureDifferenceGraph.obj
 0003:00000d14       _userActLog                1001ad14     KarlinSignatureDifferenceGraph.obj
 0003:00000d1c       _ioLog                     1001ad1c     KarlinSignatureDifferenceGraph.obj
 0003:00000d24       _coreLog                   1001ad24     KarlinSignatureDifferenceGraph.obj
 0003:00000d2c       _uiLog                     1001ad2c     KarlinSignatureDifferenceGraph.obj
 0003:00000d34       _scriptLog                 1001ad34     KarlinSignatureDifferenceGraph.obj
 0003:00000d3c       _perfLog                   1001ad3c     KarlinSignatureDifferenceGraph.obj
 0003:00000d44       _cmdLog                    1001ad44     KarlinSignatureDifferenceGraph.obj
 0003:00000d4c       __Tuple_alloc              1001ad4c     moc_BaseContentGraph.obj
 0003:00000d4d       _ignore                    1001ad4d     moc_BaseContentGraph.obj
 0003:00000d4e       _allocator_arg             1001ad4e     moc_BaseContentGraph.obj
 0003:00000d4f       _piecewise_construct       1001ad4f     moc_BaseContentGraph.obj
 0003:00000d50       _taskLog                   1001ad50     moc_BaseContentGraph.obj
 0003:00000d58       _algoLog                   1001ad58     moc_BaseContentGraph.obj
 0003:00000d60       _userActLog                1001ad60     moc_BaseContentGraph.obj
 0003:00000d68       _ioLog                     1001ad68     moc_BaseContentGraph.obj
 0003:00000d70       _coreLog                   1001ad70     moc_BaseContentGraph.obj
 0003:00000d78       _uiLog                     1001ad78     moc_BaseContentGraph.obj
 0003:00000d80       _scriptLog                 1001ad80     moc_BaseContentGraph.obj
 0003:00000d88       _perfLog                   1001ad88     moc_BaseContentGraph.obj
 0003:00000d90       _cmdLog                    1001ad90     moc_BaseContentGraph.obj
 0003:00000d98       __Tuple_alloc              1001ad98     moc_CumulativeSkew.obj
 0003:00000d99       _ignore                    1001ad99     moc_CumulativeSkew.obj
 0003:00000d9a       _allocator_arg             1001ad9a     moc_CumulativeSkew.obj
 0003:00000d9b       _piecewise_construct       1001ad9b     moc_CumulativeSkew.obj
 0003:00000d9c       _taskLog                   1001ad9c     moc_CumulativeSkew.obj
 0003:00000da4       _algoLog                   1001ada4     moc_CumulativeSkew.obj
 0003:00000dac       _userActLog                1001adac     moc_CumulativeSkew.obj
 0003:00000db4       _ioLog                     1001adb4     moc_CumulativeSkew.obj
 0003:00000dbc       _coreLog                   1001adbc     moc_CumulativeSkew.obj
 0003:00000dc4       _uiLog                     1001adc4     moc_CumulativeSkew.obj
 0003:00000dcc       _scriptLog                 1001adcc     moc_CumulativeSkew.obj
 0003:00000dd4       _perfLog                   1001add4     moc_CumulativeSkew.obj
 0003:00000ddc       _cmdLog                    1001addc     moc_CumulativeSkew.obj
 0003:00000de4       __Tuple_alloc              1001ade4     moc_DNAGraphPackPlugin.obj
 0003:00000de5       _ignore                    1001ade5     moc_DNAGraphPackPlugin.obj
 0003:00000de6       _allocator_arg             1001ade6     moc_DNAGraphPackPlugin.obj
 0003:00000de7       _piecewise_construct       1001ade7     moc_DNAGraphPackPlugin.obj
 0003:00000de8       _taskLog                   1001ade8     moc_DNAGraphPackPlugin.obj
 0003:00000df0       _algoLog                   1001adf0     moc_DNAGraphPackPlugin.obj
 0003:00000df8       _userActLog                1001adf8     moc_DNAGraphPackPlugin.obj
 0003:00000e00       _ioLog                     1001ae00     moc_DNAGraphPackPlugin.obj
 0003:00000e08       _coreLog                   1001ae08     moc_DNAGraphPackPlugin.obj
 0003:00000e10       _uiLog                     1001ae10     moc_DNAGraphPackPlugin.obj
 0003:00000e18       _scriptLog                 1001ae18     moc_DNAGraphPackPlugin.obj
 0003:00000e20       _perfLog                   1001ae20     moc_DNAGraphPackPlugin.obj
 0003:00000e28       _cmdLog                    1001ae28     moc_DNAGraphPackPlugin.obj
 0003:00000e34       __Tuple_alloc              1001ae34     moc_DeviationGraph.obj
 0003:00000e35       _ignore                    1001ae35     moc_DeviationGraph.obj
 0003:00000e36       _allocator_arg             1001ae36     moc_DeviationGraph.obj
 0003:00000e37       _piecewise_construct       1001ae37     moc_DeviationGraph.obj
 0003:00000e38       _taskLog                   1001ae38     moc_DeviationGraph.obj
 0003:00000e40       _algoLog                   1001ae40     moc_DeviationGraph.obj
 0003:00000e48       _userActLog                1001ae48     moc_DeviationGraph.obj
 0003:00000e50       _ioLog                     1001ae50     moc_DeviationGraph.obj
 0003:00000e58       _coreLog                   1001ae58     moc_DeviationGraph.obj
 0003:00000e60       _uiLog                     1001ae60     moc_DeviationGraph.obj
 0003:00000e68       _scriptLog                 1001ae68     moc_DeviationGraph.obj
 0003:00000e70       _perfLog                   1001ae70     moc_DeviationGraph.obj
 0003:00000e78       _cmdLog                    1001ae78     moc_DeviationGraph.obj
 0003:00000e80       __Tuple_alloc              1001ae80     moc_EntropyAlgorithm.obj
 0003:00000e81       _ignore                    1001ae81     moc_EntropyAlgorithm.obj
 0003:00000e82       _allocator_arg             1001ae82     moc_EntropyAlgorithm.obj
 0003:00000e83       _piecewise_construct       1001ae83     moc_EntropyAlgorithm.obj
 0003:00000e84       _taskLog                   1001ae84     moc_EntropyAlgorithm.obj
 0003:00000e8c       _algoLog                   1001ae8c     moc_EntropyAlgorithm.obj
 0003:00000e94       _userActLog                1001ae94     moc_EntropyAlgorithm.obj
 0003:00000e9c       _ioLog                     1001ae9c     moc_EntropyAlgorithm.obj
 0003:00000ea4       _coreLog                   1001aea4     moc_EntropyAlgorithm.obj
 0003:00000eac       _uiLog                     1001aeac     moc_EntropyAlgorithm.obj
 0003:00000eb4       _scriptLog                 1001aeb4     moc_EntropyAlgorithm.obj
 0003:00000ebc       _perfLog                   1001aebc     moc_EntropyAlgorithm.obj
 0003:00000ec4       _cmdLog                    1001aec4     moc_EntropyAlgorithm.obj
 0003:00000ecc       __Tuple_alloc              1001aecc     moc_GCFramePlot.obj
 0003:00000ecd       _ignore                    1001aecd     moc_GCFramePlot.obj
 0003:00000ece       _allocator_arg             1001aece     moc_GCFramePlot.obj
 0003:00000ecf       _piecewise_construct       1001aecf     moc_GCFramePlot.obj
 0003:00000ed0       _taskLog                   1001aed0     moc_GCFramePlot.obj
 0003:00000ed8       _algoLog                   1001aed8     moc_GCFramePlot.obj
 0003:00000ee0       _userActLog                1001aee0     moc_GCFramePlot.obj
 0003:00000ee8       _ioLog                     1001aee8     moc_GCFramePlot.obj
 0003:00000ef0       _coreLog                   1001aef0     moc_GCFramePlot.obj
 0003:00000ef8       _uiLog                     1001aef8     moc_GCFramePlot.obj
 0003:00000f00       _scriptLog                 1001af00     moc_GCFramePlot.obj
 0003:00000f08       _perfLog                   1001af08     moc_GCFramePlot.obj
 0003:00000f10       _cmdLog                    1001af10     moc_GCFramePlot.obj
 0003:00000f18       __Tuple_alloc              1001af18     moc_KarlinSignatureDifferenceGraph.obj
 0003:00000f19       _ignore                    1001af19     moc_KarlinSignatureDifferenceGraph.obj
 0003:00000f1a       _allocator_arg             1001af1a     moc_KarlinSignatureDifferenceGraph.obj
 0003:00000f1b       _piecewise_construct       1001af1b     moc_KarlinSignatureDifferenceGraph.obj
 0003:00000f1c       _taskLog                   1001af1c     moc_KarlinSignatureDifferenceGraph.obj
 0003:00000f24       _algoLog                   1001af24     moc_KarlinSignatureDifferenceGraph.obj
 0003:00000f2c       _userActLog                1001af2c     moc_KarlinSignatureDifferenceGraph.obj
 0003:00000f34       _ioLog                     1001af34     moc_KarlinSignatureDifferenceGraph.obj
 0003:00000f3c       _coreLog                   1001af3c     moc_KarlinSignatureDifferenceGraph.obj
 0003:00000f44       _uiLog                     1001af44     moc_KarlinSignatureDifferenceGraph.obj
 0003:00000f4c       _scriptLog                 1001af4c     moc_KarlinSignatureDifferenceGraph.obj
 0003:00000f54       _perfLog                   1001af54     moc_KarlinSignatureDifferenceGraph.obj
 0003:00000f5c       _cmdLog                    1001af5c     moc_KarlinSignatureDifferenceGraph.obj
 0003:00000f68       ___proc_attached           1001af68     MSVCRT:crtdll.obj
 0003:00000f70       _GS_ExceptionRecord        1001af70     MSVCRT:gs_report.obj
 0003:00000fc0       _GS_ContextRecord          1001afc0     MSVCRT:gs_report.obj
 0003:0000128c       _DebuggerWasPresent        1001b28c     MSVCRT:gs_report.obj
 0004:00000060       $R000000                   1001c060     * linker generated manifest res *

 Exports

  ordinal    name

        1    _ugene_plugin_init
               exported name: ugene_plugin_init
